 ptools

 Timestamp is 5dee3645 (Mon Dec 09 18:55:49 2019)

 Preferred load address is 10000000

 Start         Length     Name                   Class
 0001:00000000 00001a34H .text$di                CODE
 0001:00001a40 000168f8H .text$mn                CODE
 0001:00018340 00002554H .text$x                 CODE
 0001:0001a8a0 00000605H .text$yd                CODE
 0002:00000000 000003c4H .idata$5                DATA
 0002:000003c4 00000004H .CRT$XCA                DATA
 0002:000003c8 00000004H .CRT$XCL                DATA
 0002:000003cc 000000e0H .CRT$XCU                DATA
 0002:000004ac 00000004H .CRT$XCZ                DATA
 0002:000004b0 00000004H .CRT$XIA                DATA
 0002:000004b4 00000004H .CRT$XIAA               DATA
 0002:000004b8 00000004H .CRT$XIC                DATA
 0002:000004bc 00000004H .CRT$XIZ                DATA
 0002:000004c0 000009b8H .rdata                  DATA
 0002:00000e78 0000006cH .rdata$debug            DATA
 0002:00000ee4 00000b08H .rdata$r                DATA
 0002:000019f0 00000288H .rdata$sxdata           DATA
 0002:00001c78 00000004H .rtc$IAA                DATA
 0002:00001c7c 00000004H .rtc$IZZ                DATA
 0002:00001c80 00000004H .rtc$TAA                DATA
 0002:00001c84 00000004H .rtc$TZZ                DATA
 0002:00001c88 000028acH .xdata$x                DATA
 0002:00004540 0000004fH .edata                  DATA
 0002:00004590 000000a0H .idata$2                DATA
 0002:00004630 00000014H .idata$3                DATA
 0002:00004644 000003c4H .idata$4                DATA
 0002:00004a08 00002446H .idata$6                DATA
 0003:00000000 00000054H .data                   DATA
 0003:00000058 000006b4H .data$r                 DATA
 0003:00000710 00000504H .bss                    DATA
 0004:00000000 00000058H .rsrc$01                DATA
 0004:00000060 00000180H .rsrc$02                DATA

  Address         Publics by Value              Rva+Base       Lib:Object

 0000:00000000       ___guard_flags             00000000     <absolute>
 0000:00000000       __except_list              00000000     <absolute>
 0000:00000000       ___guard_fids_table        00000000     <absolute>
 0000:00000000       ___guard_fids_count        00000000     <absolute>
 0000:000000a2       ___safe_se_handler_count   000000a2     <absolute>
 0000:00009876       __ldused                   00009876     <absolute>
 0000:00009876       __fltused                  00009876     <absolute>
 0000:00000000       ___ImageBase               10000000     <linker-defined>
 0001:00001a40       ??$?8DD@std@@YA_NABV?$allocator@D@0@0@Z 10002a40 f i PToolsAligner.obj
 0001:00001a50       ??$?8V?$allocator@D@std@@V01@@std@@YA_NABU?$_Wrap_alloc@V?$allocator@D@std@@@0@0@Z 10002a50 f i PToolsAligner.obj
 0001:00001a60       ??$?9V?$allocator@D@std@@V01@@std@@YA_NABU?$_Wrap_alloc@V?$allocator@D@std@@@0@0@Z 10002a60 f i PToolsAligner.obj
 0001:00001a70       ??$_Allocate@D@std@@YAPADIPAD@Z 10002a70 f i PToolsAligner.obj
 0001:00001aa0       ??$addressof@D@std@@YAPADAAD@Z 10002aa0 f i PToolsAligner.obj
 0001:00001ab0       ??$atomic@H@?$QAtomicOpsBySize@$03@@CAPAJPAH@Z 10002ab0 f i PToolsAligner.obj
 0001:00001ac0       ??$construct@PADAAPAD@?$_Wrap_alloc@V?$allocator@D@std@@@std@@QAEXPAPADAAPAD@Z 10002ac0 f i PToolsAligner.obj
 0001:00001ae0       ??$construct@PADAAPAD@?$allocator@D@std@@QAEXPAPADAAPAD@Z 10002ae0 f i PToolsAligner.obj
 0001:00001b00       ??$construct@PADAAPAD@?$allocator_traits@V?$allocator@D@std@@@std@@SAXAAV?$allocator@D@1@PAPADAAPAD@Z 10002b00 f i PToolsAligner.obj
 0001:00001b20       ??$deref@H@?$QAtomicOpsBySize@$03@@SA_NAAH@Z 10002b20 f i PToolsAligner.obj
 0001:00001b40       ??$destroy@PAD@?$_Wrap_alloc@V?$allocator@D@std@@@std@@QAEXPAPAD@Z 10002b40 f i PToolsAligner.obj
 0001:00001b50       ??$destroy@PAD@?$allocator@D@std@@QAEXPAPAD@Z 10002b50 f i PToolsAligner.obj
 0001:00001b60       ??$destroy@PAD@?$allocator_traits@V?$allocator@D@std@@@std@@SAXAAV?$allocator@D@1@PAPAD@Z 10002b60 f i PToolsAligner.obj
 0001:00001b70       ??$forward@AAPAD@std@@YAAAPADAAPAD@Z 10002b70 f i PToolsAligner.obj
 0001:00001b80       ??$load@H@?$QGenericAtomicOps@U?$QAtomicOpsBySize@$03@@@@SAHABH@Z 10002b80 f i PToolsAligner.obj
 0001:00001b90       ??$qMapLessThanKey@H@@YA_NABH0@Z 10002b90 f i PToolsAligner.obj
 0001:00001bb0       ??$ref@H@?$QAtomicOpsBySize@$03@@SA_NAAH@Z 10002bb0 f i PToolsAligner.obj
 0001:00001bd0       ??0?$QFlags@W4AllocationOption@QArrayData@@@@QAE@W4AllocationOption@QArrayData@@@Z 10002bd0 f i PToolsAligner.obj
 0001:00001be0       ??0?$QForeachContainer@V?$QList@H@@@@QAE@ABV?$QList@H@@@Z 10002be0 f i PToolsAligner.obj
 0001:00001c20       ??0?$QForeachContainer@V?$QList@V?$QSharedDataPointer@VAtomData@U2@@@@@@@@QAE@ABV?$QList@V?$QSharedDataPointer@VAtomData@U2@@@@@@@Z 10002c20 f i PToolsAligner.obj
 0001:00001c60       ??0?$QList@H@@QAE@ABV0@@Z  10002c60 f i PToolsAligner.obj
 0001:00001d20       ??0?$QList@V?$QSharedDataPointer@VAtomData@U2@@@@@@QAE@ABV0@@Z 10002d20 f i PToolsAligner.obj
 0001:00001de0       ??0?$QScopedPointer@VRigidbody@PTools@@U?$QScopedPointerDeleter@VRigidbody@PTools@@@@@@QAE@PAVRigidbody@PTools@@@Z 10002de0 f i PToolsAligner.obj
 0001:00001df0       ??0?$QSharedDataPointer@VAtomData@U2@@@@QAE@ABV0@@Z 10002df0 f i PToolsAligner.obj
 0001:00001e10       ??0?$QSharedDataPointer@VMoleculeData@U2@@@@QAE@ABV0@@Z 10002e10 f i PToolsAligner.obj
 0001:00001e30       ??0?$QSharedDataPointer@VMoleculeData@U2@@@@QAE@XZ 10002e30 f i PToolsAligner.obj
 0001:00001e40       ??0?$_String_alloc@$0A@U?$_String_base_types@DV?$allocator@D@std@@@std@@@std@@QAE@ABV?$allocator@D@1@@Z 10002e40 f i PToolsAligner.obj
 0001:00001e60       ??0?$_String_val@U?$_Simple_types@D@std@@@std@@QAE@XZ 10002e60 f i PToolsAligner.obj
 0001:00001e80       ??0?$_Wrap_alloc@V?$allocator@D@std@@@std@@QAE@ABV?$allocator@D@1@@Z 10002e80 f i PToolsAligner.obj
 0001:00001e90       ??0?$_Wrap_alloc@V?$allocator@D@std@@@std@@QAE@XZ 10002e90 f i PToolsAligner.obj
 0001:00001ea0       ??0?$allocator@D@std@@QAE@ABV01@@Z 10002ea0 f i PToolsAligner.obj
 0001:00001eb0       ??0?$allocator@D@std@@QAE@XZ 10002eb0 f i PToolsAligner.obj
 0001:00001ec0       ??0?$basic_string@DU?$char_traits@D@std@@V?$allocator@D@2@@std@@QAE@ABV01@@Z 10002ec0 f i PToolsAligner.obj
 0001:00001ef0       ??0?$basic_string@DU?$char_traits@D@std@@V?$allocator@D@2@@std@@QAE@PBD@Z 10002ef0 f i PToolsAligner.obj
 0001:00001f50       ??0?$basic_string@DU?$char_traits@D@std@@V?$allocator@D@2@@std@@QAE@XZ 10002f50 f i PToolsAligner.obj
 0001:00001f70       ??0Atom@PTools@@QAE@VAtomproperty@1@UCoord3D@1@@Z 10002f70 f i PToolsAligner.obj
 0001:00001fe0       ??0Atomproperty@PTools@@QAE@ABV01@@Z 10002fe0 f i PToolsAligner.obj
 0001:000020f0       ??0Atomproperty@PTools@@QAE@XZ 100030f0 f i PToolsAligner.obj
 0001:000021f0       ??0Coord3D@PTools@@QAE@ABU01@@Z 100031f0 f i PToolsAligner.obj
 0001:00002220       ??0Coord3D@PTools@@QAE@NNN@Z 10003220 f i PToolsAligner.obj
 0001:00002250       ??0QLatin1Char@@QAE@D@Z    10003250 f i PToolsAligner.obj
 0001:00002260       ??0_Generic_error_category@std@@QAE@XZ 10003260 f i PToolsAligner.obj
 0001:00002270       ??0_Ignore@std@@QAE@XZ     10003270 f i PToolsAligner.obj
 0001:00002280       ??0_Iostream_error_category@std@@QAE@XZ 10003280 f i PToolsAligner.obj
 0001:00002290       ??0_System_error_category@std@@QAE@XZ 10003290 f i PToolsAligner.obj
 0001:000022a0       ??0const_iterator@?$QList@H@@QAE@PAUNode@1@@Z 100032a0 f i PToolsAligner.obj
 0001:000022b0       ??0const_iterator@?$QList@V?$QSharedDataPointer@VAtomData@U2@@@@@@QAE@PAUNode@1@@Z 100032b0 f i PToolsAligner.obj
 0001:000022c0       ??0error_category@std@@QAE@XZ 100032c0 f i PToolsAligner.obj
 0001:000022d0       ??0error_condition@std@@QAE@HABVerror_category@1@@Z 100032d0 f i PToolsAligner.obj
 0001:000022f0       ??1?$Array2D@N@@QAE@XZ     100032f0 f i PToolsAligner.obj
 0001:00002330       ??1?$QForeachContainer@V?$QList@H@@@@QAE@XZ 10003330 f i PToolsAligner.obj
 0001:00002360       ??1?$QForeachContainer@V?$QList@V?$QSharedDataPointer@VAtomData@U2@@@@@@@@QAE@XZ 10003360 f i PToolsAligner.obj
 0001:000023b0       ??1?$QList@H@@QAE@XZ       100033b0 f i PToolsAligner.obj
 0001:000023e0       ??1?$QList@V?$QSharedDataPointer@VAtomData@U2@@@@@@QAE@XZ 100033e0 f i PToolsAligner.obj
 0001:00002430       ??1?$QList@VBond@U2@@@@QAE@XZ 10003430 f i PToolsAligner.obj
 0001:00002480       ??1?$QMap@HVMolecule3DModel@U2@@@@QAE@XZ 10003480 f i PToolsAligner.obj
 0001:000024e0       ??1?$QMap@VResidueIndex@U2@@V?$QSharedDataPointer@VResidueData@U2@@@@@@QAE@XZ 100034e0 f i PToolsAligner.obj
 0001:00002530       ??1?$QScopedPointer@VRigidbody@PTools@@U?$QScopedPointerDeleter@VRigidbody@PTools@@@@@@QAE@XZ 10003530 f i PToolsAligner.obj
 0001:00002540       ??1?$QSharedDataPointer@VAtomData@U2@@@@QAE@XZ 10003540 f i PToolsAligner.obj
 0001:00002570       ??1?$QSharedDataPointer@VMoleculeData@U2@@@@QAE@XZ 10003570 f i PToolsAligner.obj
 0001:000025a0       ??1?$QSharedDataPointer@VResidueData@U2@@@@QAE@XZ 100035a0 f i PToolsAligner.obj
 0001:000025d0       ??1?$QVector@N@@QAE@XZ     100035d0 f i PToolsAligner.obj
 0001:00002610       ??1?$basic_string@DU?$char_traits@D@std@@V?$allocator@D@2@@std@@QAE@XZ 10003610 f i PToolsAligner.obj
 0001:00002640       ??1Atom@PTools@@QAE@XZ     10003640 f i PToolsAligner.obj
 0001:00002650       ??1AtomData@U2@@QAE@XZ     10003650 f i PToolsAligner.obj
 0001:00002660       ??1Atomproperty@PTools@@QAE@XZ 10003660 f i PToolsAligner.obj
 0001:00002720       ??1Bond@U2@@QAE@XZ         10003720 f i PToolsAligner.obj
 0001:000027c0       ??1Molecule3DModel@U2@@QAE@XZ 100037c0 f i PToolsAligner.obj
 0001:00002890       ??1MoleculeData@U2@@QAE@XZ 10003890 f i PToolsAligner.obj
 0001:00002930       ??1ResidueData@U2@@QAE@XZ  10003930 f i PToolsAligner.obj
 0001:00002940       ??1Superpose_t@@QAE@XZ     10003940 f i PToolsAligner.obj
 0001:00002980       ??1_Generic_error_category@std@@UAE@XZ 10003980 f i PToolsAligner.obj
 0001:00002990       ??1_Iostream_error_category@std@@UAE@XZ 10003990 f i PToolsAligner.obj
 0001:000029a0       ??1_System_error_category@std@@UAE@XZ 100039a0 f i PToolsAligner.obj
 0001:000029b0       ??1error_category@std@@UAE@XZ 100039b0 f i PToolsAligner.obj
 0001:000029c0       ??2@YAPAXIPAX@Z            100039c0 f i PToolsAligner.obj
 0001:000029d0       ??3@YAXPAX0@Z              100039d0 f i PToolsAligner.obj
 0001:000029e0       ??4?$basic_string@DU?$char_traits@D@std@@V?$allocator@D@2@@std@@QAEAAV01@ABV01@@Z 100039e0 f i PToolsAligner.obj
 0001:00002a00       ??4?$basic_string@DU?$char_traits@D@std@@V?$allocator@D@2@@std@@QAEAAV01@PBD@Z 10003a00 f i PToolsAligner.obj
 0001:00002a40       ??8@YA_NABVQByteArray@@PBD@Z 10003a40 f i PToolsAligner.obj
 0001:00002a70       ??8error_category@std@@QBE_NABV01@@Z 10003a70 f i PToolsAligner.obj
 0001:00002a80       ??8error_condition@std@@QBE_NABV01@@Z 10003a80 f i PToolsAligner.obj
 0001:00002aa0       ??9const_iterator@?$QList@H@@QBE_NABV01@@Z 10003aa0 f i PToolsAligner.obj
 0001:00002ac0       ??9const_iterator@?$QList@V?$QSharedDataPointer@VAtomData@U2@@@@@@QBE_NABV01@@Z 10003ac0 f i PToolsAligner.obj
 0001:00002ae0       ??A?$QVector@N@@QAEAANH@Z  10003ae0 f i PToolsAligner.obj
 0001:00002b60       ??C?$QScopedPointer@VRigidbody@PTools@@U?$QScopedPointerDeleter@VRigidbody@PTools@@@@@@QBEPAVRigidbody@PTools@@XZ 10003b60 f i PToolsAligner.obj
 0001:00002b70       ??C?$QSharedDataPointer@VAtomData@U2@@@@QBEPBVAtomData@U2@@XZ 10003b70 f i PToolsAligner.obj
 0001:00002b80       ??C?$QSharedDataPointer@VMoleculeData@U2@@@@QBEPBVMoleculeData@U2@@XZ 10003b80 f i PToolsAligner.obj
 0001:00002b90       ??D?$QScopedPointer@VRigidbody@PTools@@U?$QScopedPointerDeleter@VRigidbody@PTools@@@@@@QBEAAVRigidbody@PTools@@XZ 10003b90 f i PToolsAligner.obj
 0001:00002ba0       ??Dconst_iterator@?$QList@H@@QBEABHXZ 10003ba0 f i PToolsAligner.obj
 0001:00002bb0       ??Dconst_iterator@?$QList@V?$QSharedDataPointer@VAtomData@U2@@@@@@QBEABV?$QSharedDataPointer@VAtomData@U2@@@@XZ 10003bb0 f i PToolsAligner.obj
 0001:00002bc0       ??Econst_iterator@?$QList@H@@QAEAAV01@XZ 10003bc0 f i PToolsAligner.obj
 0001:00002bd0       ??Econst_iterator@?$QList@V?$QSharedDataPointer@VAtomData@U2@@@@@@QAEAAV01@XZ 10003bd0 f i PToolsAligner.obj
 0001:00002be0       ??R?$Array2D@N@@QAEAANHH@Z 10003be0 f i PToolsAligner.obj
 0001:00002c00       ??_G?$QSharedDataPointer@VAtomData@U2@@@@QAEPAXI@Z 10003c00 f i PToolsAligner.obj
 0001:00002c50       ??_G?$QSharedDataPointer@VResidueData@U2@@@@QAEPAXI@Z 10003c50 f i PToolsAligner.obj
 0001:00002ca0       ??_GAtomData@U2@@QAEPAXI@Z 10003ca0 f i PToolsAligner.obj
 0001:00002cd0       ??_GBond@U2@@QAEPAXI@Z     10003cd0 f i PToolsAligner.obj
 0001:00002d00       ??_GMolecule3DModel@U2@@QAEPAXI@Z 10003d00 f i PToolsAligner.obj
 0001:00002d30       ??_GMoleculeData@U2@@QAEPAXI@Z 10003d30 f i PToolsAligner.obj
 0001:00002d60       ??_GResidueData@U2@@QAEPAXI@Z 10003d60 f i PToolsAligner.obj
 0001:00002d90       ??_G_Generic_error_category@std@@UAEPAXI@Z 10003d90 f i PToolsAligner.obj
 0001:00002d90       ??_E_Generic_error_category@std@@UAEPAXI@Z 10003d90 f i PToolsAligner.obj
 0001:00002dc0       ??_E_Iostream_error_category@std@@UAEPAXI@Z 10003dc0 f i PToolsAligner.obj
 0001:00002dc0       ??_G_Iostream_error_category@std@@UAEPAXI@Z 10003dc0 f i PToolsAligner.obj
 0001:00002df0       ??_E_System_error_category@std@@UAEPAXI@Z 10003df0 f i PToolsAligner.obj
 0001:00002df0       ??_G_System_error_category@std@@UAEPAXI@Z 10003df0 f i PToolsAligner.obj
 0001:00002e20       ??_Gerror_category@std@@UAEPAXI@Z 10003e20 f i PToolsAligner.obj
 0001:00002e20       ??_Eerror_category@std@@UAEPAXI@Z 10003e20 f i PToolsAligner.obj
 0001:00002e50       ?SetResidId@Atomproperty@PTools@@QAEXI@Z 10003e50 f i PToolsAligner.obj
 0001:00002e60       ?SetType@Atomproperty@PTools@@QAEXV?$basic_string@DU?$char_traits@D@std@@V?$allocator@D@2@@std@@@Z 10003e60 f i PToolsAligner.obj
 0001:00002ec0       ?Size@CoordsArray@PTools@@QBEIXZ 10003ec0 f i PToolsAligner.obj
 0001:00002ee0       ?Size@Rigidbody@PTools@@QBEIXZ 10003ee0 f i PToolsAligner.obj
 0001:00002f00       ?_Change_alloc@?$_String_alloc@$0A@U?$_String_base_types@DV?$allocator@D@std@@@std@@@std@@QAEXABU?$_Wrap_alloc@V?$allocator@D@std@@@2@@Z 10003f00 f i PToolsAligner.obj
 0001:00002f10       ?_Copy@?$basic_string@DU?$char_traits@D@std@@V?$allocator@D@2@@std@@QAEXII@Z 10003f10 f i PToolsAligner.obj
 0001:00003060       ?_Eos@?$basic_string@DU?$char_traits@D@std@@V?$allocator@D@2@@std@@QAEXI@Z 10004060 f i PToolsAligner.obj
 0001:00003090       ?_Getal@?$_String_alloc@$0A@U?$_String_base_types@DV?$allocator@D@std@@@std@@@std@@QBE?AU?$_Wrap_alloc@V?$allocator@D@std@@@2@XZ 10004090 f i PToolsAligner.obj
 0001:000030a0       ?_Grow@?$basic_string@DU?$char_traits@D@std@@V?$allocator@D@2@@std@@QAE_NI_N@Z 100040a0 f i PToolsAligner.obj
 0001:00003150       ?_Inside@?$basic_string@DU?$char_traits@D@std@@V?$allocator@D@2@@std@@QAE_NPBD@Z 10004150 f i PToolsAligner.obj
 0001:00003190       ?_Myptr@?$_String_val@U?$_Simple_types@D@std@@@std@@QAEPADXZ 10004190 f i PToolsAligner.obj
 0001:000031a0       ?_Myptr@?$_String_val@U?$_Simple_types@D@std@@@std@@QBEPBDXZ 100041a0 f i PToolsAligner.obj
 0001:000031b0       ?_Tidy@?$basic_string@DU?$char_traits@D@std@@V?$allocator@D@2@@std@@QAEX_NI@Z 100041b0 f i PToolsAligner.obj
 0001:00003200       ?_Xlen@?$basic_string@DU?$char_traits@D@std@@V?$allocator@D@2@@std@@QBEXXZ 10004200 f i PToolsAligner.obj
 0001:00003210       ?_Xran@?$basic_string@DU?$char_traits@D@std@@V?$allocator@D@2@@std@@QBEXXZ 10004210 f i PToolsAligner.obj
 0001:00003220       ?align@PToolsAligner@U2@@UAE?AVStructuralAlignment@2@ABVStructuralAlignmentTaskSettings@2@AAVTaskStateInfo@2@@Z 10004220 f   PToolsAligner.obj
 0001:00003600       ?allocate@?$QTypedArrayData@N@@SAPAU1@IV?$QFlags@W4AllocationOption@QArrayData@@@@@Z 10004600 f i PToolsAligner.obj
 0001:00003620       ?allocate@?$_Wrap_alloc@V?$allocator@D@std@@@std@@QAEPADI@Z 10004620 f i PToolsAligner.obj
 0001:00003650       ?allocate@?$allocator@D@std@@QAEPADI@Z 10004650 f i PToolsAligner.obj
 0001:00003680       ?assign@?$basic_string@DU?$char_traits@D@std@@V?$allocator@D@2@@std@@QAEAAV12@ABV12@@Z 10004680 f i PToolsAligner.obj
 0001:000036a0       ?assign@?$basic_string@DU?$char_traits@D@std@@V?$allocator@D@2@@std@@QAEAAV12@ABV12@II@Z 100046a0 f i PToolsAligner.obj
 0001:000037c0       ?assign@?$basic_string@DU?$char_traits@D@std@@V?$allocator@D@2@@std@@QAEAAV12@PBD@Z 100047c0 f i PToolsAligner.obj
 0001:00003800       ?assign@?$basic_string@DU?$char_traits@D@std@@V?$allocator@D@2@@std@@QAEAAV12@PBDI@Z 10004800 f i PToolsAligner.obj
 0001:00003900       ?assign@?$char_traits@D@std@@SAXAADABD@Z 10004900 f i PToolsAligner.obj
 0001:00003910       ?begin@?$QList@H@@QBE?AVconst_iterator@1@XZ 10004910 f i PToolsAligner.obj
 0001:00003930       ?begin@?$QList@V?$QSharedDataPointer@VAtomData@U2@@@@@@QBE?AVconst_iterator@1@XZ 10004930 f i PToolsAligner.obj
 0001:00003950       ?begin@?$QTypedArrayData@N@@QAEPANPAN@Z 10004950 f i PToolsAligner.obj
 0001:00003960       ?category@error_code@std@@QBEABVerror_category@2@XZ 10004960 f i PToolsAligner.obj
 0001:00003970       ?category@error_condition@std@@QBEABVerror_category@2@XZ 10004970 f i PToolsAligner.obj
 0001:00003980       ?cleanup@?$QScopedPointerDeleter@VRigidbody@PTools@@@@SAXPAVRigidbody@PTools@@@Z 10004980 f i PToolsAligner.obj
 0001:000039a0       ?copy@?$char_traits@D@std@@SAPADPADPBDI@Z 100049a0 f i PToolsAligner.obj
 0001:00003ef0       ?data@?$QTypedArrayData@N@@QAEPANXZ 10004ef0 f i PToolsAligner.obj
 0001:00003f00       ?data@?$QVector@N@@QAEPANXZ 10004f00 f i PToolsAligner.obj
 0001:00003f60       ?dealloc@?$QList@H@@AAEXPAUData@QListData@@@Z 10004f60 f i PToolsAligner.obj
 0001:00003f80       ?dealloc@?$QList@V?$QSharedDataPointer@VAtomData@U2@@@@@@AAEXPAUData@QListData@@@Z 10004f80 f i PToolsAligner.obj
 0001:00003fb0       ?dealloc@?$QList@VBond@U2@@@@AAEXPAUData@QListData@@@Z 10004fb0 f i PToolsAligner.obj
 0001:00003fe0       ?deallocate@?$QTypedArrayData@N@@SAXPAUQArrayData@@@Z 10004fe0 f i PToolsAligner.obj
 0001:00004000       ?deallocate@?$_Wrap_alloc@V?$allocator@D@std@@@std@@QAEXPADI@Z 10005000 f i PToolsAligner.obj
 0001:00004020       ?deallocate@?$allocator@D@std@@QAEXPADI@Z 10005020 f i PToolsAligner.obj
 0001:00004040       ?defaultConstruct@?$QVector@N@@AAEXPAN0@Z 10005040 f i PToolsAligner.obj
 0001:00004060       ?default_error_condition@_System_error_category@std@@UBE?AVerror_condition@2@H@Z 10005060 f i PToolsAligner.obj
 0001:000040a0       ?default_error_condition@error_category@std@@UBE?AVerror_condition@2@H@Z 100050a0 f i PToolsAligner.obj
 0001:000040c0       ?deref@?$QBasicAtomicInteger@H@@QAE_NXZ 100050c0 f i PToolsAligner.obj
 0001:000040d0       ?deref@RefCount@QtPrivate@@QAE_NXZ 100050d0 f i PToolsAligner.obj
 0001:000040f0       ?destroy@?$QMapData@HVMolecule3DModel@U2@@@@QAEXXZ 100050f0 f i PToolsAligner.obj
 0001:00004140       ?destroy@?$QMapData@VResidueIndex@U2@@V?$QSharedDataPointer@VResidueData@U2@@@@@@QAEXXZ 10005140 f i PToolsAligner.obj
 0001:00004170       ?destroySubTree@?$QMapNode@HVMolecule3DModel@U2@@@@QAEXXZ 10005170 f i PToolsAligner.obj
 0001:00004190       ?destroySubTree@?$QMapNode@VResidueIndex@U2@@V?$QSharedDataPointer@VResidueData@U2@@@@@@QAEXXZ 10005190 f i PToolsAligner.obj
 0001:000041e0       ?destruct@?$QVector@N@@AAEXPAN0@Z 100051e0 f i PToolsAligner.obj
 0001:000041f0       ?detach@?$QVector@N@@QAEXXZ 100051f0 f i PToolsAligner.obj
 0001:00004240       ?end@?$QList@H@@QBE?AVconst_iterator@1@XZ 10005240 f i PToolsAligner.obj
 0001:00004260       ?end@?$QList@V?$QSharedDataPointer@VAtomData@U2@@@@@@QBE?AVconst_iterator@1@XZ 10005260 f i PToolsAligner.obj
 0001:00004280       ?end@?$QTypedArrayData@N@@QAEPANPAN@Z 10005280 f i PToolsAligner.obj
 0001:000042a0       ?equivalent@error_category@std@@UBE_NABVerror_code@2@H@Z 100052a0 f i PToolsAligner.obj
 0001:000042c0       ?equivalent@error_category@std@@UBE_NHABVerror_condition@2@@Z 100052c0 f i PToolsAligner.obj
 0001:00004300       ?erase@?$basic_string@DU?$char_traits@D@std@@V?$allocator@D@2@@std@@QAEAAV12@I@Z 10005300 f i PToolsAligner.obj
 0001:00004340       ?erase@?$basic_string@DU?$char_traits@D@std@@V?$allocator@D@2@@std@@QAEAAV12@II@Z 10005340 f i PToolsAligner.obj
 0001:000043e0       ?findNode@?$QMapData@HV?$QSharedDataPointer@VMoleculeData@U2@@@@@@QBEPAU?$QMapNode@HV?$QSharedDataPointer@VMoleculeData@U2@@@@@@ABH@Z 100053e0 f i PToolsAligner.obj
 0001:00004420       ?freeData@?$QVector@N@@AAEXPAU?$QTypedArrayData@N@@@Z 10005420 f i PToolsAligner.obj
 0001:00004450       ?generic_category@std@@YAABVerror_category@1@XZ 10005450 f i PToolsAligner.obj
 0001:000045f0       ?isDetached@?$QVector@N@@QBE_NXZ 100055f0 f i PToolsAligner.obj
 0001:00004620       ?isShared@RefCount@QtPrivate@@QBE_NXZ 10005620 f i PToolsAligner.obj
 0001:00004640       ?leftNode@?$QMapNode@HV?$QSharedDataPointer@VMoleculeData@U2@@@@@@QBEPAU1@XZ 10005640 f i PToolsAligner.obj
 0001:00004650       ?leftNode@?$QMapNode@HVMolecule3DModel@U2@@@@QBEPAU1@XZ 10005650 f i PToolsAligner.obj
 0001:00004660       ?leftNode@?$QMapNode@VResidueIndex@U2@@V?$QSharedDataPointer@VResidueData@U2@@@@@@QBEPAU1@XZ 10005660 f i PToolsAligner.obj
 0001:00004670       ?length@?$char_traits@D@std@@SAIPBD@Z 10005670 f i PToolsAligner.obj
 0001:00004690       ?load@?$QBasicAtomicInteger@H@@QBEHXZ 10005690 f i PToolsAligner.obj
 0001:000046a0       ?lowerBound@?$QMapNode@HV?$QSharedDataPointer@VMoleculeData@U2@@@@@@QAEPAU1@ABH@Z 100056a0 f i PToolsAligner.obj
 0001:000046d0       ?max_size@?$_Wrap_alloc@V?$allocator@D@std@@@std@@QBEIXZ 100056d0 f i PToolsAligner.obj
 0001:000046e0       ?max_size@?$allocator@D@std@@QBEIXZ 100056e0 f i PToolsAligner.obj
 0001:000046f0       ?max_size@?$allocator_traits@V?$allocator@D@std@@@std@@SAIABV?$allocator@D@2@@Z 100056f0 f i PToolsAligner.obj
 0001:00004700       ?max_size@?$basic_string@DU?$char_traits@D@std@@V?$allocator@D@2@@std@@QBEIXZ 10005700 f i PToolsAligner.obj
 0001:00004710       ?message@_Generic_error_category@std@@UBE?AV?$basic_string@DU?$char_traits@D@std@@V?$allocator@D@2@@2@H@Z 10005710 f i PToolsAligner.obj
 0001:00004790       ?message@_Iostream_error_category@std@@UBE?AV?$basic_string@DU?$char_traits@D@std@@V?$allocator@D@2@@2@H@Z 10005790 f i PToolsAligner.obj
 0001:000047e0       ?message@_System_error_category@std@@UBE?AV?$basic_string@DU?$char_traits@D@std@@V?$allocator@D@2@@2@H@Z 100057e0 f i PToolsAligner.obj
 0001:00004860       ?move@?$char_traits@D@std@@SAPADPADPBDI@Z 10005860 f i PToolsAligner.obj
 0001:00004880       ?name@_Generic_error_category@std@@UBEPBDXZ 10005880 f i PToolsAligner.obj
 0001:00004890       ?name@_Iostream_error_category@std@@UBEPBDXZ 10005890 f i PToolsAligner.obj
 0001:000048a0       ?name@_System_error_category@std@@UBEPBDXZ 100058a0 f i PToolsAligner.obj
 0001:000048b0       ?node_copy@?$QList@H@@AAEXPAUNode@1@00@Z 100058b0 f i PToolsAligner.obj
 0001:000048e0       ?node_copy@?$QList@V?$QSharedDataPointer@VAtomData@U2@@@@@@AAEXPAUNode@1@00@Z 100058e0 f i PToolsAligner.obj
 0001:00004920       ?node_destruct@?$QList@H@@AAEXPAUNode@1@0@Z 10005920 f i PToolsAligner.obj
 0001:00004930       ?node_destruct@?$QList@V?$QSharedDataPointer@VAtomData@U2@@@@@@AAEXPAUNode@1@0@Z 10005930 f i PToolsAligner.obj
 0001:00004980       ?node_destruct@?$QList@VBond@U2@@@@AAEXPAUNode@1@0@Z 10005980 f i PToolsAligner.obj
 0001:00004a40       ?qt_noop@@YAXXZ            10005a40 f i PToolsAligner.obj
 0001:00004a50       ?reallocData@?$QVector@N@@AAEXHHV?$QFlags@W4AllocationOption@QArrayData@@@@@Z 10005a50 f i PToolsAligner.obj
 0001:00004c90       ?ref@?$QBasicAtomicInteger@H@@QAE_NXZ 10005c90 f i PToolsAligner.obj
 0001:00004cb0       ?ref@RefCount@QtPrivate@@QAE_NXZ 10005cb0 f i PToolsAligner.obj
 0001:00004cd0       ?rightNode@?$QMapNode@HV?$QSharedDataPointer@VMoleculeData@U2@@@@@@QBEPAU1@XZ 10005cd0 f i PToolsAligner.obj
 0001:00004ce0       ?rightNode@?$QMapNode@HVMolecule3DModel@U2@@@@QBEPAU1@XZ 10005ce0 f i PToolsAligner.obj
 0001:00004cf0       ?rightNode@?$QMapNode@VResidueIndex@U2@@V?$QSharedDataPointer@VResidueData@U2@@@@@@QBEPAU1@XZ 10005cf0 f i PToolsAligner.obj
 0001:00004d00       ?root@?$QMapData@HV?$QSharedDataPointer@VMoleculeData@U2@@@@@@QBEPAU?$QMapNode@HV?$QSharedDataPointer@VMoleculeData@U2@@@@@@XZ 10005d00 f i PToolsAligner.obj
 0001:00004d10       ?root@?$QMapData@HVMolecule3DModel@U2@@@@QBEPAU?$QMapNode@HVMolecule3DModel@U2@@@@XZ 10005d10 f i PToolsAligner.obj
 0001:00004d20       ?root@?$QMapData@VResidueIndex@U2@@V?$QSharedDataPointer@VResidueData@U2@@@@@@QBEPAU?$QMapNode@VResidueIndex@U2@@V?$QSharedDataPointer@VResidueData@U2@@@@@@XZ 10005d20 f i PToolsAligner.obj
 0001:00004d30       ?select_on_container_copy_construction@?$_Wrap_alloc@V?$allocator@D@std@@@std@@QBE?AU12@XZ 10005d30 f i PToolsAligner.obj
 0001:00004d40       ?select_on_container_copy_construction@?$allocator@D@std@@QBE?AV12@XZ 10005d40 f i PToolsAligner.obj
 0001:00004d50       ?select_on_container_copy_construction@?$allocator_traits@V?$allocator@D@std@@@std@@SA?AV?$allocator@D@2@ABV32@@Z 10005d50 f i PToolsAligner.obj
 0001:00004d60       ?sharedNull@?$QTypedArrayData@N@@SAPAU1@XZ 10005d60 f i PToolsAligner.obj
 0001:00004d70       ?size@?$QList@H@@QBEHXZ    10005d70 f i PToolsAligner.obj
 0001:00004d80       ?size@?$QMap@VResidueIndex@U2@@V?$QSharedDataPointer@VResidueData@U2@@@@@@QBEHXZ 10005d80 f i PToolsAligner.obj
 0001:00004d90       ?size@?$basic_string@DU?$char_traits@D@std@@V?$allocator@D@2@@std@@QBEIXZ 10005d90 f i PToolsAligner.obj
 0001:00004da0       ?size@?$vector@UCoord3D@PTools@@V?$allocator@UCoord3D@PTools@@@std@@@std@@QBEIXZ 10005da0 f i PToolsAligner.obj
 0001:00004dc0       ?system_category@std@@YAABVerror_category@1@XZ 10005dc0 f i PToolsAligner.obj
 0001:00004dd0       ?t@Node@?$QList@H@@QAEAAHXZ 10005dd0 f i PToolsAligner.obj
 0001:00004de0       ?t@Node@?$QList@V?$QSharedDataPointer@VAtomData@U2@@@@@@QAEAAV?$QSharedDataPointer@VAtomData@U2@@@@XZ 10005de0 f i PToolsAligner.obj
 0001:00004df0       ?unsharableEmpty@?$QTypedArrayData@N@@SAPAU1@XZ 10005df0 f i PToolsAligner.obj
 0001:00004e10       ?validate@PToolsAligner@U2@@UAE?AVQString@@ABVStructuralAlignmentTaskSettings@2@@Z 10005e10 f   PToolsAligner.obj
 0001:00004e70       ?value@?$QMap@HV?$QSharedDataPointer@VMoleculeData@U2@@@@@@QBE?BV?$QSharedDataPointer@VMoleculeData@U2@@@@ABHABV2@@Z 10005e70 f i PToolsAligner.obj
 0001:00004ed0       ?value@error_code@std@@QBEHXZ 10005ed0 f i PToolsAligner.obj
 0001:00004ee0       ?value@error_condition@std@@QBEHXZ 10005ee0 f i PToolsAligner.obj
 0001:00004ef0       _hypot                     10005ef0 f i PToolsAligner.obj
 0001:00004f20       ??$_Move@AAPAUData@QListData@@@std@@YA$$QAPAUData@QListData@@AAPAU12@@Z 10005f20 f i PToolsPlugin.obj
 0001:00004f30       ??$qDeleteAll@V?$QList@PAVXMLTestFactory@U2@@@@@@YAXABV?$QList@PAVXMLTestFactory@U2@@@@@Z 10005f30 f i PToolsPlugin.obj
 0001:00004f70       ??$qDeleteAll@Vconst_iterator@?$QList@PAVXMLTestFactory@U2@@@@@@YAXVconst_iterator@?$QList@PAVXMLTestFactory@U2@@@@0@Z 10005f70 f i PToolsPlugin.obj
 0001:00004fa0       ??$qSwap@PAUData@QListData@@@@YAXAAPAUData@QListData@@0@Z 10005fa0 f i PToolsPlugin.obj
 0001:00004fc0       ??$qobject_cast@PAVXMLTestFormat@U2@@@@YAPAVXMLTestFormat@U2@@PAVQObject@@@Z 10005fc0 f i PToolsPlugin.obj
 0001:00004fe0       ??$swap@PAUData@QListData@@@std@@YAXAAPAUData@QListData@@0@Z 10005fe0 f i PToolsPlugin.obj
 0001:00005000       ??0?$GAutoDeleteList@VXMLTestFactory@U2@@@U2@@QAE@PAVQObject@@@Z 10006000 f i PToolsPlugin.obj
 0001:00005030       ??0?$QFlags@W4TaskFlag@U2@@@@QAE@VQFlag@@@Z 10006030 f i PToolsPlugin.obj
 0001:00005040       ??0?$QFlags@W4TaskFlag@U2@@@@QAE@W4TaskFlag@U2@@@Z 10006040 f i PToolsPlugin.obj
 0001:00005050       ??0?$QForeachContainer@V?$QList@PAVXMLTestFactory@U2@@@@@@QAE@ABV?$QList@PAVXMLTestFactory@U2@@@@@Z 10006050 f i PToolsPlugin.obj
 0001:00005090       ??0?$QList@PAVXMLTestFactory@U2@@@@QAE@$$QAV0@@Z 10006090 f i PToolsPlugin.obj
 0001:000050b0       ??0?$QList@PAVXMLTestFactory@U2@@@@QAE@ABV0@@Z 100060b0 f i PToolsPlugin.obj
 0001:00005170       ??0?$QList@PAVXMLTestFactory@U2@@@@QAE@XZ 10006170 f i PToolsPlugin.obj
 0001:00005180       ??0Gtest_PToolsAlignerTask@U2@@QAE@PAVXMLTestFormat@1@ABVQString@@PAVGTest@1@PBVGTestEnvironment@1@ABV?$QList@PAVGTest@U2@@@@ABVQDomElement@@@Z 10006180 f i PToolsPlugin.obj
 0001:00005230       ??0Gtest_PToolsAlignerTaskFactory@Gtest_PToolsAlignerTask@U2@@QAE@XZ 10006230 f i PToolsPlugin.obj
 0001:000052b0       ??0PToolsAligner@U2@@QAE@XZ 100062b0 f i PToolsPlugin.obj
 0001:000052c0       ??0PToolsAlignerFactory@U2@@QAE@XZ 100062c0 f i PToolsPlugin.obj
 0001:000052d0       ??0PToolsPlugin@U2@@QAE@XZ 100062d0 f   PToolsPlugin.obj
 0001:000054f0       ??0QFlag@@QAE@H@Z          100064f0 f i PToolsPlugin.obj
 0001:00005500       ??0const_iterator@?$QList@PAVXMLTestFactory@U2@@@@QAE@PAUNode@1@@Z 10006500 f i PToolsPlugin.obj
 0001:00005510       ??1?$GAutoDeleteList@VXMLTestFactory@U2@@@U2@@UAE@XZ 10006510 f i PToolsPlugin.obj
 0001:000055d0       ??1?$QForeachContainer@V?$QList@PAVXMLTestFactory@U2@@@@@@QAE@XZ 100065d0 f i PToolsPlugin.obj
 0001:00005600       ??1?$QList@PAVXMLTestFactory@U2@@@@QAE@XZ 10006600 f i PToolsPlugin.obj
 0001:00005630       ??1Gtest_PToolsAlignerTask@U2@@UAE@XZ 10006630 f i PToolsPlugin.obj
 0001:000056c0       ??1Gtest_PToolsAlignerTaskFactory@Gtest_PToolsAlignerTask@U2@@UAE@XZ 100066c0 f i PToolsPlugin.obj
 0001:000056d0       ??1PToolsAligner@U2@@UAE@XZ 100066d0 f i PToolsPlugin.obj
 0001:000056e0       ??1PToolsAlignerFactory@U2@@UAE@XZ 100066e0 f i PToolsPlugin.obj
 0001:000056f0       ??1PToolsPlugin@U2@@UAE@XZ 100066f0 f   PToolsPlugin.obj
 0001:00005700       ??4?$QList@PAVXMLTestFactory@U2@@@@QAEAAV0@$$QAV0@@Z 10006700 f i PToolsPlugin.obj
 0001:00005720       ??9const_iterator@?$QList@PAVXMLTestFactory@U2@@@@QBE_NABV01@@Z 10006720 f i PToolsPlugin.obj
 0001:00005740       ??BQFlag@@QBEHXZ           10006740 f i PToolsPlugin.obj
 0001:00005750       ??Dconst_iterator@?$QList@PAVXMLTestFactory@U2@@@@QBEABQAVXMLTestFactory@U2@@XZ 10006750 f i PToolsPlugin.obj
 0001:00005760       ??Econst_iterator@?$QList@PAVXMLTestFactory@U2@@@@QAEAAV01@XZ 10006760 f i PToolsPlugin.obj
 0001:00005770       ??U?$QFlags@W4TaskFlag@U2@@@@QBE?AV0@W4TaskFlag@U2@@@Z 10006770 f i PToolsPlugin.obj
 0001:00005790       ??_G?$GAutoDeleteList@VXMLTestFactory@U2@@@U2@@UAEPAXI@Z 10006790 f i PToolsPlugin.obj
 0001:00005790       ??_E?$GAutoDeleteList@VXMLTestFactory@U2@@@U2@@UAEPAXI@Z 10006790 f i PToolsPlugin.obj
 0001:000057c0       ??_EGtest_PToolsAlignerTask@U2@@UAEPAXI@Z 100067c0 f i PToolsPlugin.obj
 0001:000057c0       ??_GGtest_PToolsAlignerTask@U2@@UAEPAXI@Z 100067c0 f i PToolsPlugin.obj
 0001:00005860       ??_EGtest_PToolsAlignerTaskFactory@Gtest_PToolsAlignerTask@U2@@UAEPAXI@Z 10006860 f i PToolsPlugin.obj
 0001:00005860       ??_GGtest_PToolsAlignerTaskFactory@Gtest_PToolsAlignerTask@U2@@UAEPAXI@Z 10006860 f i PToolsPlugin.obj
 0001:00005890       ??_GPToolsAligner@U2@@UAEPAXI@Z 10006890 f i PToolsPlugin.obj
 0001:00005890       ??_EPToolsAligner@U2@@UAEPAXI@Z 10006890 f i PToolsPlugin.obj
 0001:000058c0       ??_EPToolsAlignerFactory@U2@@UAEPAXI@Z 100068c0 f i PToolsPlugin.obj
 0001:000058c0       ??_GPToolsAlignerFactory@U2@@UAEPAXI@Z 100068c0 f i PToolsPlugin.obj
 0001:000058f0       ??_GPToolsPlugin@U2@@UAEPAXI@Z 100068f0 f i PToolsPlugin.obj
 0001:000058f0       ??_EPToolsPlugin@U2@@UAEPAXI@Z 100068f0 f i PToolsPlugin.obj
 0001:00005920       ?append@?$QList@PAVXMLTestFactory@U2@@@@QAEXABQAVXMLTestFactory@U2@@@Z 10006920 f i PToolsPlugin.obj
 0001:000059b0       ?begin@?$QList@PAVXMLTestFactory@U2@@@@QBE?AVconst_iterator@1@XZ 100069b0 f i PToolsPlugin.obj
 0001:000059d0       ?create@PToolsAlignerFactory@U2@@UAEPAVStructuralAlignmentAlgorithm@2@XZ 100069d0 f i PToolsPlugin.obj
 0001:000059f0       ?createFactory@Gtest_PToolsAlignerTask@U2@@SAPAVXMLTestFactory@2@XZ 100069f0 f i PToolsPlugin.obj
 0001:00005a90       ?createTest@Gtest_PToolsAlignerTaskFactory@Gtest_PToolsAlignerTask@U2@@UAEPAVGTest@3@PAVXMLTestFormat@3@ABVQString@@PAV43@PBVGTestEnvironment@3@ABV?$QList@PAVGTest@U2@@@@ABVQDomElement@@@Z 10006a90 f i PToolsPlugin.obj
 0001:00005b10       ?createTestFactories@StructualAlignerTests@U2@@SA?AV?$QList@PAVXMLTestFactory@U2@@@@XZ 10006b10 f   PToolsPlugin.obj
 0001:00005b80       ?dealloc@?$QList@PAVXMLTestFactory@U2@@@@AAEXPAUData@QListData@@@Z 10006b80 f i PToolsPlugin.obj
 0001:00005ba0       ?detach_helper_grow@?$QList@PAVXMLTestFactory@U2@@@@AAEPAUNode@1@HH@Z 10006ba0 f i PToolsPlugin.obj
 0001:00005cb0       ?end@?$QList@PAVXMLTestFactory@U2@@@@QBE?AVconst_iterator@1@XZ 10006cb0 f i PToolsPlugin.obj
 0001:00005cd0       ?node_construct@?$QList@PAVXMLTestFactory@U2@@@@AAEXPAUNode@1@ABQAVXMLTestFactory@U2@@@Z 10006cd0 f i PToolsPlugin.obj
 0001:00005cf0       ?node_copy@?$QList@PAVXMLTestFactory@U2@@@@AAEXPAUNode@1@00@Z 10006cf0 f i PToolsPlugin.obj
 0001:00005d20       ?node_destruct@?$QList@PAVXMLTestFactory@U2@@@@AAEXPAUNode@1@0@Z 10006d20 f i PToolsPlugin.obj
 0001:00005d30       ?node_destruct@?$QList@PAVXMLTestFactory@U2@@@@AAEXPAUNode@1@@Z 10006d30 f i PToolsPlugin.obj
 0001:00005d40       ?t@Node@?$QList@PAVXMLTestFactory@U2@@@@QAEAAPAVXMLTestFactory@U2@@XZ 10006d40 f i PToolsPlugin.obj
 0001:00005d50       ?tr@PToolsPlugin@U2@@SA?AVQString@@PBD0H@Z 10006d50 f i PToolsPlugin.obj
 0001:00005d80       _ugene_plugin_init         10006d80 f   PToolsPlugin.obj
 0001:00005da0       ??$getContext@VBioStruct3DObject@U2@@@GTest@U2@@SAPAVBioStruct3DObject@1@PBV01@ABVQString@@@Z 10006da0 f i PToolsTests.obj
 0001:00005dc0       ??$qobject_cast@PAVBioStruct3DObject@U2@@@@YAPAVBioStruct3DObject@U2@@PAVQObject@@@Z 10006dc0 f i PToolsTests.obj
 0001:00005de0       ??0?$QForeachContainer@VQStringList@@@@QAE@ABVQStringList@@@Z 10006de0 f i PToolsTests.obj
 0001:00005e20       ??0?$QList@H@@QAE@$$QAV0@@Z 10006e20 f i PToolsTests.obj
 0001:00005e40       ??0?$QList@H@@QAE@XZ       10006e40 f i PToolsTests.obj
 0001:00005e50       ??0?$QList@VQString@@@@QAE@ABV0@@Z 10006e50 f i PToolsTests.obj
 0001:00005f10       ??0QStringList@@QAE@ABV0@@Z 10006f10 f i PToolsTests.obj
 0001:00005f30       ??0const_iterator@?$QList@VQString@@@@QAE@PAUNode@1@@Z 10006f30 f i PToolsTests.obj
 0001:00005f40       ??0const_iterator@?$QMap@HV?$QHash@HV?$QSharedDataPointer@VAtomData@U2@@@@@@@@QAE@PBU?$QMapNode@HV?$QHash@HV?$QSharedDataPointer@VAtomData@U2@@@@@@@@@Z 10006f40 f i PToolsTests.obj
 0001:00005f50       ??0const_iterator@?$QMap@HV?$QSharedDataPointer@VMoleculeData@U2@@@@@@QAE@PBU?$QMapNode@HV?$QSharedDataPointer@VMoleculeData@U2@@@@@@@Z 10006f50 f i PToolsTests.obj
 0001:00005f60       ??0iterator@?$QList@H@@QAE@PAUNode@1@@Z 10006f60 f i PToolsTests.obj
 0001:00005f70       ??1?$QForeachContainer@VQStringList@@@@QAE@XZ 10006f70 f i PToolsTests.obj
 0001:00005f80       ??1?$QList@VQString@@@@QAE@XZ 10006f80 f i PToolsTests.obj
 0001:00005fe0       ??1QStringList@@QAE@XZ     10006fe0 f i PToolsTests.obj
 0001:00005ff0       ??9const_iterator@?$QList@VQString@@@@QBE_NABV01@@Z 10006ff0 f i PToolsTests.obj
 0001:00006010       ??9const_iterator@?$QMap@HV?$QHash@HV?$QSharedDataPointer@VAtomData@U2@@@@@@@@QBE_NABV01@@Z 10007010 f i PToolsTests.obj
 0001:00006030       ??9const_iterator@?$QMap@HV?$QSharedDataPointer@VMoleculeData@U2@@@@@@QBE_NABV01@@Z 10007030 f i PToolsTests.obj
 0001:00006050       ??Dconst_iterator@?$QList@VQString@@@@QBEABVQString@@XZ 10007050 f i PToolsTests.obj
 0001:00006060       ??Diterator@?$QList@H@@QBEAAHXZ 10007060 f i PToolsTests.obj
 0001:00006070       ??Econst_iterator@?$QList@VQString@@@@QAEAAV01@XZ 10007070 f i PToolsTests.obj
 0001:00006080       ??Econst_iterator@?$QMap@HV?$QHash@HV?$QSharedDataPointer@VAtomData@U2@@@@@@@@QAEAAV01@XZ 10007080 f i PToolsTests.obj
 0001:000060a0       ??Econst_iterator@?$QMap@HV?$QSharedDataPointer@VMoleculeData@U2@@@@@@QAEAAV01@XZ 100070a0 f i PToolsTests.obj
 0001:000060c0       ??H@YA?BVQString@@ABV0@0@Z 100070c0 f i PToolsTests.obj
 0001:00006130       ??H@YA?BVQString@@ABV0@PBD@Z 10007130 f i PToolsTests.obj
 0001:000061d0       ??H@YA?BVQString@@PBDABV0@@Z 100071d0 f i PToolsTests.obj
 0001:00006240       ??_GQString@@QAEPAXI@Z     10007240 f i PToolsTests.obj
 0001:00006400       ?append@?$QList@H@@QAEXABH@Z 10007400 f i PToolsTests.obj
 0001:00006490       ?begin@?$QList@H@@QAE?AViterator@1@XZ 10007490 f i PToolsTests.obj
 0001:000064d0       ?begin@?$QList@VQString@@@@QBE?AVconst_iterator@1@XZ 100074d0 f i PToolsTests.obj
 0001:000064f0       ?begin@?$QMap@HV?$QHash@HV?$QSharedDataPointer@VAtomData@U2@@@@@@@@QBE?AVconst_iterator@1@XZ 100074f0 f i PToolsTests.obj
 0001:00006510       ?begin@?$QMap@HV?$QSharedDataPointer@VMoleculeData@U2@@@@@@QBE?AVconst_iterator@1@XZ 10007510 f i PToolsTests.obj
 0001:00006530       ?begin@?$QMapData@HV?$QHash@HV?$QSharedDataPointer@VAtomData@U2@@@@@@@@QAEPAU?$QMapNode@HV?$QHash@HV?$QSharedDataPointer@VAtomData@U2@@@@@@@@XZ 10007530 f i PToolsTests.obj
 0001:00006540       ?begin@?$QMapData@HV?$QSharedDataPointer@VMoleculeData@U2@@@@@@QAEPAU?$QMapNode@HV?$QSharedDataPointer@VMoleculeData@U2@@@@@@XZ 10007540 f i PToolsTests.obj
 0001:00006550       ?dealloc@?$QList@VQString@@@@AAEXPAUData@QListData@@@Z 10007550 f i PToolsTests.obj
 0001:00006590       ?detach@?$QList@H@@QAEXXZ  10007590 f i PToolsTests.obj
 0001:000065b0       ?detach_helper@?$QList@H@@AAEXH@Z 100075b0 f i PToolsTests.obj
 0001:00006680       ?detach_helper@?$QList@H@@AAEXXZ 10007680 f i PToolsTests.obj
 0001:00006690       ?detach_helper_grow@?$QList@H@@AAEPAUNode@1@HH@Z 10007690 f i PToolsTests.obj
 0001:000067a0       ?end@?$QList@VQString@@@@QBE?AVconst_iterator@1@XZ 100077a0 f i PToolsTests.obj
 0001:000067c0       ?end@?$QMap@HV?$QHash@HV?$QSharedDataPointer@VAtomData@U2@@@@@@@@QBE?AVconst_iterator@1@XZ 100077c0 f i PToolsTests.obj
 0001:000067e0       ?end@?$QMap@HV?$QSharedDataPointer@VMoleculeData@U2@@@@@@QBE?AVconst_iterator@1@XZ 100077e0 f i PToolsTests.obj
 0001:00006800       ?end@?$QMapData@HV?$QHash@HV?$QSharedDataPointer@VAtomData@U2@@@@@@@@QAEPAU?$QMapNode@HV?$QHash@HV?$QSharedDataPointer@VAtomData@U2@@@@@@@@XZ 10007800 f i PToolsTests.obj
 0001:00006810       ?end@?$QMapData@HV?$QSharedDataPointer@VMoleculeData@U2@@@@@@QAEPAU?$QMapNode@HV?$QSharedDataPointer@VMoleculeData@U2@@@@@@XZ 10007810 f i PToolsTests.obj
 0001:00006820       ?fabs@@YAMM@Z              10007820 f i PToolsTests.obj
 0001:00006850       ?first@?$QList@H@@QAEAAHXZ 10007850 f i PToolsTests.obj
 0001:00006880       ?init@Gtest_PToolsAlignerTask@U2@@QAEXPAVXMLTestFormat@2@ABVQDomElement@@@Z 10007880 f   PToolsTests.obj
 0001:00006e00       ?key@const_iterator@?$QMap@HV?$QHash@HV?$QSharedDataPointer@VAtomData@U2@@@@@@@@QBEABHXZ 10007e00 f i PToolsTests.obj
 0001:00006e10       ?key@const_iterator@?$QMap@HV?$QSharedDataPointer@VMoleculeData@U2@@@@@@QBEABHXZ 10007e10 f i PToolsTests.obj
 0001:00006e20       ?keys@?$QMap@HV?$QHash@HV?$QSharedDataPointer@VAtomData@U2@@@@@@@@QBE?AV?$QList@H@@XZ 10007e20 f i PToolsTests.obj
 0001:00006ee0       ?keys@?$QMap@HV?$QSharedDataPointer@VMoleculeData@U2@@@@@@QBE?AV?$QList@H@@XZ 10007ee0 f i PToolsTests.obj
 0001:00006fa0       ?nextNode@?$QMapNode@HV?$QHash@HV?$QSharedDataPointer@VAtomData@U2@@@@@@@@QBEPBU1@XZ 10007fa0 f i PToolsTests.obj
 0001:00006fb0       ?nextNode@?$QMapNode@HV?$QSharedDataPointer@VMoleculeData@U2@@@@@@QBEPBU1@XZ 10007fb0 f i PToolsTests.obj
 0001:00006fc0       ?node_construct@?$QList@H@@AAEXPAUNode@1@ABH@Z 10007fc0 f i PToolsTests.obj
 0001:00006fe0       ?node_copy@?$QList@VQString@@@@AAEXPAUNode@1@00@Z 10007fe0 f i PToolsTests.obj
 0001:00007080       ?node_destruct@?$QList@H@@AAEXPAUNode@1@@Z 10008080 f i PToolsTests.obj
 0001:00007090       ?node_destruct@?$QList@VQString@@@@AAEXPAUNode@1@0@Z 10008090 f i PToolsTests.obj
 0001:000070c0       ?report@Gtest_PToolsAlignerTask@U2@@UAE?AW4ReportResult@Task@2@XZ 100080c0 f   PToolsTests.obj
 0001:00007250       ?reserve@?$QList@H@@QAEXH@Z 10008250 f i PToolsTests.obj
 0001:00007280       ?root@?$QMapData@HV?$QHash@HV?$QSharedDataPointer@VAtomData@U2@@@@@@@@QBEPAU?$QMapNode@HV?$QHash@HV?$QSharedDataPointer@VAtomData@U2@@@@@@@@XZ 10008280 f i PToolsTests.obj
 0001:00007290       ?run@Gtest_PToolsAlignerTask@U2@@UAEXXZ 10008290 f   PToolsTests.obj
 0001:00007610       ?size@?$QList@VQString@@@@QBEHXZ 10008610 f i PToolsTests.obj
 0001:00007620       ?size@?$QMap@HV?$QHash@HV?$QSharedDataPointer@VAtomData@U2@@@@@@@@QBEHXZ 10008620 f i PToolsTests.obj
 0001:00007630       ?size@?$QMap@HV?$QSharedDataPointer@VMoleculeData@U2@@@@@@QBEHXZ 10008630 f i PToolsTests.obj
 0001:00007640       ?t@Node@?$QList@VQString@@@@QAEAAVQString@@XZ 10008640 f i PToolsTests.obj
 0001:00007650       _fabsf                     10008650 f i PToolsTests.obj
 0001:00007680       ??4Coord3D@PTools@@QAEAAU01@ABU01@@Z 10008680 f i atom.obj
 0001:000076b0       ??HPTools@@YA?AUCoord3D@0@ABU10@0@Z 100086b0 f i atom.obj
 0001:000076f0       ?GetCoords@Atom@PTools@@QBE?AUCoord3D@2@XZ 100086f0 f   atom.obj
 0001:00007720       ?Translate@Atom@PTools@@QAEXABUCoord3D@2@@Z 10008720 f   atom.obj
 0001:00007770       ??$?0AAPAIAAPAIX@?$pair@PAIPAI@std@@QAE@AAPAI0@Z 10008770 f i atomselection.obj
 0001:00007790       ??$?8II@std@@YA_NABV?$allocator@I@0@0@Z 10008790 f i atomselection.obj
 0001:000077a0       ??$?8V?$allocator@I@std@@V01@@std@@YA_NABU?$_Wrap_alloc@V?$allocator@I@std@@@0@0@Z 100087a0 f i atomselection.obj
 0001:000077b0       ??$?9V?$allocator@I@std@@V01@@std@@YA_NABU?$_Wrap_alloc@V?$allocator@I@std@@@0@0@Z 100087b0 f i atomselection.obj
 0001:000077c0       ??$?RAAIAAI@?$equal_to@X@std@@QBE_NAAI0@Z 100087c0 f i atomselection.obj
 0001:000077e0       ??$?RAAIAAI@?$less@X@std@@QBE_NAAI0@Z 100087e0 f i atomselection.obj
 0001:00007800       ??$?RAAIABI@?$less@X@std@@QBE_NAAIABI@Z 10008800 f i atomselection.obj
 0001:00007820       ??$?RABIAAI@?$less@X@std@@QBE_NABIAAI@Z 10008820 f i atomselection.obj
 0001:00007840       ??$?RABIABI@?$less@X@std@@QBE_NABI0@Z 10008840 f i atomselection.obj
 0001:00007860       ??$_Adjust_heap@PAIHIU?$less@X@std@@@std@@YAXPAIHH$$QAIU?$less@X@0@@Z 10008860 f i atomselection.obj
 0001:000078f0       ??$_Allocate@I@std@@YAPAIIPAI@Z 100088f0 f i atomselection.obj
 0001:00007920       ??$_Copy_impl@PAIPAI@std@@YAPAIPAI00@Z 10008920 f i atomselection.obj
 0001:00007950       ??$_Copy_impl@PAIPAI@std@@YAPAIPAI00U_Scalar_ptr_iterator_tag@0@@Z 10008950 f i atomselection.obj
 0001:00007980       ??$_Copy_impl@PAIV?$back_insert_iterator@V?$vector@IV?$allocator@I@std@@@std@@@std@@@std@@YA?AV?$back_insert_iterator@V?$vector@IV?$allocator@I@std@@@std@@@0@PAI0V10@@Z 10008980 f i atomselection.obj
 0001:000079a0       ??$_Copy_impl@PAIV?$back_insert_iterator@V?$vector@IV?$allocator@I@std@@@std@@@std@@@std@@YA?AV?$back_insert_iterator@V?$vector@IV?$allocator@I@std@@@std@@@0@PAI0V10@U_Nonscalar_ptr_iterator_tag@0@@Z 100089a0 f i atomselection.obj
 0001:00007a20       ??$_Destroy_range@U?$_Wrap_alloc@V?$allocator@I@std@@@std@@@std@@YAXPAI0AAU?$_Wrap_alloc@V?$allocator@I@std@@@0@@Z 10008a20 f i atomselection.obj
 0001:00007a30       ??$_Destroy_range@U?$_Wrap_alloc@V?$allocator@I@std@@@std@@@std@@YAXPAI0AAU?$_Wrap_alloc@V?$allocator@I@std@@@0@U_Scalar_ptr_iterator_tag@0@@Z 10008a30 f i atomselection.obj
 0001:00007a40       ??$_Destroy_range@U?$_Wrap_alloc@V?$allocator@UCoord3D@PTools@@@std@@@std@@@std@@YAXPAUCoord3D@PTools@@0AAU?$_Wrap_alloc@V?$allocator@UCoord3D@PTools@@@std@@@0@@Z 10008a40 f i atomselection.obj
 0001:00007a50       ??$_Destroy_range@U?$_Wrap_alloc@V?$allocator@UCoord3D@PTools@@@std@@@std@@@std@@YAXPAUCoord3D@PTools@@0AAU?$_Wrap_alloc@V?$allocator@UCoord3D@PTools@@@std@@@0@U_Nonscalar_ptr_iterator_tag@0@@Z 10008a50 f i atomselection.obj
 0001:00007a60       ??$_Destroy_range@U?$_Wrap_alloc@V?$allocator@VAtomproperty@PTools@@@std@@@std@@@std@@YAXPAVAtomproperty@PTools@@0AAU?$_Wrap_alloc@V?$allocator@VAtomproperty@PTools@@@std@@@0@@Z 10008a60 f i atomselection.obj
 0001:00007a90       ??$_Destroy_range@U?$_Wrap_alloc@V?$allocator@VAtomproperty@PTools@@@std@@@std@@@std@@YAXPAVAtomproperty@PTools@@0AAU?$_Wrap_alloc@V?$allocator@VAtomproperty@PTools@@@std@@@0@U_Nonscalar_ptr_iterator_tag@0@@Z 10008a90 f i atomselection.obj
 0001:00007ac0       ??$_Dist_type@PAI@std@@YAPAHPAI@Z 10008ac0 f i atomselection.obj
 0001:00007ad0       ??$_Insertion_sort1@PAIU?$less@X@std@@I@std@@YAXPAI0U?$less@X@0@0@Z 10008ad0 f i atomselection.obj
 0001:00007b50       ??$_Insertion_sort@PAIU?$less@X@std@@@std@@YAXPAI0U?$less@X@0@@Z 10008b50 f i atomselection.obj
 0001:00007b70       ??$_Iter_cat@V?$_Vector_iterator@V?$_Vector_val@U?$_Simple_types@I@std@@@std@@@std@@@std@@YA?AUrandom_access_iterator_tag@0@ABV?$_Vector_iterator@V?$_Vector_val@U?$_Simple_types@I@std@@@std@@@0@@Z 10008b70 f i atomselection.obj
 0001:00007b80       ??$_Make_heap@PAIHIU?$less@X@std@@@std@@YAXPAI0U?$less@X@0@PAH0@Z 10008b80 f i atomselection.obj
 0001:00007c30       ??$_Med3@PAIU?$less@X@std@@@std@@YAXPAI00U?$less@X@0@@Z 10008c30 f i atomselection.obj
 0001:00007c70       ??$_Median@PAIU?$less@X@std@@@std@@YAXPAI00U?$less@X@0@@Z 10008c70 f i atomselection.obj
 0001:00007da0       ??$_Move@AAI@std@@YA$$QAIAAI@Z 10008da0 f i atomselection.obj
 0001:00007db0       ??$_Move@AAPAI@std@@YA$$QAPAIAAPAI@Z 10008db0 f i atomselection.obj
 0001:00007dc0       ??$_Move_backward@PAIPAI@std@@YAPAIPAI00@Z 10008dc0 f i atomselection.obj
 0001:00007df0       ??$_Move_backward@PAIPAI@std@@YAPAIPAI00U_Scalar_ptr_iterator_tag@0@@Z 10008df0 f i atomselection.obj
 0001:00007e20       ??$_Pop_heap@PAIHIU?$less@X@std@@@std@@YAXPAI00$$QAIU?$less@X@0@PAH@Z 10008e20 f i atomselection.obj
 0001:00007e50       ??$_Pop_heap@PAIU?$less@X@std@@@std@@YAXPAI0U?$less@X@0@@Z 10008e50 f i atomselection.obj
 0001:00007e90       ??$_Pop_heap_0@PAIIU?$less@X@std@@@std@@YAXPAI0U?$less@X@0@0@Z 10008e90 f i atomselection.obj
 0001:00007ed0       ??$_Ptr_cat@II@std@@YA?AU_Scalar_ptr_iterator_tag@0@PAI0@Z 10008ed0 f i atomselection.obj
 0001:00007ee0       ??$_Ptr_cat@PAIV?$back_insert_iterator@V?$vector@IV?$allocator@I@std@@@std@@@std@@@std@@YA?AU_Nonscalar_ptr_iterator_tag@0@AAPAIAAV?$back_insert_iterator@V?$vector@IV?$allocator@I@std@@@std@@@0@@Z 10008ee0 f i atomselection.obj
 0001:00007ef0       ??$_Ptr_cat@UCoord3D@PTools@@U12@@std@@YA?AU_Nonscalar_ptr_iterator_tag@0@PAUCoord3D@PTools@@0@Z 10008ef0 f i atomselection.obj
 0001:00007f00       ??$_Ptr_cat@VAtomproperty@PTools@@V12@@std@@YA?AU_Nonscalar_ptr_iterator_tag@0@PAVAtomproperty@PTools@@0@Z 10008f00 f i atomselection.obj
 0001:00007f10       ??$_Push_heap@PAIHIU?$less@X@std@@@std@@YAXPAIHH$$QAIU?$less@X@0@@Z 10008f10 f i atomselection.obj
 0001:00007f60       ??$_Rechecked@PAIPAI@std@@YAAAPAIAAPAIPAI@Z 10008f60 f i atomselection.obj
 0001:00007f70       ??$_Rechecked@V?$back_insert_iterator@V?$vector@IV?$allocator@I@std@@@std@@@std@@V12@@std@@YAAAV?$back_insert_iterator@V?$vector@IV?$allocator@I@std@@@std@@@0@AAV10@V10@@Z 10008f70 f i atomselection.obj
 0001:00007f80       ??$_Set_difference@PAIPBIV?$back_insert_iterator@V?$vector@IV?$allocator@I@std@@@std@@@std@@U?$less@X@2@@std@@YA?AV?$back_insert_iterator@V?$vector@IV?$allocator@I@std@@@std@@@0@PAI0PBI1V10@U?$less@X@0@@Z 10008f80 f i atomselection.obj
 0001:00008040       ??$_Set_intersection@PBIPBIV?$back_insert_iterator@V?$vector@IV?$allocator@I@std@@@std@@@std@@U?$less@X@2@@std@@YA?AV?$back_insert_iterator@V?$vector@IV?$allocator@I@std@@@std@@@0@PBI000V10@U?$less@X@0@@Z 10009040 f i atomselection.obj
 0001:000080f0       ??$_Set_union@PAIPAIV?$back_insert_iterator@V?$vector@IV?$allocator@I@std@@@std@@@std@@U?$less@X@2@@std@@YA?AV?$back_insert_iterator@V?$vector@IV?$allocator@I@std@@@std@@@0@PAI000V10@U?$less@X@0@@Z 100090f0 f i atomselection.obj
 0001:00008280       ??$_Sort@PAIHU?$less@X@std@@@std@@YAXPAI0HU?$less@X@0@@Z 10009280 f i atomselection.obj
 0001:00008360       ??$_Sort_heap@PAIU?$less@X@std@@@std@@YAXPAI0U?$less@X@0@@Z 10009360 f i atomselection.obj
 0001:000083c0       ??$_Swap_adl@PAI@std@@YAXAAPAI0@Z 100093c0 f i atomselection.obj
 0001:000083e0       ??$_Ucopy@PAI@?$vector@IV?$allocator@I@std@@@std@@IAEPAIPAI00@Z 100093e0 f i atomselection.obj
 0001:00008410       ??$_Umove@PAI@?$vector@IV?$allocator@I@std@@@std@@IAEPAIPAI00@Z 10009410 f i atomselection.obj
 0001:00008440       ??$_Unchecked@PAI@std@@YAPAIPAI@Z 10009440 f i atomselection.obj
 0001:00008450       ??$_Unchecked@V?$_Vector_val@U?$_Simple_types@I@std@@@std@@@std@@YAPAIV?$_Vector_iterator@V?$_Vector_val@U?$_Simple_types@I@std@@@std@@@0@@Z 10009450 f i atomselection.obj
 0001:00008460       ??$_Unchecked@V?$_Vector_val@U?$_Simple_types@I@std@@@std@@@std@@YAPBIV?$_Vector_const_iterator@V?$_Vector_val@U?$_Simple_types@I@std@@@std@@@0@@Z 10009460 f i atomselection.obj
 0001:00008470       ??$_Unchecked@V?$back_insert_iterator@V?$vector@IV?$allocator@I@std@@@std@@@std@@@std@@YA?AV?$back_insert_iterator@V?$vector@IV?$allocator@I@std@@@std@@@0@V10@@Z 10009470 f i atomselection.obj
 0001:00008480       ??$_Unguarded_partition@PAIU?$less@X@std@@@std@@YA?AU?$pair@PAIPAI@0@PAI0U?$less@X@0@@Z 10009480 f i atomselection.obj
 0001:00008600       ??$_Uninit_copy@II@std@@YAPAIPAI00AAU?$_Wrap_alloc@V?$allocator@I@std@@@0@U_Scalar_ptr_iterator_tag@0@@Z 10009600 f i atomselection.obj
 0001:00008630       ??$_Uninit_copy@PAIPAIU?$_Wrap_alloc@V?$allocator@I@std@@@std@@@std@@YAPAIPAI00AAU?$_Wrap_alloc@V?$allocator@I@std@@@0@@Z 10009630 f i atomselection.obj
 0001:00008660       ??$_Uninit_move@III@std@@YAPAIPAI00AAU?$_Wrap_alloc@V?$allocator@I@std@@@0@0U_Scalar_ptr_iterator_tag@0@@Z 10009660 f i atomselection.obj
 0001:00008690       ??$_Uninit_move@PAIPAIU?$_Wrap_alloc@V?$allocator@I@std@@@std@@@std@@YAPAIPAI00AAU?$_Wrap_alloc@V?$allocator@I@std@@@0@@Z 10009690 f i atomselection.obj
 0001:000086c0       ??$_Uninitialized_copy@PAIPAIU?$_Wrap_alloc@V?$allocator@I@std@@@std@@@std@@YAPAIPAI00AAU?$_Wrap_alloc@V?$allocator@I@std@@@0@@Z 100096c0 f i atomselection.obj
 0001:000086f0       ??$_Uninitialized_move@PAIPAIU?$_Wrap_alloc@V?$allocator@I@std@@@std@@@std@@YAPAIPAI00AAU?$_Wrap_alloc@V?$allocator@I@std@@@0@@Z 100096f0 f i atomselection.obj
 0001:00008720       ??$_Unique_copy@PAIV?$back_insert_iterator@V?$vector@IV?$allocator@I@std@@@std@@@std@@U?$equal_to@X@2@@std@@YA?AV?$back_insert_iterator@V?$vector@IV?$allocator@I@std@@@std@@@0@PAI0V10@U?$equal_to@X@0@Uforward_iterator_tag@0@@Z 10009720 f i atomselection.obj
 0001:000087c0       ??$_Val_type@PAI@std@@YAPAIPAI@Z 100097c0 f i atomselection.obj
 0001:000087d0       ??$addressof@$$CBI@std@@YAPBIABI@Z 100097d0 f i atomselection.obj
 0001:000087e0       ??$addressof@V?$vector@IV?$allocator@I@std@@@std@@@std@@YAPAV?$vector@IV?$allocator@I@std@@@0@AAV10@@Z 100097e0 f i atomselection.obj
 0001:000087f0       ??$back_inserter@V?$vector@IV?$allocator@I@std@@@std@@@std@@YA?AV?$back_insert_iterator@V?$vector@IV?$allocator@I@std@@@std@@@0@AAV?$vector@IV?$allocator@I@std@@@0@@Z 100097f0 f i atomselection.obj
 0001:00008800       ??$construct@IAAI@?$_Wrap_alloc@V?$allocator@I@std@@@std@@QAEXPAIAAI@Z 10009800 f i atomselection.obj
 0001:00008820       ??$construct@IAAI@?$allocator@I@std@@QAEXPAIAAI@Z 10009820 f i atomselection.obj
 0001:00008840       ??$construct@IAAI@?$allocator_traits@V?$allocator@I@std@@@std@@SAXAAV?$allocator@I@1@PAIAAI@Z 10009840 f i atomselection.obj
 0001:00008860       ??$construct@IABI@?$_Wrap_alloc@V?$allocator@I@std@@@std@@QAEXPAIABI@Z 10009860 f i atomselection.obj
 0001:00008880       ??$construct@IABI@?$allocator_traits@V?$allocator@I@std@@@std@@SAXAAV?$allocator@I@1@PAIABI@Z 10009880 f i atomselection.obj
 0001:000088a0       ??$copy@PAIV?$back_insert_iterator@V?$vector@IV?$allocator@I@std@@@std@@@std@@@std@@YA?AV?$back_insert_iterator@V?$vector@IV?$allocator@I@std@@@std@@@0@PAI0V10@@Z 100098a0 f i atomselection.obj
 0001:000088d0       ??$destroy@UCoord3D@PTools@@@?$_Wrap_alloc@V?$allocator@UCoord3D@PTools@@@std@@@std@@QAEXPAUCoord3D@PTools@@@Z 100098d0 f i atomselection.obj
 0001:000088e0       ??$destroy@UCoord3D@PTools@@@?$allocator@UCoord3D@PTools@@@std@@QAEXPAUCoord3D@PTools@@@Z 100098e0 f i atomselection.obj
 0001:000088f0       ??$destroy@UCoord3D@PTools@@@?$allocator_traits@V?$allocator@UCoord3D@PTools@@@std@@@std@@SAXAAV?$allocator@UCoord3D@PTools@@@1@PAUCoord3D@PTools@@@Z 100098f0 f i atomselection.obj
 0001:00008900       ??$destroy@VAtomproperty@PTools@@@?$_Wrap_alloc@V?$allocator@VAtomproperty@PTools@@@std@@@std@@QAEXPAVAtomproperty@PTools@@@Z 10009900 f i atomselection.obj
 0001:00008910       ??$destroy@VAtomproperty@PTools@@@?$allocator@VAtomproperty@PTools@@@std@@QAEXPAVAtomproperty@PTools@@@Z 10009910 f i atomselection.obj
 0001:00008920       ??$destroy@VAtomproperty@PTools@@@?$allocator_traits@V?$allocator@VAtomproperty@PTools@@@std@@@std@@SAXAAV?$allocator@VAtomproperty@PTools@@@1@PAVAtomproperty@PTools@@@Z 10009920 f i atomselection.obj
 0001:00008930       ??$forward@AAI@std@@YAAAIAAI@Z 10009930 f i atomselection.obj
 0001:00008940       ??$forward@AAPAI@std@@YAAAPAIAAPAI@Z 10009940 f i atomselection.obj
 0001:00008950       ??$forward@ABI@std@@YAABIABI@Z 10009950 f i atomselection.obj
 0001:00008960       ??$iter_swap@PAIPAI@std@@YAXPAI0@Z 10009960 f i atomselection.obj
 0001:00008980       ??$make_heap@PAIU?$less@X@std@@@std@@YAXPAI0U?$less@X@0@@Z 10009980 f i atomselection.obj
 0001:000089b0       ??$set_difference@V?$_Vector_iterator@V?$_Vector_val@U?$_Simple_types@I@std@@@std@@@std@@V?$_Vector_const_iterator@V?$_Vector_val@U?$_Simple_types@I@std@@@std@@@2@V?$back_insert_iterator@V?$vector@IV?$allocator@I@std@@@std@@@2@@std@@YA?AV?$back_insert_iterator@V?$vector@IV?$allocator@I@std@@@std@@@0@V?$_Vector_iterator@V?$_Vector_val@U?$_Simple_types@I@std@@@std@@@0@0V?$_Vector_const_iterator@V?$_Vector_val@U?$_Simple_types@I@std@@@std@@@0@1V10@@Z 100099b0 f i atomselection.obj
 0001:000089e0       ??$set_difference@V?$_Vector_iterator@V?$_Vector_val@U?$_Simple_types@I@std@@@std@@@std@@V?$_Vector_const_iterator@V?$_Vector_val@U?$_Simple_types@I@std@@@std@@@2@V?$back_insert_iterator@V?$vector@IV?$allocator@I@std@@@std@@@2@U?$less@X@2@@std@@YA?AV?$back_insert_iterator@V?$vector@IV?$allocator@I@std@@@std@@@0@V?$_Vector_iterator@V?$_Vector_val@U?$_Simple_types@I@std@@@std@@@0@0V?$_Vector_const_iterator@V?$_Vector_val@U?$_Simple_types@I@std@@@std@@@0@1V10@U?$less@X@0@@Z 100099e0 f i atomselection.obj
 0001:00008a10       ??$set_intersection@V?$_Vector_const_iterator@V?$_Vector_val@U?$_Simple_types@I@std@@@std@@@std@@V12@V?$back_insert_iterator@V?$vector@IV?$allocator@I@std@@@std@@@2@@std@@YA?AV?$back_insert_iterator@V?$vector@IV?$allocator@I@std@@@std@@@0@V?$_Vector_const_iterator@V?$_Vector_val@U?$_Simple_types@I@std@@@std@@@0@000V10@@Z 10009a10 f i atomselection.obj
 0001:00008a40       ??$set_intersection@V?$_Vector_const_iterator@V?$_Vector_val@U?$_Simple_types@I@std@@@std@@@std@@V12@V?$back_insert_iterator@V?$vector@IV?$allocator@I@std@@@std@@@2@U?$less@X@2@@std@@YA?AV?$back_insert_iterator@V?$vector@IV?$allocator@I@std@@@std@@@0@V?$_Vector_const_iterator@V?$_Vector_val@U?$_Simple_types@I@std@@@std@@@0@000V10@U?$less@X@0@@Z 10009a40 f i atomselection.obj
 0001:00008a70       ??$set_union@V?$_Vector_iterator@V?$_Vector_val@U?$_Simple_types@I@std@@@std@@@std@@V12@V?$back_insert_iterator@V?$vector@IV?$allocator@I@std@@@std@@@2@@std@@YA?AV?$back_insert_iterator@V?$vector@IV?$allocator@I@std@@@std@@@0@V?$_Vector_iterator@V?$_Vector_val@U?$_Simple_types@I@std@@@std@@@0@000V10@@Z 10009a70 f i atomselection.obj
 0001:00008aa0       ??$set_union@V?$_Vector_iterator@V?$_Vector_val@U?$_Simple_types@I@std@@@std@@@std@@V12@V?$back_insert_iterator@V?$vector@IV?$allocator@I@std@@@std@@@2@U?$less@X@2@@std@@YA?AV?$back_insert_iterator@V?$vector@IV?$allocator@I@std@@@std@@@0@V?$_Vector_iterator@V?$_Vector_val@U?$_Simple_types@I@std@@@std@@@0@000V10@U?$less@X@0@@Z 10009aa0 f i atomselection.obj
 0001:00008ad0       ??$sort@V?$_Vector_iterator@V?$_Vector_val@U?$_Simple_types@I@std@@@std@@@std@@@std@@YAXV?$_Vector_iterator@V?$_Vector_val@U?$_Simple_types@I@std@@@std@@@0@0@Z 10009ad0 f i atomselection.obj
 0001:00008b00       ??$sort@V?$_Vector_iterator@V?$_Vector_val@U?$_Simple_types@I@std@@@std@@@std@@U?$less@X@2@@std@@YAXV?$_Vector_iterator@V?$_Vector_val@U?$_Simple_types@I@std@@@std@@@0@0U?$less@X@0@@Z 10009b00 f i atomselection.obj
 0001:00008b20       ??$sort_heap@PAIU?$less@X@std@@@std@@YAXPAI0U?$less@X@0@@Z 10009b20 f i atomselection.obj
 0001:00008b40       ??$swap@I@std@@YAXAAI0@Z   10009b40 f i atomselection.obj
 0001:00008b60       ??$swap@IV?$allocator@I@std@@@std@@YAXAAV?$vector@IV?$allocator@I@std@@@0@0@Z 10009b60 f i atomselection.obj
 0001:00008ba0       ??$swap@PAI@std@@YAXAAPAI0@Z 10009ba0 f i atomselection.obj
 0001:00008bc0       ??$unique_copy@V?$_Vector_iterator@V?$_Vector_val@U?$_Simple_types@I@std@@@std@@@std@@V?$back_insert_iterator@V?$vector@IV?$allocator@I@std@@@std@@@2@@std@@YA?AV?$back_insert_iterator@V?$vector@IV?$allocator@I@std@@@std@@@0@V?$_Vector_iterator@V?$_Vector_val@U?$_Simple_types@I@std@@@std@@@0@0V10@@Z 10009bc0 f i atomselection.obj
 0001:00008c10       ??$unique_copy@V?$_Vector_iterator@V?$_Vector_val@U?$_Simple_types@I@std@@@std@@@std@@V?$back_insert_iterator@V?$vector@IV?$allocator@I@std@@@std@@@2@U?$equal_to@X@2@@std@@YA?AV?$back_insert_iterator@V?$vector@IV?$allocator@I@std@@@std@@@0@V?$_Vector_iterator@V?$_Vector_val@U?$_Simple_types@I@std@@@std@@@0@0V10@U?$equal_to@X@0@@Z 10009c10 f i atomselection.obj
 0001:00008c60       ??0?$_Vector_alloc@$0A@U?$_Vec_base_types@IV?$allocator@I@std@@@std@@@std@@QAE@ABV?$allocator@I@1@@Z 10009c60 f i atomselection.obj
 0001:00008c80       ??0?$_Vector_const_iterator@V?$_Vector_val@U?$_Simple_types@I@std@@@std@@@std@@QAE@PAIPBU_Container_base0@1@@Z 10009c80 f i atomselection.obj
 0001:00008c90       ??0?$_Vector_iterator@V?$_Vector_val@U?$_Simple_types@I@std@@@std@@@std@@QAE@PAIPBU_Container_base0@1@@Z 10009c90 f i atomselection.obj
 0001:00008ca0       ??0?$_Vector_val@U?$_Simple_types@I@std@@@std@@QAE@XZ 10009ca0 f i atomselection.obj
 0001:00008cc0       ??0?$_Wrap_alloc@V?$allocator@I@std@@@std@@QAE@XZ 10009cc0 f i atomselection.obj
 0001:00008cd0       ??0?$_Wrap_alloc@V?$allocator@UCoord3D@PTools@@@std@@@std@@QAE@XZ 10009cd0 f i atomselection.obj
 0001:00008ce0       ??0?$_Wrap_alloc@V?$allocator@VAtomproperty@PTools@@@std@@@std@@QAE@XZ 10009ce0 f i atomselection.obj
 0001:00008cf0       ??0?$allocator@I@std@@QAE@ABV01@@Z 10009cf0 f i atomselection.obj
 0001:00008d00       ??0?$allocator@I@std@@QAE@XZ 10009d00 f i atomselection.obj
 0001:00008d10       ??0?$allocator@UCoord3D@PTools@@@std@@QAE@XZ 10009d10 f i atomselection.obj
 0001:00008d20       ??0?$allocator@VAtomproperty@PTools@@@std@@QAE@XZ 10009d20 f i atomselection.obj
 0001:00008d30       ??0?$back_insert_iterator@V?$vector@IV?$allocator@I@std@@@std@@@std@@QAE@AAV?$vector@IV?$allocator@I@std@@@1@@Z 10009d30 f i atomselection.obj
 0001:00008d40       ??0?$vector@IV?$allocator@I@std@@@std@@QAE@XZ 10009d40 f i atomselection.obj
 0001:00008d60       ??0AtomSelection@PTools@@QAE@ABV01@@Z 10009d60 f   atomselection.obj
 0001:00008dd0       ??0AtomSelection@PTools@@QAE@ABVRigidbody@1@@Z 10009dd0 f   atomselection.obj
 0001:00008ed0       ??0AtomSelection@PTools@@QAE@XZ 10009ed0 f i atomselection.obj
 0001:00008ef0       ??1?$vector@IV?$allocator@I@std@@@std@@QAE@XZ 10009ef0 f i atomselection.obj
 0001:00008f20       ??1?$vector@UCoord3D@PTools@@V?$allocator@UCoord3D@PTools@@@std@@@std@@QAE@XZ 10009f20 f i atomselection.obj
 0001:00008f50       ??1?$vector@VAtomproperty@PTools@@V?$allocator@VAtomproperty@PTools@@@std@@@std@@QAE@XZ 10009f50 f i atomselection.obj
 0001:00008fa0       ??1AtomSelection@PTools@@QAE@XZ 10009fa0 f   atomselection.obj
 0001:00008fd0       ??1CoordsArray@PTools@@QAE@XZ 10009fd0 f i atomselection.obj
 0001:00009020       ??1Rigidbody@PTools@@UAE@XZ 1000a020 f i atomselection.obj
 0001:00009130       ??4?$back_insert_iterator@V?$vector@IV?$allocator@I@std@@@std@@@std@@QAEAAV01@ABI@Z 1000a130 f i atomselection.obj
 0001:00009150       ??4?$vector@IV?$allocator@I@std@@@std@@QAEAAV01@ABV01@@Z 1000a150 f i atomselection.obj
 0001:00009270       ??7PTools@@YA?AVAtomSelection@0@ABV10@@Z 1000a270 f   atomselection.obj
 0001:00009330       ??8?$_Vector_const_iterator@V?$_Vector_val@U?$_Simple_types@I@std@@@std@@@std@@QBE_NABV01@@Z 1000a330 f i atomselection.obj
 0001:00009350       ??A?$vector@IV?$allocator@I@std@@@std@@QAEAAII@Z 1000a350 f i atomselection.obj
 0001:00009360       ??D?$back_insert_iterator@V?$vector@IV?$allocator@I@std@@@std@@@std@@QAEAAV01@XZ 1000a360 f i atomselection.obj
 0001:00009370       ??E?$back_insert_iterator@V?$vector@IV?$allocator@I@std@@@std@@@std@@QAE?AV01@H@Z 1000a370 f i atomselection.obj
 0001:00009380       ??E?$back_insert_iterator@V?$vector@IV?$allocator@I@std@@@std@@@std@@QAEAAV01@XZ 1000a380 f i atomselection.obj
 0001:00009390       ??G?$_Vector_const_iterator@V?$_Vector_val@U?$_Simple_types@I@std@@@std@@@std@@QBEHABV01@@Z 1000a390 f i atomselection.obj
 0001:000093b0       ??G?$_Vector_iterator@V?$_Vector_val@U?$_Simple_types@I@std@@@std@@@std@@QBEHABV?$_Vector_const_iterator@V?$_Vector_val@U?$_Simple_types@I@std@@@std@@@1@@Z 1000a3b0 f i atomselection.obj
 0001:000093d0       ??IPTools@@YA?AVAtomSelection@0@ABV10@0@Z 1000a3d0 f   atomselection.obj
 0001:000094d0       ??UPTools@@YA?AVAtomSelection@0@ABV10@0@Z 1000a4d0 f   atomselection.obj
 0001:00009740       ??_GAtomproperty@PTools@@QAEPAXI@Z 1000a740 f i atomselection.obj
 0001:00009770       ??_ERigidbody@PTools@@UAEPAXI@Z 1000a770 f i atomselection.obj
 0001:00009770       ??_GRigidbody@PTools@@UAEPAXI@Z 1000a770 f i atomselection.obj
 0001:000097a0       ?AddAtomIndex@AtomSelection@PTools@@QAEXI@Z 1000a7a0 f i atomselection.obj
 0001:000097c0       ?CreateRigid@AtomSelection@PTools@@QAE?AVRigidbody@2@XZ 1000a7c0 f   atomselection.obj
 0001:000098a0       ?SetRigid@AtomSelection@PTools@@QAEXABVRigidbody@2@@Z 1000a8a0 f i atomselection.obj
 0001:000098b0       ?Size@AtomSelection@PTools@@QBEIXZ 1000a8b0 f i atomselection.obj
 0001:000098c0       ?_Adopt@_Iterator_base0@std@@QAEXPBX@Z 1000a8c0 f i atomselection.obj
 0001:000098d0       ?_Buy@?$vector@IV?$allocator@I@std@@@std@@IAE_NI@Z 1000a8d0 f i atomselection.obj
 0001:00009940       ?_Change_alloc@?$_Vector_alloc@$0A@U?$_Vec_base_types@IV?$allocator@I@std@@@std@@@std@@QAEXABU?$_Wrap_alloc@V?$allocator@I@std@@@2@@Z 1000a940 f i atomselection.obj
 0001:00009950       ?_Compat@?$_Vector_const_iterator@V?$_Vector_val@U?$_Simple_types@I@std@@@std@@@std@@QBEXABV12@@Z 1000a950 f i atomselection.obj
 0001:00009960       ?_Destroy@?$vector@IV?$allocator@I@std@@@std@@IAEXPAI0@Z 1000a960 f i atomselection.obj
 0001:00009970       ?_Destroy@?$vector@UCoord3D@PTools@@V?$allocator@UCoord3D@PTools@@@std@@@std@@IAEXPAUCoord3D@PTools@@0@Z 1000a970 f i atomselection.obj
 0001:00009980       ?_Destroy@?$vector@VAtomproperty@PTools@@V?$allocator@VAtomproperty@PTools@@@std@@@std@@IAEXPAVAtomproperty@PTools@@0@Z 1000a980 f i atomselection.obj
 0001:000099b0       ?_Getal@?$_Vector_alloc@$0A@U?$_Vec_base_types@IV?$allocator@I@std@@@std@@@std@@QBE?AU?$_Wrap_alloc@V?$allocator@I@std@@@2@XZ 1000a9b0 f i atomselection.obj
 0001:000099c0       ?_Getal@?$_Vector_alloc@$0A@U?$_Vec_base_types@UCoord3D@PTools@@V?$allocator@UCoord3D@PTools@@@std@@@std@@@std@@QBE?AU?$_Wrap_alloc@V?$allocator@UCoord3D@PTools@@@std@@@2@XZ 1000a9c0 f i atomselection.obj
 0001:000099d0       ?_Getal@?$_Vector_alloc@$0A@U?$_Vec_base_types@VAtomproperty@PTools@@V?$allocator@VAtomproperty@PTools@@@std@@@std@@@std@@QBE?AU?$_Wrap_alloc@V?$allocator@VAtomproperty@PTools@@@std@@@2@XZ 1000a9d0 f i atomselection.obj
 0001:000099e0       ?_Grow_to@?$vector@IV?$allocator@I@std@@@std@@IBEII@Z 1000a9e0 f i atomselection.obj
 0001:00009a20       ?_Inside@?$vector@IV?$allocator@I@std@@@std@@IBE_NPBI@Z 1000aa20 f i atomselection.obj
 0001:00009a40       ?_Orphan_range@?$vector@IV?$allocator@I@std@@@std@@IBEXPAI0@Z 1000aa40 f i atomselection.obj
 0001:00009a50       ?_Reallocate@?$vector@IV?$allocator@I@std@@@std@@IAEXI@Z 1000aa50 f i atomselection.obj
 0001:00009ad0       ?_Reserve@?$vector@IV?$allocator@I@std@@@std@@IAEXI@Z 1000aad0 f i atomselection.obj
 0001:00009b50       ?_Swap_alloc@?$_Vector_alloc@$0A@U?$_Vec_base_types@IV?$allocator@I@std@@@std@@@std@@QAEXAAV12@@Z 1000ab50 f i atomselection.obj
 0001:00009b60       ?_Tidy@?$vector@IV?$allocator@I@std@@@std@@IAEXXZ 1000ab60 f i atomselection.obj
 0001:00009b90       ?_Tidy@?$vector@UCoord3D@PTools@@V?$allocator@UCoord3D@PTools@@@std@@@std@@IAEXXZ 1000ab90 f i atomselection.obj
 0001:00009bc0       ?_Tidy@?$vector@VAtomproperty@PTools@@V?$allocator@VAtomproperty@PTools@@@std@@@std@@IAEXXZ 1000abc0 f i atomselection.obj
 0001:00009c10       ?_Unchecked@?$_Vector_const_iterator@V?$_Vector_val@U?$_Simple_types@I@std@@@std@@@std@@QBEPBIXZ 1000ac10 f i atomselection.obj
 0001:00009c20       ?_Unchecked@?$_Vector_iterator@V?$_Vector_val@U?$_Simple_types@I@std@@@std@@@std@@QBEPAIXZ 1000ac20 f i atomselection.obj
 0001:00009c30       ?_Unused_capacity@?$vector@IV?$allocator@I@std@@@std@@QBEIXZ 1000ac30 f i atomselection.obj
 0001:00009c40       ?_Xlen@?$vector@IV?$allocator@I@std@@@std@@IBEXXZ 1000ac40 f i atomselection.obj
 0001:00009c50       ?allocate@?$_Wrap_alloc@V?$allocator@I@std@@@std@@QAEPAII@Z 1000ac50 f i atomselection.obj
 0001:00009c90       ?allocate@?$allocator@I@std@@QAEPAII@Z 1000ac90 f i atomselection.obj
 0001:00009cd0       ?begin@?$vector@IV?$allocator@I@std@@@std@@QAE?AV?$_Vector_iterator@V?$_Vector_val@U?$_Simple_types@I@std@@@std@@@2@XZ 1000acd0 f i atomselection.obj
 0001:00009ce0       ?begin@?$vector@IV?$allocator@I@std@@@std@@QBE?AV?$_Vector_const_iterator@V?$_Vector_val@U?$_Simple_types@I@std@@@std@@@2@XZ 1000ace0 f i atomselection.obj
 0001:00009cf0       ?capacity@?$vector@IV?$allocator@I@std@@@std@@QBEIXZ 1000acf0 f i atomselection.obj
 0001:00009d00       ?clear@?$vector@IV?$allocator@I@std@@@std@@QAEXXZ 1000ad00 f i atomselection.obj
 0001:00009d10       ?construct@?$allocator@I@std@@QAEXPAIABI@Z 1000ad10 f i atomselection.obj
 0001:00009d30       ?deallocate@?$_Wrap_alloc@V?$allocator@I@std@@@std@@QAEXPAII@Z 1000ad30 f i atomselection.obj
 0001:00009d50       ?deallocate@?$_Wrap_alloc@V?$allocator@UCoord3D@PTools@@@std@@@std@@QAEXPAUCoord3D@PTools@@I@Z 1000ad50 f i atomselection.obj
 0001:00009d70       ?deallocate@?$_Wrap_alloc@V?$allocator@VAtomproperty@PTools@@@std@@@std@@QAEXPAVAtomproperty@PTools@@I@Z 1000ad70 f i atomselection.obj
 0001:00009d90       ?deallocate@?$allocator@I@std@@QAEXPAII@Z 1000ad90 f i atomselection.obj
 0001:00009db0       ?deallocate@?$allocator@UCoord3D@PTools@@@std@@QAEXPAUCoord3D@PTools@@I@Z 1000adb0 f i atomselection.obj
 0001:00009dd0       ?deallocate@?$allocator@VAtomproperty@PTools@@@std@@QAEXPAVAtomproperty@PTools@@I@Z 1000add0 f i atomselection.obj
 0001:00009df0       ?empty@?$vector@IV?$allocator@I@std@@@std@@QBE_NXZ 1000adf0 f i atomselection.obj
 0001:00009e00       ?end@?$vector@IV?$allocator@I@std@@@std@@QAE?AV?$_Vector_iterator@V?$_Vector_val@U?$_Simple_types@I@std@@@std@@@2@XZ 1000ae00 f i atomselection.obj
 0001:00009e10       ?end@?$vector@IV?$allocator@I@std@@@std@@QBE?AV?$_Vector_const_iterator@V?$_Vector_val@U?$_Simple_types@I@std@@@std@@@2@XZ 1000ae10 f i atomselection.obj
 0001:00009e20       ?isAtomActive@Rigidbody@PTools@@UBE_NI@Z 1000ae20 f i atomselection.obj
 0001:00009e30       ?max_size@?$_Wrap_alloc@V?$allocator@I@std@@@std@@QBEIXZ 1000ae30 f i atomselection.obj
 0001:00009e40       ?max_size@?$allocator@I@std@@QBEIXZ 1000ae40 f i atomselection.obj
 0001:00009e50       ?max_size@?$allocator_traits@V?$allocator@I@std@@@std@@SAIABV?$allocator@I@2@@Z 1000ae50 f i atomselection.obj
 0001:00009e60       ?max_size@?$vector@IV?$allocator@I@std@@@std@@QBEIXZ 1000ae60 f i atomselection.obj
 0001:00009e70       ?non@AtomSelection@PTools@@QAE?AV12@ABV12@@Z 1000ae70 f   atomselection.obj
 0001:00009ea0       ?push_back@?$vector@IV?$allocator@I@std@@@std@@QAEXABI@Z 1000aea0 f i atomselection.obj
 0001:00009f10       ?size@?$vector@IV?$allocator@I@std@@@std@@QBEIXZ 1000af10 f i atomselection.obj
 0001:00009f20       ?swap@?$vector@IV?$allocator@I@std@@@std@@QAEXAAV12@@Z 1000af20 f i atomselection.obj
 0001:00009f60       ??$?0HHX@?$pair@HH@std@@QAE@$$QAU01@@Z 1000af60 f i basetypes.obj
 0001:00009f80       ??$forward@H@std@@YA$$QAHAAH@Z 1000af80 f i basetypes.obj
 0001:00009f90       ??0?$pair@HH@std@@QAE@XZ   1000af90 f i basetypes.obj
 0001:00009fa0       ?MakeIdentity@PTools@@YAXAAV?$Array2D@N@@@Z 1000afa0 f   basetypes.obj
 0001:0000a0d0       ?getDim@?$Array2D@N@@QAE?AU?$pair@HH@std@@XZ 1000b0d0 f i basetypes.obj
 0001:0000a0f0       ??$?6U?$char_traits@D@std@@@std@@YAAAV?$basic_ostream@DU?$char_traits@D@std@@@0@AAV10@PBD@Z 1000b0f0 f i coord3d.obj
 0001:0000a320       ??$forward@V?$basic_string@DU?$char_traits@D@std@@V?$allocator@D@2@@std@@@std@@YA$$QAV?$basic_string@DU?$char_traits@D@std@@V?$allocator@D@2@@0@AAV10@@Z 1000b320 f i coord3d.obj
 0001:0000a330       ??0?$basic_string@DU?$char_traits@D@std@@V?$allocator@D@2@@std@@QAE@$$QAV01@@Z 1000b330 f i coord3d.obj
 0001:0000a3a0       ??0?$basic_string@DU?$char_traits@D@std@@V?$allocator@D@2@@std@@QAE@PBDI@Z 1000b3a0 f i coord3d.obj
 0001:0000a3d0       ??0?$basic_stringbuf@DU?$char_traits@D@std@@V?$allocator@D@2@@std@@QAE@H@Z 1000b3d0 f i coord3d.obj
 0001:0000a450       ??0?$basic_stringstream@DU?$char_traits@D@std@@V?$allocator@D@2@@std@@QAE@H@Z 1000b450 f i coord3d.obj
 0001:0000a540       ??0?$fpos@H@std@@QAE@_J@Z  1000b540 f i coord3d.obj
 0001:0000a570       ??0_Sentry_base@?$basic_ostream@DU?$char_traits@D@std@@@std@@QAE@AAV12@@Z 1000b570 f i coord3d.obj
 0001:0000a5a0       ??0sentry@?$basic_ostream@DU?$char_traits@D@std@@@std@@QAE@AAV12@@Z 1000b5a0 f i coord3d.obj
 0001:0000a630       ??1?$basic_stringbuf@DU?$char_traits@D@std@@V?$allocator@D@2@@std@@UAE@XZ 1000b630 f i coord3d.obj
 0001:0000a650       ??1?$basic_stringstream@DU?$char_traits@D@std@@V?$allocator@D@2@@std@@UAE@XZ 1000b650 f i coord3d.obj
 0001:0000a6a0       ??1_Sentry_base@?$basic_ostream@DU?$char_traits@D@std@@@std@@QAE@XZ 1000b6a0 f i coord3d.obj
 0001:0000a6c0       ??1sentry@?$basic_ostream@DU?$char_traits@D@std@@@std@@QAE@XZ 1000b6c0 f i coord3d.obj
 0001:0000a6f0       ??B?$fpos@H@std@@QBE_JXZ   1000b6f0 f i coord3d.obj
 0001:0000a700       ??Bsentry@?$basic_ostream@DU?$char_traits@D@std@@@std@@QBE_NXZ 1000b700 f i coord3d.obj
 0001:0000a710       ??_D?$basic_stringstream@DU?$char_traits@D@std@@V?$allocator@D@2@@std@@QAEXXZ 1000b710 f i coord3d.obj
 0001:0000a76b       ??_E?$basic_stringstream@DU?$char_traits@D@std@@V?$allocator@D@2@@std@@$4PPPPPPPM@A@AEPAXI@Z 1000b76b f i coord3d.obj
 0001:0000a780       ??_E?$basic_stringbuf@DU?$char_traits@D@std@@V?$allocator@D@2@@std@@UAEPAXI@Z 1000b780 f i coord3d.obj
 0001:0000a780       ??_G?$basic_stringbuf@DU?$char_traits@D@std@@V?$allocator@D@2@@std@@UAEPAXI@Z 1000b780 f i coord3d.obj
 0001:0000a7b0       ??_E?$basic_stringstream@DU?$char_traits@D@std@@V?$allocator@D@2@@std@@UAEPAXI@Z 1000b7b0 f i coord3d.obj
 0001:0000a7b0       ??_G?$basic_stringstream@DU?$char_traits@D@std@@V?$allocator@D@2@@std@@UAEPAXI@Z 1000b7b0 f i coord3d.obj
 0001:0000a7e0       ?Norm@PTools@@YANABUCoord3D@1@@Z 1000b7e0 f i coord3d.obj
 0001:0000a820       ?Normalize@Coord3D@PTools@@QAEAAU12@XZ 1000b820 f   coord3d.obj
 0001:0000a8b0       ?_Assign_rv@?$basic_string@DU?$char_traits@D@std@@V?$allocator@D@2@@std@@QAEX$$QAV12@@Z 1000b8b0 f i coord3d.obj
 0001:0000a910       ?_Getstate@?$basic_stringbuf@DU?$char_traits@D@std@@V?$allocator@D@2@@std@@AAEHH@Z 1000b910 f i coord3d.obj
 0001:0000a940       ?_Init@?$basic_stringbuf@DU?$char_traits@D@std@@V?$allocator@D@2@@std@@IAEXPBDIH@Z 1000b940 f i coord3d.obj
 0001:0000aa00       ?_Tidy@?$basic_stringbuf@DU?$char_traits@D@std@@V?$allocator@D@2@@std@@IAEXXZ 1000ba00 f i coord3d.obj
 0001:0000aa60       ?eof@?$char_traits@D@std@@SAHXZ 1000ba60 f i coord3d.obj
 0001:0000aa70       ?eq@?$char_traits@D@std@@SA_NABD0@Z 1000ba70 f i coord3d.obj
 0001:0000aa90       ?eq_int_type@?$char_traits@D@std@@SA_NABH0@Z 1000ba90 f i coord3d.obj
 0001:0000aab0       ?not_eof@?$char_traits@D@std@@SAHABH@Z 1000bab0 f i coord3d.obj
 0001:0000aad0       ?overflow@?$basic_stringbuf@DU?$char_traits@D@std@@V?$allocator@D@2@@std@@MAEHH@Z 1000bad0 f i coord3d.obj
 0001:0000aca0       ?pbackfail@?$basic_stringbuf@DU?$char_traits@D@std@@V?$allocator@D@2@@std@@MAEHH@Z 1000bca0 f i coord3d.obj
 0001:0000ad00       ?seekoff@?$basic_stringbuf@DU?$char_traits@D@std@@V?$allocator@D@2@@std@@MAE?AV?$fpos@H@2@_JHH@Z 1000bd00 f i coord3d.obj
 0001:0000aed0       ?seekpos@?$basic_stringbuf@DU?$char_traits@D@std@@V?$allocator@D@2@@std@@MAE?AV?$fpos@H@2@V32@H@Z 1000bed0 f i coord3d.obj
 0001:0000aff0       ?str@?$basic_stringbuf@DU?$char_traits@D@std@@V?$allocator@D@2@@std@@QBE?AV?$basic_string@DU?$char_traits@D@std@@V?$allocator@D@2@@2@XZ 1000bff0 f i coord3d.obj
 0001:0000b100       ?str@?$basic_stringstream@DU?$char_traits@D@std@@V?$allocator@D@2@@std@@QBE?AV?$basic_string@DU?$char_traits@D@std@@V?$allocator@D@2@@2@XZ 1000c100 f i coord3d.obj
 0001:0000b120       ?toString@Coord3D@PTools@@QAE?AV?$basic_string@DU?$char_traits@D@std@@V?$allocator@D@2@@std@@_N@Z 1000c120 f   coord3d.obj
 0001:0000b300       ?to_char_type@?$char_traits@D@std@@SADABH@Z 1000c300 f i coord3d.obj
 0001:0000b310       ?to_int_type@?$char_traits@D@std@@SAHABD@Z 1000c310 f i coord3d.obj
 0001:0000b320       ?underflow@?$basic_stringbuf@DU?$char_traits@D@std@@V?$allocator@D@2@@std@@MAEHXZ 1000c320 f i coord3d.obj
 0001:0000b380       ??$?8UCoord3D@PTools@@U01@@std@@YA_NABV?$allocator@UCoord3D@PTools@@@0@0@Z 1000c380 f i coordsarray.obj
 0001:0000b390       ??$?8V?$allocator@UCoord3D@PTools@@@std@@V01@@std@@YA_NABU?$_Wrap_alloc@V?$allocator@UCoord3D@PTools@@@std@@@0@0@Z 1000c390 f i coordsarray.obj
 0001:0000b3a0       ??$?9V?$allocator@UCoord3D@PTools@@@std@@V01@@std@@YA_NABU?$_Wrap_alloc@V?$allocator@UCoord3D@PTools@@@std@@@0@0@Z 1000c3a0 f i coordsarray.obj
 0001:0000b3b0       ??$_Allocate@UCoord3D@PTools@@@std@@YAPAUCoord3D@PTools@@IPAU12@@Z 1000c3b0 f i coordsarray.obj
 0001:0000b3f0       ??$_Copy_impl@PAUCoord3D@PTools@@PAU12@@std@@YAPAUCoord3D@PTools@@PAU12@00@Z 1000c3f0 f i coordsarray.obj
 0001:0000b440       ??$_Copy_impl@PAUCoord3D@PTools@@PAU12@@std@@YAPAUCoord3D@PTools@@PAU12@00U_Nonscalar_ptr_iterator_tag@0@@Z 1000c440 f i coordsarray.obj
 0001:0000b480       ??$_Rechecked@PAUCoord3D@PTools@@PAU12@@std@@YAAAPAUCoord3D@PTools@@AAPAU12@PAU12@@Z 1000c480 f i coordsarray.obj
 0001:0000b490       ??$_Ucopy@PAUCoord3D@PTools@@@?$vector@UCoord3D@PTools@@V?$allocator@UCoord3D@PTools@@@std@@@std@@IAEPAUCoord3D@PTools@@PAU23@00@Z 1000c490 f i coordsarray.obj
 0001:0000b4c0       ??$_Unchecked@PAUCoord3D@PTools@@@std@@YAPAUCoord3D@PTools@@PAU12@@Z 1000c4c0 f i coordsarray.obj
 0001:0000b4d0       ??$_Uninit_copy@PAUCoord3D@PTools@@PAU12@U?$_Wrap_alloc@V?$allocator@UCoord3D@PTools@@@std@@@std@@@std@@YAPAUCoord3D@PTools@@PAU12@00AAU?$_Wrap_alloc@V?$allocator@UCoord3D@PTools@@@std@@@0@@Z 1000c4d0 f i coordsarray.obj
 0001:0000b4f0       ??$_Uninit_copy@PAUCoord3D@PTools@@PAU12@V?$allocator@UCoord3D@PTools@@@std@@@std@@YAPAUCoord3D@PTools@@PAU12@00AAU?$_Wrap_alloc@V?$allocator@UCoord3D@PTools@@@std@@@0@U_Nonscalar_ptr_iterator_tag@0@@Z 1000c4f0 f i coordsarray.obj
 0001:0000b530       ??$_Uninitialized_copy@PAUCoord3D@PTools@@PAU12@U?$_Wrap_alloc@V?$allocator@UCoord3D@PTools@@@std@@@std@@@std@@YAPAUCoord3D@PTools@@PAU12@00AAU?$_Wrap_alloc@V?$allocator@UCoord3D@PTools@@@std@@@0@@Z 1000c530 f i coordsarray.obj
 0001:0000b550       ??$construct@UCoord3D@PTools@@AAU12@@?$_Wrap_alloc@V?$allocator@UCoord3D@PTools@@@std@@@std@@QAEXPAUCoord3D@PTools@@AAU23@@Z 1000c550 f i coordsarray.obj
 0001:0000b580       ??$construct@UCoord3D@PTools@@AAU12@@?$allocator@UCoord3D@PTools@@@std@@QAEXPAUCoord3D@PTools@@AAU23@@Z 1000c580 f i coordsarray.obj
 0001:0000b5b0       ??$construct@UCoord3D@PTools@@AAU12@@?$allocator_traits@V?$allocator@UCoord3D@PTools@@@std@@@std@@SAXAAV?$allocator@UCoord3D@PTools@@@1@PAUCoord3D@PTools@@AAU34@@Z 1000c5b0 f i coordsarray.obj
 0001:0000b5e0       ??$forward@AAUCoord3D@PTools@@@std@@YAAAUCoord3D@PTools@@AAU12@@Z 1000c5e0 f i coordsarray.obj
 0001:0000b5f0       ??0?$Array2D@N@@QAE@ABV0@@Z 1000c5f0 f i coordsarray.obj
 0001:0000b620       ??0?$Array2D@N@@QAE@HH@Z   1000c620 f i coordsarray.obj
 0001:0000b6c0       ??0?$QFlags@W4AllocationOption@QArrayData@@@@QAE@PQPrivate@0@H@Z 1000c6c0 f i coordsarray.obj
 0001:0000b6d0       ??0?$QVector@N@@QAE@ABV0@@Z 1000c6d0 f i coordsarray.obj
 0001:0000b790       ??0?$QVector@N@@QAE@XZ     1000c790 f i coordsarray.obj
 0001:0000b7a0       ??0?$_Vector_alloc@$0A@U?$_Vec_base_types@UCoord3D@PTools@@V?$allocator@UCoord3D@PTools@@@std@@@std@@@std@@QAE@ABV?$allocator@UCoord3D@PTools@@@1@@Z 1000c7a0 f i coordsarray.obj
 0001:0000b7c0       ??0?$_Vector_val@U?$_Simple_types@UCoord3D@PTools@@@std@@@std@@QAE@XZ 1000c7c0 f i coordsarray.obj
 0001:0000b7e0       ??0?$allocator@UCoord3D@PTools@@@std@@QAE@ABV01@@Z 1000c7e0 f i coordsarray.obj
 0001:0000b7f0       ??0?$vector@UCoord3D@PTools@@V?$allocator@UCoord3D@PTools@@@std@@@std@@QAE@XZ 1000c7f0 f i coordsarray.obj
 0001:0000b810       ??0Coord3D@PTools@@QAE@XZ  1000c810 f i coordsarray.obj
 0001:0000b820       ??0CoordsArray@PTools@@QAE@ABV01@@Z 1000c820 f   coordsarray.obj
 0001:0000b910       ??0CoordsArray@PTools@@QAE@XZ 1000c910 f   coordsarray.obj
 0001:0000b9b0       ??0logic_error@std@@QAE@ABV01@@Z 1000c9b0 f i coordsarray.obj
 0001:0000b9d0       ??0logic_error@std@@QAE@PBD@Z 1000c9d0 f i coordsarray.obj
 0001:0000b9f0       ??0out_of_range@std@@QAE@ABV01@@Z 1000c9f0 f i coordsarray.obj
 0001:0000ba10       ??0out_of_range@std@@QAE@ABV?$basic_string@DU?$char_traits@D@std@@V?$allocator@D@2@@1@@Z 1000ca10 f i coordsarray.obj
 0001:0000ba40       ??1logic_error@std@@UAE@XZ 1000ca40 f i coordsarray.obj
 0001:0000ba50       ??1out_of_range@std@@UAE@XZ 1000ca50 f i coordsarray.obj
 0001:0000ba60       ??4?$vector@UCoord3D@PTools@@V?$allocator@UCoord3D@PTools@@@std@@@std@@QAEAAV01@ABV01@@Z 1000ca60 f i coordsarray.obj
 0001:0000bbe0       ??A?$vector@UCoord3D@PTools@@V?$allocator@UCoord3D@PTools@@@std@@@std@@QAEAAUCoord3D@PTools@@I@Z 1000cbe0 f i coordsarray.obj
 0001:0000bc00       ??A?$vector@UCoord3D@PTools@@V?$allocator@UCoord3D@PTools@@@std@@@std@@QBEABUCoord3D@PTools@@I@Z 1000cc00 f i coordsarray.obj
 0001:0000bc20       ??Y?$basic_string@DU?$char_traits@D@std@@V?$allocator@D@2@@std@@QAEAAV01@D@Z 1000cc20 f i coordsarray.obj
 0001:0000bc40       ??Y?$basic_string@DU?$char_traits@D@std@@V?$allocator@D@2@@std@@QAEAAV01@PBD@Z 1000cc40 f i coordsarray.obj
 0001:0000bc80       ??_Glogic_error@std@@UAEPAXI@Z 1000cc80 f i coordsarray.obj
 0001:0000bc80       ??_Elogic_error@std@@UAEPAXI@Z 1000cc80 f i coordsarray.obj
 0001:0000bcb0       ??_Eout_of_range@std@@UAEPAXI@Z 1000ccb0 f i coordsarray.obj
 0001:0000bcb0       ??_Gout_of_range@std@@UAEPAXI@Z 1000ccb0 f i coordsarray.obj
 0001:0000bce0       ?AttractEulerRotate@CoordsArray@PTools@@QAEXNNN@Z 1000cce0 f   coordsarray.obj
 0001:0000bed0       ?GetCoords@CoordsArray@PTools@@QBEXIAAUCoord3D@2@@Z 1000ced0 f   coordsarray.obj
 0001:0000bff0       ?GetMatrix@CoordsArray@PTools@@QBE?AV?$Array2D@N@@XZ 1000cff0 f   coordsarray.obj
 0001:0000c140       ?MatrixMultiply@CoordsArray@PTools@@IAEXQAY03$$CBN@Z 1000d140 f   coordsarray.obj
 0001:0000c170       ?ResetMatrix@CoordsArray@PTools@@QAEXXZ 1000d170 f   coordsarray.obj
 0001:0000c200       ?SetCoords@CoordsArray@PTools@@QAEXIABUCoord3D@2@@Z 1000d200 f   coordsarray.obj
 0001:0000c300       ?Translate@CoordsArray@PTools@@QAEXABUCoord3D@2@@Z 1000d300 f   coordsarray.obj
 0001:0000c350       ?_Buy@?$vector@UCoord3D@PTools@@V?$allocator@UCoord3D@PTools@@@std@@@std@@IAE_NI@Z 1000d350 f i coordsarray.obj
 0001:0000c3c0       ?_Change_alloc@?$_Vector_alloc@$0A@U?$_Vec_base_types@UCoord3D@PTools@@V?$allocator@UCoord3D@PTools@@@std@@@std@@@std@@QAEXABU?$_Wrap_alloc@V?$allocator@UCoord3D@PTools@@@std@@@2@@Z 1000d3c0 f i coordsarray.obj
 0001:0000c3d0       ?_Chassign@?$basic_string@DU?$char_traits@D@std@@V?$allocator@D@2@@std@@QAEXIID@Z 1000d3d0 f i coordsarray.obj
 0001:0000c420       ?_Xlen@?$vector@UCoord3D@PTools@@V?$allocator@UCoord3D@PTools@@@std@@@std@@IBEXXZ 1000d420 f i coordsarray.obj
 0001:0000c430       ?_modified@CoordsArray@PTools@@AAEXXZ 1000d430 f i coordsarray.obj
 0001:0000c450       ?_safegetcoords@CoordsArray@PTools@@ABEXIAAUCoord3D@2@@Z 1000d450 f i coordsarray.obj
 0001:0000c560       ?allocate@?$_Wrap_alloc@V?$allocator@UCoord3D@PTools@@@std@@@std@@QAEPAUCoord3D@PTools@@I@Z 1000d560 f i coordsarray.obj
 0001:0000c5a0       ?allocate@?$allocator@UCoord3D@PTools@@@std@@QAEPAUCoord3D@PTools@@I@Z 1000d5a0 f i coordsarray.obj
 0001:0000c5e0       ?append@?$basic_string@DU?$char_traits@D@std@@V?$allocator@D@2@@std@@QAEAAV12@ABV12@II@Z 1000d5e0 f i coordsarray.obj
 0001:0000c6a0       ?append@?$basic_string@DU?$char_traits@D@std@@V?$allocator@D@2@@std@@QAEAAV12@ID@Z 1000d6a0 f i coordsarray.obj
 0001:0000c750       ?append@?$basic_string@DU?$char_traits@D@std@@V?$allocator@D@2@@std@@QAEAAV12@PBD@Z 1000d750 f i coordsarray.obj
 0001:0000c790       ?append@?$basic_string@DU?$char_traits@D@std@@V?$allocator@D@2@@std@@QAEAAV12@PBDI@Z 1000d790 f i coordsarray.obj
 0001:0000c880       ?assign@?$char_traits@D@std@@SAPADPADID@Z 1000d880 f i coordsarray.obj
 0001:0000c8a0       ?c_str@?$basic_string@DU?$char_traits@D@std@@V?$allocator@D@2@@std@@QBEPBDXZ 1000d8a0 f i coordsarray.obj
 0001:0000c8b0       ?capacity@?$vector@UCoord3D@PTools@@V?$allocator@UCoord3D@PTools@@@std@@@std@@QBEIXZ 1000d8b0 f i coordsarray.obj
 0001:0000c8d0       ?clear@?$vector@UCoord3D@PTools@@V?$allocator@UCoord3D@PTools@@@std@@@std@@QAEXXZ 1000d8d0 f i coordsarray.obj
 0001:0000c8e0       ?copyConstruct@?$QVector@N@@AAEXPBN0PAN@Z 1000d8e0 f i coordsarray.obj
 0001:0000c900       ?empty@?$vector@UCoord3D@PTools@@V?$allocator@UCoord3D@PTools@@@std@@@std@@QBE_NXZ 1000d900 f i coordsarray.obj
 0001:0000c910       ?matrix44xVect@PTools@@YAXQAY03$$CBNABUCoord3D@1@AAU21@@Z 1000d910 f i coordsarray.obj
 0001:0000c9b0       ?max_size@?$_Wrap_alloc@V?$allocator@UCoord3D@PTools@@@std@@@std@@QBEIXZ 1000d9b0 f i coordsarray.obj
 0001:0000c9c0       ?max_size@?$allocator@UCoord3D@PTools@@@std@@QBEIXZ 1000d9c0 f i coordsarray.obj
 0001:0000c9d0       ?max_size@?$allocator_traits@V?$allocator@UCoord3D@PTools@@@std@@@std@@SAIABV?$allocator@UCoord3D@PTools@@@2@@Z 1000d9d0 f i coordsarray.obj
 0001:0000c9e0       ?max_size@?$vector@UCoord3D@PTools@@V?$allocator@UCoord3D@PTools@@@std@@@std@@QBEIXZ 1000d9e0 f i coordsarray.obj
 0001:0000c9f0       ?resize@?$QVector@N@@QAEXH@Z 1000d9f0 f i coordsarray.obj
 0001:0000ca40       ?unsafeGetCoords@CoordsArray@PTools@@QBEXIAAUCoord3D@2@@Z 1000da40 f i coordsarray.obj
 0001:0000ca80       ??GPTools@@YA?AUCoord3D@0@ABU10@0@Z 1000da80 f i geometry.obj
 0001:0000cac0       ?ABrotate@PTools@@YAXUCoord3D@1@0AAVRigidbody@1@N@Z 1000dac0 f   geometry.obj
 0001:0000cb60       ?Angle@PTools@@YANABUCoord3D@1@0@Z 1000db60 f   geometry.obj
 0001:0000cc20       ?Dihedral@PTools@@YANABUCoord3D@1@000@Z 1000dc20 f   geometry.obj
 0001:0000cde0       ?MakeRotationMatrix@PTools@@YAXUCoord3D@1@0NQAY03N@Z 1000dde0 f   geometry.obj
 0001:0000d3f0       ?MakeTranslationMat44@PTools@@YAXUCoord3D@1@QAY03N@Z 1000e3f0 f   geometry.obj
 0001:0000d480       ?MakeVect@PTools@@YAXABUCoord3D@1@0AAU21@@Z 1000e480 f   geometry.obj
 0001:0000d4c0       ?ScalProd@PTools@@YANABUCoord3D@1@0@Z 1000e4c0 f i geometry.obj
 0001:0000d4e0       ?VectProd@PTools@@YAXABUCoord3D@1@0AAU21@@Z 1000e4e0 f   geometry.obj
 0001:0000d540       ?mat44xmat44@PTools@@YAXQAY03$$CBN0QAY03N@Z 1000e540 f   geometry.obj
 0001:0000d610       ?real@@YAAANAAN@Z          1000e610 f i geometry.obj
 0001:0000d620       ??$?8DU?$char_traits@D@std@@V?$allocator@D@1@@std@@YA_NABV?$basic_string@DU?$char_traits@D@std@@V?$allocator@D@2@@0@0@Z 1000e620 f i pdbio.obj
 0001:0000d650       ??$?8DU?$char_traits@D@std@@V?$allocator@D@1@@std@@YA_NABV?$basic_string@DU?$char_traits@D@std@@V?$allocator@D@2@@0@PBD@Z 1000e650 f i pdbio.obj
 0001:0000d690       ??$?HDU?$char_traits@D@std@@V?$allocator@D@1@@std@@YA?AV?$basic_string@DU?$char_traits@D@std@@V?$allocator@D@2@@0@$$QAV10@PBD@Z 1000e690 f i pdbio.obj
 0001:0000d730       ??$?HDU?$char_traits@D@std@@V?$allocator@D@1@@std@@YA?AV?$basic_string@DU?$char_traits@D@std@@V?$allocator@D@2@@0@PBDABV10@@Z 1000e730 f i pdbio.obj
 0001:0000d820       ??$_Fgetc@D@std@@YA_NAADPAU_iobuf@@@Z 1000e820 f i pdbio.obj
 0001:0000d850       ??$_Fputc@D@std@@YA_NDPAU_iobuf@@@Z 1000e850 f i pdbio.obj
 0001:0000d870       ??$_Transform@PADV?$_String_iterator@V?$_String_val@U?$_Simple_types@D@std@@@std@@@std@@P6AHH@Z@std@@YA?AV?$_String_iterator@V?$_String_val@U?$_Simple_types@D@std@@@std@@@0@PAD0V10@P6AHH@Z@Z 1000e870 f i pdbio.obj
 0001:0000d8d0       ??$_Unchecked@V?$_String_val@U?$_Simple_types@D@std@@@std@@@std@@YAPADV?$_String_iterator@V?$_String_val@U?$_Simple_types@D@std@@@std@@@0@@Z 1000e8d0 f i pdbio.obj
 0001:0000d8e0       ??$_Ungetc@D@std@@YA_NABDPAU_iobuf@@@Z 1000e8e0 f i pdbio.obj
 0001:0000d900       ??$assign@V?$_String_iterator@V?$_String_val@U?$_Simple_types@D@std@@@std@@@std@@@?$basic_string@DU?$char_traits@D@std@@V?$allocator@D@2@@std@@QAEAAV01@V?$_String_iterator@V?$_String_val@U?$_Simple_types@D@std@@@std@@@1@0@Z 1000e900 f i pdbio.obj
 0001:0000d940       ??$getline@DU?$char_traits@D@std@@V?$allocator@D@2@@std@@YAAAV?$basic_istream@DU?$char_traits@D@std@@@0@$$QAV10@AAV?$basic_string@DU?$char_traits@D@std@@V?$allocator@D@2@@0@D@Z 1000e940 f i pdbio.obj
 0001:0000dab0       ??$getline@DU?$char_traits@D@std@@V?$allocator@D@2@@std@@YAAAV?$basic_istream@DU?$char_traits@D@std@@@0@AAV10@AAV?$basic_string@DU?$char_traits@D@std@@V?$allocator@D@2@@0@@Z 1000eab0 f i pdbio.obj
 0001:0000dae0       ??$move@AAV?$basic_istream@DU?$char_traits@D@std@@@std@@@std@@YA$$QAV?$basic_istream@DU?$char_traits@D@std@@@0@AAV10@@Z 1000eae0 f i pdbio.obj
 0001:0000daf0       ??$move@AAV?$basic_string@DU?$char_traits@D@std@@V?$allocator@D@2@@std@@@std@@YA$$QAV?$basic_string@DU?$char_traits@D@std@@V?$allocator@D@2@@0@AAV10@@Z 1000eaf0 f i pdbio.obj
 0001:0000db00       ??$transform@V?$_String_iterator@V?$_String_val@U?$_Simple_types@D@std@@@std@@@std@@V12@P6AHH@Z@std@@YA?AV?$_String_iterator@V?$_String_val@U?$_Simple_types@D@std@@@std@@@0@V10@00P6AHH@Z@Z 1000eb00 f i pdbio.obj
 0001:0000db30       ??$use_facet@V?$codecvt@DDH@std@@@std@@YAABV?$codecvt@DDH@0@ABVlocale@0@@Z 1000eb30 f i pdbio.obj
 0001:0000dc20       ??0?$_String_const_iterator@V?$_String_val@U?$_Simple_types@D@std@@@std@@@std@@QAE@PBDPBU_Container_base0@1@@Z 1000ec20 f i pdbio.obj
 0001:0000dc30       ??0?$_String_iterator@V?$_String_val@U?$_Simple_types@D@std@@@std@@@std@@QAE@PADPBU_Container_base0@1@@Z 1000ec30 f i pdbio.obj
 0001:0000dc40       ??0?$basic_filebuf@DU?$char_traits@D@std@@@std@@QAE@PAU_iobuf@@@Z 1000ec40 f i pdbio.obj
 0001:0000dce0       ??0?$basic_ifstream@DU?$char_traits@D@std@@@std@@QAE@PBDHH@Z 1000ece0 f i pdbio.obj
 0001:0000ddf0       ??0?$basic_ostringstream@DU?$char_traits@D@std@@V?$allocator@D@2@@std@@QAE@H@Z 1000edf0 f i pdbio.obj
 0001:0000dee0       ??0?$basic_string@DU?$char_traits@D@std@@V?$allocator@D@2@@std@@QAE@ABV01@IIABV?$allocator@D@1@@Z 1000eee0 f i pdbio.obj
 0001:0000df10       ??0?$basic_string@DU?$char_traits@D@std@@V?$allocator@D@2@@std@@QAE@ID@Z 1000ef10 f i pdbio.obj
 0001:0000df40       ??0?$fpos@H@std@@QAE@H_J@Z 1000ef40 f i pdbio.obj
 0001:0000df70       ??0_Sentry_base@?$basic_istream@DU?$char_traits@D@std@@@std@@QAE@AAV12@@Z 1000ef70 f i pdbio.obj
 0001:0000dfa0       ??0invalid_argument@std@@QAE@ABV01@@Z 1000efa0 f i pdbio.obj
 0001:0000dfc0       ??0invalid_argument@std@@QAE@ABV?$basic_string@DU?$char_traits@D@std@@V?$allocator@D@2@@1@@Z 1000efc0 f i pdbio.obj
 0001:0000dff0       ??0sentry@?$basic_istream@DU?$char_traits@D@std@@@std@@QAE@AAV12@_N@Z 1000eff0 f i pdbio.obj
 0001:0000e060       ??1?$basic_filebuf@DU?$char_traits@D@std@@@std@@UAE@XZ 1000f060 f i pdbio.obj
 0001:0000e0b0       ??1?$basic_ifstream@DU?$char_traits@D@std@@@std@@UAE@XZ 1000f0b0 f i pdbio.obj
 0001:0000e120       ??1?$basic_ostringstream@DU?$char_traits@D@std@@V?$allocator@D@2@@std@@UAE@XZ 1000f120 f i pdbio.obj
 0001:0000e170       ??1_Sentry_base@?$basic_istream@DU?$char_traits@D@std@@@std@@QAE@XZ 1000f170 f i pdbio.obj
 0001:0000e190       ??1invalid_argument@std@@UAE@XZ 1000f190 f i pdbio.obj
 0001:0000e1a0       ??1locale@std@@QAE@XZ      1000f1a0 f i pdbio.obj
 0001:0000e1c0       ??1sentry@?$basic_istream@DU?$char_traits@D@std@@@std@@QAE@XZ 1000f1c0 f i pdbio.obj
 0001:0000e1e0       ??4?$basic_string@DU?$char_traits@D@std@@V?$allocator@D@2@@std@@QAEAAV01@$$QAV01@@Z 1000f1e0 f i pdbio.obj
 0001:0000e220       ??8?$_String_const_iterator@V?$_String_val@U?$_Simple_types@D@std@@@std@@@std@@QBE_NABV01@@Z 1000f220 f i pdbio.obj
 0001:0000e240       ??9?$_String_const_iterator@V?$_String_val@U?$_Simple_types@D@std@@@std@@@std@@QBE_NABV01@@Z 1000f240 f i pdbio.obj
 0001:0000e260       ??A?$basic_string@DU?$char_traits@D@std@@V?$allocator@D@2@@std@@QBEABDI@Z 1000f260 f i pdbio.obj
 0001:0000e280       ??Bsentry@?$basic_istream@DU?$char_traits@D@std@@@std@@QBE_NXZ 1000f280 f i pdbio.obj
 0001:0000e290       ??D?$_String_const_iterator@V?$_String_val@U?$_Simple_types@D@std@@@std@@@std@@QBEABDXZ 1000f290 f i pdbio.obj
 0001:0000e2a0       ??D?$_String_iterator@V?$_String_val@U?$_Simple_types@D@std@@@std@@@std@@QBEAADXZ 1000f2a0 f i pdbio.obj
 0001:0000e2b0       ??E?$_String_const_iterator@V?$_String_val@U?$_Simple_types@D@std@@@std@@@std@@QAEAAV01@XZ 1000f2b0 f i pdbio.obj
 0001:0000e2c0       ??E?$_String_iterator@V?$_String_val@U?$_Simple_types@D@std@@@std@@@std@@QAEAAV01@XZ 1000f2c0 f i pdbio.obj
 0001:0000e2d0       ??G?$_String_const_iterator@V?$_String_val@U?$_Simple_types@D@std@@@std@@@std@@QBEHABV01@@Z 1000f2d0 f i pdbio.obj
 0001:0000e2e0       ??G?$_String_iterator@V?$_String_val@U?$_Simple_types@D@std@@@std@@@std@@QBEHABV?$_String_const_iterator@V?$_String_val@U?$_Simple_types@D@std@@@std@@@1@@Z 1000f2e0 f i pdbio.obj
 0001:0000e2f0       ??Y?$basic_string@DU?$char_traits@D@std@@V?$allocator@D@2@@std@@QAEAAV01@ABV01@@Z 1000f2f0 f i pdbio.obj
 0001:0000e310       ??_D?$basic_ifstream@DU?$char_traits@D@std@@@std@@QAEXXZ 1000f310 f i pdbio.obj
 0001:0000e340       ??_D?$basic_ostringstream@DU?$char_traits@D@std@@V?$allocator@D@2@@std@@QAEXXZ 1000f340 f i pdbio.obj
 0001:0000e39b       ??_E?$basic_ifstream@DU?$char_traits@D@std@@@std@@$4PPPPPPPM@A@AEPAXI@Z 1000f39b f i pdbio.obj
 0001:0000e3a3       ??_E?$basic_ostringstream@DU?$char_traits@D@std@@V?$allocator@D@2@@std@@$4PPPPPPPM@A@AEPAXI@Z 1000f3a3 f i pdbio.obj
 0001:0000e3b0       ??_E?$basic_filebuf@DU?$char_traits@D@std@@@std@@UAEPAXI@Z 1000f3b0 f i pdbio.obj
 0001:0000e3b0       ??_G?$basic_filebuf@DU?$char_traits@D@std@@@std@@UAEPAXI@Z 1000f3b0 f i pdbio.obj
 0001:0000e410       ??_E?$basic_ifstream@DU?$char_traits@D@std@@@std@@UAEPAXI@Z 1000f410 f i pdbio.obj
 0001:0000e410       ??_G?$basic_ifstream@DU?$char_traits@D@std@@@std@@UAEPAXI@Z 1000f410 f i pdbio.obj
 0001:0000e460       ??_E?$basic_ostringstream@DU?$char_traits@D@std@@V?$allocator@D@2@@std@@UAEPAXI@Z 1000f460 f i pdbio.obj
 0001:0000e460       ??_G?$basic_ostringstream@DU?$char_traits@D@std@@V?$allocator@D@2@@std@@UAEPAXI@Z 1000f460 f i pdbio.obj
 0001:0000e490       ??_Ginvalid_argument@std@@UAEPAXI@Z 1000f490 f i pdbio.obj
 0001:0000e490       ??_Einvalid_argument@std@@UAEPAXI@Z 1000f490 f i pdbio.obj
 0001:0000e4c0       ?GetAtomId@Atomproperty@PTools@@QBEIXZ 1000f4c0 f i pdbio.obj
 0001:0000e4d0       ?GetChainId@Atomproperty@PTools@@QBE?AV?$basic_string@DU?$char_traits@D@std@@V?$allocator@D@2@@std@@XZ 1000f4d0 f i pdbio.obj
 0001:0000e510       ?GetExtra@Atomproperty@PTools@@QBE?AV?$basic_string@DU?$char_traits@D@std@@V?$allocator@D@2@@std@@XZ 1000f510 f i pdbio.obj
 0001:0000e550       ?GetResidId@Atomproperty@PTools@@QBEIXZ 1000f550 f i pdbio.obj
 0001:0000e560       ?GetResidType@Atomproperty@PTools@@QBE?AV?$basic_string@DU?$char_traits@D@std@@V?$allocator@D@2@@std@@XZ 1000f560 f i pdbio.obj
 0001:0000e5a0       ?GetType@Atomproperty@PTools@@QBE?AV?$basic_string@DU?$char_traits@D@std@@V?$allocator@D@2@@std@@XZ 1000f5a0 f i pdbio.obj
 0001:0000e5e0       ?ReadPDB@PTools@@YAXAAV?$basic_ifstream@DU?$char_traits@D@std@@@std@@AAVRigidbody@1@@Z 1000f5e0 f   pdbio.obj
 0001:0000ebd0       ?ReadPDB@PTools@@YAXV?$basic_string@DU?$char_traits@D@std@@V?$allocator@D@2@@std@@AAVRigidbody@1@@Z 1000fbd0 f   pdbio.obj
 0001:0000ed80       ?SetAtomId@Atomproperty@PTools@@QAEXI@Z 1000fd80 f i pdbio.obj
 0001:0000ed90       ?SetChainId@Atomproperty@PTools@@QAEXV?$basic_string@DU?$char_traits@D@std@@V?$allocator@D@2@@std@@@Z 1000fd90 f i pdbio.obj
 0001:0000edf0       ?SetExtra@Atomproperty@PTools@@QAEXV?$basic_string@DU?$char_traits@D@std@@V?$allocator@D@2@@std@@@Z 1000fdf0 f i pdbio.obj
 0001:0000ee50       ?SetResidType@Atomproperty@PTools@@QAEXV?$basic_string@DU?$char_traits@D@std@@V?$allocator@D@2@@std@@@Z 1000fe50 f i pdbio.obj
 0001:0000eeb0       ?WritePDB@PTools@@YAXABVRigidbody@1@V?$basic_string@DU?$char_traits@D@std@@V?$allocator@D@2@@std@@@Z 1000feb0 f   pdbio.obj
 0001:0000f160       ?_Compat@?$_String_const_iterator@V?$_String_val@U?$_Simple_types@D@std@@@std@@@std@@QBEXABV12@@Z 10010160 f i pdbio.obj
 0001:0000f170       ?_Endwrite@?$basic_filebuf@DU?$char_traits@D@std@@@std@@IAE_NXZ 10010170 f i pdbio.obj
 0001:0000f2c0       ?_Getfacet@locale@std@@QBEPBVfacet@12@I@Z 100102c0 f i pdbio.obj
 0001:0000f300       ?_Init@?$basic_filebuf@DU?$char_traits@D@std@@@std@@IAEXPAU_iobuf@@W4_Initfl@12@@Z 10010300 f i pdbio.obj
 0001:0000f350       ?_Initcvt@?$basic_filebuf@DU?$char_traits@D@std@@@std@@IAEXPBV?$codecvt@DDH@2@@Z 10010350 f i pdbio.obj
 0001:0000f390       ?_Lock@?$basic_filebuf@DU?$char_traits@D@std@@@std@@UAEXXZ 10010390 f i pdbio.obj
 0001:0000f3a0       ?_Pdif@?$basic_string@DU?$char_traits@D@std@@V?$allocator@D@2@@std@@SAIV?$_String_const_iterator@V?$_String_val@U?$_Simple_types@D@std@@@std@@@2@0@Z 100103a0 f i pdbio.obj
 0001:0000f3c0       ?_Reset_back@?$basic_filebuf@DU?$char_traits@D@std@@@std@@AAEXXZ 100103c0 f i pdbio.obj
 0001:0000f3f0       ?_Set_back@?$basic_filebuf@DU?$char_traits@D@std@@@std@@AAEXXZ 100103f0 f i pdbio.obj
 0001:0000f430       ?_Unchecked@?$_String_iterator@V?$_String_val@U?$_Simple_types@D@std@@@std@@@std@@QBEPADXZ 10010430 f i pdbio.obj
 0001:0000f440       ?_Unlock@?$basic_filebuf@DU?$char_traits@D@std@@@std@@UAEXXZ 10010440 f i pdbio.obj
 0001:0000f450       ?append@?$basic_string@DU?$char_traits@D@std@@V?$allocator@D@2@@std@@QAEAAV12@ABV12@@Z 10010450 f i pdbio.obj
 0001:0000f470       ?assign@?$basic_string@DU?$char_traits@D@std@@V?$allocator@D@2@@std@@QAEAAV12@ID@Z 10010470 f i pdbio.obj
 0001:0000f540       ?begin@?$basic_string@DU?$char_traits@D@std@@V?$allocator@D@2@@std@@QAE?AV?$_String_iterator@V?$_String_val@U?$_Simple_types@D@std@@@std@@@2@XZ 10010540 f i pdbio.obj
 0001:0000f560       ?close@?$basic_filebuf@DU?$char_traits@D@std@@@std@@QAEPAV12@XZ 10010560 f i pdbio.obj
 0001:0000f5c0       ?close@?$basic_ifstream@DU?$char_traits@D@std@@@std@@QAEXXZ 100105c0 f i pdbio.obj
 0001:0000f5f0       ?compare@?$basic_string@DU?$char_traits@D@std@@V?$allocator@D@2@@std@@QBEHABV12@@Z 100105f0 f i pdbio.obj
 0001:0000f620       ?compare@?$basic_string@DU?$char_traits@D@std@@V?$allocator@D@2@@std@@QBEHIIPBDI@Z 10010620 f i pdbio.obj
 0001:0000f690       ?compare@?$basic_string@DU?$char_traits@D@std@@V?$allocator@D@2@@std@@QBEHPBD@Z 10010690 f i pdbio.obj
 0001:0000f6d0       ?compare@?$char_traits@D@std@@SAHPBD0I@Z 100106d0 f i pdbio.obj
 0001:0000f740       ?end@?$basic_string@DU?$char_traits@D@std@@V?$allocator@D@2@@std@@QAE?AV?$_String_iterator@V?$_String_val@U?$_Simple_types@D@std@@@std@@@2@XZ 10010740 f i pdbio.obj
 0001:0000f770       ?find@?$char_traits@D@std@@SAPBDPBDIABD@Z 10010770 f i pdbio.obj
 0001:0000f7a0       ?find_first_not_of@?$basic_string@DU?$char_traits@D@std@@V?$allocator@D@2@@std@@QBEIPBDI@Z 100107a0 f i pdbio.obj
 0001:0000f7e0       ?find_first_not_of@?$basic_string@DU?$char_traits@D@std@@V?$allocator@D@2@@std@@QBEIPBDII@Z 100107e0 f i pdbio.obj
 0001:0000f870       ?find_last_not_of@?$basic_string@DU?$char_traits@D@std@@V?$allocator@D@2@@std@@QBEIPBDI@Z 10010870 f i pdbio.obj
 0001:0000f8b0       ?find_last_not_of@?$basic_string@DU?$char_traits@D@std@@V?$allocator@D@2@@std@@QBEIPBDII@Z 100108b0 f i pdbio.obj
 0001:0000f930       ?get_allocator@?$basic_string@DU?$char_traits@D@std@@V?$allocator@D@2@@std@@QBE?AV?$allocator@D@2@XZ 10010930 f i pdbio.obj
 0001:0000f940       ?imbue@?$basic_filebuf@DU?$char_traits@D@std@@@std@@MAEXABVlocale@2@@Z 10010940 f i pdbio.obj
 0001:0000f980       ?isAtom@PTools@@YA_NABV?$basic_string@DU?$char_traits@D@std@@V?$allocator@D@2@@std@@@Z 10010980 f   pdbio.obj
 0001:0000fa70       ?isHeteroAtom@PTools@@YA_NABV?$basic_string@DU?$char_traits@D@std@@V?$allocator@D@2@@std@@@Z 10010a70 f   pdbio.obj
 0001:0000fb30       ?open@?$basic_filebuf@DU?$char_traits@D@std@@@std@@QAEPAV12@PBDHH@Z 10010b30 f i pdbio.obj
 0001:0000fc40       ?overflow@?$basic_filebuf@DU?$char_traits@D@std@@@std@@MAEHH@Z 10010c40 f i pdbio.obj
 0001:0000fe30       ?pbackfail@?$basic_filebuf@DU?$char_traits@D@std@@@std@@MAEHH@Z 10010e30 f i pdbio.obj
 0001:0000fec0       ?readatomtype@PTools@@YA?AV?$basic_string@DU?$char_traits@D@std@@V?$allocator@D@2@@std@@ABV23@@Z 10010ec0 f   pdbio.obj
 0001:00010030       ?readresidtype@PTools@@YA?AV?$basic_string@DU?$char_traits@D@std@@V?$allocator@D@2@@std@@ABV23@@Z 10011030 f   pdbio.obj
 0001:000101a0       ?replace@?$basic_string@DU?$char_traits@D@std@@V?$allocator@D@2@@std@@QAEAAV12@IIABV12@II@Z 100111a0 f i pdbio.obj
 0001:00010500       ?replace@?$basic_string@DU?$char_traits@D@std@@V?$allocator@D@2@@std@@QAEAAV12@IIPBDI@Z 10011500 f i pdbio.obj
 0001:000106a0       ?replace@?$basic_string@DU?$char_traits@D@std@@V?$allocator@D@2@@std@@QAEAAV12@V?$_String_const_iterator@V?$_String_val@U?$_Simple_types@D@std@@@std@@@2@0V?$_String_iterator@V?$_String_val@U?$_Simple_types@D@std@@@std@@@2@1@Z 100116a0 f i pdbio.obj
 0001:00010730       ?reserve@?$basic_string@DU?$char_traits@D@std@@V?$allocator@D@2@@std@@QAEXI@Z 10011730 f i pdbio.obj
 0001:00010770       ?seekoff@?$basic_filebuf@DU?$char_traits@D@std@@@std@@MAE?AV?$fpos@H@2@_JHH@Z 10011770 f i pdbio.obj
 0001:00010870       ?seekpos@?$basic_filebuf@DU?$char_traits@D@std@@@std@@MAE?AV?$fpos@H@2@V32@H@Z 10011870 f i pdbio.obj
 0001:00010950       ?seekpos@?$fpos@H@std@@QBE_JXZ 10011950 f i pdbio.obj
 0001:00010960       ?setbuf@?$basic_filebuf@DU?$char_traits@D@std@@@std@@MAEPAV?$basic_streambuf@DU?$char_traits@D@std@@@2@PAD_J@Z 10011960 f i pdbio.obj
 0001:000109f0       ?state@?$fpos@H@std@@QBEHXZ 100119f0 f i pdbio.obj
 0001:00010a00       ?strip@PTools@@YA?AV?$basic_string@DU?$char_traits@D@std@@V?$allocator@D@2@@std@@ABV23@PBD@Z 10011a00 f   pdbio.obj
 0001:00010b80       ?substr@?$basic_string@DU?$char_traits@D@std@@V?$allocator@D@2@@std@@QBE?AV12@II@Z 10011b80 f i pdbio.obj
 0001:00010bc0       ?sync@?$basic_filebuf@DU?$char_traits@D@std@@@std@@MAEHXZ 10011bc0 f i pdbio.obj
 0001:00010bf0       ?uflow@?$basic_filebuf@DU?$char_traits@D@std@@@std@@MAEHXZ 10011bf0 f i pdbio.obj
 0001:00010de0       ?underflow@?$basic_filebuf@DU?$char_traits@D@std@@@std@@MAEHXZ 10011de0 f i pdbio.obj
 0001:00010e20       ??$?8V?$allocator@VAtomproperty@PTools@@@std@@V01@@std@@YA_NABU?$_Wrap_alloc@V?$allocator@VAtomproperty@PTools@@@std@@@0@0@Z 10011e20 f i rigidbody.obj
 0001:00010e30       ??$?8VAtomproperty@PTools@@V01@@std@@YA_NABV?$allocator@VAtomproperty@PTools@@@0@0@Z 10011e30 f i rigidbody.obj
 0001:00010e40       ??$?9V?$allocator@VAtomproperty@PTools@@@std@@V01@@std@@YA_NABU?$_Wrap_alloc@V?$allocator@VAtomproperty@PTools@@@std@@@0@0@Z 10011e40 f i rigidbody.obj
 0001:00010e50       ??$_Allocate@VAtomproperty@PTools@@@std@@YAPAVAtomproperty@PTools@@IPAV12@@Z 10011e50 f i rigidbody.obj
 0001:00010e90       ??$_Copy_impl@PAVAtomproperty@PTools@@PAV12@@std@@YAPAVAtomproperty@PTools@@PAV12@00@Z 10011e90 f i rigidbody.obj
 0001:00010eb0       ??$_Copy_impl@PAVAtomproperty@PTools@@PAV12@@std@@YAPAVAtomproperty@PTools@@PAV12@00U_Nonscalar_ptr_iterator_tag@0@@Z 10011eb0 f i rigidbody.obj
 0001:00010f80       ??$_Rechecked@PAVAtomproperty@PTools@@PAV12@@std@@YAAAPAVAtomproperty@PTools@@AAPAV12@PAV12@@Z 10011f80 f i rigidbody.obj
 0001:00010f90       ??$_Ucopy@PAVAtomproperty@PTools@@@?$vector@VAtomproperty@PTools@@V?$allocator@VAtomproperty@PTools@@@std@@@std@@IAEPAVAtomproperty@PTools@@PAV23@00@Z 10011f90 f i rigidbody.obj
 0001:00010fc0       ??$_Umove@PAUCoord3D@PTools@@@?$vector@UCoord3D@PTools@@V?$allocator@UCoord3D@PTools@@@std@@@std@@IAEPAUCoord3D@PTools@@PAU23@00@Z 10011fc0 f i rigidbody.obj
 0001:00010ff0       ??$_Umove@PAVAtomproperty@PTools@@@?$vector@VAtomproperty@PTools@@V?$allocator@VAtomproperty@PTools@@@std@@@std@@IAEPAVAtomproperty@PTools@@PAV23@00@Z 10011ff0 f i rigidbody.obj
 0001:00011020       ??$_Unchecked@PAVAtomproperty@PTools@@@std@@YAPAVAtomproperty@PTools@@PAV12@@Z 10012020 f i rigidbody.obj
 0001:00011030       ??$_Uninit_copy@PAVAtomproperty@PTools@@PAV12@U?$_Wrap_alloc@V?$allocator@VAtomproperty@PTools@@@std@@@std@@@std@@YAPAVAtomproperty@PTools@@PAV12@00AAU?$_Wrap_alloc@V?$allocator@VAtomproperty@PTools@@@std@@@0@@Z 10012030 f i rigidbody.obj
 0001:00011050       ??$_Uninit_copy@PAVAtomproperty@PTools@@PAV12@V?$allocator@VAtomproperty@PTools@@@std@@@std@@YAPAVAtomproperty@PTools@@PAV12@00AAU?$_Wrap_alloc@V?$allocator@VAtomproperty@PTools@@@std@@@0@U_Nonscalar_ptr_iterator_tag@0@@Z 10012050 f i rigidbody.obj
 0001:00011100       ??$_Uninit_move@PAUCoord3D@PTools@@PAU12@U?$_Wrap_alloc@V?$allocator@UCoord3D@PTools@@@std@@@std@@@std@@YAPAUCoord3D@PTools@@PAU12@00AAU?$_Wrap_alloc@V?$allocator@UCoord3D@PTools@@@std@@@0@@Z 10012100 f i rigidbody.obj
 0001:00011130       ??$_Uninit_move@PAUCoord3D@PTools@@PAU12@V?$allocator@UCoord3D@PTools@@@std@@U12@@std@@YAPAUCoord3D@PTools@@PAU12@00AAU?$_Wrap_alloc@V?$allocator@UCoord3D@PTools@@@std@@@0@0U_Nonscalar_ptr_iterator_tag@0@@Z 10012130 f i rigidbody.obj
 0001:00011170       ??$_Uninit_move@PAVAtomproperty@PTools@@PAV12@U?$_Wrap_alloc@V?$allocator@VAtomproperty@PTools@@@std@@@std@@@std@@YAPAVAtomproperty@PTools@@PAV12@00AAU?$_Wrap_alloc@V?$allocator@VAtomproperty@PTools@@@std@@@0@@Z 10012170 f i rigidbody.obj
 0001:000111a0       ??$_Uninit_move@PAVAtomproperty@PTools@@PAV12@V?$allocator@VAtomproperty@PTools@@@std@@V12@@std@@YAPAVAtomproperty@PTools@@PAV12@00AAU?$_Wrap_alloc@V?$allocator@VAtomproperty@PTools@@@std@@@0@0U_Nonscalar_ptr_iterator_tag@0@@Z 100121a0 f i rigidbody.obj
 0001:00011250       ??$_Uninitialized_copy@PAVAtomproperty@PTools@@PAV12@U?$_Wrap_alloc@V?$allocator@VAtomproperty@PTools@@@std@@@std@@@std@@YAPAVAtomproperty@PTools@@PAV12@00AAU?$_Wrap_alloc@V?$allocator@VAtomproperty@PTools@@@std@@@0@@Z 10012250 f i rigidbody.obj
 0001:00011270       ??$_Uninitialized_move@PAUCoord3D@PTools@@PAU12@U?$_Wrap_alloc@V?$allocator@UCoord3D@PTools@@@std@@@std@@@std@@YAPAUCoord3D@PTools@@PAU12@00AAU?$_Wrap_alloc@V?$allocator@UCoord3D@PTools@@@std@@@0@@Z 10012270 f i rigidbody.obj
 0001:00011290       ??$_Uninitialized_move@PAVAtomproperty@PTools@@PAV12@U?$_Wrap_alloc@V?$allocator@VAtomproperty@PTools@@@std@@@std@@@std@@YAPAVAtomproperty@PTools@@PAV12@00AAU?$_Wrap_alloc@V?$allocator@VAtomproperty@PTools@@@std@@@0@@Z 10012290 f i rigidbody.obj
 0001:000112b0       ??$_Val_type@PAUCoord3D@PTools@@@std@@YAPAUCoord3D@PTools@@PAU12@@Z 100122b0 f i rigidbody.obj
 0001:000112c0       ??$_Val_type@PAVAtomproperty@PTools@@@std@@YAPAVAtomproperty@PTools@@PAV12@@Z 100122c0 f i rigidbody.obj
 0001:000112d0       ??$addressof@$$CBUCoord3D@PTools@@@std@@YAPBUCoord3D@PTools@@ABU12@@Z 100122d0 f i rigidbody.obj
 0001:000112e0       ??$addressof@$$CBVAtomproperty@PTools@@@std@@YAPBVAtomproperty@PTools@@ABV12@@Z 100122e0 f i rigidbody.obj
 0001:000112f0       ??$construct@UCoord3D@PTools@@ABU12@@?$_Wrap_alloc@V?$allocator@UCoord3D@PTools@@@std@@@std@@QAEXPAUCoord3D@PTools@@ABU23@@Z 100122f0 f i rigidbody.obj
 0001:00011320       ??$construct@UCoord3D@PTools@@ABU12@@?$allocator_traits@V?$allocator@UCoord3D@PTools@@@std@@@std@@SAXAAV?$allocator@UCoord3D@PTools@@@1@PAUCoord3D@PTools@@ABU34@@Z 10012320 f i rigidbody.obj
 0001:00011350       ??$construct@UCoord3D@PTools@@U12@@?$_Wrap_alloc@V?$allocator@UCoord3D@PTools@@@std@@@std@@QAEXPAUCoord3D@PTools@@$$QAU23@@Z 10012350 f i rigidbody.obj
 0001:00011380       ??$construct@UCoord3D@PTools@@U12@@?$allocator@UCoord3D@PTools@@@std@@QAEXPAUCoord3D@PTools@@$$QAU23@@Z 10012380 f i rigidbody.obj
 0001:000113b0       ??$construct@UCoord3D@PTools@@U12@@?$allocator_traits@V?$allocator@UCoord3D@PTools@@@std@@@std@@SAXAAV?$allocator@UCoord3D@PTools@@@1@PAUCoord3D@PTools@@$$QAU34@@Z 100123b0 f i rigidbody.obj
 0001:000113e0       ??$construct@VAtomproperty@PTools@@AAV12@@?$_Wrap_alloc@V?$allocator@VAtomproperty@PTools@@@std@@@std@@QAEXPAVAtomproperty@PTools@@AAV23@@Z 100123e0 f i rigidbody.obj
 0001:00011430       ??$construct@VAtomproperty@PTools@@AAV12@@?$allocator@VAtomproperty@PTools@@@std@@QAEXPAVAtomproperty@PTools@@AAV23@@Z 10012430 f i rigidbody.obj
 0001:00011480       ??$construct@VAtomproperty@PTools@@AAV12@@?$allocator_traits@V?$allocator@VAtomproperty@PTools@@@std@@@std@@SAXAAV?$allocator@VAtomproperty@PTools@@@1@PAVAtomproperty@PTools@@AAV34@@Z 10012480 f i rigidbody.obj
 0001:000114d0       ??$construct@VAtomproperty@PTools@@ABV12@@?$_Wrap_alloc@V?$allocator@VAtomproperty@PTools@@@std@@@std@@QAEXPAVAtomproperty@PTools@@ABV23@@Z 100124d0 f i rigidbody.obj
 0001:00011520       ??$construct@VAtomproperty@PTools@@ABV12@@?$allocator_traits@V?$allocator@VAtomproperty@PTools@@@std@@@std@@SAXAAV?$allocator@VAtomproperty@PTools@@@1@PAVAtomproperty@PTools@@ABV34@@Z 10012520 f i rigidbody.obj
 0001:00011570       ??$construct@VAtomproperty@PTools@@V12@@?$_Wrap_alloc@V?$allocator@VAtomproperty@PTools@@@std@@@std@@QAEXPAVAtomproperty@PTools@@$$QAV23@@Z 10012570 f i rigidbody.obj
 0001:000115c0       ??$construct@VAtomproperty@PTools@@V12@@?$allocator@VAtomproperty@PTools@@@std@@QAEXPAVAtomproperty@PTools@@$$QAV23@@Z 100125c0 f i rigidbody.obj
 0001:00011610       ??$construct@VAtomproperty@PTools@@V12@@?$allocator_traits@V?$allocator@VAtomproperty@PTools@@@std@@@std@@SAXAAV?$allocator@VAtomproperty@PTools@@@1@PAVAtomproperty@PTools@@$$QAV34@@Z 10012610 f i rigidbody.obj
 0001:00011660       ??$forward@AAVAtomproperty@PTools@@@std@@YAAAVAtomproperty@PTools@@AAV12@@Z 10012660 f i rigidbody.obj
 0001:00011670       ??$forward@ABUCoord3D@PTools@@@std@@YAABUCoord3D@PTools@@ABU12@@Z 10012670 f i rigidbody.obj
 0001:00011680       ??$forward@ABVAtomproperty@PTools@@@std@@YAABVAtomproperty@PTools@@ABV12@@Z 10012680 f i rigidbody.obj
 0001:00011690       ??$forward@UCoord3D@PTools@@@std@@YA$$QAUCoord3D@PTools@@AAU12@@Z 10012690 f i rigidbody.obj
 0001:000116a0       ??$forward@VAtomproperty@PTools@@@std@@YA$$QAVAtomproperty@PTools@@AAV12@@Z 100126a0 f i rigidbody.obj
 0001:000116b0       ??0?$_Vector_alloc@$0A@U?$_Vec_base_types@VAtomproperty@PTools@@V?$allocator@VAtomproperty@PTools@@@std@@@std@@@std@@QAE@ABV?$allocator@VAtomproperty@PTools@@@1@@Z 100126b0 f i rigidbody.obj
 0001:000116d0       ??0?$_Vector_val@U?$_Simple_types@VAtomproperty@PTools@@@std@@@std@@QAE@XZ 100126d0 f i rigidbody.obj
 0001:000116f0       ??0?$allocator@VAtomproperty@PTools@@@std@@QAE@ABV01@@Z 100126f0 f i rigidbody.obj
 0001:00011700       ??0?$vector@VAtomproperty@PTools@@V?$allocator@VAtomproperty@PTools@@@std@@@std@@QAE@XZ 10012700 f i rigidbody.obj
 0001:00011720       ??0Atom@PTools@@QAE@ABV01@@Z 10012720 f i rigidbody.obj
 0001:00011770       ??0Rigidbody@PTools@@QAE@ABV01@@Z 10012770 f   rigidbody.obj
 0001:00011870       ??0Rigidbody@PTools@@QAE@V?$basic_string@DU?$char_traits@D@std@@V?$allocator@D@2@@std@@@Z 10012870 f   rigidbody.obj
 0001:00011970       ??0Rigidbody@PTools@@QAE@XZ 10012970 f   rigidbody.obj
 0001:00011a30       ??4?$vector@VAtomproperty@PTools@@V?$allocator@VAtomproperty@PTools@@@std@@@std@@QAEAAV01@ABV01@@Z 10012a30 f i rigidbody.obj
 0001:00011be0       ??4Atomproperty@PTools@@QAEAAV01@ABV01@@Z 10012be0 f i rigidbody.obj
 0001:00011c70       ??A?$QVector@N@@QBEABNH@Z  10012c70 f i rigidbody.obj
 0001:00011c90       ??A?$vector@VAtomproperty@PTools@@V?$allocator@VAtomproperty@PTools@@@std@@@std@@QAEAAVAtomproperty@PTools@@I@Z 10012c90 f i rigidbody.obj
 0001:00011ca0       ??A?$vector@VAtomproperty@PTools@@V?$allocator@VAtomproperty@PTools@@@std@@@std@@QBEABVAtomproperty@PTools@@I@Z 10012ca0 f i rigidbody.obj
 0001:00011cb0       ??DPTools@@YA?AUCoord3D@0@ABU10@N@Z 10012cb0 f i rigidbody.obj
 0001:00011ce0       ??DPTools@@YA?AUCoord3D@0@NABU10@@Z 10012ce0 f i rigidbody.obj
 0001:00011d10       ??HRigidbody@PTools@@QAE?AV01@ABV01@@Z 10012d10 f   rigidbody.obj
 0001:00011f70       ??R?$Array2D@N@@QBEABNHH@Z 10012f70 f i rigidbody.obj
 0001:00011f90       ?ABrotate@Rigidbody@PTools@@QAEXABUCoord3D@2@0N@Z 10012f90 f   rigidbody.obj
 0001:00012000       ?AddAtom@Rigidbody@PTools@@QAEXABVAtom@2@@Z 10013000 f   rigidbody.obj
 0001:000120e0       ?AddAtom@Rigidbody@PTools@@QAEXABVAtomproperty@2@UCoord3D@2@@Z 100130e0 f   rigidbody.obj
 0001:00012130       ?AddCoord@CoordsArray@PTools@@QAEXABUCoord3D@2@@Z 10013130 f i rigidbody.obj
 0001:00012160       ?ApplyMatrix@Rigidbody@PTools@@QAEXABV?$Array2D@N@@@Z 10013160 f   rigidbody.obj
 0001:00012200       ?AttractEulerRotate@Rigidbody@PTools@@QAEXNNN@Z 10013200 f   rigidbody.obj
 0001:00012240       ?Backbone@Rigidbody@PTools@@QAE?AVAtomSelection@2@XZ 10013240 f   rigidbody.obj
 0001:00012400       ?CA@Rigidbody@PTools@@QAE?AVAtomSelection@2@XZ 10013400 f   rigidbody.obj
 0001:00012450       ?CenterToOrigin@Rigidbody@PTools@@QAEXXZ 10013450 f   rigidbody.obj
 0001:000124a0       ?CopyAtom@Rigidbody@PTools@@UBE?AVAtom@2@I@Z 100134a0 f   rigidbody.obj
 0001:00012560       ?FindCenter@Rigidbody@PTools@@QBE?AUCoord3D@2@XZ 10013560 f   rigidbody.obj
 0001:00012690       ?GetCoords@Rigidbody@PTools@@QBE?AUCoord3D@2@I@Z 10013690 f i rigidbody.obj
 0001:000126c0       ?Norm2@PTools@@YANABUCoord3D@1@@Z 100136c0 f i rigidbody.obj
 0001:00012700       ?Radius@Rigidbody@PTools@@QAENXZ 10013700 f   rigidbody.obj
 0001:000127c0       ?RadiusGyration@Rigidbody@PTools@@QAENXZ 100137c0 f   rigidbody.obj
 0001:000128d0       ?SelectAllAtoms@Rigidbody@PTools@@QBE?AVAtomSelection@2@XZ 100138d0 f   rigidbody.obj
 0001:000129e0       ?SelectAtomType@Rigidbody@PTools@@QAE?AVAtomSelection@2@V?$basic_string@DU?$char_traits@D@std@@V?$allocator@D@2@@std@@@Z 100139e0 f   rigidbody.obj
 0001:00012bf0       ?SelectChainId@Rigidbody@PTools@@QAE?AVAtomSelection@2@V?$basic_string@DU?$char_traits@D@std@@V?$allocator@D@2@@std@@@Z 10013bf0 f   rigidbody.obj
 0001:00012e00       ?SelectResRange@Rigidbody@PTools@@QAE?AVAtomSelection@2@II@Z 10013e00 f   rigidbody.obj
 0001:00012f40       ?SelectResidType@Rigidbody@PTools@@QAE?AVAtomSelection@2@V?$basic_string@DU?$char_traits@D@std@@V?$allocator@D@2@@std@@@Z 10013f40 f   rigidbody.obj
 0001:00013150       ?SetAtom@Rigidbody@PTools@@QAEXIABVAtom@2@@Z 10014150 f   rigidbody.obj
 0001:000132b0       ?SetAtomProperty@Rigidbody@PTools@@QAEXIABVAtomproperty@2@@Z 100142b0 f i rigidbody.obj
 0001:000132d0       ?SetCoords@Rigidbody@PTools@@QAEXIABUCoord3D@2@@Z 100142d0 f i rigidbody.obj
 0001:000132e0       ?Translate@Rigidbody@PTools@@QAEXABUCoord3D@2@@Z 100142e0 f   rigidbody.obj
 0001:000132f0       ?_Buy@?$vector@VAtomproperty@PTools@@V?$allocator@VAtomproperty@PTools@@@std@@@std@@IAE_NI@Z 100142f0 f i rigidbody.obj
 0001:00013360       ?_Change_alloc@?$_Vector_alloc@$0A@U?$_Vec_base_types@VAtomproperty@PTools@@V?$allocator@VAtomproperty@PTools@@@std@@@std@@@std@@QAEXABU?$_Wrap_alloc@V?$allocator@VAtomproperty@PTools@@@std@@@2@@Z 10014360 f i rigidbody.obj
 0001:00013370       ?_Grow_to@?$vector@UCoord3D@PTools@@V?$allocator@UCoord3D@PTools@@@std@@@std@@IBEII@Z 10014370 f i rigidbody.obj
 0001:000133c0       ?_Grow_to@?$vector@VAtomproperty@PTools@@V?$allocator@VAtomproperty@PTools@@@std@@@std@@IBEII@Z 100143c0 f i rigidbody.obj
 0001:00013410       ?_Inside@?$vector@UCoord3D@PTools@@V?$allocator@UCoord3D@PTools@@@std@@@std@@IBE_NPBUCoord3D@PTools@@@Z 10014410 f i rigidbody.obj
 0001:00013430       ?_Inside@?$vector@VAtomproperty@PTools@@V?$allocator@VAtomproperty@PTools@@@std@@@std@@IBE_NPBVAtomproperty@PTools@@@Z 10014430 f i rigidbody.obj
 0001:00013450       ?_Orphan_range@?$vector@UCoord3D@PTools@@V?$allocator@UCoord3D@PTools@@@std@@@std@@IBEXPAUCoord3D@PTools@@0@Z 10014450 f i rigidbody.obj
 0001:00013460       ?_Orphan_range@?$vector@VAtomproperty@PTools@@V?$allocator@VAtomproperty@PTools@@@std@@@std@@IBEXPAVAtomproperty@PTools@@0@Z 10014460 f i rigidbody.obj
 0001:00013470       ?_Reallocate@?$vector@UCoord3D@PTools@@V?$allocator@UCoord3D@PTools@@@std@@@std@@IAEXI@Z 10014470 f i rigidbody.obj
 0001:00013560       ?_Reallocate@?$vector@VAtomproperty@PTools@@V?$allocator@VAtomproperty@PTools@@@std@@@std@@IAEXI@Z 10014560 f i rigidbody.obj
 0001:00013670       ?_Reserve@?$vector@UCoord3D@PTools@@V?$allocator@UCoord3D@PTools@@@std@@@std@@IAEXI@Z 10014670 f i rigidbody.obj
 0001:00013720       ?_Reserve@?$vector@VAtomproperty@PTools@@V?$allocator@VAtomproperty@PTools@@@std@@@std@@IAEXI@Z 10014720 f i rigidbody.obj
 0001:000137d0       ?_Unused_capacity@?$vector@UCoord3D@PTools@@V?$allocator@UCoord3D@PTools@@@std@@@std@@QBEIXZ 100147d0 f i rigidbody.obj
 0001:000137f0       ?_Unused_capacity@?$vector@VAtomproperty@PTools@@V?$allocator@VAtomproperty@PTools@@@std@@@std@@QBEIXZ 100147f0 f i rigidbody.obj
 0001:00013810       ?_Xlen@?$vector@VAtomproperty@PTools@@V?$allocator@VAtomproperty@PTools@@@std@@@std@@IBEXXZ 10014810 f i rigidbody.obj
 0001:00013820       ?allocate@?$_Wrap_alloc@V?$allocator@VAtomproperty@PTools@@@std@@@std@@QAEPAVAtomproperty@PTools@@I@Z 10014820 f i rigidbody.obj
 0001:00013860       ?allocate@?$allocator@VAtomproperty@PTools@@@std@@QAEPAVAtomproperty@PTools@@I@Z 10014860 f i rigidbody.obj
 0001:000138a0       ?capacity@?$vector@VAtomproperty@PTools@@V?$allocator@VAtomproperty@PTools@@@std@@@std@@QBEIXZ 100148a0 f i rigidbody.obj
 0001:000138c0       ?clear@?$vector@VAtomproperty@PTools@@V?$allocator@VAtomproperty@PTools@@@std@@@std@@QAEXXZ 100148c0 f i rigidbody.obj
 0001:00013900       ?construct@?$allocator@UCoord3D@PTools@@@std@@QAEXPAUCoord3D@PTools@@ABU34@@Z 10014900 f i rigidbody.obj
 0001:00013930       ?construct@?$allocator@VAtomproperty@PTools@@@std@@QAEXPAVAtomproperty@PTools@@ABV34@@Z 10014930 f i rigidbody.obj
 0001:00013980       ?empty@?$vector@VAtomproperty@PTools@@V?$allocator@VAtomproperty@PTools@@@std@@@std@@QBE_NXZ 10014980 f i rigidbody.obj
 0001:00013990       ?isBackbone@PTools@@YA_NABV?$basic_string@DU?$char_traits@D@std@@V?$allocator@D@2@@std@@@Z 10014990 f   rigidbody.obj
 0001:00013b60       ?max_size@?$_Wrap_alloc@V?$allocator@VAtomproperty@PTools@@@std@@@std@@QBEIXZ 10014b60 f i rigidbody.obj
 0001:00013b70       ?max_size@?$allocator@VAtomproperty@PTools@@@std@@QBEIXZ 10014b70 f i rigidbody.obj
 0001:00013b80       ?max_size@?$allocator_traits@V?$allocator@VAtomproperty@PTools@@@std@@@std@@SAIABV?$allocator@VAtomproperty@PTools@@@2@@Z 10014b80 f i rigidbody.obj
 0001:00013b90       ?max_size@?$vector@VAtomproperty@PTools@@V?$allocator@VAtomproperty@PTools@@@std@@@std@@QBEIXZ 10014b90 f i rigidbody.obj
 0001:00013ba0       ?push_back@?$vector@UCoord3D@PTools@@V?$allocator@UCoord3D@PTools@@@std@@@std@@QAEXABUCoord3D@PTools@@@Z 10014ba0 f i rigidbody.obj
 0001:00013c50       ?push_back@?$vector@VAtomproperty@PTools@@V?$allocator@VAtomproperty@PTools@@@std@@@std@@QAEXABVAtomproperty@PTools@@@Z 10014c50 f i rigidbody.obj
 0001:00013d10       ?size@?$vector@VAtomproperty@PTools@@V?$allocator@VAtomproperty@PTools@@@std@@@std@@QBEIXZ 10014d10 f i rigidbody.obj
 0001:00013d30       ??0invalid_argument@std@@QAE@PBD@Z 10014d30 f i rmsd.obj
 0001:00013d60       ??A?$vector@IV?$allocator@I@std@@@std@@QBEABII@Z 10014d60 f i rmsd.obj
 0001:00013d70       ?CopyAtom@AtomSelection@PTools@@QBE?AVAtom@2@I@Z 10014d70 f i rmsd.obj
 0001:00013da0       ?Dist2@PTools@@YANABVAtom@1@0@Z 10014da0 f i rmsd.obj
 0001:00013e00       ?Rmsd@PTools@@YANABVAtomSelection@1@0@Z 10014e00 f   rmsd.obj
 0001:00013fe0       ??$_Allocate@N@std@@YAPANIPAN@Z 10014fe0 f i superpose.obj
 0001:00014010       ??$_Allocate@V?$vector@NV?$allocator@N@std@@@std@@@std@@YAPAV?$vector@NV?$allocator@N@std@@@0@IPAV10@@Z 10015010 f i superpose.obj
 0001:00014050       ??$_Destroy_range@U?$_Wrap_alloc@V?$allocator@N@std@@@std@@@std@@YAXPAN0AAU?$_Wrap_alloc@V?$allocator@N@std@@@0@@Z 10015050 f i superpose.obj
 0001:00014060       ??$_Destroy_range@U?$_Wrap_alloc@V?$allocator@N@std@@@std@@@std@@YAXPAN0AAU?$_Wrap_alloc@V?$allocator@N@std@@@0@U_Scalar_ptr_iterator_tag@0@@Z 10015060 f i superpose.obj
 0001:00014070       ??$_Destroy_range@U?$_Wrap_alloc@V?$allocator@V?$vector@NV?$allocator@N@std@@@std@@@std@@@std@@@std@@YAXPAV?$vector@NV?$allocator@N@std@@@0@0AAU?$_Wrap_alloc@V?$allocator@V?$vector@NV?$allocator@N@std@@@std@@@std@@@0@@Z 10015070 f i superpose.obj
 0001:00014090       ??$_Destroy_range@U?$_Wrap_alloc@V?$allocator@V?$vector@NV?$allocator@N@std@@@std@@@std@@@std@@@std@@YAXPAV?$vector@NV?$allocator@N@std@@@0@0AAU?$_Wrap_alloc@V?$allocator@V?$vector@NV?$allocator@N@std@@@std@@@std@@@0@U_Nonscalar_ptr_iterator_tag@0@@Z 10015090 f i superpose.obj
 0001:000140d0       ??$_Fill_n@PANIN@std@@YAPANPANIABN@Z 100150d0 f i superpose.obj
 0001:000140f0       ??$_Move@AAPAU?$QTypedArrayData@N@@@std@@YA$$QAPAU?$QTypedArrayData@N@@AAPAU1@@Z 100150f0 f i superpose.obj
 0001:00014100       ??$_Ptr_cat@NN@std@@YA?AU_Scalar_ptr_iterator_tag@0@PAN0@Z 10015100 f i superpose.obj
 0001:00014110       ??$_Ptr_cat@NN@std@@YA?AU_Scalar_ptr_iterator_tag@0@PBNPAN@Z 10015110 f i superpose.obj
 0001:00014120       ??$_Ptr_cat@V?$vector@NV?$allocator@N@std@@@std@@V12@@std@@YA?AU_Nonscalar_ptr_iterator_tag@0@PAV?$vector@NV?$allocator@N@std@@@0@0@Z 10015120 f i superpose.obj
 0001:00014130       ??$_Rechecked@PANPAN@std@@YAAAPANAAPANPAN@Z 10015130 f i superpose.obj
 0001:00014140       ??$_Ucopy@V?$_Vector_const_iterator@V?$_Vector_val@U?$_Simple_types@N@std@@@std@@@std@@@?$vector@NV?$allocator@N@std@@@std@@IAEPANV?$_Vector_const_iterator@V?$_Vector_val@U?$_Simple_types@N@std@@@std@@@1@0PAN@Z 10015140 f i superpose.obj
 0001:00014170       ??$_Unchecked@PAN@std@@YAPANPAN@Z 10015170 f i superpose.obj
 0001:00014180       ??$_Unchecked@V?$_Vector_val@U?$_Simple_types@N@std@@@std@@@std@@YAPBNV?$_Vector_const_iterator@V?$_Vector_val@U?$_Simple_types@N@std@@@std@@@0@@Z 10015180 f i superpose.obj
 0001:00014190       ??$_Uninit_copy@$$CBNN@std@@YAPANPBN0PANAAU?$_Wrap_alloc@V?$allocator@N@std@@@0@U_Scalar_ptr_iterator_tag@0@@Z 10015190 f i superpose.obj
 0001:000141c0       ??$_Uninit_copy@PBNPANU?$_Wrap_alloc@V?$allocator@N@std@@@std@@@std@@YAPANPBN0PANAAU?$_Wrap_alloc@V?$allocator@N@std@@@0@@Z 100151c0 f i superpose.obj
 0001:000141f0       ??$_Uninit_def_fill_n@NIN@std@@YAXPANIAAU?$_Wrap_alloc@V?$allocator@N@std@@@0@0U_Scalar_ptr_iterator_tag@0@@Z 100151f0 f i superpose.obj
 0001:00014210       ??$_Uninit_fill_n@PAV?$vector@NV?$allocator@N@std@@@std@@IV12@V?$allocator@V?$vector@NV?$allocator@N@std@@@std@@@2@V12@@std@@YAXPAV?$vector@NV?$allocator@N@std@@@0@IPBV10@AAU?$_Wrap_alloc@V?$allocator@V?$vector@NV?$allocator@N@std@@@std@@@std@@@0@0U_Nonscalar_ptr_iterator_tag@0@@Z 10015210 f i superpose.obj
 0001:000142b0       ??$_Uninitialized_copy@V?$_Vector_const_iterator@V?$_Vector_val@U?$_Simple_types@N@std@@@std@@@std@@PANU?$_Wrap_alloc@V?$allocator@N@std@@@2@@std@@YAPANV?$_Vector_const_iterator@V?$_Vector_val@U?$_Simple_types@N@std@@@std@@@0@0PANAAU?$_Wrap_alloc@V?$allocator@N@std@@@0@@Z 100152b0 f i superpose.obj
 0001:000142e0       ??$_Uninitialized_default_fill_n@PANIU?$_Wrap_alloc@V?$allocator@N@std@@@std@@@std@@YAXPANIAAU?$_Wrap_alloc@V?$allocator@N@std@@@0@@Z 100152e0 f i superpose.obj
 0001:00014300       ??$_Uninitialized_fill_n@PAV?$vector@NV?$allocator@N@std@@@std@@IV12@U?$_Wrap_alloc@V?$allocator@V?$vector@NV?$allocator@N@std@@@std@@@std@@@2@@std@@YAXPAV?$vector@NV?$allocator@N@std@@@0@IPBV10@AAU?$_Wrap_alloc@V?$allocator@V?$vector@NV?$allocator@N@std@@@std@@@std@@@0@@Z 10015300 f i superpose.obj
 0001:00014330       ??$_Val_type@PAN@std@@YAPANPAN@Z 10015330 f i superpose.obj
 0001:00014340       ??$_Val_type@PAV?$vector@NV?$allocator@N@std@@@std@@@std@@YAPAV?$vector@NV?$allocator@N@std@@@0@PAV10@@Z 10015340 f i superpose.obj
 0001:00014350       ??$addressof@$$CBV?$vector@NV?$allocator@N@std@@@std@@@std@@YAPBV?$vector@NV?$allocator@N@std@@@0@ABV10@@Z 10015350 f i superpose.obj
 0001:00014360       ??$construct@V?$vector@NV?$allocator@N@std@@@std@@ABV12@@?$_Wrap_alloc@V?$allocator@V?$vector@NV?$allocator@N@std@@@std@@@std@@@std@@QAEXPAV?$vector@NV?$allocator@N@std@@@1@ABV21@@Z 10015360 f i superpose.obj
 0001:000143b0       ??$construct@V?$vector@NV?$allocator@N@std@@@std@@ABV12@@?$allocator_traits@V?$allocator@V?$vector@NV?$allocator@N@std@@@std@@@std@@@std@@SAXAAV?$allocator@V?$vector@NV?$allocator@N@std@@@std@@@1@PAV?$vector@NV?$allocator@N@std@@@1@ABV31@@Z 100153b0 f i superpose.obj
 0001:00014400       ??$destroy@V?$vector@NV?$allocator@N@std@@@std@@@?$_Wrap_alloc@V?$allocator@V?$vector@NV?$allocator@N@std@@@std@@@std@@@std@@QAEXPAV?$vector@NV?$allocator@N@std@@@1@@Z 10015400 f i superpose.obj
 0001:00014430       ??$destroy@V?$vector@NV?$allocator@N@std@@@std@@@?$allocator@V?$vector@NV?$allocator@N@std@@@std@@@std@@QAEXPAV?$vector@NV?$allocator@N@std@@@1@@Z 10015430 f i superpose.obj
 0001:00014460       ??$destroy@V?$vector@NV?$allocator@N@std@@@std@@@?$allocator_traits@V?$allocator@V?$vector@NV?$allocator@N@std@@@std@@@std@@@std@@SAXAAV?$allocator@V?$vector@NV?$allocator@N@std@@@std@@@1@PAV?$vector@NV?$allocator@N@std@@@1@@Z 10015460 f i superpose.obj
 0001:00014490       ??$forward@ABV?$vector@NV?$allocator@N@std@@@std@@@std@@YAABV?$vector@NV?$allocator@N@std@@@0@ABV10@@Z 10015490 f i superpose.obj
 0001:000144a0       ??$qSwap@PAU?$QTypedArrayData@N@@@@YAXAAPAU?$QTypedArrayData@N@@0@Z 100154a0 f i superpose.obj
 0001:000144c0       ??$swap@PAU?$QTypedArrayData@N@@@std@@YAXAAPAU?$QTypedArrayData@N@@0@Z 100154c0 f i superpose.obj
 0001:000144e0       ??0?$Array2D@N@@QAE@XZ     100154e0 f i superpose.obj
 0001:00014500       ??0?$_Vector_alloc@$0A@U?$_Vec_base_types@NV?$allocator@N@std@@@std@@@std@@QAE@ABV?$allocator@N@1@@Z 10015500 f i superpose.obj
 0001:00014520       ??0?$_Vector_alloc@$0A@U?$_Vec_base_types@V?$vector@NV?$allocator@N@std@@@std@@V?$allocator@V?$vector@NV?$allocator@N@std@@@std@@@2@@std@@@std@@QAE@ABV?$allocator@V?$vector@NV?$allocator@N@std@@@std@@@1@@Z 10015520 f i superpose.obj
 0001:00014540       ??0?$_Vector_const_iterator@V?$_Vector_val@U?$_Simple_types@N@std@@@std@@@std@@QAE@PANPBU_Container_base0@1@@Z 10015540 f i superpose.obj
 0001:00014550       ??0?$_Vector_val@U?$_Simple_types@N@std@@@std@@QAE@XZ 10015550 f i superpose.obj
 0001:00014570       ??0?$_Vector_val@U?$_Simple_types@V?$vector@NV?$allocator@N@std@@@std@@@std@@@std@@QAE@XZ 10015570 f i superpose.obj
 0001:00014590       ??0?$_Wrap_alloc@V?$allocator@N@std@@@std@@QAE@ABV?$allocator@N@1@@Z 10015590 f i superpose.obj
 0001:000145a0       ??0?$_Wrap_alloc@V?$allocator@N@std@@@std@@QAE@XZ 100155a0 f i superpose.obj
 0001:000145b0       ??0?$_Wrap_alloc@V?$allocator@V?$vector@NV?$allocator@N@std@@@std@@@std@@@std@@QAE@XZ 100155b0 f i superpose.obj
 0001:000145c0       ??0?$allocator@N@std@@QAE@ABV01@@Z 100155c0 f i superpose.obj
 0001:000145d0       ??0?$allocator@N@std@@QAE@XZ 100155d0 f i superpose.obj
 0001:000145e0       ??0?$allocator@V?$vector@NV?$allocator@N@std@@@std@@@std@@QAE@XZ 100155e0 f i superpose.obj
 0001:000145f0       ??0?$vector@NV?$allocator@N@std@@@std@@QAE@ABV01@@Z 100155f0 f i superpose.obj
 0001:00014650       ??0?$vector@NV?$allocator@N@std@@@std@@QAE@I@Z 10015650 f i superpose.obj
 0001:000146a0       ??0?$vector@V?$vector@NV?$allocator@N@std@@@std@@V?$allocator@V?$vector@NV?$allocator@N@std@@@std@@@2@@std@@QAE@IABV?$vector@NV?$allocator@N@std@@@1@@Z 100156a0 f i superpose.obj
 0001:000146d0       ??0Screw@PTools@@QAE@ABU01@@Z 100156d0 f i superpose.obj
 0001:00014730       ??0Screw@PTools@@QAE@XZ    10015730 f i superpose.obj
 0001:00014750       ??0Superpose_t@@QAE@ABU0@@Z 10015750 f i superpose.obj
 0001:00014790       ??0Superpose_t@@QAE@XZ     10015790 f i superpose.obj
 0001:000147b0       ??0runtime_error@std@@QAE@ABV01@@Z 100157b0 f i superpose.obj
 0001:000147d0       ??0runtime_error@std@@QAE@ABV?$basic_string@DU?$char_traits@D@std@@V?$allocator@D@2@@1@@Z 100157d0 f i superpose.obj
 0001:00014800       ??1?$vector@NV?$allocator@N@std@@@std@@QAE@XZ 10015800 f i superpose.obj
 0001:00014830       ??1?$vector@V?$vector@NV?$allocator@N@std@@@std@@V?$allocator@V?$vector@NV?$allocator@N@std@@@std@@@2@@std@@QAE@XZ 10015830 f i superpose.obj
 0001:00014880       ??1runtime_error@std@@UAE@XZ 10015880 f i superpose.obj
 0001:00014890       ??4?$Array2D@N@@QAEAAV0@ABV0@@Z 10015890 f i superpose.obj
 0001:000148c0       ??4?$QVector@N@@QAEAAV0@ABV0@@Z 100158c0 f i superpose.obj
 0001:00014930       ??A?$vector@NV?$allocator@N@std@@@std@@QAEAANI@Z 10015930 f i superpose.obj
 0001:00014940       ??A?$vector@V?$vector@NV?$allocator@N@std@@@std@@V?$allocator@V?$vector@NV?$allocator@N@std@@@std@@@2@@std@@QAEAAV?$vector@NV?$allocator@N@std@@@1@I@Z 10015940 f i superpose.obj
 0001:00014960       ??KPTools@@YA?AUCoord3D@0@ABU10@N@Z 10015960 f i superpose.obj
 0001:000149a0       ??_G?$vector@NV?$allocator@N@std@@@std@@QAEPAXI@Z 100159a0 f i superpose.obj
 0001:000149e0       ??_Gruntime_error@std@@UAEPAXI@Z 100159e0 f i superpose.obj
 0001:000149e0       ??_Eruntime_error@std@@UAEPAXI@Z 100159e0 f i superpose.obj
 0001:00014ef0       ?Mat44toMat33trans@PTools@@YAXQAY03NQAY02NAAUCoord3D@1@@Z 10015ef0 f   superpose.obj
 0001:00014f80       ?MatTrans2screw@PTools@@YA?AUScrew@1@ABV?$Array2D@N@@@Z 10015f80 f   superpose.obj
 0001:00015870       ?Rotate@PTools@@YAXAAVRigidbody@1@QAY02N@Z 10016870 f   superpose.obj
 0001:00015ad0       ?_Buy@?$vector@NV?$allocator@N@std@@@std@@IAE_NI@Z 10016ad0 f i superpose.obj
 0001:00015b40       ?_Buy@?$vector@V?$vector@NV?$allocator@N@std@@@std@@V?$allocator@V?$vector@NV?$allocator@N@std@@@std@@@2@@std@@IAE_NI@Z 10016b40 f i superpose.obj
 0001:00015bb0       ?_Construct_n@?$vector@V?$vector@NV?$allocator@N@std@@@std@@V?$allocator@V?$vector@NV?$allocator@N@std@@@std@@@2@@std@@QAEXIPBV?$vector@NV?$allocator@N@std@@@2@@Z 10016bb0 f i superpose.obj
 0001:00015c40       ?_Destroy@?$vector@NV?$allocator@N@std@@@std@@IAEXPAN0@Z 10016c40 f i superpose.obj
 0001:00015c50       ?_Destroy@?$vector@V?$vector@NV?$allocator@N@std@@@std@@V?$allocator@V?$vector@NV?$allocator@N@std@@@std@@@2@@std@@IAEXPAV?$vector@NV?$allocator@N@std@@@2@0@Z 10016c50 f i superpose.obj
 0001:00015c70       ?_Getal@?$_Vector_alloc@$0A@U?$_Vec_base_types@NV?$allocator@N@std@@@std@@@std@@QBE?AU?$_Wrap_alloc@V?$allocator@N@std@@@2@XZ 10016c70 f i superpose.obj
 0001:00015c80       ?_Getal@?$_Vector_alloc@$0A@U?$_Vec_base_types@V?$vector@NV?$allocator@N@std@@@std@@V?$allocator@V?$vector@NV?$allocator@N@std@@@std@@@2@@std@@@std@@QBE?AU?$_Wrap_alloc@V?$allocator@V?$vector@NV?$allocator@N@std@@@std@@@std@@@2@XZ 10016c80 f i superpose.obj
 0001:00015c90       ?_Tidy@?$vector@NV?$allocator@N@std@@@std@@IAEXXZ 10016c90 f i superpose.obj
 0001:00015cc0       ?_Tidy@?$vector@V?$vector@NV?$allocator@N@std@@@std@@V?$allocator@V?$vector@NV?$allocator@N@std@@@std@@@2@@std@@IAEXXZ 10016cc0 f i superpose.obj
 0001:00015d10       ?_Ufill@?$vector@V?$vector@NV?$allocator@N@std@@@std@@V?$allocator@V?$vector@NV?$allocator@N@std@@@std@@@2@@std@@IAEPAV?$vector@NV?$allocator@N@std@@@2@PAV32@IPBV32@@Z 10016d10 f i superpose.obj
 0001:00015d40       ?_Unchecked@?$_Vector_const_iterator@V?$_Vector_val@U?$_Simple_types@N@std@@@std@@@std@@QBEPBNXZ 10016d40 f i superpose.obj
 0001:00015d50       ?_Xlen@?$vector@NV?$allocator@N@std@@@std@@IBEXXZ 10016d50 f i superpose.obj
 0001:00015d60       ?_Xlen@?$vector@V?$vector@NV?$allocator@N@std@@@std@@V?$allocator@V?$vector@NV?$allocator@N@std@@@std@@@2@@std@@IBEXXZ 10016d60 f i superpose.obj
 0001:00015d70       ?allocate@?$_Wrap_alloc@V?$allocator@N@std@@@std@@QAEPANI@Z 10016d70 f i superpose.obj
 0001:00015db0       ?allocate@?$_Wrap_alloc@V?$allocator@V?$vector@NV?$allocator@N@std@@@std@@@std@@@std@@QAEPAV?$vector@NV?$allocator@N@std@@@2@I@Z 10016db0 f i superpose.obj
 0001:00015df0       ?allocate@?$allocator@N@std@@QAEPANI@Z 10016df0 f i superpose.obj
 0001:00015e30       ?allocate@?$allocator@V?$vector@NV?$allocator@N@std@@@std@@@std@@QAEPAV?$vector@NV?$allocator@N@std@@@2@I@Z 10016e30 f i superpose.obj
 0001:00015e70       ?begin@?$vector@NV?$allocator@N@std@@@std@@QBE?AV?$_Vector_const_iterator@V?$_Vector_val@U?$_Simple_types@N@std@@@std@@@2@XZ 10016e70 f i superpose.obj
 0001:00015e80       ?construct@?$allocator@V?$vector@NV?$allocator@N@std@@@std@@@std@@QAEXPAV?$vector@NV?$allocator@N@std@@@2@ABV32@@Z 10016e80 f i superpose.obj
 0001:00015ed0       ?deallocate@?$_Wrap_alloc@V?$allocator@N@std@@@std@@QAEXPANI@Z 10016ed0 f i superpose.obj
 0001:00015ef0       ?deallocate@?$_Wrap_alloc@V?$allocator@V?$vector@NV?$allocator@N@std@@@std@@@std@@@std@@QAEXPAV?$vector@NV?$allocator@N@std@@@2@I@Z 10016ef0 f i superpose.obj
 0001:00015f10       ?deallocate@?$allocator@N@std@@QAEXPANI@Z 10016f10 f i superpose.obj
 0001:00015f30       ?deallocate@?$allocator@V?$vector@NV?$allocator@N@std@@@std@@@std@@QAEXPAV?$vector@NV?$allocator@N@std@@@2@I@Z 10016f30 f i superpose.obj
 0001:00015f50       ?end@?$vector@NV?$allocator@N@std@@@std@@QBE?AV?$_Vector_const_iterator@V?$_Vector_val@U?$_Simple_types@N@std@@@std@@@2@XZ 10016f50 f i superpose.obj
 0001:00015f60       ?max_size@?$_Wrap_alloc@V?$allocator@N@std@@@std@@QBEIXZ 10016f60 f i superpose.obj
 0001:00015f70       ?max_size@?$_Wrap_alloc@V?$allocator@V?$vector@NV?$allocator@N@std@@@std@@@std@@@std@@QBEIXZ 10016f70 f i superpose.obj
 0001:00015f80       ?max_size@?$allocator@N@std@@QBEIXZ 10016f80 f i superpose.obj
 0001:00015f90       ?max_size@?$allocator@V?$vector@NV?$allocator@N@std@@@std@@@std@@QBEIXZ 10016f90 f i superpose.obj
 0001:00015fa0       ?max_size@?$allocator_traits@V?$allocator@N@std@@@std@@SAIABV?$allocator@N@2@@Z 10016fa0 f i superpose.obj
 0001:00015fb0       ?max_size@?$allocator_traits@V?$allocator@V?$vector@NV?$allocator@N@std@@@std@@@std@@@std@@SAIABV?$allocator@V?$vector@NV?$allocator@N@std@@@std@@@2@@Z 10016fb0 f i superpose.obj
 0001:00015fc0       ?max_size@?$vector@NV?$allocator@N@std@@@std@@QBEIXZ 10016fc0 f i superpose.obj
 0001:00015fd0       ?max_size@?$vector@V?$vector@NV?$allocator@N@std@@@std@@V?$allocator@V?$vector@NV?$allocator@N@std@@@std@@@2@@std@@QBEIXZ 10016fd0 f i superpose.obj
 0001:00016080       ?select_on_container_copy_construction@?$_Wrap_alloc@V?$allocator@N@std@@@std@@QBE?AU12@XZ 10017080 f i superpose.obj
 0001:00016090       ?select_on_container_copy_construction@?$allocator@N@std@@QBE?AV12@XZ 10017090 f i superpose.obj
 0001:000160a0       ?select_on_container_copy_construction@?$allocator_traits@V?$allocator@N@std@@@std@@SA?AV?$allocator@N@2@ABV32@@Z 100170a0 f i superpose.obj
 0001:000160b0       ?size@?$vector@NV?$allocator@N@std@@@std@@QBEIXZ 100170b0 f i superpose.obj
 0001:000160c0       ?superpose@PTools@@YA?AUSuperpose_t@@ABVRigidbody@1@0H@Z 100170c0 f   superpose.obj
 0001:00017030       ?swap@?$QVector@N@@QAEXAAV1@@Z 10018030 f i superpose.obj
 0001:00017050       ??C?$QScopedPointer@VQObjectData@@U?$QScopedPointerDeleter@VQObjectData@@@@@@QBEPAVQObjectData@@XZ 10018050 f i moc_PToolsPlugin.obj
 0001:00017060       ?metaObject@PToolsPlugin@U2@@UBEPBUQMetaObject@@XZ 10018060 f   moc_PToolsPlugin.obj
 0001:00017080       ?qt_metacall@PToolsPlugin@U2@@UAEHW4Call@QMetaObject@@HPAPAX@Z 10018080 f   moc_PToolsPlugin.obj
 0001:00017090       ?qt_metacast@PToolsPlugin@U2@@UAEPAXPBD@Z 10018090 f   moc_PToolsPlugin.obj
 0001:000170f0       ?qt_static_metacall@PToolsPlugin@U2@@CAXPAVQObject@@W4Call@QMetaObject@@HPAPAX@Z 100180f0 f   moc_PToolsPlugin.obj
 0001:00017100       ?metaObject@Gtest_PToolsAlignerTask@U2@@UBEPBUQMetaObject@@XZ 10018100 f   moc_PToolsTests.obj
 0001:00017120       ?qt_metacall@Gtest_PToolsAlignerTask@U2@@UAEHW4Call@QMetaObject@@HPAPAX@Z 10018120 f   moc_PToolsTests.obj
 0001:00017130       ?qt_metacast@Gtest_PToolsAlignerTask@U2@@UAEPAXPBD@Z 10018130 f   moc_PToolsTests.obj
 0001:00017190       ?qt_static_metacall@Gtest_PToolsAlignerTask@U2@@CAXPAVQObject@@W4Call@QMetaObject@@HPAPAX@Z 10018190 f   moc_PToolsTests.obj
 0001:00017192       ??AMatrix44@U2@@QAEAAMI@Z  10018192 f   U2Core:U2Core.dll
 0001:00017198       ??0Logger@U2@@QAE@ABVQString@@@Z 10018198 f   U2Core:U2Core.dll
 0001:0001719e       ??1Logger@U2@@UAE@XZ       1001819e f   U2Core:U2Core.dll
 0001:000171a4       ?trace@Logger@U2@@QAEXABVQString@@@Z 100181a4 f   U2Core:U2Core.dll
 0001:000171aa       ?error@Logger@U2@@QAEXABVQString@@@Z 100181aa f   U2Core:U2Core.dll
 0001:000171b0       ?getModelByName@BioStruct3D@U2@@QBE?BVMolecule3DModel@2@HH@Z 100181b0 f   U2Core:U2Core.dll
 0001:000171b6       ?getBioStruct3D@BioStruct3DObject@U2@@QBEABVBioStruct3D@2@XZ 100181b6 f   U2Core:U2Core.dll
 0001:000171bc       ??0Plugin@U2@@QAE@ABVQString@@0_NW4PluginState@1@@Z 100181bc f   U2Core:U2Core.dll
 0001:000171c2       ??1Plugin@U2@@UAE@XZ       100181c2 f   U2Core:U2Core.dll
 0001:000171c8       ?getTestFramework@AppContext@U2@@SAPAVTestFramework@2@XZ 100181c8 f   U2Core:U2Core.dll
 0001:000171ce       ?getStructuralAlignmentAlgorithmRegistry@AppContext@U2@@SAPAVStructuralAlignmentAlgorithmRegistry@2@XZ 100181ce f   U2Core:U2Core.dll
 0001:000171d4       ?cleanup@Task@U2@@UAEXXZ   100181d4 f   U2Core:U2Core.dll
 0001:000171da       ?generateReport@Task@U2@@UBE?AVQString@@XZ 100181da f   U2Core:U2Core.dll
 0001:000171e0       ?getNumParallelSubtasks@Task@U2@@UBEHXZ 100181e0 f   U2Core:U2Core.dll
 0001:000171e6       ?getParentTask@Task@U2@@UBEPAV12@XZ 100181e6 f   U2Core:U2Core.dll
 0001:000171ec       ?getSubtaskWithErrors@Task@U2@@UBEPAV12@XZ 100181ec f   U2Core:U2Core.dll
 0001:000171f2       ?getTaskId@Task@U2@@UBE_JXZ 100181f2 f   U2Core:U2Core.dll
 0001:000171f8       ?getTopLevelParentTask@Task@U2@@UAEPAV12@XZ 100181f8 f   U2Core:U2Core.dll
 0001:000171fe       ?getWarnings@Task@U2@@UBE?AVQStringList@@XZ 100181fe f   U2Core:U2Core.dll
 0001:00017204       ?hasSubtasksWithErrors@Task@U2@@UBE_NXZ 10018204 f   U2Core:U2Core.dll
 0001:0001720a       ?hasWarning@Task@U2@@UBE_NXZ 1001820a f   U2Core:U2Core.dll
 0001:00017210       ?isNotificationReport@Task@U2@@UBE_NXZ 10018210 f   U2Core:U2Core.dll
 0001:00017216       ?isReportingEnabled@Task@U2@@UBE_NXZ 10018216 f   U2Core:U2Core.dll
 0001:0001721c       ?isReportingSupported@Task@U2@@UBE_NXZ 1001821c f   U2Core:U2Core.dll
 0001:00017222       ?isTopLevelTask@Task@U2@@UBE_NXZ 10018222 f   U2Core:U2Core.dll
 0001:00017228       ?onSubTaskFinished@Task@U2@@MAE?AV?$QList@PAVTask@U2@@@@PAV12@@Z 10018228 f   U2Core:U2Core.dll
 0001:0001722e       ?prepare@Task@U2@@UAEXXZ   1001822e f   U2Core:U2Core.dll
 0001:00017234       ?propagateSubtaskError@Task@U2@@UAE_NXZ 10018234 f   U2Core:U2Core.dll
 0001:0001723a       ?setCollectChildrensWarningsFlag@Task@U2@@UAEX_N@Z 1001823a f   U2Core:U2Core.dll
 0001:00017240       ?setNoAutoDelete@Task@U2@@UAEX_N@Z 10018240 f   U2Core:U2Core.dll
 0001:00017246       ?setNotificationReport@Task@U2@@UAEX_N@Z 10018246 f   U2Core:U2Core.dll
 0001:0001724c       ?setReportingEnabled@Task@U2@@UAEX_N@Z 1001824c f   U2Core:U2Core.dll
 0001:00017252       ?setReportingSupported@Task@U2@@UAEX_N@Z 10018252 f   U2Core:U2Core.dll
 0001:00017258       ??4Matrix44@U2@@QAEAAV01@ABV01@@Z 10018258 f   U2Core:U2Core.dll
 0001:0001725e       ??AMatrix44@U2@@QBEMI@Z    1001825e f   U2Core:U2Core.dll
 0001:00017264       ?setError@Task@U2@@QAEXABVQString@@@Z 10018264 f   U2Core:U2Core.dll
 0001:0001726a       ?qt_metacast@Plugin@U2@@UAEPAXPBD@Z 1001826a f   U2Core:U2Core.dll
 0001:00017270       ?qt_metacall@Plugin@U2@@UAEHW4Call@QMetaObject@@HPAPAX@Z 10018270 f   U2Core:U2Core.dll
 0001:00017276       ?print@BioStruct3DReference@U2@@QBE?AVQString@@XZ 10018276 f   U2Algorithm:U2Algorithm.dll
 0001:0001727c       ??0StructuralAlignment@U2@@QAE@XZ 1001827c f   U2Algorithm:U2Algorithm.dll
 0001:00017282       ??1StructuralAlignment@U2@@QAE@XZ 10018282 f   U2Algorithm:U2Algorithm.dll
 0001:00017288       ?registerAlgorithmFactory@StructuralAlignmentAlgorithmRegistry@U2@@QAEXPAVStructuralAlignmentAlgorithmFactory@2@ABVQString@@@Z 10018288 f   U2Algorithm:U2Algorithm.dll
 0001:0001728e       ??0BioStruct3DReference@U2@@QAE@PBVBioStruct3DObject@1@ABV?$QList@H@@H@Z 1001828e f   U2Algorithm:U2Algorithm.dll
 0001:00017294       ??1BioStruct3DReference@U2@@QAE@XZ 10018294 f   U2Algorithm:U2Algorithm.dll
 0001:0001729a       ??0StructuralAlignmentTaskSettings@U2@@QAE@ABVBioStruct3DReference@1@0@Z 1001829a f   U2Algorithm:U2Algorithm.dll
 0001:000172a0       ??1StructuralAlignmentTaskSettings@U2@@QAE@XZ 100182a0 f   U2Algorithm:U2Algorithm.dll
 0001:000172a6       ??0XMLTestFactory@U2@@QAE@ABVQString@@@Z 100182a6 f   U2Test:U2Test.dll
 0001:000172ac       ??1XMLTestFactory@U2@@UAE@XZ 100182ac f   U2Test:U2Test.dll
 0001:000172b2       ??0XmlTest@U2@@QAE@ABVQString@@PAVGTest@1@PBVGTestEnvironment@1@V?$QFlags@W4TaskFlag@U2@@@@ABV?$QList@PAVGTest@U2@@@@@Z 100182b2 f   U2Test:U2Test.dll
 0001:000172b8       ??1XmlTest@U2@@UAE@XZ      100182b8 f   U2Test:U2Test.dll
 0001:000172be       ?findFormat@GTestFormatRegistry@U2@@QAEPAVGTestFormat@2@ABVQString@@@Z 100182be f   U2Test:U2Test.dll
 0001:000172c4       ?getContext@GTest@U2@@QBEPAVQObject@@ABVQString@@@Z 100182c4 f   U2Test:U2Test.dll
 0001:000172ca       ?failMissingValue@GTest@U2@@IAEXABVQString@@@Z 100182ca f   U2Test:U2Test.dll
 0001:000172d0       ?qt_metacast@GTest@U2@@UAEPAXPBD@Z 100182d0 f   U2Test:U2Test.dll
 0001:000172d6       ?qt_metacall@GTest@U2@@UAEHW4Call@QMetaObject@@HPAPAX@Z 100182d6 f   U2Test:U2Test.dll
 0001:000172dc       ?attribute@QDomElement@@QBE?AVQString@@ABV2@0@Z 100182dc f   Qt5Xml:Qt5Xml.dll
 0001:000172e2       ?qBadAlloc@@YAXXZ          100182e2 f   Qt5Core:Qt5Core.dll
 0001:000172e8       ??0QChar@@QAE@UQLatin1Char@@@Z 100182e8 f   Qt5Core:Qt5Core.dll
 0001:000172ee       ?data@QArrayData@@QAEPAXXZ 100182ee f   Qt5Core:Qt5Core.dll
 0001:000172f4       ?allocate@QArrayData@@SAPAU1@IIIV?$QFlags@W4AllocationOption@QArrayData@@@@@Z 100182f4 f   Qt5Core:Qt5Core.dll
 0001:000172fa       ?deallocate@QArrayData@@SAXPAU1@II@Z 100182fa f   Qt5Core:Qt5Core.dll
 0001:00017300       ?qstrcmp@@YAHABVQByteArray@@PBD@Z 10018300 f   Qt5Core:Qt5Core.dll
 0001:00017306       ??1QByteArray@@QAE@XZ      10018306 f   Qt5Core:Qt5Core.dll
 0001:0001730c       ?data@QByteArray@@QBEPBDXZ 1001830c f   Qt5Core:Qt5Core.dll
 0001:00017312       ??0QString@@QAE@XZ         10018312 f   Qt5Core:Qt5Core.dll
 0001:00017318       ??1QString@@QAE@XZ         10018318 f   Qt5Core:Qt5Core.dll
 0001:0001731e       ??4QString@@QAEAAV0@$$QAV0@@Z 1001831e f   Qt5Core:Qt5Core.dll
 0001:00017324       ?arg@QString@@QBE?AV1@ABV1@HVQChar@@@Z 10018324 f   Qt5Core:Qt5Core.dll
 0001:0001732a       ?arg@QString@@QBE?AV1@ABV1@0@Z 1001832a f   Qt5Core:Qt5Core.dll
 0001:00017330       ?fromAscii_helper@QString@@CAPAU?$QTypedArrayData@G@@PBDH@Z 10018330 f   Qt5Core:Qt5Core.dll
 0001:00017336       ?detach@QListData@@QAEPAUData@1@H@Z 10018336 f   Qt5Core:Qt5Core.dll
 0001:0001733c       ?dispose@QListData@@SAXPAUData@1@@Z 1001833c f   Qt5Core:Qt5Core.dll
 0001:00017342       ?freeTree@QMapDataBase@@QAEXPAUQMapNodeBase@@H@Z 10018342 f   Qt5Core:Qt5Core.dll
 0001:00017348       ?freeData@QMapDataBase@@SAXPAU1@@Z 10018348 f   Qt5Core:Qt5Core.dll
 0001:0001734e       ?detach_grow@QListData@@QAEPAUData@1@PAHH@Z 1001834e f   Qt5Core:Qt5Core.dll
 0001:00017354       ?append@QListData@@QAEPAPAXXZ 10018354 f   Qt5Core:Qt5Core.dll
 0001:0001735a       ?cast@QMetaObject@@QBEPAVQObject@@PAV2@@Z 1001835a f   Qt5Core:Qt5Core.dll
 0001:00017360       ?tr@QMetaObject@@QBE?AVQString@@PBD0H@Z 10018360 f   Qt5Core:Qt5Core.dll
 0001:00017366       ??0QObject@@QAE@PAV0@@Z    10018366 f   Qt5Core:Qt5Core.dll
 0001:0001736c       ??1QObject@@UAE@XZ         1001836c f   Qt5Core:Qt5Core.dll
 0001:00017372       ?childEvent@QObject@@MAEXPAVQChildEvent@@@Z 10018372 f   Qt5Core:Qt5Core.dll
 0001:00017378       ?connectNotify@QObject@@MAEXABVQMetaMethod@@@Z 10018378 f   Qt5Core:Qt5Core.dll
 0001:0001737e       ?customEvent@QObject@@MAEXPAVQEvent@@@Z 1001837e f   Qt5Core:Qt5Core.dll
 0001:00017384       ?disconnectNotify@QObject@@MAEXABVQMetaMethod@@@Z 10018384 f   Qt5Core:Qt5Core.dll
 0001:0001738a       ?event@QObject@@UAE_NPAVQEvent@@@Z 1001838a f   Qt5Core:Qt5Core.dll
 0001:00017390       ?eventFilter@QObject@@UAE_NPAV1@PAVQEvent@@@Z 10018390 f   Qt5Core:Qt5Core.dll
 0001:00017396       ?metaObject@QObject@@UBEPBUQMetaObject@@XZ 10018396 f   Qt5Core:Qt5Core.dll
 0001:0001739c       ?qt_metacall@QObject@@UAEHW4Call@QMetaObject@@HPAPAX@Z 1001839c f   Qt5Core:Qt5Core.dll
 0001:000173a2       ?qt_metacast@QObject@@UAEPAXPBD@Z 100183a2 f   Qt5Core:Qt5Core.dll
 0001:000173a8       ?timerEvent@QObject@@MAEXPAVQTimerEvent@@@Z 100183a8 f   Qt5Core:Qt5Core.dll
 0001:000173ae       ??0QString@@QAE@ABV0@@Z    100183ae f   Qt5Core:Qt5Core.dll
 0001:000173b4       ?chop@QString@@QAEXH@Z     100183b4 f   Qt5Core:Qt5Core.dll
 0001:000173ba       ?arg@QString@@QBE?AV1@NHDHVQChar@@@Z 100183ba f   Qt5Core:Qt5Core.dll
 0001:000173c0       ?trimmed@QString@@QBE?AV1@XZ 100183c0 f   Qt5Core:Qt5Core.dll
 0001:000173c6       ?append@QString@@QAEAAV1@ABV1@@Z 100183c6 f   Qt5Core:Qt5Core.dll
 0001:000173cc       ?split@QString@@QBE?AVQStringList@@ABV1@W4SplitBehavior@1@W4CaseSensitivity@Qt@@@Z 100183cc f   Qt5Core:Qt5Core.dll
 0001:000173d2       ?fromUtf8@QString@@SA?AV1@PBDH@Z 100183d2 f   Qt5Core:Qt5Core.dll
 0001:000173d8       ?toDouble@QString@@QBENPA_N@Z 100183d8 f   Qt5Core:Qt5Core.dll
 0001:000173de       ?number@QString@@SA?AV1@NDH@Z 100183de f   Qt5Core:Qt5Core.dll
 0001:000173e4       ??YQString@@QAEAAV0@PBD@Z  100183e4 f   Qt5Core:Qt5Core.dll
 0001:000173ea       ?realloc@QListData@@QAEXH@Z 100183ea f   Qt5Core:Qt5Core.dll
 0001:000173f0       ?nextNode@QMapNodeBase@@QBEPBU1@XZ 100183f0 f   Qt5Core:Qt5Core.dll
 0001:000173f6       ?dynamicMetaObject@QObjectData@@QBEPAUQMetaObject@@XZ 100183f6 f   Qt5Core:Qt5Core.dll
 0001:000173fc       ?_Xbad_alloc@std@@YAXXZ    100183fc f   msvcprt:MSVCP120.dll
 0001:00017402       ?_Xlength_error@std@@YAXPBD@Z 10018402 f   msvcprt:MSVCP120.dll
 0001:00017408       ?_Xout_of_range@std@@YAXPBD@Z 10018408 f   msvcprt:MSVCP120.dll
 0001:0001740e       ?_Syserror_map@std@@YAPBDH@Z 1001840e f   msvcprt:MSVCP120.dll
 0001:00017414       ?_Winerror_map@std@@YAPBDH@Z 10018414 f   msvcprt:MSVCP120.dll
 0001:0001741a       ?uncaught_exception@std@@YA_NXZ 1001841a f   msvcprt:MSVCP120.dll
 0001:00017420       ?_Ios_base_dtor@ios_base@std@@CAXPAV12@@Z 10018420 f   msvcprt:MSVCP120.dll
 0001:00017426       ??0?$basic_streambuf@DU?$char_traits@D@std@@@std@@IAE@XZ 10018426 f   msvcprt:MSVCP120.dll
 0001:0001742c       ??1?$basic_streambuf@DU?$char_traits@D@std@@@std@@UAE@XZ 1001842c f   msvcprt:MSVCP120.dll
 0001:00017432       ?sputc@?$basic_streambuf@DU?$char_traits@D@std@@@std@@QAEHD@Z 10018432 f   msvcprt:MSVCP120.dll
 0001:00017438       ?sputn@?$basic_streambuf@DU?$char_traits@D@std@@@std@@QAE_JPBD_J@Z 10018438 f   msvcprt:MSVCP120.dll
 0001:0001743e       ?_Pninc@?$basic_streambuf@DU?$char_traits@D@std@@@std@@IAEPADXZ 1001843e f   msvcprt:MSVCP120.dll
 0001:00017444       ??1?$basic_ios@DU?$char_traits@D@std@@@std@@UAE@XZ 10018444 f   msvcprt:MSVCP120.dll
 0001:0001744a       ?setstate@?$basic_ios@DU?$char_traits@D@std@@@std@@QAEXH_N@Z 1001844a f   msvcprt:MSVCP120.dll
 0001:00017450       ?_Osfx@?$basic_ostream@DU?$char_traits@D@std@@@std@@QAEXXZ 10018450 f   msvcprt:MSVCP120.dll
 0001:00017456       ??6?$basic_ostream@DU?$char_traits@D@std@@@std@@QAEAAV01@N@Z 10018456 f   msvcprt:MSVCP120.dll
 0001:0001745c       ?flush@?$basic_ostream@DU?$char_traits@D@std@@@std@@QAEAAV12@XZ 1001845c f   msvcprt:MSVCP120.dll
 0001:00017462       ??0?$basic_iostream@DU?$char_traits@D@std@@@std@@QAE@PAV?$basic_streambuf@DU?$char_traits@D@std@@@1@@Z 10018462 f   msvcprt:MSVCP120.dll
 0001:00017468       ??1?$basic_iostream@DU?$char_traits@D@std@@@std@@UAE@XZ 10018468 f   msvcprt:MSVCP120.dll
 0001:0001746e       ?_Lock@?$basic_streambuf@DU?$char_traits@D@std@@@std@@UAEXXZ 1001846e f   msvcprt:MSVCP120.dll
 0001:00017474       ?_Unlock@?$basic_streambuf@DU?$char_traits@D@std@@@std@@UAEXXZ 10018474 f   msvcprt:MSVCP120.dll
 0001:0001747a       ?imbue@?$basic_streambuf@DU?$char_traits@D@std@@@std@@MAEXABVlocale@2@@Z 1001847a f   msvcprt:MSVCP120.dll
 0001:00017480       ?setbuf@?$basic_streambuf@DU?$char_traits@D@std@@@std@@MAEPAV12@PAD_J@Z 10018480 f   msvcprt:MSVCP120.dll
 0001:00017486       ?showmanyc@?$basic_streambuf@DU?$char_traits@D@std@@@std@@MAE_JXZ 10018486 f   msvcprt:MSVCP120.dll
 0001:0001748c       ?sync@?$basic_streambuf@DU?$char_traits@D@std@@@std@@MAEHXZ 1001848c f   msvcprt:MSVCP120.dll
 0001:00017492       ?uflow@?$basic_streambuf@DU?$char_traits@D@std@@@std@@MAEHXZ 10018492 f   msvcprt:MSVCP120.dll
 0001:00017498       ?xsgetn@?$basic_streambuf@DU?$char_traits@D@std@@@std@@MAE_JPAD_J@Z 10018498 f   msvcprt:MSVCP120.dll
 0001:0001749e       ?xsputn@?$basic_streambuf@DU?$char_traits@D@std@@@std@@MAE_JPBD_J@Z 1001849e f   msvcprt:MSVCP120.dll
 0001:000174a4       ??0_Lockit@std@@QAE@H@Z    100184a4 f   msvcprt:MSVCP120.dll
 0001:000174aa       ??1_Lockit@std@@QAE@XZ     100184aa f   msvcprt:MSVCP120.dll
 0001:000174b0       ??0_Fac_node@std@@QAE@PAU01@PAV_Facet_base@1@@Z 100184b0 f i msvcprt:locale0_implib.obj
 0001:000174c4       ??1_Fac_node@std@@QAE@XZ   100184c4 f i msvcprt:locale0_implib.obj
 0001:000174d9       ??1_Fac_tidy_reg_t@std@@QAE@XZ 100184d9 f i msvcprt:locale0_implib.obj
 0001:000174fd       ??_G_Fac_node@std@@QAEPAXI@Z 100184fd f i msvcprt:locale0_implib.obj
 0001:0001751c       ?_Facet_Register@std@@YAXPAV_Facet_base@1@@Z 1001851c f   msvcprt:locale0_implib.obj
 0001:00017544       ??Bid@locale@std@@QAEIXZ   10018544 f   msvcprt:MSVCP120.dll
 0001:0001754a       ?_Getgloballocale@locale@std@@CAPAV_Locimp@12@XZ 1001854a f   msvcprt:MSVCP120.dll
 0001:00017550       ?always_noconv@codecvt_base@std@@QBE_NXZ 10018550 f   msvcprt:MSVCP120.dll
 0001:00017556       ?in@?$codecvt@DDH@std@@QBEHAAHPBD1AAPBDPAD3AAPAD@Z 10018556 f   msvcprt:MSVCP120.dll
 0001:0001755c       ?out@?$codecvt@DDH@std@@QBEHAAHPBD1AAPBDPAD3AAPAD@Z 1001855c f   msvcprt:MSVCP120.dll
 0001:00017562       ?unshift@?$codecvt@DDH@std@@QBEHAAHPAD1AAPAD@Z 10018562 f   msvcprt:MSVCP120.dll
 0001:00017568       ?_Getcat@?$codecvt@DDH@std@@SAIPAPBVfacet@locale@2@PBV42@@Z 10018568 f   msvcprt:MSVCP120.dll
 0001:0001756e       ?getloc@?$basic_streambuf@DU?$char_traits@D@std@@@std@@QBE?AVlocale@2@XZ 1001856e f   msvcprt:MSVCP120.dll
 0001:00017574       ?sbumpc@?$basic_streambuf@DU?$char_traits@D@std@@@std@@QAEHXZ 10018574 f   msvcprt:MSVCP120.dll
 0001:0001757a       ?sgetc@?$basic_streambuf@DU?$char_traits@D@std@@@std@@QAEHXZ 1001857a f   msvcprt:MSVCP120.dll
 0001:00017580       ?snextc@?$basic_streambuf@DU?$char_traits@D@std@@@std@@QAEHXZ 10018580 f   msvcprt:MSVCP120.dll
 0001:00017586       ?setg@?$basic_streambuf@DU?$char_traits@D@std@@@std@@IAEXPAD00@Z 10018586 f   msvcprt:MSVCP120.dll
 0001:0001758c       ?_Init@?$basic_streambuf@DU?$char_traits@D@std@@@std@@IAEXXZ 1001858c f   msvcprt:MSVCP120.dll
 0001:00017592       ?widen@?$basic_ios@DU?$char_traits@D@std@@@std@@QBEDD@Z 10018592 f   msvcprt:MSVCP120.dll
 0001:00017598       ??0?$basic_ostream@DU?$char_traits@D@std@@@std@@QAE@PAV?$basic_streambuf@DU?$char_traits@D@std@@@1@_N@Z 10018598 f   msvcprt:MSVCP120.dll
 0001:0001759e       ??1?$basic_ostream@DU?$char_traits@D@std@@@std@@UAE@XZ 1001859e f   msvcprt:MSVCP120.dll
 0001:000175a4       ??0?$basic_istream@DU?$char_traits@D@std@@@std@@QAE@PAV?$basic_streambuf@DU?$char_traits@D@std@@@1@_N@Z 100185a4 f   msvcprt:MSVCP120.dll
 0001:000175aa       ??1?$basic_istream@DU?$char_traits@D@std@@@std@@UAE@XZ 100185aa f   msvcprt:MSVCP120.dll
 0001:000175b0       ?_Ipfx@?$basic_istream@DU?$char_traits@D@std@@@std@@QAE_N_N@Z 100185b0 f   msvcprt:MSVCP120.dll
 0001:000175b6       ?_Fiopen@std@@YAPAU_iobuf@@PBDHH@Z 100185b6 f   msvcprt:MSVCP120.dll
 0001:000175bc       __purecall                 100185bc f   MSVCRT:MSVCR120.dll
 0001:000175c2       ??2@YAPAXI@Z               100185c2 f   MSVCRT:MSVCR120.dll
 0001:000175c8       ??3@YAXPAX@Z               100185c8 f   MSVCRT:MSVCR120.dll
 0001:000175ce       ___atonexitinit            100185ce f   MSVCRT:atonexit.obj
 0001:0001760a       __onexit                   1001860a f   MSVCRT:atonexit.obj
 0001:000176b3       _atexit                    100186b3 f   MSVCRT:atonexit.obj
 0001:000176c8       _memmove                   100186c8 f   MSVCRT:MSVCR120.dll
 0001:000176ce       __hypot                    100186ce f   MSVCRT:MSVCR120.dll
 0001:000176d4       @__security_check_cookie@4 100186d4 f   MSVCRT:secchk.obj
 0001:000176e4       __CxxThrowException@8      100186e4 f   MSVCRT:MSVCR120.dll
 0001:000176ea       ___CxxFrameHandler3        100186ea f   MSVCRT:MSVCR120.dll
 0001:000176f0       _memcpy                    100186f0 f   MSVCRT:MSVCR120.dll
 0001:000176f6       _memset                    100186f6 f   MSVCRT:MSVCR120.dll
 0001:000176fc       ??0type_info@@AAE@ABV0@@Z  100186fc f   MSVCRT:ti_inst.obj
 0001:00017707       ??4type_info@@AAEAAV0@ABV0@@Z 10018707 f   MSVCRT:ti_inst.obj
 0001:0001770c       ??_Etype_info@@UAEPAXI@Z   1001870c f i MSVCRT:ti_inst.obj
 0001:00017760       __libm_sse2_log10_precise  10018760 f   MSVCRT:MSVCR120.dll
 0001:00017766       __libm_sse2_sqrt_precise   10018766 f   MSVCRT:MSVCR120.dll
 0001:0001776c       ??0exception@std@@QAE@ABQBD@Z 1001876c f   MSVCRT:MSVCR120.dll
 0001:00017772       ??0exception@std@@QAE@ABV01@@Z 10018772 f   MSVCRT:MSVCR120.dll
 0001:00017778       ??1exception@std@@UAE@XZ   10018778 f   MSVCRT:MSVCR120.dll
 0001:0001777e       ?what@exception@std@@UBEPBDXZ 1001877e f   MSVCRT:MSVCR120.dll
 0001:00017784       __libm_sse2_cos_precise    10018784 f   MSVCRT:MSVCR120.dll
 0001:0001778a       __libm_sse2_sin_precise    1001878a f   MSVCRT:MSVCR120.dll
 0001:00017790       __CIatan2                  10018790 f   MSVCRT:MSVCR120.dll
 0001:00017796       __libm_sse2_acos_precise   10018796 f   MSVCRT:MSVCR120.dll
 0001:0001779c       _atof                      1001879c f   MSVCRT:MSVCR120.dll
 0001:000177a2       _atoi                      100187a2 f   MSVCRT:MSVCR120.dll
 0001:000177a8       _memcpy_s                  100187a8 f   MSVCRT:MSVCR120.dll
 0001:000177ae       _memchr                    100187ae f   MSVCRT:MSVCR120.dll
 0001:000177b4       _fclose                    100187b4 f   MSVCRT:MSVCR120.dll
 0001:000177ba       _fflush                    100187ba f   MSVCRT:MSVCR120.dll
 0001:000177c0       _fgetc                     100187c0 f   MSVCRT:MSVCR120.dll
 0001:000177c6       _fgetpos                   100187c6 f   MSVCRT:MSVCR120.dll
 0001:000177cc       _fopen                     100187cc f   MSVCRT:MSVCR120.dll
 0001:000177d2       _fprintf                   100187d2 f   MSVCRT:MSVCR120.dll
 0001:000177d8       _fputc                     100187d8 f   MSVCRT:MSVCR120.dll
 0001:000177de       _fsetpos                   100187de f   MSVCRT:MSVCR120.dll
 0001:000177e4       __fseeki64                 100187e4 f   MSVCRT:MSVCR120.dll
 0001:000177ea       _fwrite                    100187ea f   MSVCRT:MSVCR120.dll
 0001:000177f0       _setvbuf                   100187f0 f   MSVCRT:MSVCR120.dll
 0001:000177f6       _ungetc                    100187f6 f   MSVCRT:MSVCR120.dll
 0001:000177fc       __lock_file                100187fc f   MSVCRT:MSVCR120.dll
 0001:00017802       __unlock_file              10018802 f   MSVCRT:MSVCR120.dll
 0001:00017808       _toupper                   10018808 f   MSVCRT:MSVCR120.dll
 0001:0001780e       ??0bad_cast@std@@QAE@PBD@Z 1001880e f   MSVCRT:MSVCR120.dll
 0001:00017814       ??0bad_cast@std@@QAE@ABV01@@Z 10018814 f   MSVCRT:MSVCR120.dll
 0001:0001781a       ??1bad_cast@std@@UAE@XZ    1001881a f   MSVCRT:MSVCR120.dll
 0001:00017820       ??_M@YGXPAXIHP6EX0@Z@Z     10018820 f   MSVCRT:ehvecdtr.obj
 0001:000178a8       ?__ArrayUnwind@@YGXPAXIHP6EX0@Z@Z 100188a8 f   MSVCRT:ehvecdtr.obj
 0001:00017952       _NtCurrentTeb              10018952 f i MSVCRT:crtdll.obj
 0001:00017959       __CRT_INIT@12              10018959 f   MSVCRT:crtdll.obj
 0001:00017b50       __DllMainCRTStartup@12     10018b50 f   MSVCRT:crtdll.obj
 0001:00017ca6       __lock                     10018ca6 f   MSVCRT:MSVCR120.dll
 0001:00017cac       __unlock                   10018cac f   MSVCRT:MSVCR120.dll
 0001:00017cb2       __calloc_crt               10018cb2 f   MSVCRT:MSVCR120.dll
 0001:00017cb8       ___dllonexit               10018cb8 f   MSVCRT:MSVCR120.dll
 0001:00017cc0       __SEH_prolog4              10018cc0 f   MSVCRT:sehprolg4.obj
 0001:00017d05       __SEH_epilog4              10018d05 f   MSVCRT:sehprolg4.obj
 0001:00017d19       __except_handler4          10018d19 f   MSVCRT:chandler4gs.obj
 0001:00017d3c       ___raise_securityfailure   10018d3c f   MSVCRT:gs_report.obj
 0001:00017d79       ___report_gsfailure        10018d79 f   MSVCRT:gs_report.obj
 0001:00017e74       ___report_rangecheckfailure 10018e74 f   MSVCRT:gs_report.obj
 0001:00017e80       ___report_securityfailure  10018e80 f   MSVCRT:gs_report.obj
 0001:00017f50       ___report_securityfailureEx 10018f50 f   MSVCRT:gs_report.obj
 0001:00018066       ??1type_info@@UAE@XZ       10019066 f   MSVCRT:MSVCR120.dll
 0001:0001806c       ?terminate@@YAXXZ          1001906c f   MSVCRT:MSVCR120.dll
 0001:00018072       ___CppXcptFilter           10019072 f   MSVCRT:MSVCR120.dll
 0001:00018078       __amsg_exit                10019078 f   MSVCRT:MSVCR120.dll
 0001:00018080       __FindPESection            10019080 f   MSVCRT:pesect.obj
 0001:000180d0       __IsNonwritableInCurrentImage 100190d0 f   MSVCRT:pesect.obj
 0001:00018190       __ValidateImageBase        10019190 f   MSVCRT:pesect.obj
 0001:000181c2       _free                      100191c2 f   MSVCRT:MSVCR120.dll
 0001:000181c8       ___security_init_cookie    100191c8 f   MSVCRT:gs_support.obj
 0001:00018264       _DllMain@12                10019264 f   MSVCRT:dllmain.obj
 0001:00018286       __malloc_crt               10019286 f   MSVCRT:MSVCR120.dll
 0001:0001828c       __RTC_Initialize           1001928c f   MSVCRT:initsect.obj
 0001:000182ac       __RTC_Terminate            100192ac f   MSVCRT:initsect.obj
 0001:000182cc       __initterm                 100192cc f   MSVCRT:MSVCR120.dll
 0001:000182d2       __initterm_e               100192d2 f   MSVCRT:MSVCR120.dll
 0001:000182d8       ___clean_type_info_names   100192d8 f   MSVCRT:tncleanup.obj
 0001:000182e4       __except_handler4_common   100192e4 f   MSVCRT:MSVCR120.dll
 0001:000182ea       __crt_debugger_hook        100192ea f   MSVCRT:MSVCR120.dll
 0001:000182f0       ___crtUnhandledException   100192f0 f   MSVCRT:MSVCR120.dll
 0001:000182f6       ___crtTerminateProcess     100192f6 f   MSVCRT:MSVCR120.dll
 0001:000182fc       ___clean_type_info_names_internal 100192fc f   MSVCRT:MSVCR120.dll
 0001:00018302       _EncodePointer@4           10019302 f   kernel32:KERNEL32.dll
 0001:00018308       _DecodePointer@4           10019308 f   kernel32:KERNEL32.dll
 0001:0001830e       _IsDebuggerPresent@0       1001930e f   kernel32:KERNEL32.dll
 0001:00018314       _IsProcessorFeaturePresent@4 10019314 f   kernel32:KERNEL32.dll
 0001:0001831a       _QueryPerformanceCounter@4 1001931a f   kernel32:KERNEL32.dll
 0001:00018320       _GetCurrentProcessId@0     10019320 f   kernel32:KERNEL32.dll
 0001:00018326       _GetCurrentThreadId@0      10019326 f   kernel32:KERNEL32.dll
 0001:0001832c       _GetSystemTimeAsFileTime@4 1001932c f   kernel32:KERNEL32.dll
 0001:00018332       _DisableThreadLibraryCalls@4 10019332 f   kernel32:KERNEL32.dll
 0002:00000000       __imp__DisableThreadLibraryCalls@4 1001c000     kernel32:KERNEL32.dll
 0002:00000004       __imp__GetSystemTimeAsFileTime@4 1001c004     kernel32:KERNEL32.dll
 0002:00000008       __imp__GetCurrentThreadId@0 1001c008     kernel32:KERNEL32.dll
 0002:0000000c       __imp__GetCurrentProcessId@0 1001c00c     kernel32:KERNEL32.dll
 0002:00000010       __imp__QueryPerformanceCounter@4 1001c010     kernel32:KERNEL32.dll
 0002:00000014       __imp__IsProcessorFeaturePresent@4 1001c014     kernel32:KERNEL32.dll
 0002:00000018       __imp__IsDebuggerPresent@0 1001c018     kernel32:KERNEL32.dll
 0002:0000001c       __imp__DecodePointer@4     1001c01c     kernel32:KERNEL32.dll
 0002:00000020       __imp__EncodePointer@4     1001c020     kernel32:KERNEL32.dll
 0002:00000024       \177KERNEL32_NULL_THUNK_DATA 1001c024     kernel32:KERNEL32.dll
 0002:00000028       __imp_?id@?$codecvt@DDH@std@@2V0locale@2@A 1001c028     msvcprt:MSVCP120.dll
 0002:0000002c       __imp_?_Fiopen@std@@YAPAU_iobuf@@PBDHH@Z 1001c02c     msvcprt:MSVCP120.dll
 0002:00000030       __imp_?_Ipfx@?$basic_istream@DU?$char_traits@D@std@@@std@@QAE_N_N@Z 1001c030     msvcprt:MSVCP120.dll
 0002:00000034       __imp_??1?$basic_istream@DU?$char_traits@D@std@@@std@@UAE@XZ 1001c034     msvcprt:MSVCP120.dll
 0002:00000038       __imp_??0?$basic_istream@DU?$char_traits@D@std@@@std@@QAE@PAV?$basic_streambuf@DU?$char_traits@D@std@@@1@_N@Z 1001c038     msvcprt:MSVCP120.dll
 0002:0000003c       __imp_??1?$basic_ostream@DU?$char_traits@D@std@@@std@@UAE@XZ 1001c03c     msvcprt:MSVCP120.dll
 0002:00000040       __imp_??0?$basic_ostream@DU?$char_traits@D@std@@@std@@QAE@PAV?$basic_streambuf@DU?$char_traits@D@std@@@1@_N@Z 1001c040     msvcprt:MSVCP120.dll
 0002:00000044       __imp_?widen@?$basic_ios@DU?$char_traits@D@std@@@std@@QBEDD@Z 1001c044     msvcprt:MSVCP120.dll
 0002:00000048       __imp_?_Init@?$basic_streambuf@DU?$char_traits@D@std@@@std@@IAEXXZ 1001c048     msvcprt:MSVCP120.dll
 0002:0000004c       __imp_?setg@?$basic_streambuf@DU?$char_traits@D@std@@@std@@IAEXPAD00@Z 1001c04c     msvcprt:MSVCP120.dll
 0002:00000050       __imp_?snextc@?$basic_streambuf@DU?$char_traits@D@std@@@std@@QAEHXZ 1001c050     msvcprt:MSVCP120.dll
 0002:00000054       __imp_?sgetc@?$basic_streambuf@DU?$char_traits@D@std@@@std@@QAEHXZ 1001c054     msvcprt:MSVCP120.dll
 0002:00000058       __imp_?sbumpc@?$basic_streambuf@DU?$char_traits@D@std@@@std@@QAEHXZ 1001c058     msvcprt:MSVCP120.dll
 0002:0000005c       __imp_?getloc@?$basic_streambuf@DU?$char_traits@D@std@@@std@@QBE?AVlocale@2@XZ 1001c05c     msvcprt:MSVCP120.dll
 0002:00000060       __imp_?_Getcat@?$codecvt@DDH@std@@SAIPAPBVfacet@locale@2@PBV42@@Z 1001c060     msvcprt:MSVCP120.dll
 0002:00000064       __imp_?unshift@?$codecvt@DDH@std@@QBEHAAHPAD1AAPAD@Z 1001c064     msvcprt:MSVCP120.dll
 0002:00000068       __imp_?out@?$codecvt@DDH@std@@QBEHAAHPBD1AAPBDPAD3AAPAD@Z 1001c068     msvcprt:MSVCP120.dll
 0002:0000006c       __imp_?in@?$codecvt@DDH@std@@QBEHAAHPBD1AAPBDPAD3AAPAD@Z 1001c06c     msvcprt:MSVCP120.dll
 0002:00000070       __imp_?always_noconv@codecvt_base@std@@QBE_NXZ 1001c070     msvcprt:MSVCP120.dll
 0002:00000074       __imp_?_Getgloballocale@locale@std@@CAPAV_Locimp@12@XZ 1001c074     msvcprt:MSVCP120.dll
 0002:00000078       __imp_??Bid@locale@std@@QAEIXZ 1001c078     msvcprt:MSVCP120.dll
 0002:0000007c       __imp_??1_Lockit@std@@QAE@XZ 1001c07c     msvcprt:MSVCP120.dll
 0002:00000080       __imp_??0_Lockit@std@@QAE@H@Z 1001c080     msvcprt:MSVCP120.dll
 0002:00000084       __imp_??_7?$basic_ios@DU?$char_traits@D@std@@@std@@6B@ 1001c084     msvcprt:MSVCP120.dll
 0002:00000088       __imp_??_7ios_base@std@@6B@ 1001c088     msvcprt:MSVCP120.dll
 0002:0000008c       __imp_?_BADOFF@std@@3_JB   1001c08c     msvcprt:MSVCP120.dll
 0002:00000090       __imp_?xsputn@?$basic_streambuf@DU?$char_traits@D@std@@@std@@MAE_JPBD_J@Z 1001c090     msvcprt:MSVCP120.dll
 0002:00000094       __imp_?xsgetn@?$basic_streambuf@DU?$char_traits@D@std@@@std@@MAE_JPAD_J@Z 1001c094     msvcprt:MSVCP120.dll
 0002:00000098       __imp_?uflow@?$basic_streambuf@DU?$char_traits@D@std@@@std@@MAEHXZ 1001c098     msvcprt:MSVCP120.dll
 0002:0000009c       __imp_?sync@?$basic_streambuf@DU?$char_traits@D@std@@@std@@MAEHXZ 1001c09c     msvcprt:MSVCP120.dll
 0002:000000a0       __imp_?showmanyc@?$basic_streambuf@DU?$char_traits@D@std@@@std@@MAE_JXZ 1001c0a0     msvcprt:MSVCP120.dll
 0002:000000a4       __imp_?setbuf@?$basic_streambuf@DU?$char_traits@D@std@@@std@@MAEPAV12@PAD_J@Z 1001c0a4     msvcprt:MSVCP120.dll
 0002:000000a8       __imp_?imbue@?$basic_streambuf@DU?$char_traits@D@std@@@std@@MAEXABVlocale@2@@Z 1001c0a8     msvcprt:MSVCP120.dll
 0002:000000ac       __imp_?_Unlock@?$basic_streambuf@DU?$char_traits@D@std@@@std@@UAEXXZ 1001c0ac     msvcprt:MSVCP120.dll
 0002:000000b0       __imp_?_Lock@?$basic_streambuf@DU?$char_traits@D@std@@@std@@UAEXXZ 1001c0b0     msvcprt:MSVCP120.dll
 0002:000000b4       __imp_??1?$basic_iostream@DU?$char_traits@D@std@@@std@@UAE@XZ 1001c0b4     msvcprt:MSVCP120.dll
 0002:000000b8       __imp_??0?$basic_iostream@DU?$char_traits@D@std@@@std@@QAE@PAV?$basic_streambuf@DU?$char_traits@D@std@@@1@@Z 1001c0b8     msvcprt:MSVCP120.dll
 0002:000000bc       __imp_?flush@?$basic_ostream@DU?$char_traits@D@std@@@std@@QAEAAV12@XZ 1001c0bc     msvcprt:MSVCP120.dll
 0002:000000c0       __imp_??6?$basic_ostream@DU?$char_traits@D@std@@@std@@QAEAAV01@N@Z 1001c0c0     msvcprt:MSVCP120.dll
 0002:000000c4       __imp_?_Osfx@?$basic_ostream@DU?$char_traits@D@std@@@std@@QAEXXZ 1001c0c4     msvcprt:MSVCP120.dll
 0002:000000c8       __imp_?setstate@?$basic_ios@DU?$char_traits@D@std@@@std@@QAEXH_N@Z 1001c0c8     msvcprt:MSVCP120.dll
 0002:000000cc       __imp_??1?$basic_ios@DU?$char_traits@D@std@@@std@@UAE@XZ 1001c0cc     msvcprt:MSVCP120.dll
 0002:000000d0       __imp_?_Pninc@?$basic_streambuf@DU?$char_traits@D@std@@@std@@IAEPADXZ 1001c0d0     msvcprt:MSVCP120.dll
 0002:000000d4       __imp_?sputn@?$basic_streambuf@DU?$char_traits@D@std@@@std@@QAE_JPBD_J@Z 1001c0d4     msvcprt:MSVCP120.dll
 0002:000000d8       __imp_?sputc@?$basic_streambuf@DU?$char_traits@D@std@@@std@@QAEHD@Z 1001c0d8     msvcprt:MSVCP120.dll
 0002:000000dc       __imp_??1?$basic_streambuf@DU?$char_traits@D@std@@@std@@UAE@XZ 1001c0dc     msvcprt:MSVCP120.dll
 0002:000000e0       __imp_??0?$basic_streambuf@DU?$char_traits@D@std@@@std@@IAE@XZ 1001c0e0     msvcprt:MSVCP120.dll
 0002:000000e4       __imp_?_Ios_base_dtor@ios_base@std@@CAXPAV12@@Z 1001c0e4     msvcprt:MSVCP120.dll
 0002:000000e8       __imp_?uncaught_exception@std@@YA_NXZ 1001c0e8     msvcprt:MSVCP120.dll
 0002:000000ec       __imp_?_Winerror_map@std@@YAPBDH@Z 1001c0ec     msvcprt:MSVCP120.dll
 0002:000000f0       __imp_?_Syserror_map@std@@YAPBDH@Z 1001c0f0     msvcprt:MSVCP120.dll
 0002:000000f4       __imp_?_Xout_of_range@std@@YAXPBD@Z 1001c0f4     msvcprt:MSVCP120.dll
 0002:000000f8       __imp_?_Xlength_error@std@@YAXPBD@Z 1001c0f8     msvcprt:MSVCP120.dll
 0002:000000fc       __imp_?_Xbad_alloc@std@@YAXXZ 1001c0fc     msvcprt:MSVCP120.dll
 0002:00000100       \177MSVCP120_NULL_THUNK_DATA 1001c100     msvcprt:MSVCP120.dll
 0002:00000104       __imp___crt_debugger_hook  1001c104     MSVCRT:MSVCR120.dll
 0002:00000108       __imp___hypot              1001c108     MSVCRT:MSVCR120.dll
 0002:0000010c       __imp__memmove             1001c10c     MSVCRT:MSVCR120.dll
 0002:00000110       __imp_??3@YAXPAX@Z         1001c110     MSVCRT:MSVCR120.dll
 0002:00000114       __imp_??2@YAPAXI@Z         1001c114     MSVCRT:MSVCR120.dll
 0002:00000118       __imp___purecall           1001c118     MSVCRT:MSVCR120.dll
 0002:0000011c       __imp____CxxFrameHandler3  1001c11c     MSVCRT:MSVCR120.dll
 0002:00000120       __imp__memcpy              1001c120     MSVCRT:MSVCR120.dll
 0002:00000124       __imp__memset              1001c124     MSVCRT:MSVCR120.dll
 0002:00000128       __imp___libm_sse2_log10_precise 1001c128     MSVCRT:MSVCR120.dll
 0002:0000012c       __imp___libm_sse2_sqrt_precise 1001c12c     MSVCRT:MSVCR120.dll
 0002:00000130       __imp_??0exception@std@@QAE@ABQBD@Z 1001c130     MSVCRT:MSVCR120.dll
 0002:00000134       __imp_??0exception@std@@QAE@ABV01@@Z 1001c134     MSVCRT:MSVCR120.dll
 0002:00000138       __imp_??1exception@std@@UAE@XZ 1001c138     MSVCRT:MSVCR120.dll
 0002:0000013c       __imp_?what@exception@std@@UBEPBDXZ 1001c13c     MSVCRT:MSVCR120.dll
 0002:00000140       __imp___libm_sse2_cos_precise 1001c140     MSVCRT:MSVCR120.dll
 0002:00000144       __imp___libm_sse2_sin_precise 1001c144     MSVCRT:MSVCR120.dll
 0002:00000148       __imp___CIatan2            1001c148     MSVCRT:MSVCR120.dll
 0002:0000014c       __imp___libm_sse2_acos_precise 1001c14c     MSVCRT:MSVCR120.dll
 0002:00000150       __imp__atof                1001c150     MSVCRT:MSVCR120.dll
 0002:00000154       __imp__atoi                1001c154     MSVCRT:MSVCR120.dll
 0002:00000158       __imp__memcpy_s            1001c158     MSVCRT:MSVCR120.dll
 0002:0000015c       __imp__memchr              1001c15c     MSVCRT:MSVCR120.dll
 0002:00000160       __imp__fclose              1001c160     MSVCRT:MSVCR120.dll
 0002:00000164       __imp__fflush              1001c164     MSVCRT:MSVCR120.dll
 0002:00000168       __imp__fgetc               1001c168     MSVCRT:MSVCR120.dll
 0002:0000016c       __imp__fgetpos             1001c16c     MSVCRT:MSVCR120.dll
 0002:00000170       __imp__fopen               1001c170     MSVCRT:MSVCR120.dll
 0002:00000174       __imp__fprintf             1001c174     MSVCRT:MSVCR120.dll
 0002:00000178       __imp__fputc               1001c178     MSVCRT:MSVCR120.dll
 0002:0000017c       __imp__fsetpos             1001c17c     MSVCRT:MSVCR120.dll
 0002:00000180       __imp___fseeki64           1001c180     MSVCRT:MSVCR120.dll
 0002:00000184       __imp__fwrite              1001c184     MSVCRT:MSVCR120.dll
 0002:00000188       __imp__setvbuf             1001c188     MSVCRT:MSVCR120.dll
 0002:0000018c       __imp__ungetc              1001c18c     MSVCRT:MSVCR120.dll
 0002:00000190       __imp___lock_file          1001c190     MSVCRT:MSVCR120.dll
 0002:00000194       __imp___unlock_file        1001c194     MSVCRT:MSVCR120.dll
 0002:00000198       __imp__toupper             1001c198     MSVCRT:MSVCR120.dll
 0002:0000019c       __imp_??0bad_cast@std@@QAE@PBD@Z 1001c19c     MSVCRT:MSVCR120.dll
 0002:000001a0       __imp_??0bad_cast@std@@QAE@ABV01@@Z 1001c1a0     MSVCRT:MSVCR120.dll
 0002:000001a4       __imp_??1bad_cast@std@@UAE@XZ 1001c1a4     MSVCRT:MSVCR120.dll
 0002:000001a8       __imp___lock               1001c1a8     MSVCRT:MSVCR120.dll
 0002:000001ac       __imp___unlock             1001c1ac     MSVCRT:MSVCR120.dll
 0002:000001b0       __imp___calloc_crt         1001c1b0     MSVCRT:MSVCR120.dll
 0002:000001b4       __imp____dllonexit         1001c1b4     MSVCRT:MSVCR120.dll
 0002:000001b8       __imp___onexit             1001c1b8     MSVCRT:MSVCR120.dll
 0002:000001bc       __imp_??1type_info@@UAE@XZ 1001c1bc     MSVCRT:MSVCR120.dll
 0002:000001c0       __imp____crtUnhandledException 1001c1c0     MSVCRT:MSVCR120.dll
 0002:000001c4       __imp____crtTerminateProcess 1001c1c4     MSVCRT:MSVCR120.dll
 0002:000001c8       __imp____clean_type_info_names_internal 1001c1c8     MSVCRT:MSVCR120.dll
 0002:000001cc       __imp_?terminate@@YAXXZ    1001c1cc     MSVCRT:MSVCR120.dll
 0002:000001d0       __imp____CppXcptFilter     1001c1d0     MSVCRT:MSVCR120.dll
 0002:000001d4       __imp___except_handler4_common 1001c1d4     MSVCRT:MSVCR120.dll
 0002:000001d8       __imp___initterm_e         1001c1d8     MSVCRT:MSVCR120.dll
 0002:000001dc       __imp___initterm           1001c1dc     MSVCRT:MSVCR120.dll
 0002:000001e0       __imp___malloc_crt         1001c1e0     MSVCRT:MSVCR120.dll
 0002:000001e4       __imp__free                1001c1e4     MSVCRT:MSVCR120.dll
 0002:000001e8       __imp___amsg_exit          1001c1e8     MSVCRT:MSVCR120.dll
 0002:000001ec       __imp___CxxThrowException@8 1001c1ec     MSVCRT:MSVCR120.dll
 0002:000001f0       \177MSVCR120_NULL_THUNK_DATA 1001c1f0     MSVCRT:MSVCR120.dll
 0002:000001f4       __imp_?dynamicMetaObject@QObjectData@@QBEPAUQMetaObject@@XZ 1001c1f4     Qt5Core:Qt5Core.dll
 0002:000001f8       __imp_?nextNode@QMapNodeBase@@QBEPBU1@XZ 1001c1f8     Qt5Core:Qt5Core.dll
 0002:000001fc       __imp_?realloc@QListData@@QAEXH@Z 1001c1fc     Qt5Core:Qt5Core.dll
 0002:00000200       __imp_??YQString@@QAEAAV0@PBD@Z 1001c200     Qt5Core:Qt5Core.dll
 0002:00000204       __imp_?number@QString@@SA?AV1@NDH@Z 1001c204     Qt5Core:Qt5Core.dll
 0002:00000208       __imp_?toDouble@QString@@QBENPA_N@Z 1001c208     Qt5Core:Qt5Core.dll
 0002:0000020c       __imp_?fromUtf8@QString@@SA?AV1@PBDH@Z 1001c20c     Qt5Core:Qt5Core.dll
 0002:00000210       __imp_?split@QString@@QBE?AVQStringList@@ABV1@W4SplitBehavior@1@W4CaseSensitivity@Qt@@@Z 1001c210     Qt5Core:Qt5Core.dll
 0002:00000214       __imp_?append@QString@@QAEAAV1@ABV1@@Z 1001c214     Qt5Core:Qt5Core.dll
 0002:00000218       __imp_?trimmed@QString@@QBE?AV1@XZ 1001c218     Qt5Core:Qt5Core.dll
 0002:0000021c       __imp_?arg@QString@@QBE?AV1@NHDHVQChar@@@Z 1001c21c     Qt5Core:Qt5Core.dll
 0002:00000220       __imp_?chop@QString@@QAEXH@Z 1001c220     Qt5Core:Qt5Core.dll
 0002:00000224       __imp_??0QString@@QAE@ABV0@@Z 1001c224     Qt5Core:Qt5Core.dll
 0002:00000228       __imp_?shared_null@QListData@@2UData@1@B 1001c228     Qt5Core:Qt5Core.dll
 0002:0000022c       __imp_?timerEvent@QObject@@MAEXPAVQTimerEvent@@@Z 1001c22c     Qt5Core:Qt5Core.dll
 0002:00000230       __imp_?qt_metacast@QObject@@UAEPAXPBD@Z 1001c230     Qt5Core:Qt5Core.dll
 0002:00000234       __imp_?qt_metacall@QObject@@UAEHW4Call@QMetaObject@@HPAPAX@Z 1001c234     Qt5Core:Qt5Core.dll
 0002:00000238       __imp_?metaObject@QObject@@UBEPBUQMetaObject@@XZ 1001c238     Qt5Core:Qt5Core.dll
 0002:0000023c       __imp_?eventFilter@QObject@@UAE_NPAV1@PAVQEvent@@@Z 1001c23c     Qt5Core:Qt5Core.dll
 0002:00000240       __imp_?event@QObject@@UAE_NPAVQEvent@@@Z 1001c240     Qt5Core:Qt5Core.dll
 0002:00000244       __imp_?qBadAlloc@@YAXXZ    1001c244     Qt5Core:Qt5Core.dll
 0002:00000248       __imp_?disconnectNotify@QObject@@MAEXABVQMetaMethod@@@Z 1001c248     Qt5Core:Qt5Core.dll
 0002:0000024c       __imp_?customEvent@QObject@@MAEXPAVQEvent@@@Z 1001c24c     Qt5Core:Qt5Core.dll
 0002:00000250       __imp_?connectNotify@QObject@@MAEXABVQMetaMethod@@@Z 1001c250     Qt5Core:Qt5Core.dll
 0002:00000254       __imp_?childEvent@QObject@@MAEXPAVQChildEvent@@@Z 1001c254     Qt5Core:Qt5Core.dll
 0002:00000258       __imp_??1QObject@@UAE@XZ   1001c258     Qt5Core:Qt5Core.dll
 0002:0000025c       __imp_??0QObject@@QAE@PAV0@@Z 1001c25c     Qt5Core:Qt5Core.dll
 0002:00000260       __imp_?tr@QMetaObject@@QBE?AVQString@@PBD0H@Z 1001c260     Qt5Core:Qt5Core.dll
 0002:00000264       __imp_?cast@QMetaObject@@QBEPAVQObject@@PAV2@@Z 1001c264     Qt5Core:Qt5Core.dll
 0002:00000268       __imp_?append@QListData@@QAEPAPAXXZ 1001c268     Qt5Core:Qt5Core.dll
 0002:0000026c       __imp_?detach_grow@QListData@@QAEPAUData@1@PAHH@Z 1001c26c     Qt5Core:Qt5Core.dll
 0002:00000270       __imp_?shared_null@QArrayData@@2QBU1@B 1001c270     Qt5Core:Qt5Core.dll
 0002:00000274       __imp_?freeData@QMapDataBase@@SAXPAU1@@Z 1001c274     Qt5Core:Qt5Core.dll
 0002:00000278       __imp_?freeTree@QMapDataBase@@QAEXPAUQMapNodeBase@@H@Z 1001c278     Qt5Core:Qt5Core.dll
 0002:0000027c       __imp_?dispose@QListData@@SAXPAUData@1@@Z 1001c27c     Qt5Core:Qt5Core.dll
 0002:00000280       __imp_?detach@QListData@@QAEPAUData@1@H@Z 1001c280     Qt5Core:Qt5Core.dll
 0002:00000284       __imp_?fromAscii_helper@QString@@CAPAU?$QTypedArrayData@G@@PBDH@Z 1001c284     Qt5Core:Qt5Core.dll
 0002:00000288       __imp_?arg@QString@@QBE?AV1@ABV1@0@Z 1001c288     Qt5Core:Qt5Core.dll
 0002:0000028c       __imp_?arg@QString@@QBE?AV1@ABV1@HVQChar@@@Z 1001c28c     Qt5Core:Qt5Core.dll
 0002:00000290       __imp_??4QString@@QAEAAV0@$$QAV0@@Z 1001c290     Qt5Core:Qt5Core.dll
 0002:00000294       __imp_??1QString@@QAE@XZ   1001c294     Qt5Core:Qt5Core.dll
 0002:00000298       __imp_??0QString@@QAE@XZ   1001c298     Qt5Core:Qt5Core.dll
 0002:0000029c       __imp_?data@QByteArray@@QBEPBDXZ 1001c29c     Qt5Core:Qt5Core.dll
 0002:000002a0       __imp_??1QByteArray@@QAE@XZ 1001c2a0     Qt5Core:Qt5Core.dll
 0002:000002a4       __imp_?qstrcmp@@YAHABVQByteArray@@PBD@Z 1001c2a4     Qt5Core:Qt5Core.dll
 0002:000002a8       __imp_?deallocate@QArrayData@@SAXPAU1@II@Z 1001c2a8     Qt5Core:Qt5Core.dll
 0002:000002ac       __imp_?allocate@QArrayData@@SAPAU1@IIIV?$QFlags@W4AllocationOption@QArrayData@@@@@Z 1001c2ac     Qt5Core:Qt5Core.dll
 0002:000002b0       __imp_?data@QArrayData@@QAEPAXXZ 1001c2b0     Qt5Core:Qt5Core.dll
 0002:000002b4       __imp_??0QChar@@QAE@UQLatin1Char@@@Z 1001c2b4     Qt5Core:Qt5Core.dll
 0002:000002b8       \177Qt5Core_NULL_THUNK_DATA 1001c2b8     Qt5Core:Qt5Core.dll
 0002:000002bc       __imp_?attribute@QDomElement@@QBE?AVQString@@ABV2@0@Z 1001c2bc     Qt5Xml:Qt5Xml.dll
 0002:000002c0       \177Qt5Xml_NULL_THUNK_DATA 1001c2c0     Qt5Xml:Qt5Xml.dll
 0002:000002c4       __imp_??0StructuralAlignmentTaskSettings@U2@@QAE@ABVBioStruct3DReference@1@0@Z 1001c2c4     U2Algorithm:U2Algorithm.dll
 0002:000002c8       __imp_??1BioStruct3DReference@U2@@QAE@XZ 1001c2c8     U2Algorithm:U2Algorithm.dll
 0002:000002cc       __imp_??0BioStruct3DReference@U2@@QAE@PBVBioStruct3DObject@1@ABV?$QList@H@@H@Z 1001c2cc     U2Algorithm:U2Algorithm.dll
 0002:000002d0       __imp_??_7StructuralAlignmentAlgorithmFactory@U2@@6B@ 1001c2d0     U2Algorithm:U2Algorithm.dll
 0002:000002d4       __imp_??_7StructuralAlignmentAlgorithm@U2@@6B@ 1001c2d4     U2Algorithm:U2Algorithm.dll
 0002:000002d8       __imp_?registerAlgorithmFactory@StructuralAlignmentAlgorithmRegistry@U2@@QAEXPAVStructuralAlignmentAlgorithmFactory@2@ABVQString@@@Z 1001c2d8     U2Algorithm:U2Algorithm.dll
 0002:000002dc       __imp_??1StructuralAlignment@U2@@QAE@XZ 1001c2dc     U2Algorithm:U2Algorithm.dll
 0002:000002e0       __imp_??0StructuralAlignment@U2@@QAE@XZ 1001c2e0     U2Algorithm:U2Algorithm.dll
 0002:000002e4       __imp_?print@BioStruct3DReference@U2@@QBE?AVQString@@XZ 1001c2e4     U2Algorithm:U2Algorithm.dll
 0002:000002e8       __imp_??1StructuralAlignmentTaskSettings@U2@@QAE@XZ 1001c2e8     U2Algorithm:U2Algorithm.dll
 0002:000002ec       \177U2Algorithm_NULL_THUNK_DATA 1001c2ec     U2Algorithm:U2Algorithm.dll
 0002:000002f0       __imp_?isNotificationReport@Task@U2@@UBE_NXZ 1001c2f0     U2Core:U2Core.dll
 0002:000002f4       __imp_?isReportingEnabled@Task@U2@@UBE_NXZ 1001c2f4     U2Core:U2Core.dll
 0002:000002f8       __imp_?isReportingSupported@Task@U2@@UBE_NXZ 1001c2f8     U2Core:U2Core.dll
 0002:000002fc       __imp_?isTopLevelTask@Task@U2@@UBE_NXZ 1001c2fc     U2Core:U2Core.dll
 0002:00000300       __imp_?onSubTaskFinished@Task@U2@@MAE?AV?$QList@PAVTask@U2@@@@PAV12@@Z 1001c300     U2Core:U2Core.dll
 0002:00000304       __imp_?prepare@Task@U2@@UAEXXZ 1001c304     U2Core:U2Core.dll
 0002:00000308       __imp_?propagateSubtaskError@Task@U2@@UAE_NXZ 1001c308     U2Core:U2Core.dll
 0002:0000030c       __imp_?setCollectChildrensWarningsFlag@Task@U2@@UAEX_N@Z 1001c30c     U2Core:U2Core.dll
 0002:00000310       __imp_?setNoAutoDelete@Task@U2@@UAEX_N@Z 1001c310     U2Core:U2Core.dll
 0002:00000314       __imp_?hasWarning@Task@U2@@UBE_NXZ 1001c314     U2Core:U2Core.dll
 0002:00000318       __imp_?setReportingEnabled@Task@U2@@UAEX_N@Z 1001c318     U2Core:U2Core.dll
 0002:0000031c       __imp_?setReportingSupported@Task@U2@@UAEX_N@Z 1001c31c     U2Core:U2Core.dll
 0002:00000320       __imp_??4Matrix44@U2@@QAEAAV01@ABV01@@Z 1001c320     U2Core:U2Core.dll
 0002:00000324       __imp_?setError@Task@U2@@QAEXABVQString@@@Z 1001c324     U2Core:U2Core.dll
 0002:00000328       __imp_?staticMetaObject@BioStruct3DObject@U2@@2UQMetaObject@@B 1001c328     U2Core:U2Core.dll
 0002:0000032c       __imp_?qt_metacast@Plugin@U2@@UAEPAXPBD@Z 1001c32c     U2Core:U2Core.dll
 0002:00000330       __imp_?qt_metacall@Plugin@U2@@UAEHW4Call@QMetaObject@@HPAPAX@Z 1001c330     U2Core:U2Core.dll
 0002:00000334       __imp_?staticMetaObject@Plugin@U2@@2UQMetaObject@@B 1001c334     U2Core:U2Core.dll
 0002:00000338       __imp_?hasSubtasksWithErrors@Task@U2@@UBE_NXZ 1001c338     U2Core:U2Core.dll
 0002:0000033c       __imp_?getWarnings@Task@U2@@UBE?AVQStringList@@XZ 1001c33c     U2Core:U2Core.dll
 0002:00000340       __imp_?getTopLevelParentTask@Task@U2@@UAEPAV12@XZ 1001c340     U2Core:U2Core.dll
 0002:00000344       __imp_?getTaskId@Task@U2@@UBE_JXZ 1001c344     U2Core:U2Core.dll
 0002:00000348       __imp_?getSubtaskWithErrors@Task@U2@@UBEPAV12@XZ 1001c348     U2Core:U2Core.dll
 0002:0000034c       __imp_?getParentTask@Task@U2@@UBEPAV12@XZ 1001c34c     U2Core:U2Core.dll
 0002:00000350       __imp_?getNumParallelSubtasks@Task@U2@@UBEHXZ 1001c350     U2Core:U2Core.dll
 0002:00000354       __imp_?generateReport@Task@U2@@UBE?AVQString@@XZ 1001c354     U2Core:U2Core.dll
 0002:00000358       __imp_?cleanup@Task@U2@@UAEXXZ 1001c358     U2Core:U2Core.dll
 0002:0000035c       __imp_?setNotificationReport@Task@U2@@UAEX_N@Z 1001c35c     U2Core:U2Core.dll
 0002:00000360       __imp_?getStructuralAlignmentAlgorithmRegistry@AppContext@U2@@SAPAVStructuralAlignmentAlgorithmRegistry@2@XZ 1001c360     U2Core:U2Core.dll
 0002:00000364       __imp_?getTestFramework@AppContext@U2@@SAPAVTestFramework@2@XZ 1001c364     U2Core:U2Core.dll
 0002:00000368       __imp_??1Plugin@U2@@UAE@XZ 1001c368     U2Core:U2Core.dll
 0002:0000036c       __imp_??0Plugin@U2@@QAE@ABVQString@@0_NW4PluginState@1@@Z 1001c36c     U2Core:U2Core.dll
 0002:00000370       __imp_?getBioStruct3D@BioStruct3DObject@U2@@QBEABVBioStruct3D@2@XZ 1001c370     U2Core:U2Core.dll
 0002:00000374       __imp_?getModelByName@BioStruct3D@U2@@QBE?BVMolecule3DModel@2@HH@Z 1001c374     U2Core:U2Core.dll
 0002:00000378       __imp_?error@Logger@U2@@QAEXABVQString@@@Z 1001c378     U2Core:U2Core.dll
 0002:0000037c       __imp_?trace@Logger@U2@@QAEXABVQString@@@Z 1001c37c     U2Core:U2Core.dll
 0002:00000380       __imp_??1Logger@U2@@UAE@XZ 1001c380     U2Core:U2Core.dll
 0002:00000384       __imp_??0Logger@U2@@QAE@ABVQString@@@Z 1001c384     U2Core:U2Core.dll
 0002:00000388       __imp_??AMatrix44@U2@@QBEMI@Z 1001c388     U2Core:U2Core.dll
 0002:0000038c       __imp_??AMatrix44@U2@@QAEAAMI@Z 1001c38c     U2Core:U2Core.dll
 0002:00000390       \177U2Core_NULL_THUNK_DATA 1001c390     U2Core:U2Core.dll
 0002:00000394       __imp_??1XMLTestFactory@U2@@UAE@XZ 1001c394     U2Test:U2Test.dll
 0002:00000398       __imp_??0XmlTest@U2@@QAE@ABVQString@@PAVGTest@1@PBVGTestEnvironment@1@V?$QFlags@W4TaskFlag@U2@@@@ABV?$QList@PAVGTest@U2@@@@@Z 1001c398     U2Test:U2Test.dll
 0002:0000039c       __imp_??1XmlTest@U2@@UAE@XZ 1001c39c     U2Test:U2Test.dll
 0002:000003a0       __imp_?findFormat@GTestFormatRegistry@U2@@QAEPAVGTestFormat@2@ABVQString@@@Z 1001c3a0     U2Test:U2Test.dll
 0002:000003a4       __imp_?staticMetaObject@XMLTestFormat@U2@@2UQMetaObject@@B 1001c3a4     U2Test:U2Test.dll
 0002:000003a8       __imp_?getContext@GTest@U2@@QBEPAVQObject@@ABVQString@@@Z 1001c3a8     U2Test:U2Test.dll
 0002:000003ac       __imp_?failMissingValue@GTest@U2@@IAEXABVQString@@@Z 1001c3ac     U2Test:U2Test.dll
 0002:000003b0       __imp_?qt_metacast@GTest@U2@@UAEPAXPBD@Z 1001c3b0     U2Test:U2Test.dll
 0002:000003b4       __imp_?qt_metacall@GTest@U2@@UAEHW4Call@QMetaObject@@HPAPAX@Z 1001c3b4     U2Test:U2Test.dll
 0002:000003b8       __imp_?staticMetaObject@GTest@U2@@2UQMetaObject@@B 1001c3b8     U2Test:U2Test.dll
 0002:000003bc       __imp_??0XMLTestFactory@U2@@QAE@ABVQString@@@Z 1001c3bc     U2Test:U2Test.dll
 0002:000003c0       \177U2Test_NULL_THUNK_DATA 1001c3c0     U2Test:U2Test.dll
 0002:000003c4       ___xc_a                    1001c3c4     MSVCRT:cinitexe.obj
 0002:000004ac       ___xc_z                    1001c4ac     MSVCRT:cinitexe.obj
 0002:000004b0       ___xi_a                    1001c4b0     MSVCRT:cinitexe.obj
 0002:000004bc       ___xi_z                    1001c4bc     MSVCRT:cinitexe.obj
 0002:000004fc       ??_7error_category@std@@6B@ 1001c4fc     PToolsAligner.obj
 0002:00000518       ??_7_Generic_error_category@std@@6B@ 1001c518     PToolsAligner.obj
 0002:00000530       ??_C@_07DCLBNMLN@generic?$AA@ 1001c530     PToolsAligner.obj
 0002:00000538       ??_C@_0O@BFJCFAAK@unknown?5error?$AA@ 1001c538     PToolsAligner.obj
 0002:0000054c       ??_7_Iostream_error_category@std@@6B@ 1001c54c     PToolsAligner.obj
 0002:00000564       ??_C@_08LLGCOLLL@iostream?$AA@ 1001c564     PToolsAligner.obj
 0002:00000570       ??_C@_0BG@PADBLCHM@iostream?5stream?5error?$AA@ 1001c570     PToolsAligner.obj
 0002:0000058c       ??_7_System_error_category@std@@6B@ 1001c58c     PToolsAligner.obj
 0002:000005a4       ??_C@_06FHFOAHML@system?$AA@ 1001c5a4     PToolsAligner.obj
 0002:000005ac       ??_C@_0L@JLHNEGIN@Algorithms?$AA@ 1001c5ac     PToolsAligner.obj
 0002:000005b8       ??_C@_07PGLPGHFC@Console?$AA@ 1001c5b8     PToolsAligner.obj
 0002:000005c0       ??_C@_0O@BOFHOPCF@Core?5Services?$AA@ 1001c5c0     PToolsAligner.obj
 0002:000005d0       ??_C@_0N@PPADAKBM@Input?1Output?$AA@ 1001c5d0     PToolsAligner.obj
 0002:000005e0       ??_C@_0M@KPPBKPKK@Performance?$AA@ 1001c5e0     PToolsAligner.obj
 0002:000005ec       ??_C@_07BFDHHBBI@Scripts?$AA@ 1001c5ec     PToolsAligner.obj
 0002:000005f4       ??_C@_05EEGKELMG@Tasks?$AA@ 1001c5f4     PToolsAligner.obj
 0002:000005fc       ??_C@_0P@NIIOBHGA@User?5Interface?$AA@ 1001c5fc     PToolsAligner.obj
 0002:0000060c       ??_C@_0N@JINCGGMN@User?5Actions?$AA@ 1001c60c     PToolsAligner.obj
 0002:0000061c       ??_C@_01MMEEDKFM@X?$AA@    1001c61c     PToolsAligner.obj
 0002:00000620       ??_C@_03MAMPKPPK@XXX?$AA@  1001c620     PToolsAligner.obj
 0002:00000624       ??_C@_02JLAAGLDA@CA?$AA@   1001c624     PToolsAligner.obj
 0002:00000628       ??_C@_0DK@ENAMFNDC@structure?5subsets?5has?5different?5@ 1001c628     PToolsAligner.obj
 0002:00000664       ??_C@_0CO@LHCCMO@PToolsAligner?5started?5on?5?$CF1?5?$CIref@ 1001c664     PToolsAligner.obj
 0002:00000698       ??_C@_0EB@OADKJMLA@Failed?5to?5align?0?5subsets?5turn?5to@ 1001c698     PToolsAligner.obj
 0002:000006dc       ??_C@_0BK@LMCGAOAJ@Internal?5ptools?5error?3?5?$CF1?$AA@ 1001c6dc     PToolsAligner.obj
 0002:000006f8       ??_C@_0BG@JJBFMAJH@Internal?5ptools?5error?$AA@ 1001c6f8     PToolsAligner.obj
 0002:00000710       ??_C@_0BA@JFNIOLAK@string?5too?5long?$AA@ 1001c710     PToolsAligner.obj
 0002:00000720       ??_C@_0BI@CFPLBAOH@invalid?5string?5position?$AA@ 1001c720     PToolsAligner.obj
 0002:0000073c       ??_7PToolsPlugin@U2@@6B@   1001c73c     PToolsPlugin.obj
 0002:0000076c       ??_7PToolsAligner@U2@@6B@  1001c76c     PToolsPlugin.obj
 0002:0000077c       ??_7PToolsAlignerFactory@U2@@6B@ 1001c77c     PToolsPlugin.obj
 0002:00000788       ??_7Gtest_PToolsAlignerTaskFactory@Gtest_PToolsAlignerTask@U2@@6B@ 1001c788     PToolsPlugin.obj
 0002:00000794       ??_7Gtest_PToolsAlignerTask@U2@@6B@ 1001c794     PToolsPlugin.obj
 0002:00000820       ??_C@_0BJ@JJBEOFKB@ptools?9align?9and?9compare?$AA@ 1001c820     PToolsPlugin.obj
 0002:0000083c       ??_C@_06OLKBJMGP@PTools?$AA@ 1001c83c     PToolsPlugin.obj
 0002:00000848       ??_C@_0EN@GFJMIOHC@Structural?5alignment?5algorithm?5?$CI@ 1001c848     PToolsPlugin.obj
 0002:00000898       ??_C@_03PEIMBJDE@XML?$AA@  1001c898     PToolsPlugin.obj
 0002:000008a0       ??_7?$GAutoDeleteList@VXMLTestFactory@U2@@@U2@@6B@ 1001c8a0     PToolsPlugin.obj
 0002:000008cc       ??_C@_04BIAIHMIG@refo?$AA@ 1001c8cc     PToolsTests.obj
 0002:000008d4       ??_C@_04JCAMDEGN@mobo?$AA@ 1001c8d4     PToolsTests.obj
 0002:000008dc       ??_C@_04CEKFOMDJ@rmsd?$AA@ 1001c8dc     PToolsTests.obj
 0002:000008e4       ??_C@_08FJNPIHOL@accuracy?$AA@ 1001c8e4     PToolsTests.obj
 0002:000008f0       ??_C@_09IFONHNKG@transform?$AA@ 1001c8f0     PToolsTests.obj
 0002:000008fc       ??_C@_0BJ@PDNKHEPB@Error?3?5bad?5rmsd?5value?5?$CF1?$AA@ 1001c8fc     PToolsTests.obj
 0002:00000918       ??_C@_01GBGANLPD@0?$AA@    1001c918     PToolsTests.obj
 0002:0000091c       ??_C@_01IHBHIGKO@?0?$AA@   1001c91c     PToolsTests.obj
 0002:00000920       ??_C@_0CF@OAPCHGGH@Error?3?5bad?5transform?5matrix?5valu@ 1001c920     PToolsTests.obj
 0002:00000948       ??_C@_0CN@GCDEHOBE@Error?3?5bad?5transform?5matrix?5elem@ 1001c948     PToolsTests.obj
 0002:00000978       ??_C@_0DI@HDONGGMA@Error?3?5can?8t?5cast?5to?5BioSrtuct3D@ 1001c978     PToolsTests.obj
 0002:000009b0       ??_C@_06LCKCPPDI@RMSD?3?5?$AA@ 1001c9b0     PToolsTests.obj
 0002:000009b8       ??_C@_0BA@CPIHLHLE@?$DL?5Transform?3?5?$FL?5?$AA@ 1001c9b8     PToolsTests.obj
 0002:000009c8       ??_C@_02KEGNLNML@?0?5?$AA@ 1001c9c8     PToolsTests.obj
 0002:000009cc       ??_C@_02DHOGEDBE@?5?$FN?$AA@ 1001c9cc     PToolsTests.obj
 0002:000009d0       ??_C@_0DD@JMPNIACK@Alignment?5results?5are?5not?5equal?5@ 1001c9d0     PToolsTests.obj
 0002:00000a04       ??_C@_0BA@DJNGKFJA@?5Calculated?5?9?5?6?$AA@ 1001ca04     PToolsTests.obj
 0002:00000a14       ??_C@_0BA@MDNPLFJI@?5Expected?5?5?5?9?5?6?$AA@ 1001ca14     PToolsTests.obj
 0002:00000a28       __real@0000000000000000    1001ca28     PToolsTests.obj
 0002:00000a30       __real@3ff0000000000000    1001ca30     PToolsTests.obj
 0002:00000a40       __xmm@7fffffffffffffff7fffffffffffffff 1001ca40     PToolsTests.obj
 0002:00000a54       ??_7Rigidbody@PTools@@6B@  1001ca54     atomselection.obj
 0002:00000a60       ??_C@_0BD@OLBABOEK@vector?$DMT?$DO?5too?5long?$AA@ 1001ca60     atomselection.obj
 0002:00000a78       ??_7?$basic_stringbuf@DU?$char_traits@D@std@@V?$allocator@D@2@@std@@6B@ 1001ca78     coord3d.obj
 0002:00000ab8       ??_7?$basic_stringstream@DU?$char_traits@D@std@@V?$allocator@D@2@@std@@6B@ 1001cab8     coord3d.obj
 0002:00000abc       ??_8?$basic_stringstream@DU?$char_traits@D@std@@V?$allocator@D@2@@std@@7B?$basic_istream@DU?$char_traits@D@std@@@1@@ 1001cabc     coord3d.obj
 0002:00000ac4       ??_8?$basic_stringstream@DU?$char_traits@D@std@@V?$allocator@D@2@@std@@7B?$basic_ostream@DU?$char_traits@D@std@@@1@@ 1001cac4     coord3d.obj
 0002:00000acc       ??_C@_02KNHHEEKP@?5?5?$AA@ 1001cacc     coord3d.obj
 0002:00000ad0       ??_C@_01EEMJAFIK@?6?$AA@   1001cad0     coord3d.obj
 0002:00000ad8       ??_7logic_error@std@@6B@   1001cad8     coordsarray.obj
 0002:00000ae4       ??_7out_of_range@std@@6B@  1001cae4     coordsarray.obj
 0002:00000aec       ??_C@_0CK@HDODJKKG@CoordsArray?3?3GetCoords?5?3?5out?5of?5@ 1001caec     coordsarray.obj
 0002:00000b18       ??_C@_0CB@CJBLNFJD@?5is?5out?5of?5bounds?5?$CIobject?5size?3?5@ 1001cb18     coordsarray.obj
 0002:00000b3c       ??_C@_02MNMNLDAI@?$CJ?6?$AA@ 1001cb3c     coordsarray.obj
 0002:00000b40       __xmm@80000000000000008000000000000000 1001cb40     coordsarray.obj
 0002:00000b50       __xmm@00000000000000003ff0000000000000 1001cb50     geometry.obj
 0002:00000b60       __xmm@3ff00000000000000000000000000000 1001cb60     geometry.obj
 0002:00000b74       ??_7invalid_argument@std@@6B@ 1001cb74     pdbio.obj
 0002:00000b7c       ??_C@_00CNPNBAHC@?$AA@     1001cb7c     pdbio.obj
 0002:00000b80       ??_C@_06JOEDJJH@ATOM?5?5?$AA@ 1001cb80     pdbio.obj
 0002:00000b88       ??_C@_06IKLLGBDH@HETATM?$AA@ 1001cb88     pdbio.obj
 0002:00000b94       ??_7?$basic_filebuf@DU?$char_traits@D@std@@@std@@6B@ 1001cb94     pdbio.obj
 0002:00000bd4       ??_7?$basic_ifstream@DU?$char_traits@D@std@@@std@@6B@ 1001cbd4     pdbio.obj
 0002:00000bd8       ??_8?$basic_ifstream@DU?$char_traits@D@std@@@std@@7B@ 1001cbd8     pdbio.obj
 0002:00000be4       ??_7?$basic_ostringstream@DU?$char_traits@D@std@@V?$allocator@D@2@@std@@6B@ 1001cbe4     pdbio.obj
 0002:00000be8       ??_8?$basic_ostringstream@DU?$char_traits@D@std@@V?$allocator@D@2@@std@@7B@ 1001cbe8     pdbio.obj
 0002:00000bf0       ??_C@_07NPEPNBGF@?$CC?5?$CD?$CD?$CD?$CD?$CD?$AA@ 1001cbf0     pdbio.obj
 0002:00000bf8       ??_C@_0CE@ELABADMI@?$CD?$CD?$CD?$CD?$CD?5ReadPDB?3Could?5not?5open?5fil@ 1001cbf8     pdbio.obj
 0002:00000c1c       ??_C@_01NOFIACDB@w?$AA@    1001cc1c     pdbio.obj
 0002:00000c20       ??_C@_0CP@PHILIGMB@ATOM?5?5?$CF5d?5?5?$CF?94s?$CF3s?5?$CF1s?$CF4d?5?5?5?5?$CF8?4@ 1001cc20     pdbio.obj
 0002:00000c50       ??_C@_08EPJLHIJG@bad?5cast?$AA@ 1001cc50     pdbio.obj
 0002:00000c5c       ??_C@_01GFHCPBMG@C?$AA@    1001cc5c     rigidbody.obj
 0002:00000c60       ??_C@_0BD@NCDPAEGH@SetAtom?3?5position?5?$AA@ 1001cc60     rigidbody.obj
 0002:00000c74       ??_C@_0BB@IELAECFH@?5is?5out?5of?5range?$AA@ 1001cc74     rigidbody.obj
 0002:00000c88       ??_C@_01NANMIPIL@N?$AA@    1001cc88     rigidbody.obj
 0002:00000c8c       ??_C@_01MJMHLOMK@O?$AA@    1001cc8c     rigidbody.obj
 0002:00000c90       __xmm@41f00000000000000000000000000000 1001cc90     rigidbody.obj
 0002:00000ca0       ??_C@_0BB@NNAPBAPB@RmsdSizesDiffers?$AA@ 1001cca0     rmsd.obj
 0002:00000cb8       ??_7runtime_error@std@@6B@ 1001ccb8     superpose.obj
 0002:00000cc0       ??_C@_0FJ@DICMNFHM@in?5superpose?4cpp?0?5in?5MakeTensor?3@ 1001ccc0     superpose.obj
 0002:00000d20       __real@3ee4f8b588e368f1    1001cd20     superpose.obj
 0002:00000d28       __real@3fb999999999999a    1001cd28     superpose.obj
 0002:00000d30       __real@bff0000000000000    1001cd30     superpose.obj
 0002:00000e00       ?value@?$integral_constant@_N$0A@@std@@2_NB 1001ce00     MSVCRT:ti_inst.obj
 0002:00000e01       ?value@?$integral_constant@_N$00@std@@2_NB 1001ce01     MSVCRT:ti_inst.obj
 0002:00000e08       ??_7type_info@@6B@         1001ce08     MSVCRT:ti_inst.obj
 0002:00000e0c       __pDefaultRawDllMain       1001ce0c     MSVCRT:crtdll.obj
 0002:00000e0c       __pRawDllMain              1001ce0c     MSVCRT:crtdll.obj
 0002:00000e18       ?ProcessDetach@NativeDll@<CrtImplementationDetails>@@0IB 1001ce18     MSVCRT:initsect.obj
 0002:00000e1c       ?ProcessAttach@NativeDll@<CrtImplementationDetails>@@0IB 1001ce1c     MSVCRT:initsect.obj
 0002:00000e20       ?ThreadAttach@NativeDll@<CrtImplementationDetails>@@0IB 1001ce20     MSVCRT:initsect.obj
 0002:00000e24       ?ThreadDetach@NativeDll@<CrtImplementationDetails>@@0IB 1001ce24     MSVCRT:initsect.obj
 0002:00000e28       ?ProcessVerifier@NativeDll@<CrtImplementationDetails>@@0IB 1001ce28     MSVCRT:initsect.obj
 0002:00000e30       __load_config_used         1001ce30     MSVCRT:loadcfg.obj
 0002:00000ee4       ??_R4error_category@std@@6B@ 1001cee4     PToolsAligner.obj
 0002:00000ef8       ??_R3error_category@std@@8 1001cef8     PToolsAligner.obj
 0002:00000f08       ??_R2error_category@std@@8 1001cf08     PToolsAligner.obj
 0002:00000f10       ??_R1A@?0A@EA@error_category@std@@8 1001cf10     PToolsAligner.obj
 0002:00000f2c       ??_R4_Generic_error_category@std@@6B@ 1001cf2c     PToolsAligner.obj
 0002:00000f40       ??_R3_Generic_error_category@std@@8 1001cf40     PToolsAligner.obj
 0002:00000f50       ??_R2_Generic_error_category@std@@8 1001cf50     PToolsAligner.obj
 0002:00000f5c       ??_R1A@?0A@EA@_Generic_error_category@std@@8 1001cf5c     PToolsAligner.obj
 0002:00000f78       ??_R4_Iostream_error_category@std@@6B@ 1001cf78     PToolsAligner.obj
 0002:00000f8c       ??_R3_Iostream_error_category@std@@8 1001cf8c     PToolsAligner.obj
 0002:00000f9c       ??_R2_Iostream_error_category@std@@8 1001cf9c     PToolsAligner.obj
 0002:00000fac       ??_R1A@?0A@EA@_Iostream_error_category@std@@8 1001cfac     PToolsAligner.obj
 0002:00000fc8       ??_R4_System_error_category@std@@6B@ 1001cfc8     PToolsAligner.obj
 0002:00000fdc       ??_R3_System_error_category@std@@8 1001cfdc     PToolsAligner.obj
 0002:00000fec       ??_R2_System_error_category@std@@8 1001cfec     PToolsAligner.obj
 0002:00000ffc       ??_R1A@?0A@EA@_System_error_category@std@@8 1001cffc     PToolsAligner.obj
 0002:00001018       ??_R1A@?0A@EA@XmlTest@U2@@8 1001d018     PToolsPlugin.obj
 0002:00001034       ??_R3XmlTest@U2@@8         1001d034     PToolsPlugin.obj
 0002:00001044       ??_R2XmlTest@U2@@8         1001d044     PToolsPlugin.obj
 0002:00001058       ??_R1A@?0A@EA@GTest@U2@@8  1001d058     PToolsPlugin.obj
 0002:00001074       ??_R3GTest@U2@@8           1001d074     PToolsPlugin.obj
 0002:00001084       ??_R2GTest@U2@@8           1001d084     PToolsPlugin.obj
 0002:00001094       ??_R1A@?0A@EA@Task@U2@@8   1001d094     PToolsPlugin.obj
 0002:000010b0       ??_R3Task@U2@@8            1001d0b0     PToolsPlugin.obj
 0002:000010c0       ??_R2Task@U2@@8            1001d0c0     PToolsPlugin.obj
 0002:000010cc       ??_R1A@?0A@EA@QObject@@8   1001d0cc     PToolsPlugin.obj
 0002:000010e8       ??_R3QObject@@8            1001d0e8     PToolsPlugin.obj
 0002:000010f8       ??_R2QObject@@8            1001d0f8     PToolsPlugin.obj
 0002:00001100       ??_R1A@?0A@EA@XMLTestFactory@U2@@8 1001d100     PToolsPlugin.obj
 0002:0000111c       ??_R3XMLTestFactory@U2@@8  1001d11c     PToolsPlugin.obj
 0002:0000112c       ??_R2XMLTestFactory@U2@@8  1001d12c     PToolsPlugin.obj
 0002:00001134       ??_R4PToolsPlugin@U2@@6B@  1001d134     PToolsPlugin.obj
 0002:00001148       ??_R3PToolsPlugin@U2@@8    1001d148     PToolsPlugin.obj
 0002:00001158       ??_R2PToolsPlugin@U2@@8    1001d158     PToolsPlugin.obj
 0002:00001168       ??_R1A@?0A@EA@PToolsPlugin@U2@@8 1001d168     PToolsPlugin.obj
 0002:00001184       ??_R1A@?0A@EA@Plugin@U2@@8 1001d184     PToolsPlugin.obj
 0002:000011a0       ??_R3Plugin@U2@@8          1001d1a0     PToolsPlugin.obj
 0002:000011b0       ??_R2Plugin@U2@@8          1001d1b0     PToolsPlugin.obj
 0002:000011bc       ??_R4PToolsAligner@U2@@6B@ 1001d1bc     PToolsPlugin.obj
 0002:000011d0       ??_R3PToolsAligner@U2@@8   1001d1d0     PToolsPlugin.obj
 0002:000011e0       ??_R2PToolsAligner@U2@@8   1001d1e0     PToolsPlugin.obj
 0002:000011ec       ??_R1A@?0A@EA@PToolsAligner@U2@@8 1001d1ec     PToolsPlugin.obj
 0002:00001208       ??_R1A@?0A@EA@StructuralAlignmentAlgorithm@U2@@8 1001d208     PToolsPlugin.obj
 0002:00001224       ??_R3StructuralAlignmentAlgorithm@U2@@8 1001d224     PToolsPlugin.obj
 0002:00001234       ??_R2StructuralAlignmentAlgorithm@U2@@8 1001d234     PToolsPlugin.obj
 0002:0000123c       ??_R4PToolsAlignerFactory@U2@@6B@ 1001d23c     PToolsPlugin.obj
 0002:00001250       ??_R3PToolsAlignerFactory@U2@@8 1001d250     PToolsPlugin.obj
 0002:00001260       ??_R2PToolsAlignerFactory@U2@@8 1001d260     PToolsPlugin.obj
 0002:0000126c       ??_R1A@?0A@EA@PToolsAlignerFactory@U2@@8 1001d26c     PToolsPlugin.obj
 0002:00001288       ??_R1A@?0A@EA@StructuralAlignmentAlgorithmFactory@U2@@8 1001d288     PToolsPlugin.obj
 0002:000012a4       ??_R3StructuralAlignmentAlgorithmFactory@U2@@8 1001d2a4     PToolsPlugin.obj
 0002:000012b4       ??_R2StructuralAlignmentAlgorithmFactory@U2@@8 1001d2b4     PToolsPlugin.obj
 0002:000012bc       ??_R4Gtest_PToolsAlignerTask@U2@@6B@ 1001d2bc     PToolsPlugin.obj
 0002:000012d0       ??_R3Gtest_PToolsAlignerTask@U2@@8 1001d2d0     PToolsPlugin.obj
 0002:000012e0       ??_R2Gtest_PToolsAlignerTask@U2@@8 1001d2e0     PToolsPlugin.obj
 0002:000012f8       ??_R1A@?0A@EA@Gtest_PToolsAlignerTask@U2@@8 1001d2f8     PToolsPlugin.obj
 0002:00001314       ??_R4Gtest_PToolsAlignerTaskFactory@Gtest_PToolsAlignerTask@U2@@6B@ 1001d314     PToolsPlugin.obj
 0002:00001328       ??_R3Gtest_PToolsAlignerTaskFactory@Gtest_PToolsAlignerTask@U2@@8 1001d328     PToolsPlugin.obj
 0002:00001338       ??_R2Gtest_PToolsAlignerTaskFactory@Gtest_PToolsAlignerTask@U2@@8 1001d338     PToolsPlugin.obj
 0002:00001344       ??_R1A@?0A@EA@Gtest_PToolsAlignerTaskFactory@Gtest_PToolsAlignerTask@U2@@8 1001d344     PToolsPlugin.obj
 0002:00001360       ??_R4?$GAutoDeleteList@VXMLTestFactory@U2@@@U2@@6B@ 1001d360     PToolsPlugin.obj
 0002:00001374       ??_R3?$GAutoDeleteList@VXMLTestFactory@U2@@@U2@@8 1001d374     PToolsPlugin.obj
 0002:00001384       ??_R2?$GAutoDeleteList@VXMLTestFactory@U2@@@U2@@8 1001d384     PToolsPlugin.obj
 0002:00001390       ??_R1A@?0A@EA@?$GAutoDeleteList@VXMLTestFactory@U2@@@U2@@8 1001d390     PToolsPlugin.obj
 0002:000013ac       ??_R4Rigidbody@PTools@@6B@ 1001d3ac     atomselection.obj
 0002:000013c0       ??_R3Rigidbody@PTools@@8   1001d3c0     atomselection.obj
 0002:000013d0       ??_R2Rigidbody@PTools@@8   1001d3d0     atomselection.obj
 0002:000013dc       ??_R1A@?0A@EA@Rigidbody@PTools@@8 1001d3dc     atomselection.obj
 0002:000013f8       ??_R17?0A@EN@CoordsArray@PTools@@8 1001d3f8     atomselection.obj
 0002:00001414       ??_R3CoordsArray@PTools@@8 1001d414     atomselection.obj
 0002:00001424       ??_R2CoordsArray@PTools@@8 1001d424     atomselection.obj
 0002:0000142c       ??_R1A@?0A@EA@CoordsArray@PTools@@8 1001d42c     atomselection.obj
 0002:00001448       ??_R4?$basic_stringbuf@DU?$char_traits@D@std@@V?$allocator@D@2@@std@@6B@ 1001d448     coord3d.obj
 0002:0000145c       ??_R3?$basic_stringbuf@DU?$char_traits@D@std@@V?$allocator@D@2@@std@@8 1001d45c     coord3d.obj
 0002:0000146c       ??_R2?$basic_stringbuf@DU?$char_traits@D@std@@V?$allocator@D@2@@std@@8 1001d46c     coord3d.obj
 0002:00001478       ??_R1A@?0A@EA@?$basic_stringbuf@DU?$char_traits@D@std@@V?$allocator@D@2@@std@@8 1001d478     coord3d.obj
 0002:00001494       ??_R1A@?0A@EA@?$basic_streambuf@DU?$char_traits@D@std@@@std@@8 1001d494     coord3d.obj
 0002:000014b0       ??_R3?$basic_streambuf@DU?$char_traits@D@std@@@std@@8 1001d4b0     coord3d.obj
 0002:000014c0       ??_R2?$basic_streambuf@DU?$char_traits@D@std@@@std@@8 1001d4c0     coord3d.obj
 0002:000014c8       ??_R4?$basic_stringstream@DU?$char_traits@D@std@@V?$allocator@D@2@@std@@6B@ 1001d4c8     coord3d.obj
 0002:000014dc       ??_R3?$basic_stringstream@DU?$char_traits@D@std@@V?$allocator@D@2@@std@@8 1001d4dc     coord3d.obj
 0002:000014ec       ??_R2?$basic_stringstream@DU?$char_traits@D@std@@V?$allocator@D@2@@std@@8 1001d4ec     coord3d.obj
 0002:00001518       ??_R1A@?0A@EA@?$basic_stringstream@DU?$char_traits@D@std@@V?$allocator@D@2@@std@@8 1001d518     coord3d.obj
 0002:00001534       ??_R1A@?0A@EA@?$basic_iostream@DU?$char_traits@D@std@@@std@@8 1001d534     coord3d.obj
 0002:00001550       ??_R3?$basic_iostream@DU?$char_traits@D@std@@@std@@8 1001d550     coord3d.obj
 0002:00001560       ??_R2?$basic_iostream@DU?$char_traits@D@std@@@std@@8 1001d560     coord3d.obj
 0002:00001588       ??_R1A@?0A@EA@?$basic_istream@DU?$char_traits@D@std@@@std@@8 1001d588     coord3d.obj
 0002:000015a4       ??_R3?$basic_istream@DU?$char_traits@D@std@@@std@@8 1001d5a4     coord3d.obj
 0002:000015b4       ??_R2?$basic_istream@DU?$char_traits@D@std@@@std@@8 1001d5b4     coord3d.obj
 0002:000015c8       ??_R1A@A@3FA@?$basic_ios@DU?$char_traits@D@std@@@std@@8 1001d5c8     coord3d.obj
 0002:000015e4       ??_R3?$basic_ios@DU?$char_traits@D@std@@@std@@8 1001d5e4     coord3d.obj
 0002:000015f4       ??_R2?$basic_ios@DU?$char_traits@D@std@@@std@@8 1001d5f4     coord3d.obj
 0002:00001604       ??_R1A@?0A@EA@?$basic_ios@DU?$char_traits@D@std@@@std@@8 1001d604     coord3d.obj
 0002:00001620       ??_R1A@?0A@EA@ios_base@std@@8 1001d620     coord3d.obj
 0002:0000163c       ??_R3ios_base@std@@8       1001d63c     coord3d.obj
 0002:0000164c       ??_R2ios_base@std@@8       1001d64c     coord3d.obj
 0002:00001658       ??_R17?0A@EA@?$_Iosb@H@std@@8 1001d658     coord3d.obj
 0002:00001674       ??_R3?$_Iosb@H@std@@8      1001d674     coord3d.obj
 0002:00001684       ??_R2?$_Iosb@H@std@@8      1001d684     coord3d.obj
 0002:0000168c       ??_R1A@?0A@EA@?$_Iosb@H@std@@8 1001d68c     coord3d.obj
 0002:000016a8       ??_R1A@A@3EA@ios_base@std@@8 1001d6a8     coord3d.obj
 0002:000016c4       ??_R17A@3EA@?$_Iosb@H@std@@8 1001d6c4     coord3d.obj
 0002:000016e0       ??_R1BA@?0A@EA@?$basic_ostream@DU?$char_traits@D@std@@@std@@8 1001d6e0     coord3d.obj
 0002:000016fc       ??_R3?$basic_ostream@DU?$char_traits@D@std@@@std@@8 1001d6fc     coord3d.obj
 0002:0000170c       ??_R2?$basic_ostream@DU?$char_traits@D@std@@@std@@8 1001d70c     coord3d.obj
 0002:00001720       ??_R1A@?0A@EA@?$basic_ostream@DU?$char_traits@D@std@@@std@@8 1001d720     coord3d.obj
 0002:0000173c       ??_R1A@?0A@EA@exception@std@@8 1001d73c     coordsarray.obj
 0002:00001758       ??_R3exception@std@@8      1001d758     coordsarray.obj
 0002:00001768       ??_R2exception@std@@8      1001d768     coordsarray.obj
 0002:00001770       ??_R4logic_error@std@@6B@  1001d770     coordsarray.obj
 0002:00001784       ??_R3logic_error@std@@8    1001d784     coordsarray.obj
 0002:00001794       ??_R2logic_error@std@@8    1001d794     coordsarray.obj
 0002:000017a0       ??_R1A@?0A@EA@logic_error@std@@8 1001d7a0     coordsarray.obj
 0002:000017bc       ??_R4out_of_range@std@@6B@ 1001d7bc     coordsarray.obj
 0002:000017d0       ??_R3out_of_range@std@@8   1001d7d0     coordsarray.obj
 0002:000017e0       ??_R2out_of_range@std@@8   1001d7e0     coordsarray.obj
 0002:000017f0       ??_R1A@?0A@EA@out_of_range@std@@8 1001d7f0     coordsarray.obj
 0002:0000180c       ??_R4?$basic_ostringstream@DU?$char_traits@D@std@@V?$allocator@D@2@@std@@6B@ 1001d80c     pdbio.obj
 0002:00001820       ??_R3?$basic_ostringstream@DU?$char_traits@D@std@@V?$allocator@D@2@@std@@8 1001d820     pdbio.obj
 0002:00001830       ??_R2?$basic_ostringstream@DU?$char_traits@D@std@@V?$allocator@D@2@@std@@8 1001d830     pdbio.obj
 0002:00001848       ??_R1A@?0A@EA@?$basic_ostringstream@DU?$char_traits@D@std@@V?$allocator@D@2@@std@@8 1001d848     pdbio.obj
 0002:00001864       ??_R4?$basic_filebuf@DU?$char_traits@D@std@@@std@@6B@ 1001d864     pdbio.obj
 0002:00001878       ??_R3?$basic_filebuf@DU?$char_traits@D@std@@@std@@8 1001d878     pdbio.obj
 0002:00001888       ??_R2?$basic_filebuf@DU?$char_traits@D@std@@@std@@8 1001d888     pdbio.obj
 0002:00001894       ??_R1A@?0A@EA@?$basic_filebuf@DU?$char_traits@D@std@@@std@@8 1001d894     pdbio.obj
 0002:000018b0       ??_R4?$basic_ifstream@DU?$char_traits@D@std@@@std@@6B@ 1001d8b0     pdbio.obj
 0002:000018c4       ??_R3?$basic_ifstream@DU?$char_traits@D@std@@@std@@8 1001d8c4     pdbio.obj
 0002:000018d4       ??_R2?$basic_ifstream@DU?$char_traits@D@std@@@std@@8 1001d8d4     pdbio.obj
 0002:000018ec       ??_R1A@?0A@EA@?$basic_ifstream@DU?$char_traits@D@std@@@std@@8 1001d8ec     pdbio.obj
 0002:00001908       ??_R4invalid_argument@std@@6B@ 1001d908     pdbio.obj
 0002:0000191c       ??_R3invalid_argument@std@@8 1001d91c     pdbio.obj
 0002:0000192c       ??_R2invalid_argument@std@@8 1001d92c     pdbio.obj
 0002:0000193c       ??_R1A@?0A@EA@invalid_argument@std@@8 1001d93c     pdbio.obj
 0002:00001958       ??_R4runtime_error@std@@6B@ 1001d958     superpose.obj
 0002:0000196c       ??_R3runtime_error@std@@8  1001d96c     superpose.obj
 0002:0000197c       ??_R2runtime_error@std@@8  1001d97c     superpose.obj
 0002:00001988       ??_R1A@?0A@EA@runtime_error@std@@8 1001d988     superpose.obj
 0002:000019a4       ??_R4type_info@@6B@        1001d9a4     MSVCRT:ti_inst.obj
 0002:000019b8       ??_R3type_info@@8          1001d9b8     MSVCRT:ti_inst.obj
 0002:000019c8       ??_R2type_info@@8          1001d9c8     MSVCRT:ti_inst.obj
 0002:000019d0       ??_R1A@?0A@EA@type_info@@8 1001d9d0     MSVCRT:ti_inst.obj
 0002:000019f0       ___safe_se_handler_table   1001d9f0     <linker-defined>
 0002:00001c78       ___rtc_iaa                 1001dc78     MSVCRT:initsect.obj
 0002:00001c7c       ___rtc_izz                 1001dc7c     MSVCRT:initsect.obj
 0002:00001c80       ___rtc_taa                 1001dc80     MSVCRT:initsect.obj
 0002:00001c84       ___rtc_tzz                 1001dc84     MSVCRT:initsect.obj
 0002:000032d4       __CT??_R0?AVexception@std@@@8??0exception@std@@QAE@ABV01@@Z12 1001f2d4     coordsarray.obj
 0002:000032f0       __TI3?AVout_of_range@std@@ 1001f2f0     coordsarray.obj
 0002:00003300       __CTA3?AVout_of_range@std@@ 1001f300     coordsarray.obj
 0002:00003310       __CT??_R0?AVout_of_range@std@@@8??0out_of_range@std@@QAE@ABV01@@Z12 1001f310     coordsarray.obj
 0002:0000332c       __CT??_R0?AVlogic_error@std@@@8??0logic_error@std@@QAE@ABV01@@Z12 1001f32c     coordsarray.obj
 0002:000037f4       __TI3?AVinvalid_argument@std@@ 1001f7f4     pdbio.obj
 0002:00003804       __CTA3?AVinvalid_argument@std@@ 1001f804     pdbio.obj
 0002:00003814       __CT??_R0?AVinvalid_argument@std@@@8??0invalid_argument@std@@QAE@ABV01@@Z12 1001f814     pdbio.obj
 0002:00003830       __TI2?AVbad_cast@std@@     1001f830     pdbio.obj
 0002:00003840       __CTA2?AVbad_cast@std@@    1001f840     pdbio.obj
 0002:0000384c       __CT??_R0?AVbad_cast@std@@@8??0bad_cast@std@@QAE@ABV01@@Z12 1001f84c     pdbio.obj
 0002:00004140       __TI2?AVruntime_error@std@@ 10020140     superpose.obj
 0002:00004150       __CTA2?AVruntime_error@std@@ 10020150     superpose.obj
 0002:0000415c       __CT??_R0?AVruntime_error@std@@@8??0runtime_error@std@@QAE@ABV01@@Z12 1002015c     superpose.obj
 0002:00004590       __IMPORT_DESCRIPTOR_U2Core 10020590     U2Core:U2Core.dll
 0002:000045a4       __IMPORT_DESCRIPTOR_U2Algorithm 100205a4     U2Algorithm:U2Algorithm.dll
 0002:000045b8       __IMPORT_DESCRIPTOR_U2Test 100205b8     U2Test:U2Test.dll
 0002:000045cc       __IMPORT_DESCRIPTOR_Qt5Xml 100205cc     Qt5Xml:Qt5Xml.dll
 0002:000045e0       __IMPORT_DESCRIPTOR_Qt5Core 100205e0     Qt5Core:Qt5Core.dll
 0002:000045f4       __IMPORT_DESCRIPTOR_MSVCP120 100205f4     msvcprt:MSVCP120.dll
 0002:00004608       __IMPORT_DESCRIPTOR_MSVCR120 10020608     MSVCRT:MSVCR120.dll
 0002:0000461c       __IMPORT_DESCRIPTOR_KERNEL32 1002061c     kernel32:KERNEL32.dll
 0002:00004630       __NULL_IMPORT_DESCRIPTOR   10020630     U2Core:U2Core.dll
 0003:00000000       ?_Generic_object@?$_Error_objects@H@std@@2V_Generic_error_category@2@A 10023000     PToolsAligner.obj
 0003:00000004       ?_Iostream_object@?$_Error_objects@H@std@@2V_Iostream_error_category@2@A 10023004     PToolsAligner.obj
 0003:00000008       ?_System_object@?$_Error_objects@H@std@@2V_System_error_category@2@A 10023008     PToolsAligner.obj
 0003:0000000c       ?staticMetaObject@PToolsPlugin@U2@@2UQMetaObject@@B 1002300c     moc_PToolsPlugin.obj
 0003:00000024       ?staticMetaObject@Gtest_PToolsAlignerTask@U2@@2UQMetaObject@@B 10023024     moc_PToolsTests.obj
 0003:0000003c       ___security_cookie         1002303c     MSVCRT:gs_cookie.obj
 0003:00000040       ___security_cookie_complement 10023040     MSVCRT:gs_cookie.obj
 0003:00000050       ___native_dllmain_reason   10023050     MSVCRT:natstart.obj
 0003:00000058       ??_R0?AVexception@std@@@8  10023058     PToolsAligner.obj
 0003:00000074       ??_R0?AVerror_category@std@@@8 10023074     PToolsAligner.obj
 0003:00000098       ??_R0?AV_Generic_error_category@std@@@8 10023098     PToolsAligner.obj
 0003:000000c4       ??_R0?AV_Iostream_error_category@std@@@8 100230c4     PToolsAligner.obj
 0003:000000f0       ??_R0?AV_System_error_category@std@@@8 100230f0     PToolsAligner.obj
 0003:0000011c       ??_R0?AVXmlTest@U2@@@8     1002311c     PToolsPlugin.obj
 0003:00000138       ??_R0?AVGTest@U2@@@8       10023138     PToolsPlugin.obj
 0003:00000150       ??_R0?AVTask@U2@@@8        10023150     PToolsPlugin.obj
 0003:00000168       ??_R0?AVQObject@@@8        10023168     PToolsPlugin.obj
 0003:00000180       ??_R0?AVXMLTestFactory@U2@@@8 10023180     PToolsPlugin.obj
 0003:000001a0       ??_R0?AVPToolsPlugin@U2@@@8 100231a0     PToolsPlugin.obj
 0003:000001c0       ??_R0?AVPlugin@U2@@@8      100231c0     PToolsPlugin.obj
 0003:000001d8       ??_R0?AVPToolsAligner@U2@@@8 100231d8     PToolsPlugin.obj
 0003:000001f8       ??_R0?AVStructuralAlignmentAlgorithm@U2@@@8 100231f8     PToolsPlugin.obj
 0003:00000228       ??_R0?AVPToolsAlignerFactory@U2@@@8 10023228     PToolsPlugin.obj
 0003:00000250       ??_R0?AVStructuralAlignmentAlgorithmFactory@U2@@@8 10023250     PToolsPlugin.obj
 0003:00000288       ??_R0?AVGtest_PToolsAlignerTask@U2@@@8 10023288     PToolsPlugin.obj
 0003:000002b8       ??_R0?AVGtest_PToolsAlignerTaskFactory@Gtest_PToolsAlignerTask@U2@@@8 100232b8     PToolsPlugin.obj
 0003:00000300       ??_R0?AV?$GAutoDeleteList@VXMLTestFactory@U2@@@U2@@@8 10023300     PToolsPlugin.obj
 0003:00000338       ??_R0?AVRigidbody@PTools@@@8 10023338     atomselection.obj
 0003:00000358       ??_R0?AVCoordsArray@PTools@@@8 10023358     atomselection.obj
 0003:00000380       ??_R0?AV?$basic_stringbuf@DU?$char_traits@D@std@@V?$allocator@D@2@@std@@@8 10023380     coord3d.obj
 0003:000003d0       ??_R0?AV?$basic_streambuf@DU?$char_traits@D@std@@@std@@@8 100233d0     coord3d.obj
 0003:00000410       ??_R0?AV?$basic_stringstream@DU?$char_traits@D@std@@V?$allocator@D@2@@std@@@8 10023410     coord3d.obj
 0003:00000460       ??_R0?AV?$basic_iostream@DU?$char_traits@D@std@@@std@@@8 10023460     coord3d.obj
 0003:0000049c       ??_R0?AV?$basic_istream@DU?$char_traits@D@std@@@std@@@8 1002349c     coord3d.obj
 0003:000004d8       ??_R0?AV?$basic_ios@DU?$char_traits@D@std@@@std@@@8 100234d8     coord3d.obj
 0003:00000510       ??_R0?AVios_base@std@@@8   10023510     coord3d.obj
 0003:0000052c       ??_R0?AV?$_Iosb@H@std@@@8  1002352c     coord3d.obj
 0003:00000548       ??_R0?AV?$basic_ostream@DU?$char_traits@D@std@@@std@@@8 10023548     coord3d.obj
 0003:00000584       ??_R0?AVout_of_range@std@@@8 10023584     coordsarray.obj
 0003:000005a4       ??_R0?AVlogic_error@std@@@8 100235a4     coordsarray.obj
 0003:000005c4       ??_R0?AVinvalid_argument@std@@@8 100235c4     pdbio.obj
 0003:000005e8       ??_R0?AVbad_cast@std@@@8   100235e8     pdbio.obj
 0003:00000608       ??_R0?AV?$basic_ostringstream@DU?$char_traits@D@std@@V?$allocator@D@2@@std@@@8 10023608     pdbio.obj
 0003:0000065c       ??_R0?AV?$basic_filebuf@DU?$char_traits@D@std@@@std@@@8 1002365c     pdbio.obj
 0003:00000698       ??_R0?AV?$basic_ifstream@DU?$char_traits@D@std@@@std@@@8 10023698     pdbio.obj
 0003:000006d4       ??_R0?AVruntime_error@std@@@8 100236d4     superpose.obj
 0003:000006f4       ??_R0?AVtype_info@@@8      100236f4     MSVCRT:ti_inst.obj
 0003:0000075c       ?id@?$num_put@DV?$back_insert_iterator@V?$basic_string@DU?$char_traits@D@std@@V?$allocator@D@2@@std@@@std@@@std@@2V0locale@2@A 1002375c     PToolsAligner.obj
 0003:00000760       ?id@?$num_put@_WV?$back_insert_iterator@V?$basic_string@_WU?$char_traits@_W@std@@V?$allocator@_W@2@@std@@@std@@@std@@2V0locale@2@A 10023760     PToolsAligner.obj
 0003:000007e8       ?RMSD_ATTR@Gtest_PToolsAlignerTask@U2@@2VQString@@B 100237e8     PToolsTests.obj
 0003:000007ec       ?MOBO_ATTR@Gtest_PToolsAlignerTask@U2@@2VQString@@B 100237ec     PToolsTests.obj
 0003:00000808       ?TRANSFORM_ATTR@Gtest_PToolsAlignerTask@U2@@2VQString@@B 10023808     PToolsTests.obj
 0003:0000080c       ?REFO_ATTR@Gtest_PToolsAlignerTask@U2@@2VQString@@B 1002380c     PToolsTests.obj
 0003:00000810       ?ACCURACY_ATTR@Gtest_PToolsAlignerTask@U2@@2VQString@@B 10023810     PToolsTests.obj
 0003:00000824       ?_Stinit@?1??_Init@?$basic_filebuf@DU?$char_traits@D@std@@@std@@IAEXPAU_iobuf@@W4_Initfl@23@@Z@4HA 10023824     pdbio.obj
 0003:00000828       ?_Psave@?$_Facetptr@V?$codecvt@DDH@std@@@std@@2PBVfacet@locale@2@B 10023828     pdbio.obj
 0003:00000bf8       ?__type_info_root_node@@3U__type_info_node@@A 10023bf8     MSVCRT:tncleanup.obj
 0003:00000c00       ___native_startup_lock     10023c00     <common>
 0003:00000c04       ___native_startup_state    10023c04     <common>
 0003:00000c08       ___dyn_tls_init_callback   10023c08     <common>
 0003:00000c0c       ___onexitend               10023c0c     <common>
 0003:00000c10       ___onexitbegin             10023c10     <common>

 entry point at        0001:00017b50

 Static symbols

 0002:fffe4000       __catchsym$?_Copy@?$basic_string@DU?$char_traits@D@std@@V?$allocator@D@2@@std@@QAEXII@Z$5 10000000     atom.obj
 0000:fffd9000       .debug$S                   10000000     MSVCRT:MSVCR120.dll
 0000:fffd9000       .debug$S                   10000000     MSVCRT:MSVCR120.dll
 0000:fffd9000       .debug$S                   10000000     MSVCRT:MSVCR120.dll
 0000:fffd9000       .debug$S                   10000000     MSVCRT:MSVCR120.dll
 0000:fffd9000       .debug$S                   10000000     MSVCRT:MSVCR120.dll
 0000:fffd9000       .debug$S                   10000000     MSVCRT:MSVCR120.dll
 0000:fffd9000       .debug$S                   10000000     MSVCRT:MSVCR120.dll
 0000:fffd9000       .debug$S                   10000000     MSVCRT:MSVCR120.dll
 0000:fffd9000       .debug$S                   10000000     MSVCRT:MSVCR120.dll
 0000:fffd9000       .debug$S                   10000000     MSVCRT:MSVCR120.dll
 0000:fffd9000       .debug$S                   10000000     MSVCRT:MSVCR120.dll
 0000:fffd9000       .debug$S                   10000000     MSVCRT:MSVCR120.dll
 0000:fffd9000       .debug$S                   10000000     MSVCRT:MSVCR120.dll
 0000:fffd9000       .debug$S                   10000000     MSVCRT:MSVCR120.dll
 0000:fffd9000       .debug$S                   10000000     MSVCRT:MSVCR120.dll
 0000:fffd9000       .debug$S                   10000000     MSVCRT:MSVCR120.dll
 0000:fffd9000       .debug$S                   10000000     MSVCRT:MSVCR120.dll
 0000:fffd9000       .debug$S                   10000000     MSVCRT:MSVCR120.dll
 0000:fffd9000       .debug$S                   10000000     MSVCRT:MSVCR120.dll
 0000:fffd9000       .debug$S                   10000000     MSVCRT:MSVCR120.dll
 0000:fffd9000       .debug$S                   10000000     MSVCRT:MSVCR120.dll
 0000:fffd9000       .debug$S                   10000000     MSVCRT:MSVCR120.dll
 0000:fffd9000       .debug$S                   10000000     MSVCRT:MSVCR120.dll
 0000:fffd9000       .debug$S                   10000000     MSVCRT:MSVCR120.dll
 0000:fffd9000       .debug$S                   10000000     MSVCRT:MSVCR120.dll
 0000:fffd9000       .debug$S                   10000000     MSVCRT:MSVCR120.dll
 0000:fffd9000       .debug$S                   10000000     MSVCRT:MSVCR120.dll
 0000:fffd9000       .debug$S                   10000000     MSVCRT:MSVCR120.dll
 0000:fffd9000       .debug$S                   10000000     MSVCRT:MSVCR120.dll
 0000:fffd9000       .debug$S                   10000000     MSVCRT:MSVCR120.dll
 0000:fffd9000       .debug$S                   10000000     MSVCRT:MSVCR120.dll
 0000:fffd9000       .debug$S                   10000000     MSVCRT:MSVCR120.dll
 0000:fffd9000       .debug$S                   10000000     MSVCRT:MSVCR120.dll
 0001:fffff000       __ehhandler$?_Copy@?$basic_string@DU?$char_traits@D@std@@V?$allocator@D@2@@std@@QAEXII@Z 10000000 f   moc_PToolsTests.obj
 0000:fffd9000       .debug$S                   10000000     MSVCRT:MSVCR120.dll
 0000:fffd9000       .debug$S                   10000000     MSVCRT:MSVCR120.dll
 0000:fffd9000       .debug$S                   10000000     MSVCRT:MSVCR120.dll
 0000:fffd9000       .debug$S                   10000000     MSVCRT:MSVCR120.dll
 0000:fffd9000       .debug$S                   10000000     MSVCRT:MSVCR120.dll
 0000:fffd9000       .debug$S                   10000000     MSVCRT:MSVCR120.dll
 0000:fffd9000       .debug$S                   10000000     MSVCRT:MSVCR120.dll
 0000:fffd9000       .debug$S                   10000000     MSVCRT:MSVCR120.dll
 0000:fffd9000       .debug$S                   10000000     MSVCRT:MSVCR120.dll
 0000:fffd9000       .debug$S                   10000000     MSVCRT:MSVCR120.dll
 0000:fffd9000       .debug$S                   10000000     MSVCRT:MSVCR120.dll
 0000:fffd9000       .debug$S                   10000000     MSVCRT:MSVCR120.dll
 0000:fffd9000       .debug$S                   10000000     MSVCRT:MSVCR120.dll
 0000:fffd9000       .debug$S                   10000000     MSVCRT:MSVCR120.dll
 0000:fffd9000       .debug$S                   10000000     MSVCRT:MSVCR120.dll
 0000:fffd9000       .debug$S                   10000000     MSVCRT:MSVCR120.dll
 0000:fffd9000       .debug$S                   10000000     MSVCRT:MSVCR120.dll
 0000:fffd9000       .debug$S                   10000000     MSVCRT:MSVCR120.dll
 0000:fffd9000       .debug$S                   10000000     MSVCRT:MSVCR120.dll
 0000:fffd9000       .debug$S                   10000000     MSVCRT:MSVCR120.dll
 0000:fffd9000       .debug$S                   10000000     MSVCRT:MSVCR120.dll
 0000:fffd9000       .debug$S                   10000000     MSVCRT:MSVCR120.dll
 0000:fffd9000       .debug$S                   10000000     MSVCRT:MSVCR120.dll
 0000:fffd9000       .debug$S                   10000000     MSVCRT:MSVCR120.dll
 0002:fffe4000       __catchsym$?_Copy@?$basic_string@DU?$char_traits@D@std@@V?$allocator@D@2@@std@@QAEXII@Z$5 10000000     moc_PToolsTests.obj
 0000:fffd9000       .debug$S                   10000000     MSVCRT:MSVCR120.dll
 0000:fffd9000       .debug$S                   10000000     msvcprt:MSVCP120.dll
 0000:fffd9000       .debug$S                   10000000     msvcprt:MSVCP120.dll
 0000:fffd9000       .debug$S                   10000000     msvcprt:MSVCP120.dll
 0000:fffd9000       .debug$S                   10000000     msvcprt:MSVCP120.dll
 0000:fffd9000       .debug$S                   10000000     msvcprt:MSVCP120.dll
 0000:fffd9000       .debug$S                   10000000     msvcprt:MSVCP120.dll
 0000:fffd9000       .debug$S                   10000000     msvcprt:MSVCP120.dll
 0000:fffd9000       .debug$S                   10000000     msvcprt:MSVCP120.dll
 0000:fffd9000       .debug$S                   10000000     msvcprt:MSVCP120.dll
 0000:fffd9000       .debug$S                   10000000     msvcprt:MSVCP120.dll
 0000:fffd9000       .debug$S                   10000000     msvcprt:MSVCP120.dll
 0000:fffd9000       .debug$S                   10000000     msvcprt:MSVCP120.dll
 0000:fffd9000       .debug$S                   10000000     msvcprt:MSVCP120.dll
 0000:fffd9000       .debug$S                   10000000     msvcprt:MSVCP120.dll
 0000:fffd9000       .debug$S                   10000000     msvcprt:MSVCP120.dll
 0000:fffd9000       .debug$S                   10000000     msvcprt:MSVCP120.dll
 0000:fffd9000       .debug$S                   10000000     msvcprt:MSVCP120.dll
 0000:fffd9000       .debug$S                   10000000     msvcprt:MSVCP120.dll
 0000:fffd9000       .debug$S                   10000000     msvcprt:MSVCP120.dll
 0000:fffd9000       .debug$S                   10000000     msvcprt:MSVCP120.dll
 0000:fffd9000       .debug$S                   10000000     msvcprt:MSVCP120.dll
 0000:fffd9000       .debug$S                   10000000     msvcprt:MSVCP120.dll
 0000:fffd9000       .debug$S                   10000000     msvcprt:MSVCP120.dll
 0000:fffd9000       .debug$S                   10000000     msvcprt:MSVCP120.dll
 0000:fffd9000       .debug$S                   10000000     msvcprt:MSVCP120.dll
 0000:fffd9000       .debug$S                   10000000     msvcprt:MSVCP120.dll
 0000:fffd9000       .debug$S                   10000000     msvcprt:MSVCP120.dll
 0000:fffd9000       .debug$S                   10000000     msvcprt:MSVCP120.dll
 0000:fffd9000       .debug$S                   10000000     msvcprt:MSVCP120.dll
 0000:fffd9000       .debug$S                   10000000     msvcprt:MSVCP120.dll
 0000:fffd9000       .debug$S                   10000000     msvcprt:MSVCP120.dll
 0000:fffd9000       .debug$S                   10000000     msvcprt:MSVCP120.dll
 0000:fffd9000       .debug$S                   10000000     msvcprt:MSVCP120.dll
 0000:fffd9000       .debug$S                   10000000     msvcprt:MSVCP120.dll
 0000:fffd9000       .debug$S                   10000000     msvcprt:MSVCP120.dll
 0000:fffd9000       .debug$S                   10000000     msvcprt:MSVCP120.dll
 0000:fffd9000       .debug$S                   10000000     msvcprt:MSVCP120.dll
 0000:fffd9000       .debug$S                   10000000     msvcprt:MSVCP120.dll
 0000:fffd9000       .debug$S                   10000000     msvcprt:MSVCP120.dll
 0000:fffd9000       .debug$S                   10000000     msvcprt:MSVCP120.dll
 0002:fffe4000       ?_Generic_object$initializer$@?$_Error_objects@H@std@@2P6AXXZA 10000000     moc_PToolsTests.obj
 0002:fffe4000       ?_Iostream_object$initializer$@?$_Error_objects@H@std@@2P6AXXZA 10000000     moc_PToolsTests.obj
 0002:fffe4000       ?_System_object$initializer$@?$_Error_objects@H@std@@2P6AXXZA 10000000     moc_PToolsTests.obj
 0000:fffd9000       .debug$S                   10000000     msvcprt:MSVCP120.dll
 0000:fffd9000       .debug$S                   10000000     msvcprt:MSVCP120.dll
 0000:fffd9000       .debug$S                   10000000     msvcprt:MSVCP120.dll
 0000:fffd9000       .debug$S                   10000000     msvcprt:MSVCP120.dll
 0000:fffd9000       .debug$S                   10000000     msvcprt:MSVCP120.dll
 0000:fffd9000       .debug$S                   10000000     msvcprt:MSVCP120.dll
 0000:fffd9000       .debug$S                   10000000     msvcprt:MSVCP120.dll
 0000:fffd9000       .debug$S                   10000000     msvcprt:MSVCP120.dll
 0000:fffd9000       .debug$S                   10000000     msvcprt:MSVCP120.dll
 0000:fffd9000       .debug$S                   10000000     msvcprt:MSVCP120.dll
 0000:fffd9000       .debug$S                   10000000     msvcprt:MSVCP120.dll
 0000:fffd9000       .debug$S                   10000000     msvcprt:MSVCP120.dll
 0000:fffd9000       .debug$S                   10000000     msvcprt:MSVCP120.dll
 0000:fffd9000       .debug$S                   10000000     msvcprt:MSVCP120.dll
 0000:fffd9000       .debug$S                   10000000     kernel32:KERNEL32.dll
 0000:fffd9000       .debug$S                   10000000     kernel32:KERNEL32.dll
 0000:fffd9000       .debug$S                   10000000     kernel32:KERNEL32.dll
 0000:fffd9000       .debug$S                   10000000     kernel32:KERNEL32.dll
 0000:fffd9000       .debug$S                   10000000     kernel32:KERNEL32.dll
 0000:fffd9000       .debug$S                   10000000     kernel32:KERNEL32.dll
 0000:fffd9000       .debug$S                   10000000     kernel32:KERNEL32.dll
 0000:fffd9000       .debug$S                   10000000     kernel32:KERNEL32.dll
 0000:fffd9000       .debug$S                   10000000     kernel32:KERNEL32.dll
 0000:fffd9000       .debug$S                   10000000     Qt5Core:Qt5Core.dll
 0000:fffd9000       .debug$S                   10000000     Qt5Core:Qt5Core.dll
 0000:fffd9000       .debug$S                   10000000     Qt5Core:Qt5Core.dll
 0000:fffd9000       .debug$S                   10000000     Qt5Core:Qt5Core.dll
 0001:fffff000       __ehhandler$?_Copy@?$basic_string@DU?$char_traits@D@std@@V?$allocator@D@2@@std@@QAEXII@Z 10000000 f   moc_PToolsPlugin.obj
 0000:fffd9000       .debug$S                   10000000     Qt5Core:Qt5Core.dll
 0000:fffd9000       .debug$S                   10000000     Qt5Core:Qt5Core.dll
 0000:fffd9000       .debug$S                   10000000     Qt5Core:Qt5Core.dll
 0000:fffd9000       .debug$S                   10000000     Qt5Core:Qt5Core.dll
 0000:fffd9000       .debug$S                   10000000     Qt5Core:Qt5Core.dll
 0000:fffd9000       .debug$S                   10000000     Qt5Core:Qt5Core.dll
 0000:fffd9000       .debug$S                   10000000     Qt5Core:Qt5Core.dll
 0000:fffd9000       .debug$S                   10000000     Qt5Core:Qt5Core.dll
 0000:fffd9000       .debug$S                   10000000     Qt5Core:Qt5Core.dll
 0000:fffd9000       .debug$S                   10000000     Qt5Core:Qt5Core.dll
 0000:fffd9000       .debug$S                   10000000     Qt5Core:Qt5Core.dll
 0000:fffd9000       .debug$S                   10000000     Qt5Core:Qt5Core.dll
 0000:fffd9000       .debug$S                   10000000     Qt5Core:Qt5Core.dll
 0000:fffd9000       .debug$S                   10000000     Qt5Core:Qt5Core.dll
 0000:fffd9000       .debug$S                   10000000     Qt5Core:Qt5Core.dll
 0000:fffd9000       .debug$S                   10000000     Qt5Core:Qt5Core.dll
 0000:fffd9000       .debug$S                   10000000     Qt5Core:Qt5Core.dll
 0000:fffd9000       .debug$S                   10000000     Qt5Core:Qt5Core.dll
 0000:fffd9000       .debug$S                   10000000     Qt5Core:Qt5Core.dll
 0000:fffd9000       .debug$S                   10000000     Qt5Core:Qt5Core.dll
 0000:fffd9000       .debug$S                   10000000     Qt5Core:Qt5Core.dll
 0000:fffd9000       .debug$S                   10000000     Qt5Core:Qt5Core.dll
 0000:fffd9000       .debug$S                   10000000     Qt5Core:Qt5Core.dll
 0000:fffd9000       .debug$S                   10000000     Qt5Core:Qt5Core.dll
 0002:fffe4000       __catchsym$?_Copy@?$basic_string@DU?$char_traits@D@std@@V?$allocator@D@2@@std@@QAEXII@Z$5 10000000     moc_PToolsPlugin.obj
 0000:fffd9000       .debug$S                   10000000     Qt5Core:Qt5Core.dll
 0000:fffd9000       .debug$S                   10000000     Qt5Core:Qt5Core.dll
 0000:fffd9000       .debug$S                   10000000     Qt5Core:Qt5Core.dll
 0000:fffd9000       .debug$S                   10000000     Qt5Core:Qt5Core.dll
 0000:fffd9000       .debug$S                   10000000     Qt5Core:Qt5Core.dll
 0000:fffd9000       .debug$S                   10000000     Qt5Core:Qt5Core.dll
 0000:fffd9000       .debug$S                   10000000     Qt5Core:Qt5Core.dll
 0000:fffd9000       .debug$S                   10000000     Qt5Core:Qt5Core.dll
 0000:fffd9000       .debug$S                   10000000     Qt5Core:Qt5Core.dll
 0000:fffd9000       .debug$S                   10000000     Qt5Core:Qt5Core.dll
 0000:fffd9000       .debug$S                   10000000     Qt5Core:Qt5Core.dll
 0000:fffd9000       .debug$S                   10000000     Qt5Core:Qt5Core.dll
 0000:fffd9000       .debug$S                   10000000     Qt5Core:Qt5Core.dll
 0000:fffd9000       .debug$S                   10000000     Qt5Core:Qt5Core.dll
 0000:fffd9000       .debug$S                   10000000     Qt5Core:Qt5Core.dll
 0000:fffd9000       .debug$S                   10000000     Qt5Core:Qt5Core.dll
 0000:fffd9000       .debug$S                   10000000     Qt5Core:Qt5Core.dll
 0000:fffd9000       .debug$S                   10000000     Qt5Core:Qt5Core.dll
 0000:fffd9000       .debug$S                   10000000     Qt5Core:Qt5Core.dll
 0000:fffd9000       .debug$S                   10000000     Qt5Core:Qt5Core.dll
 0000:fffd9000       .debug$S                   10000000     Qt5Core:Qt5Core.dll
 0000:fffd9000       .debug$S                   10000000     Qt5Xml:Qt5Xml.dll
 0000:fffd9000       .debug$S                   10000000     U2Test:U2Test.dll
 0000:fffd9000       .debug$S                   10000000     U2Test:U2Test.dll
 0000:fffd9000       .debug$S                   10000000     U2Test:U2Test.dll
 0000:fffd9000       .debug$S                   10000000     U2Test:U2Test.dll
 0000:fffd9000       .debug$S                   10000000     U2Test:U2Test.dll
 0000:fffd9000       .debug$S                   10000000     U2Test:U2Test.dll
 0000:fffd9000       .debug$S                   10000000     U2Test:U2Test.dll
 0000:fffd9000       .debug$S                   10000000     U2Test:U2Test.dll
 0000:fffd9000       .debug$S                   10000000     U2Test:U2Test.dll
 0000:fffd9000       .debug$S                   10000000     U2Test:U2Test.dll
 0000:fffd9000       .debug$S                   10000000     U2Test:U2Test.dll
 0000:fffd9000       .debug$S                   10000000     U2Algorithm:U2Algorithm.dll
 0000:fffd9000       .debug$S                   10000000     U2Algorithm:U2Algorithm.dll
 0000:fffd9000       .debug$S                   10000000     U2Algorithm:U2Algorithm.dll
 0000:fffd9000       .debug$S                   10000000     U2Algorithm:U2Algorithm.dll
 0000:fffd9000       .debug$S                   10000000     U2Algorithm:U2Algorithm.dll
 0000:fffd9000       .debug$S                   10000000     U2Algorithm:U2Algorithm.dll
 0000:fffd9000       .debug$S                   10000000     U2Algorithm:U2Algorithm.dll
 0000:fffd9000       .debug$S                   10000000     U2Algorithm:U2Algorithm.dll
 0002:fffe4000       ?_Generic_object$initializer$@?$_Error_objects@H@std@@2P6AXXZA 10000000     moc_PToolsPlugin.obj
 0002:fffe4000       ?_Iostream_object$initializer$@?$_Error_objects@H@std@@2P6AXXZA 10000000     moc_PToolsPlugin.obj
 0002:fffe4000       ?_System_object$initializer$@?$_Error_objects@H@std@@2P6AXXZA 10000000     moc_PToolsPlugin.obj
 0000:fffd9000       .debug$S                   10000000     U2Algorithm:U2Algorithm.dll
 0000:fffd9000       .debug$S                   10000000     U2Algorithm:U2Algorithm.dll
 0000:fffd9000       .debug$S                   10000000     U2Core:U2Core.dll
 0000:fffd9000       .debug$S                   10000000     U2Core:U2Core.dll
 0000:fffd9000       .debug$S                   10000000     U2Core:U2Core.dll
 0000:fffd9000       .debug$S                   10000000     U2Core:U2Core.dll
 0000:fffd9000       .debug$S                   10000000     U2Core:U2Core.dll
 0000:fffd9000       .debug$S                   10000000     U2Core:U2Core.dll
 0000:fffd9000       .debug$S                   10000000     U2Core:U2Core.dll
 0000:fffd9000       .debug$S                   10000000     U2Core:U2Core.dll
 0000:fffd9000       .debug$S                   10000000     U2Core:U2Core.dll
 0000:fffd9000       .debug$S                   10000000     U2Core:U2Core.dll
 0000:fffd9000       .debug$S                   10000000     U2Core:U2Core.dll
 0001:fffff000       __ehhandler$?_Copy@?$basic_string@DU?$char_traits@D@std@@V?$allocator@D@2@@std@@QAEXII@Z 10000000 f   superpose.obj
 0000:fffd9000       .debug$S                   10000000     U2Core:U2Core.dll
 0000:fffd9000       .debug$S                   10000000     U2Core:U2Core.dll
 0000:fffd9000       .debug$S                   10000000     U2Core:U2Core.dll
 0001:fffff000       __unwindfunclet$??0?$Array2D@N@@QAE@HH@Z$0 10000000 f   superpose.obj
 0001:fffff000       __ehhandler$?reallocData@?$QVector@N@@AAEXHHV?$QFlags@W4AllocationOption@QArrayData@@@@@Z 10000000 f   superpose.obj
 0000:fffd9000       .debug$S                   10000000     U2Core:U2Core.dll
 0000:fffd9000       .debug$S                   10000000     U2Core:U2Core.dll
 0000:fffd9000       .debug$S                   10000000     U2Core:U2Core.dll
 0000:fffd9000       .debug$S                   10000000     U2Core:U2Core.dll
 0000:fffd9000       .debug$S                   10000000     U2Core:U2Core.dll
 0000:fffd9000       .debug$S                   10000000     U2Core:U2Core.dll
 0000:fffd9000       .debug$S                   10000000     U2Core:U2Core.dll
 0000:fffd9000       .debug$S                   10000000     U2Core:U2Core.dll
 0000:fffd9000       .debug$S                   10000000     U2Core:U2Core.dll
 0000:fffd9000       .debug$S                   10000000     U2Core:U2Core.dll
 0000:fffd9000       .debug$S                   10000000     U2Core:U2Core.dll
 0000:fffd9000       .debug$S                   10000000     U2Core:U2Core.dll
 0000:fffd9000       .debug$S                   10000000     U2Core:U2Core.dll
 0000:fffd9000       .debug$S                   10000000     U2Core:U2Core.dll
 0000:fffd9000       .debug$S                   10000000     U2Core:U2Core.dll
 0000:fffd9000       .debug$S                   10000000     U2Core:U2Core.dll
 0000:fffd9000       .debug$S                   10000000     U2Core:U2Core.dll
 0000:fffd9000       .debug$S                   10000000     U2Core:U2Core.dll
 0000:fffd9000       .debug$S                   10000000     U2Core:U2Core.dll
 0000:fffd9000       .debug$S                   10000000     U2Core:U2Core.dll
 0000:fffd9000       .debug$S                   10000000     U2Core:U2Core.dll
 0000:fffd9000       .debug$S                   10000000     U2Core:U2Core.dll
 0000:fffd9000       .debug$S                   10000000     U2Core:U2Core.dll
 0000:fffd9000       .debug$S                   10000000     U2Core:U2Core.dll
 0000:fffd9000       .debug$S                   10000000     U2Core:U2Core.dll
 0000:fffd9000       .debug$S                   10000000     U2Core:U2Core.dll
 0002:fffe4000       ?_System_object$initializer$@?$_Error_objects@H@std@@2P6AXXZA 10000000     PToolsPlugin.obj
 0002:fffe4000       ?_Iostream_object$initializer$@?$_Error_objects@H@std@@2P6AXXZA 10000000     PToolsPlugin.obj
 0002:fffe4000       ?_Generic_object$initializer$@?$_Error_objects@H@std@@2P6AXXZA 10000000     PToolsPlugin.obj
 0002:fffe4000       __catchsym$?_Copy@?$basic_string@DU?$char_traits@D@std@@V?$allocator@D@2@@std@@QAEXII@Z$5 10000000     PToolsPlugin.obj
 0001:fffff000       __ehhandler$?_Copy@?$basic_string@DU?$char_traits@D@std@@V?$allocator@D@2@@std@@QAEXII@Z 10000000 f   PToolsPlugin.obj
 0002:fffe4000       ?_System_object$initializer$@?$_Error_objects@H@std@@2P6AXXZA 10000000     PToolsTests.obj
 0002:fffe4000       ?_Iostream_object$initializer$@?$_Error_objects@H@std@@2P6AXXZA 10000000     PToolsTests.obj
 0002:fffe4000       __catchsym$?_Copy@?$basic_string@DU?$char_traits@D@std@@V?$allocator@D@2@@std@@QAEXII@Z$5 10000000     superpose.obj
 0002:fffe4000       ?_Generic_object$initializer$@?$_Error_objects@H@std@@2P6AXXZA 10000000     PToolsTests.obj
 0002:fffe4000       __unwindtable$??0?$Array2D@N@@QAE@HH@Z 10000000     superpose.obj
 0002:fffe4000       __catchsym$?_Copy@?$basic_string@DU?$char_traits@D@std@@V?$allocator@D@2@@std@@QAEXII@Z$5 10000000     PToolsTests.obj
 0001:fffff000       __ehhandler$?_Copy@?$basic_string@DU?$char_traits@D@std@@V?$allocator@D@2@@std@@QAEXII@Z 10000000 f   PToolsTests.obj
 0002:fffe4000       ?_System_object$initializer$@?$_Error_objects@H@std@@2P6AXXZA 10000000     atom.obj
 0002:fffe4000       ?_Iostream_object$initializer$@?$_Error_objects@H@std@@2P6AXXZA 10000000     atom.obj
 0002:fffe4000       __catchsym$?reallocData@?$QVector@N@@AAEXHHV?$QFlags@W4AllocationOption@QArrayData@@@@@Z$5 10000000     superpose.obj
 0002:fffe4000       ?_Generic_object$initializer$@?$_Error_objects@H@std@@2P6AXXZA 10000000     atom.obj
 0000:fffd9000       .debug$S                   10000000     MSVCRT:MSVCR120.dll
 0001:fffff000       __ehhandler$?_Copy@?$basic_string@DU?$char_traits@D@std@@V?$allocator@D@2@@std@@QAEXII@Z 10000000 f   atom.obj
 0002:fffe4000       ?_System_object$initializer$@?$_Error_objects@H@std@@2P6AXXZA 10000000     atomselection.obj
 0002:fffe4000       ?_Iostream_object$initializer$@?$_Error_objects@H@std@@2P6AXXZA 10000000     atomselection.obj
 0002:fffe4000       ?_Generic_object$initializer$@?$_Error_objects@H@std@@2P6AXXZA 10000000     atomselection.obj
 0002:fffe4000       __catchsym$?_Copy@?$basic_string@DU?$char_traits@D@std@@V?$allocator@D@2@@std@@QAEXII@Z$5 10000000     atomselection.obj
 0001:fffff000       __ehhandler$?_Copy@?$basic_string@DU?$char_traits@D@std@@V?$allocator@D@2@@std@@QAEXII@Z 10000000 f   atomselection.obj
 0002:fffe4000       ?_System_object$initializer$@?$_Error_objects@H@std@@2P6AXXZA 10000000     basetypes.obj
 0002:fffe4000       ?_Iostream_object$initializer$@?$_Error_objects@H@std@@2P6AXXZA 10000000     basetypes.obj
 0002:fffe4000       ?_Generic_object$initializer$@?$_Error_objects@H@std@@2P6AXXZA 10000000     basetypes.obj
 0002:fffe4000       __catchsym$?reallocData@?$QVector@N@@AAEXHHV?$QFlags@W4AllocationOption@QArrayData@@@@@Z$5 10000000     basetypes.obj
 0002:fffe4000       __catchsym$?_Copy@?$basic_string@DU?$char_traits@D@std@@V?$allocator@D@2@@std@@QAEXII@Z$5 10000000     basetypes.obj
 0001:fffff000       __ehhandler$?reallocData@?$QVector@N@@AAEXHHV?$QFlags@W4AllocationOption@QArrayData@@@@@Z 10000000 f   basetypes.obj
 0001:fffff000       __ehhandler$?_Copy@?$basic_string@DU?$char_traits@D@std@@V?$allocator@D@2@@std@@QAEXII@Z 10000000 f   basetypes.obj
 0002:fffe4000       ?_System_object$initializer$@?$_Error_objects@H@std@@2P6AXXZA 10000000     coord3d.obj
 0002:fffe4000       ?_Iostream_object$initializer$@?$_Error_objects@H@std@@2P6AXXZA 10000000     coord3d.obj
 0002:fffe4000       ?_Generic_object$initializer$@?$_Error_objects@H@std@@2P6AXXZA 10000000     coord3d.obj
 0002:fffe4000       __catchsym$?_Copy@?$basic_string@DU?$char_traits@D@std@@V?$allocator@D@2@@std@@QAEXII@Z$5 10000000     coord3d.obj
 0001:fffff000       __ehhandler$?_Copy@?$basic_string@DU?$char_traits@D@std@@V?$allocator@D@2@@std@@QAEXII@Z 10000000 f   coord3d.obj
 0002:fffe4000       ?_Generic_object$initializer$@?$_Error_objects@H@std@@2P6AXXZA 10000000     superpose.obj
 0002:fffe4000       ?_Iostream_object$initializer$@?$_Error_objects@H@std@@2P6AXXZA 10000000     superpose.obj
 0002:fffe4000       ?_System_object$initializer$@?$_Error_objects@H@std@@2P6AXXZA 10000000     superpose.obj
 0002:fffe4000       ?_System_object$initializer$@?$_Error_objects@H@std@@2P6AXXZA 10000000     coordsarray.obj
 0002:fffe4000       ?_Iostream_object$initializer$@?$_Error_objects@H@std@@2P6AXXZA 10000000     coordsarray.obj
 0002:fffe4000       ?_Generic_object$initializer$@?$_Error_objects@H@std@@2P6AXXZA 10000000     coordsarray.obj
 0002:fffe4000       __catchsym$?reallocData@?$QVector@N@@AAEXHHV?$QFlags@W4AllocationOption@QArrayData@@@@@Z$5 10000000     coordsarray.obj
 0002:fffe4000       __catchsym$?_Copy@?$basic_string@DU?$char_traits@D@std@@V?$allocator@D@2@@std@@QAEXII@Z$5 10000000     coordsarray.obj
 0001:fffff000       __ehhandler$?reallocData@?$QVector@N@@AAEXHHV?$QFlags@W4AllocationOption@QArrayData@@@@@Z 10000000 f   coordsarray.obj
 0001:fffff000       __ehhandler$?_Copy@?$basic_string@DU?$char_traits@D@std@@V?$allocator@D@2@@std@@QAEXII@Z 10000000 f   rmsd.obj
 0001:fffff000       __ehhandler$?_Copy@?$basic_string@DU?$char_traits@D@std@@V?$allocator@D@2@@std@@QAEXII@Z 10000000 f   coordsarray.obj
 0002:fffe4000       ?_System_object$initializer$@?$_Error_objects@H@std@@2P6AXXZA 10000000     geometry.obj
 0002:fffe4000       ?_Iostream_object$initializer$@?$_Error_objects@H@std@@2P6AXXZA 10000000     geometry.obj
 0002:fffe4000       ?_Generic_object$initializer$@?$_Error_objects@H@std@@2P6AXXZA 10000000     geometry.obj
 0002:fffe4000       __catchsym$?_Copy@?$basic_string@DU?$char_traits@D@std@@V?$allocator@D@2@@std@@QAEXII@Z$5 10000000     geometry.obj
 0001:fffff000       __ehhandler$?_Copy@?$basic_string@DU?$char_traits@D@std@@V?$allocator@D@2@@std@@QAEXII@Z 10000000 f   geometry.obj
 0002:fffe4000       ?_System_object$initializer$@?$_Error_objects@H@std@@2P6AXXZA 10000000     pdbio.obj
 0002:fffe4000       ?_Iostream_object$initializer$@?$_Error_objects@H@std@@2P6AXXZA 10000000     pdbio.obj
 0002:fffe4000       ?_Generic_object$initializer$@?$_Error_objects@H@std@@2P6AXXZA 10000000     pdbio.obj
 0002:fffe4000       __catchsym$?_Copy@?$basic_string@DU?$char_traits@D@std@@V?$allocator@D@2@@std@@QAEXII@Z$5 10000000     rmsd.obj
 0002:fffe4000       __unwindtable$??0?$basic_stringbuf@DU?$char_traits@D@std@@V?$allocator@D@2@@std@@QAE@H@Z 10000000     pdbio.obj
 0002:fffe4000       __unwindtable$?SetType@Atomproperty@PTools@@QAEXV?$basic_string@DU?$char_traits@D@std@@V?$allocator@D@2@@std@@@Z 10000000     pdbio.obj
 0002:fffe4000       __ehfuncinfo$??0Atomproperty@PTools@@QAE@XZ 10000000     pdbio.obj
 0002:fffe4000       __catchsym$?_Copy@?$basic_string@DU?$char_traits@D@std@@V?$allocator@D@2@@std@@QAEXII@Z$5 10000000     pdbio.obj
 0002:fffe4000       ?_Generic_object$initializer$@?$_Error_objects@H@std@@2P6AXXZA 10000000     rmsd.obj
 0002:fffe4000       ?_Iostream_object$initializer$@?$_Error_objects@H@std@@2P6AXXZA 10000000     rmsd.obj
 0002:fffe4000       ?_System_object$initializer$@?$_Error_objects@H@std@@2P6AXXZA 10000000     rmsd.obj
 0001:fffff000       __unwindfunclet$??0?$basic_stringbuf@DU?$char_traits@D@std@@V?$allocator@D@2@@std@@QAE@H@Z$0 10000000 f   pdbio.obj
 0001:fffff000       __unwindfunclet$?SetType@Atomproperty@PTools@@QAEXV?$basic_string@DU?$char_traits@D@std@@V?$allocator@D@2@@std@@@Z$0 10000000 f   pdbio.obj
 0001:fffff000       __unwindfunclet$??0Atomproperty@PTools@@QAE@XZ$0 10000000 f   pdbio.obj
 0001:fffff000       __ehhandler$?_Copy@?$basic_string@DU?$char_traits@D@std@@V?$allocator@D@2@@std@@QAEXII@Z 10000000 f   pdbio.obj
 0002:fffe4000       ?_System_object$initializer$@?$_Error_objects@H@std@@2P6AXXZA 10000000     rigidbody.obj
 0002:fffe4000       ?_Iostream_object$initializer$@?$_Error_objects@H@std@@2P6AXXZA 10000000     rigidbody.obj
 0001:fffff000       __ehhandler$?_Copy@?$basic_string@DU?$char_traits@D@std@@V?$allocator@D@2@@std@@QAEXII@Z 10000000 f   rigidbody.obj
 0002:fffe4000       ?_Generic_object$initializer$@?$_Error_objects@H@std@@2P6AXXZA 10000000     rigidbody.obj
 0002:fffe4000       __catchsym$??4?$vector@UCoord3D@PTools@@V?$allocator@UCoord3D@PTools@@@std@@@std@@QAEAAV01@ABV01@@Z$2 10000000     rigidbody.obj
 0002:fffe4000       __unwindtable$??0Atom@PTools@@QAE@VAtomproperty@1@UCoord3D@1@@Z 10000000     rigidbody.obj
 0001:fffff000       __unwindfunclet$??0Atomproperty@PTools@@QAE@ABV01@@Z$0 10000000 f   rigidbody.obj
 0002:fffe4000       __unwindtable$??0Atomproperty@PTools@@QAE@ABV01@@Z 10000000     rigidbody.obj
 0002:fffe4000       __catchsym$?_Copy@?$basic_string@DU?$char_traits@D@std@@V?$allocator@D@2@@std@@QAEXII@Z$5 10000000     rigidbody.obj
 0001:fffff000       __ehhandler$??4?$vector@UCoord3D@PTools@@V?$allocator@UCoord3D@PTools@@@std@@@std@@QAEAAV01@ABV01@@Z 10000000 f   rigidbody.obj
 0001:fffff000       __unwindfunclet$??0Atom@PTools@@QAE@VAtomproperty@1@UCoord3D@1@@Z$0 10000000 f   rigidbody.obj
 0001:fffff008       __ehhandler$??0Atom@PTools@@QAE@VAtomproperty@1@UCoord3D@1@@Z 10000008 f   rigidbody.obj
 0001:fffff008       __unwindfunclet$??0Atomproperty@PTools@@QAE@ABV01@@Z$1 10000008 f   rigidbody.obj
 0001:fffff008       __unwindfunclet$??0Atomproperty@PTools@@QAE@XZ$1 10000008 f   pdbio.obj
 0002:fffe4008       __ehfuncinfo$??0Atom@PTools@@QAE@VAtomproperty@1@UCoord3D@1@@Z 10000008     rigidbody.obj
 0001:fffff008       __ehhandler$??0?$Array2D@N@@QAE@HH@Z 10000008 f   superpose.obj
 0002:fffe4008       __ehfuncinfo$??0?$Array2D@N@@QAE@HH@Z 10000008     superpose.obj
 0002:fffe4008       __ehfuncinfo$?SetType@Atomproperty@PTools@@QAEXV?$basic_string@DU?$char_traits@D@std@@V?$allocator@D@2@@std@@@Z 10000008     pdbio.obj
 0002:fffe4008       __ehfuncinfo$??0?$basic_stringbuf@DU?$char_traits@D@std@@V?$allocator@D@2@@std@@QAE@H@Z 10000008     pdbio.obj
 0001:fffff008       __ehhandler$?SetType@Atomproperty@PTools@@QAEXV?$basic_string@DU?$char_traits@D@std@@V?$allocator@D@2@@std@@@Z 10000008 f   pdbio.obj
 0001:fffff009       __ehhandler$??0?$basic_stringbuf@DU?$char_traits@D@std@@V?$allocator@D@2@@std@@QAE@H@Z 10000009 f   pdbio.obj
 0002:fffe4010       __catchsym$?reallocData@?$QVector@N@@AAEXHHV?$QFlags@W4AllocationOption@QArrayData@@@@@Z$4 10000010     coordsarray.obj
 0002:fffe4010       __unwindtable$??4?$vector@UCoord3D@PTools@@V?$allocator@UCoord3D@PTools@@@std@@@std@@QAEAAV01@ABV01@@Z 10000010     rigidbody.obj
 0002:fffe4010       __catchsym$?_Copy@?$basic_string@DU?$char_traits@D@std@@V?$allocator@D@2@@std@@QAEXII@Z$4 10000010     coordsarray.obj
 0002:fffe4010       __catchsym$?_Copy@?$basic_string@DU?$char_traits@D@std@@V?$allocator@D@2@@std@@QAEXII@Z$4 10000010     superpose.obj
 0002:fffe4010       __catchsym$?_Copy@?$basic_string@DU?$char_traits@D@std@@V?$allocator@D@2@@std@@QAEXII@Z$4 10000010     moc_PToolsPlugin.obj
 0002:fffe4010       __catchsym$?_Copy@?$basic_string@DU?$char_traits@D@std@@V?$allocator@D@2@@std@@QAEXII@Z$4 10000010     coord3d.obj
 0002:fffe4010       __catchsym$?_Copy@?$basic_string@DU?$char_traits@D@std@@V?$allocator@D@2@@std@@QAEXII@Z$4 10000010     pdbio.obj
 0002:fffe4010       __catchsym$?_Copy@?$basic_string@DU?$char_traits@D@std@@V?$allocator@D@2@@std@@QAEXII@Z$4 10000010     moc_PToolsTests.obj
 0002:fffe4010       __catchsym$?_Copy@?$basic_string@DU?$char_traits@D@std@@V?$allocator@D@2@@std@@QAEXII@Z$4 10000010     rmsd.obj
 0002:fffe4010       __catchsym$?_Copy@?$basic_string@DU?$char_traits@D@std@@V?$allocator@D@2@@std@@QAEXII@Z$4 10000010     PToolsTests.obj
 0002:fffe4010       __catchsym$?_Copy@?$basic_string@DU?$char_traits@D@std@@V?$allocator@D@2@@std@@QAEXII@Z$4 10000010     basetypes.obj
 0002:fffe4010       __catchsym$?_Copy@?$basic_string@DU?$char_traits@D@std@@V?$allocator@D@2@@std@@QAEXII@Z$4 10000010     geometry.obj
 0002:fffe4010       __catchsym$?reallocData@?$QVector@N@@AAEXHHV?$QFlags@W4AllocationOption@QArrayData@@@@@Z$4 10000010     basetypes.obj
 0002:fffe4010       __catchsym$?_Copy@?$basic_string@DU?$char_traits@D@std@@V?$allocator@D@2@@std@@QAEXII@Z$4 10000010     PToolsPlugin.obj
 0002:fffe4010       __catchsym$?_Copy@?$basic_string@DU?$char_traits@D@std@@V?$allocator@D@2@@std@@QAEXII@Z$4 10000010     atomselection.obj
 0002:fffe4010       __catchsym$?_Copy@?$basic_string@DU?$char_traits@D@std@@V?$allocator@D@2@@std@@QAEXII@Z$4 10000010     rigidbody.obj
 0002:fffe4010       __catchsym$?_Copy@?$basic_string@DU?$char_traits@D@std@@V?$allocator@D@2@@std@@QAEXII@Z$4 10000010     atom.obj
 0002:fffe4010       __catchsym$?reallocData@?$QVector@N@@AAEXHHV?$QFlags@W4AllocationOption@QArrayData@@@@@Z$4 10000010     superpose.obj
 0001:fffff013       __unwindfunclet$??0Atomproperty@PTools@@QAE@XZ$2 10000013 f   pdbio.obj
 0001:fffff013       __unwindfunclet$??0Atomproperty@PTools@@QAE@ABV01@@Z$2 10000013 f   rigidbody.obj
 0001:fffff01e       __unwindfunclet$??0Atomproperty@PTools@@QAE@XZ$3 1000001e f   pdbio.obj
 0001:fffff01e       __unwindfunclet$??0Atomproperty@PTools@@QAE@ABV01@@Z$3 1000001e f   rigidbody.obj
 0002:fffe4020       __unwindtable$?reallocData@?$QVector@N@@AAEXHHV?$QFlags@W4AllocationOption@QArrayData@@@@@Z 10000020     superpose.obj
 0002:fffe4020       __unwindtable$?_Copy@?$basic_string@DU?$char_traits@D@std@@V?$allocator@D@2@@std@@QAEXII@Z 10000020     geometry.obj
 0002:fffe4020       __unwindtable$?_Copy@?$basic_string@DU?$char_traits@D@std@@V?$allocator@D@2@@std@@QAEXII@Z 10000020     PToolsTests.obj
 0002:fffe4020       __unwindtable$?_Copy@?$basic_string@DU?$char_traits@D@std@@V?$allocator@D@2@@std@@QAEXII@Z 10000020     basetypes.obj
 0002:fffe4020       __unwindtable$?_Copy@?$basic_string@DU?$char_traits@D@std@@V?$allocator@D@2@@std@@QAEXII@Z 10000020     coord3d.obj
 0002:fffe4020       __unwindtable$?reallocData@?$QVector@N@@AAEXHHV?$QFlags@W4AllocationOption@QArrayData@@@@@Z 10000020     basetypes.obj
 0002:fffe4020       __unwindtable$?reallocData@?$QVector@N@@AAEXHHV?$QFlags@W4AllocationOption@QArrayData@@@@@Z 10000020     coordsarray.obj
 0002:fffe4020       __unwindtable$?_Copy@?$basic_string@DU?$char_traits@D@std@@V?$allocator@D@2@@std@@QAEXII@Z 10000020     moc_PToolsTests.obj
 0002:fffe4020       __unwindtable$?_Copy@?$basic_string@DU?$char_traits@D@std@@V?$allocator@D@2@@std@@QAEXII@Z 10000020     superpose.obj
 0002:fffe4020       __unwindtable$?_Copy@?$basic_string@DU?$char_traits@D@std@@V?$allocator@D@2@@std@@QAEXII@Z 10000020     PToolsPlugin.obj
 0002:fffe4020       __unwindtable$?_Copy@?$basic_string@DU?$char_traits@D@std@@V?$allocator@D@2@@std@@QAEXII@Z 10000020     coordsarray.obj
 0002:fffe4020       __tryblocktable$??4?$vector@UCoord3D@PTools@@V?$allocator@UCoord3D@PTools@@@std@@@std@@QAEAAV01@ABV01@@Z 10000020     rigidbody.obj
 0002:fffe4020       __unwindtable$?_Copy@?$basic_string@DU?$char_traits@D@std@@V?$allocator@D@2@@std@@QAEXII@Z 10000020     moc_PToolsPlugin.obj
 0002:fffe4020       __unwindtable$?_Copy@?$basic_string@DU?$char_traits@D@std@@V?$allocator@D@2@@std@@QAEXII@Z 10000020     rmsd.obj
 0002:fffe4020       __unwindtable$?_Copy@?$basic_string@DU?$char_traits@D@std@@V?$allocator@D@2@@std@@QAEXII@Z 10000020     pdbio.obj
 0002:fffe4020       __ehfuncinfo$??0Atomproperty@PTools@@QAE@ABV01@@Z 10000020     rigidbody.obj
 0002:fffe4020       __unwindtable$?_Copy@?$basic_string@DU?$char_traits@D@std@@V?$allocator@D@2@@std@@QAEXII@Z 10000020     atomselection.obj
 0002:fffe4020       __unwindtable$?_Copy@?$basic_string@DU?$char_traits@D@std@@V?$allocator@D@2@@std@@QAEXII@Z 10000020     atom.obj
 0002:fffe4020       __unwindtable$?_Copy@?$basic_string@DU?$char_traits@D@std@@V?$allocator@D@2@@std@@QAEXII@Z 10000020     rigidbody.obj
 0002:fffe4024       __unwindtable$??0Atomproperty@PTools@@QAE@XZ 10000024     pdbio.obj
 0001:fffff029       __ehhandler$??0Atomproperty@PTools@@QAE@ABV01@@Z 10000029 f   rigidbody.obj
 0001:fffff029       __unwindfunclet$??0Atomproperty@PTools@@QAE@XZ$4 10000029 f   pdbio.obj
 0002:fffe4034       __ehfuncinfo$??4?$vector@UCoord3D@PTools@@V?$allocator@UCoord3D@PTools@@@std@@@std@@QAEAAV01@ABV01@@Z 10000034     rigidbody.obj
 0001:fffff034       __ehhandler$??0Atomproperty@PTools@@QAE@XZ 10000034 f   pdbio.obj
 0002:fffe4040       __ehfuncinfo$?_Copy@?$basic_string@DU?$char_traits@D@std@@V?$allocator@D@2@@std@@QAEXII@Z 10000040     rmsd.obj
 0002:fffe4040       __ehfuncinfo$?_Copy@?$basic_string@DU?$char_traits@D@std@@V?$allocator@D@2@@std@@QAEXII@Z 10000040     rigidbody.obj
 0002:fffe4040       __ehfuncinfo$?_Copy@?$basic_string@DU?$char_traits@D@std@@V?$allocator@D@2@@std@@QAEXII@Z 10000040     PToolsTests.obj
 0002:fffe4040       __ehfuncinfo$?_Copy@?$basic_string@DU?$char_traits@D@std@@V?$allocator@D@2@@std@@QAEXII@Z 10000040     geometry.obj
 0002:fffe4040       __ehfuncinfo$?_Copy@?$basic_string@DU?$char_traits@D@std@@V?$allocator@D@2@@std@@QAEXII@Z 10000040     PToolsPlugin.obj
 0002:fffe4040       __ehfuncinfo$?reallocData@?$QVector@N@@AAEXHHV?$QFlags@W4AllocationOption@QArrayData@@@@@Z 10000040     superpose.obj
 0002:fffe4040       __ehfuncinfo$?_Copy@?$basic_string@DU?$char_traits@D@std@@V?$allocator@D@2@@std@@QAEXII@Z 10000040     atomselection.obj
 0002:fffe4040       __ehfuncinfo$?_Copy@?$basic_string@DU?$char_traits@D@std@@V?$allocator@D@2@@std@@QAEXII@Z 10000040     atom.obj
 0002:fffe4040       __ehfuncinfo$?_Copy@?$basic_string@DU?$char_traits@D@std@@V?$allocator@D@2@@std@@QAEXII@Z 10000040     coordsarray.obj
 0002:fffe4040       __ehfuncinfo$?_Copy@?$basic_string@DU?$char_traits@D@std@@V?$allocator@D@2@@std@@QAEXII@Z 10000040     moc_PToolsPlugin.obj
 0002:fffe4040       __ehfuncinfo$?_Copy@?$basic_string@DU?$char_traits@D@std@@V?$allocator@D@2@@std@@QAEXII@Z 10000040     basetypes.obj
 0002:fffe4040       __ehfuncinfo$?reallocData@?$QVector@N@@AAEXHHV?$QFlags@W4AllocationOption@QArrayData@@@@@Z 10000040     basetypes.obj
 0002:fffe4040       __ehfuncinfo$?_Copy@?$basic_string@DU?$char_traits@D@std@@V?$allocator@D@2@@std@@QAEXII@Z 10000040     superpose.obj
 0002:fffe4040       __ehfuncinfo$?_Copy@?$basic_string@DU?$char_traits@D@std@@V?$allocator@D@2@@std@@QAEXII@Z 10000040     pdbio.obj
 0002:fffe4040       __ehfuncinfo$?_Copy@?$basic_string@DU?$char_traits@D@std@@V?$allocator@D@2@@std@@QAEXII@Z 10000040     moc_PToolsTests.obj
 0002:fffe4040       __ehfuncinfo$?_Copy@?$basic_string@DU?$char_traits@D@std@@V?$allocator@D@2@@std@@QAEXII@Z 10000040     coord3d.obj
 0002:fffe4040       __ehfuncinfo$?reallocData@?$QVector@N@@AAEXHHV?$QFlags@W4AllocationOption@QArrayData@@@@@Z 10000040     coordsarray.obj
 0002:fffe4064       __tryblocktable$?reallocData@?$QVector@N@@AAEXHHV?$QFlags@W4AllocationOption@QArrayData@@@@@Z 10000064     superpose.obj
 0002:fffe4064       __tryblocktable$?_Copy@?$basic_string@DU?$char_traits@D@std@@V?$allocator@D@2@@std@@QAEXII@Z 10000064     basetypes.obj
 0002:fffe4064       __tryblocktable$?_Copy@?$basic_string@DU?$char_traits@D@std@@V?$allocator@D@2@@std@@QAEXII@Z 10000064     moc_PToolsPlugin.obj
 0002:fffe4064       __tryblocktable$?_Copy@?$basic_string@DU?$char_traits@D@std@@V?$allocator@D@2@@std@@QAEXII@Z 10000064     atom.obj
 0002:fffe4064       __tryblocktable$?_Copy@?$basic_string@DU?$char_traits@D@std@@V?$allocator@D@2@@std@@QAEXII@Z 10000064     coordsarray.obj
 0002:fffe4064       __tryblocktable$?reallocData@?$QVector@N@@AAEXHHV?$QFlags@W4AllocationOption@QArrayData@@@@@Z 10000064     basetypes.obj
 0002:fffe4064       __tryblocktable$?_Copy@?$basic_string@DU?$char_traits@D@std@@V?$allocator@D@2@@std@@QAEXII@Z 10000064     coord3d.obj
 0002:fffe4064       __tryblocktable$?_Copy@?$basic_string@DU?$char_traits@D@std@@V?$allocator@D@2@@std@@QAEXII@Z 10000064     rmsd.obj
 0002:fffe4064       __tryblocktable$?_Copy@?$basic_string@DU?$char_traits@D@std@@V?$allocator@D@2@@std@@QAEXII@Z 10000064     superpose.obj
 0002:fffe4064       __tryblocktable$?_Copy@?$basic_string@DU?$char_traits@D@std@@V?$allocator@D@2@@std@@QAEXII@Z 10000064     atomselection.obj
 0002:fffe4064       __tryblocktable$?_Copy@?$basic_string@DU?$char_traits@D@std@@V?$allocator@D@2@@std@@QAEXII@Z 10000064     pdbio.obj
 0002:fffe4064       __tryblocktable$?_Copy@?$basic_string@DU?$char_traits@D@std@@V?$allocator@D@2@@std@@QAEXII@Z 10000064     geometry.obj
 0002:fffe4064       __tryblocktable$?_Copy@?$basic_string@DU?$char_traits@D@std@@V?$allocator@D@2@@std@@QAEXII@Z 10000064     PToolsTests.obj
 0002:fffe4064       __tryblocktable$?_Copy@?$basic_string@DU?$char_traits@D@std@@V?$allocator@D@2@@std@@QAEXII@Z 10000064     moc_PToolsTests.obj
 0002:fffe4064       __tryblocktable$?_Copy@?$basic_string@DU?$char_traits@D@std@@V?$allocator@D@2@@std@@QAEXII@Z 10000064     PToolsPlugin.obj
 0002:fffe4064       __tryblocktable$?_Copy@?$basic_string@DU?$char_traits@D@std@@V?$allocator@D@2@@std@@QAEXII@Z 10000064     rigidbody.obj
 0002:fffe4064       __tryblocktable$?reallocData@?$QVector@N@@AAEXHHV?$QFlags@W4AllocationOption@QArrayData@@@@@Z 10000064     coordsarray.obj
 0001:fffff096       __catch$?_Copy@?$basic_string@DU?$char_traits@D@std@@V?$allocator@D@2@@std@@QAEXII@Z$0 10000096 f   atom.obj
 0001:fffff096       __catch$?_Copy@?$basic_string@DU?$char_traits@D@std@@V?$allocator@D@2@@std@@QAEXII@Z$0 10000096 f   moc_PToolsPlugin.obj
 0001:fffff096       __catch$?_Copy@?$basic_string@DU?$char_traits@D@std@@V?$allocator@D@2@@std@@QAEXII@Z$0 10000096 f   atomselection.obj
 0001:fffff096       __catch$?_Copy@?$basic_string@DU?$char_traits@D@std@@V?$allocator@D@2@@std@@QAEXII@Z$0 10000096 f   coordsarray.obj
 0001:fffff096       __catch$?_Copy@?$basic_string@DU?$char_traits@D@std@@V?$allocator@D@2@@std@@QAEXII@Z$0 10000096 f   basetypes.obj
 0001:fffff096       __catch$?_Copy@?$basic_string@DU?$char_traits@D@std@@V?$allocator@D@2@@std@@QAEXII@Z$0 10000096 f   pdbio.obj
 0001:fffff096       __catch$?_Copy@?$basic_string@DU?$char_traits@D@std@@V?$allocator@D@2@@std@@QAEXII@Z$0 10000096 f   superpose.obj
 0001:fffff096       __catch$?_Copy@?$basic_string@DU?$char_traits@D@std@@V?$allocator@D@2@@std@@QAEXII@Z$0 10000096 f   PToolsTests.obj
 0001:fffff096       __catch$?_Copy@?$basic_string@DU?$char_traits@D@std@@V?$allocator@D@2@@std@@QAEXII@Z$0 10000096 f   rigidbody.obj
 0001:fffff096       __catch$?_Copy@?$basic_string@DU?$char_traits@D@std@@V?$allocator@D@2@@std@@QAEXII@Z$0 10000096 f   geometry.obj
 0001:fffff096       __catch$?_Copy@?$basic_string@DU?$char_traits@D@std@@V?$allocator@D@2@@std@@QAEXII@Z$0 10000096 f   moc_PToolsTests.obj
 0001:fffff096       __catch$?_Copy@?$basic_string@DU?$char_traits@D@std@@V?$allocator@D@2@@std@@QAEXII@Z$0 10000096 f   PToolsPlugin.obj
 0001:fffff096       __catch$?_Copy@?$basic_string@DU?$char_traits@D@std@@V?$allocator@D@2@@std@@QAEXII@Z$0 10000096 f   coord3d.obj
 0001:fffff096       __catch$?_Copy@?$basic_string@DU?$char_traits@D@std@@V?$allocator@D@2@@std@@QAEXII@Z$0 10000096 f   rmsd.obj
 0001:fffff0d3       __catch$?_Copy@?$basic_string@DU?$char_traits@D@std@@V?$allocator@D@2@@std@@QAEXII@Z$1 100000d3 f   PToolsPlugin.obj
 0001:fffff0d3       __catch$?_Copy@?$basic_string@DU?$char_traits@D@std@@V?$allocator@D@2@@std@@QAEXII@Z$1 100000d3 f   moc_PToolsTests.obj
 0001:fffff0d3       __catch$?_Copy@?$basic_string@DU?$char_traits@D@std@@V?$allocator@D@2@@std@@QAEXII@Z$1 100000d3 f   basetypes.obj
 0001:fffff0d3       __catch$?_Copy@?$basic_string@DU?$char_traits@D@std@@V?$allocator@D@2@@std@@QAEXII@Z$1 100000d3 f   PToolsTests.obj
 0001:fffff0d3       __catch$?_Copy@?$basic_string@DU?$char_traits@D@std@@V?$allocator@D@2@@std@@QAEXII@Z$1 100000d3 f   rigidbody.obj
 0001:fffff0d3       __catch$?_Copy@?$basic_string@DU?$char_traits@D@std@@V?$allocator@D@2@@std@@QAEXII@Z$1 100000d3 f   superpose.obj
 0001:fffff0d3       __catch$?_Copy@?$basic_string@DU?$char_traits@D@std@@V?$allocator@D@2@@std@@QAEXII@Z$1 100000d3 f   geometry.obj
 0001:fffff0d3       __catch$?_Copy@?$basic_string@DU?$char_traits@D@std@@V?$allocator@D@2@@std@@QAEXII@Z$1 100000d3 f   pdbio.obj
 0001:fffff0d3       __catch$?_Copy@?$basic_string@DU?$char_traits@D@std@@V?$allocator@D@2@@std@@QAEXII@Z$1 100000d3 f   coord3d.obj
 0001:fffff0d3       __catch$?_Copy@?$basic_string@DU?$char_traits@D@std@@V?$allocator@D@2@@std@@QAEXII@Z$1 100000d3 f   coordsarray.obj
 0001:fffff0d3       __catch$?_Copy@?$basic_string@DU?$char_traits@D@std@@V?$allocator@D@2@@std@@QAEXII@Z$1 100000d3 f   atomselection.obj
 0001:fffff0d3       __catch$?_Copy@?$basic_string@DU?$char_traits@D@std@@V?$allocator@D@2@@std@@QAEXII@Z$1 100000d3 f   atom.obj
 0001:fffff0d3       __catch$?_Copy@?$basic_string@DU?$char_traits@D@std@@V?$allocator@D@2@@std@@QAEXII@Z$1 100000d3 f   rmsd.obj
 0001:fffff0d3       __catch$?_Copy@?$basic_string@DU?$char_traits@D@std@@V?$allocator@D@2@@std@@QAEXII@Z$1 100000d3 f   moc_PToolsPlugin.obj
 0001:fffff15f       __catch$??4?$vector@UCoord3D@PTools@@V?$allocator@UCoord3D@PTools@@@std@@@std@@QAEAAV01@ABV01@@Z$0 1000015f f   rigidbody.obj
 0001:fffff1a4       __catch$?reallocData@?$QVector@N@@AAEXHHV?$QFlags@W4AllocationOption@QArrayData@@@@@Z$0 100001a4 f   superpose.obj
 0001:fffff1a4       __catch$?reallocData@?$QVector@N@@AAEXHHV?$QFlags@W4AllocationOption@QArrayData@@@@@Z$0 100001a4 f   basetypes.obj
 0001:fffff1a4       __catch$?reallocData@?$QVector@N@@AAEXHHV?$QFlags@W4AllocationOption@QArrayData@@@@@Z$0 100001a4 f   coordsarray.obj
 0001:fffff1b6       __catch$?reallocData@?$QVector@N@@AAEXHHV?$QFlags@W4AllocationOption@QArrayData@@@@@Z$2 100001b6 f   basetypes.obj
 0001:fffff1b6       __catch$?reallocData@?$QVector@N@@AAEXHHV?$QFlags@W4AllocationOption@QArrayData@@@@@Z$2 100001b6 f   coordsarray.obj
 0001:fffff1b6       __catch$?reallocData@?$QVector@N@@AAEXHHV?$QFlags@W4AllocationOption@QArrayData@@@@@Z$2 100001b6 f   superpose.obj
 0001:00000000       ??__E?_Generic_object@?$_Error_objects@H@std@@2V_Generic_error_category@2@A@@YAXXZ 10001000 f   PToolsAligner.obj
 0001:00000010       ??__E?_Iostream_object@?$_Error_objects@H@std@@2V_Iostream_error_category@2@A@@YAXXZ 10001010 f   PToolsAligner.obj
 0001:00000020       ??__E?_System_object@?$_Error_objects@H@std@@2V_System_error_category@2@A@@YAXXZ 10001020 f   PToolsAligner.obj
 0001:00000030       ??__EalgoLog@U2@@YAXXZ     10001030 f   PToolsAligner.obj
 0001:000000b0       ??__EcmdLog@U2@@YAXXZ      100010b0 f   PToolsAligner.obj
 0001:00000130       ??__EcoreLog@U2@@YAXXZ     10001130 f   PToolsAligner.obj
 0001:000001b0       ??__EioLog@U2@@YAXXZ       100011b0 f   PToolsAligner.obj
 0001:00000230       ??__EperfLog@U2@@YAXXZ     10001230 f   PToolsAligner.obj
 0001:000002b0       ??__EscriptLog@U2@@YAXXZ   100012b0 f   PToolsAligner.obj
 0001:00000330       ??__EtaskLog@U2@@YAXXZ     10001330 f   PToolsAligner.obj
 0001:000003b0       ??__EuiLog@U2@@YAXXZ       100013b0 f   PToolsAligner.obj
 0001:00000430       ??__EuserActLog@U2@@YAXXZ  10001430 f   PToolsAligner.obj
 0001:000004b0       ??__E?_Generic_object@?$_Error_objects@H@std@@2V_Generic_error_category@2@A@@YAXXZ 100014b0 f   PToolsPlugin.obj
 0001:000004c0       ??__E?_Iostream_object@?$_Error_objects@H@std@@2V_Iostream_error_category@2@A@@YAXXZ 100014c0 f   PToolsPlugin.obj
 0001:000004d0       ??__E?_System_object@?$_Error_objects@H@std@@2V_System_error_category@2@A@@YAXXZ 100014d0 f   PToolsPlugin.obj
 0001:000004e0       ??__EPTOOLS_ID@U2@@YAXXZ   100014e0 f   PToolsPlugin.obj
 0001:00000500       ??__EalgoLog@U2@@YAXXZ     10001500 f   PToolsPlugin.obj
 0001:00000580       ??__EcmdLog@U2@@YAXXZ      10001580 f   PToolsPlugin.obj
 0001:00000600       ??__EcoreLog@U2@@YAXXZ     10001600 f   PToolsPlugin.obj
 0001:00000680       ??__EioLog@U2@@YAXXZ       10001680 f   PToolsPlugin.obj
 0001:00000700       ??__EperfLog@U2@@YAXXZ     10001700 f   PToolsPlugin.obj
 0001:00000780       ??__EscriptLog@U2@@YAXXZ   10001780 f   PToolsPlugin.obj
 0001:00000800       ??__EtaskLog@U2@@YAXXZ     10001800 f   PToolsPlugin.obj
 0001:00000880       ??__EuiLog@U2@@YAXXZ       10001880 f   PToolsPlugin.obj
 0001:00000900       ??__EuserActLog@U2@@YAXXZ  10001900 f   PToolsPlugin.obj
 0001:00000980       ??__E?ACCURACY_ATTR@Gtest_PToolsAlignerTask@U2@@2VQString@@B@@YAXXZ 10001980 f   PToolsTests.obj
 0001:000009a0       ??__E?MOBO_ATTR@Gtest_PToolsAlignerTask@U2@@2VQString@@B@@YAXXZ 100019a0 f   PToolsTests.obj
 0001:000009c0       ??__E?REFO_ATTR@Gtest_PToolsAlignerTask@U2@@2VQString@@B@@YAXXZ 100019c0 f   PToolsTests.obj
 0001:000009e0       ??__E?RMSD_ATTR@Gtest_PToolsAlignerTask@U2@@2VQString@@B@@YAXXZ 100019e0 f   PToolsTests.obj
 0001:00000a00       ??__E?TRANSFORM_ATTR@Gtest_PToolsAlignerTask@U2@@2VQString@@B@@YAXXZ 10001a00 f   PToolsTests.obj
 0001:00000a20       ??__E?_Generic_object@?$_Error_objects@H@std@@2V_Generic_error_category@2@A@@YAXXZ 10001a20 f   PToolsTests.obj
 0001:00000a30       ??__E?_Iostream_object@?$_Error_objects@H@std@@2V_Iostream_error_category@2@A@@YAXXZ 10001a30 f   PToolsTests.obj
 0001:00000a40       ??__E?_System_object@?$_Error_objects@H@std@@2V_System_error_category@2@A@@YAXXZ 10001a40 f   PToolsTests.obj
 0001:00000a50       ??__EalgoLog@U2@@YAXXZ     10001a50 f   PToolsTests.obj
 0001:00000ad0       ??__EcmdLog@U2@@YAXXZ      10001ad0 f   PToolsTests.obj
 0001:00000b50       ??__EcoreLog@U2@@YAXXZ     10001b50 f   PToolsTests.obj
 0001:00000bd0       ??__EioLog@U2@@YAXXZ       10001bd0 f   PToolsTests.obj
 0001:00000c50       ??__EperfLog@U2@@YAXXZ     10001c50 f   PToolsTests.obj
 0001:00000cd0       ??__EscriptLog@U2@@YAXXZ   10001cd0 f   PToolsTests.obj
 0001:00000d50       ??__EtaskLog@U2@@YAXXZ     10001d50 f   PToolsTests.obj
 0001:00000dd0       ??__EuiLog@U2@@YAXXZ       10001dd0 f   PToolsTests.obj
 0001:00000e50       ??__EuserActLog@U2@@YAXXZ  10001e50 f   PToolsTests.obj
 0001:00000ed0       ??__E?_Generic_object@?$_Error_objects@H@std@@2V_Generic_error_category@2@A@@YAXXZ 10001ed0 f   atom.obj
 0001:00000ee0       ??__E?_Iostream_object@?$_Error_objects@H@std@@2V_Iostream_error_category@2@A@@YAXXZ 10001ee0 f   atom.obj
 0001:00000ef0       ??__E?_System_object@?$_Error_objects@H@std@@2V_System_error_category@2@A@@YAXXZ 10001ef0 f   atom.obj
 0001:00000f00       ??__E?_Generic_object@?$_Error_objects@H@std@@2V_Generic_error_category@2@A@@YAXXZ 10001f00 f   atomselection.obj
 0001:00000f10       ??__E?_Iostream_object@?$_Error_objects@H@std@@2V_Iostream_error_category@2@A@@YAXXZ 10001f10 f   atomselection.obj
 0001:00000f20       ??__E?_System_object@?$_Error_objects@H@std@@2V_System_error_category@2@A@@YAXXZ 10001f20 f   atomselection.obj
 0001:00000f30       ??__E?_Generic_object@?$_Error_objects@H@std@@2V_Generic_error_category@2@A@@YAXXZ 10001f30 f   basetypes.obj
 0001:00000f40       ??__E?_Iostream_object@?$_Error_objects@H@std@@2V_Iostream_error_category@2@A@@YAXXZ 10001f40 f   basetypes.obj
 0001:00000f50       ??__E?_System_object@?$_Error_objects@H@std@@2V_System_error_category@2@A@@YAXXZ 10001f50 f   basetypes.obj
 0001:00000f60       ??__E?_Generic_object@?$_Error_objects@H@std@@2V_Generic_error_category@2@A@@YAXXZ 10001f60 f   coord3d.obj
 0001:00000f70       ??__E?_Iostream_object@?$_Error_objects@H@std@@2V_Iostream_error_category@2@A@@YAXXZ 10001f70 f   coord3d.obj
 0001:00000f80       ??__E?_System_object@?$_Error_objects@H@std@@2V_System_error_category@2@A@@YAXXZ 10001f80 f   coord3d.obj
 0001:00000f90       ??__E?_Generic_object@?$_Error_objects@H@std@@2V_Generic_error_category@2@A@@YAXXZ 10001f90 f   coordsarray.obj
 0001:00000fa0       ??__E?_Iostream_object@?$_Error_objects@H@std@@2V_Iostream_error_category@2@A@@YAXXZ 10001fa0 f   coordsarray.obj
 0001:00000fb0       ??__E?_System_object@?$_Error_objects@H@std@@2V_System_error_category@2@A@@YAXXZ 10001fb0 f   coordsarray.obj
 0001:00000fc0       ??__E?_Generic_object@?$_Error_objects@H@std@@2V_Generic_error_category@2@A@@YAXXZ 10001fc0 f   geometry.obj
 0001:00000fd0       ??__E?_Iostream_object@?$_Error_objects@H@std@@2V_Iostream_error_category@2@A@@YAXXZ 10001fd0 f   geometry.obj
 0001:00000fe0       ??__E?_System_object@?$_Error_objects@H@std@@2V_System_error_category@2@A@@YAXXZ 10001fe0 f   geometry.obj
 0001:00000ff0       ??__E?_Generic_object@?$_Error_objects@H@std@@2V_Generic_error_category@2@A@@YAXXZ 10001ff0 f   pdbio.obj
 0001:00001000       ??__E?_Iostream_object@?$_Error_objects@H@std@@2V_Iostream_error_category@2@A@@YAXXZ 10002000 f   pdbio.obj
 0001:00001010       ??__E?_System_object@?$_Error_objects@H@std@@2V_System_error_category@2@A@@YAXXZ 10002010 f   pdbio.obj
 0001:00001020       ??__E?_Generic_object@?$_Error_objects@H@std@@2V_Generic_error_category@2@A@@YAXXZ 10002020 f   rigidbody.obj
 0001:00001030       ??__E?_Iostream_object@?$_Error_objects@H@std@@2V_Iostream_error_category@2@A@@YAXXZ 10002030 f   rigidbody.obj
 0001:00001040       ??__E?_System_object@?$_Error_objects@H@std@@2V_System_error_category@2@A@@YAXXZ 10002040 f   rigidbody.obj
 0001:00001050       ??__E?_Generic_object@?$_Error_objects@H@std@@2V_Generic_error_category@2@A@@YAXXZ 10002050 f   rmsd.obj
 0001:00001060       ??__E?_Iostream_object@?$_Error_objects@H@std@@2V_Iostream_error_category@2@A@@YAXXZ 10002060 f   rmsd.obj
 0001:00001070       ??__E?_System_object@?$_Error_objects@H@std@@2V_System_error_category@2@A@@YAXXZ 10002070 f   rmsd.obj
 0001:00001080       ??__E?_Generic_object@?$_Error_objects@H@std@@2V_Generic_error_category@2@A@@YAXXZ 10002080 f   superpose.obj
 0001:00001090       ??__E?_Iostream_object@?$_Error_objects@H@std@@2V_Iostream_error_category@2@A@@YAXXZ 10002090 f   superpose.obj
 0001:000010a0       ??__E?_System_object@?$_Error_objects@H@std@@2V_System_error_category@2@A@@YAXXZ 100020a0 f   superpose.obj
 0001:000010b0       ??__E?_Generic_object@?$_Error_objects@H@std@@2V_Generic_error_category@2@A@@YAXXZ 100020b0 f   moc_PToolsPlugin.obj
 0001:000010c0       ??__E?_Iostream_object@?$_Error_objects@H@std@@2V_Iostream_error_category@2@A@@YAXXZ 100020c0 f   moc_PToolsPlugin.obj
 0001:000010d0       ??__E?_System_object@?$_Error_objects@H@std@@2V_System_error_category@2@A@@YAXXZ 100020d0 f   moc_PToolsPlugin.obj
 0001:000010e0       ??__E?staticMetaObject@PToolsPlugin@U2@@2UQMetaObject@@B@@YAXXZ 100020e0 f   moc_PToolsPlugin.obj
 0001:000010f0       ??__EalgoLog@U2@@YAXXZ     100020f0 f   moc_PToolsPlugin.obj
 0001:00001170       ??__EcmdLog@U2@@YAXXZ      10002170 f   moc_PToolsPlugin.obj
 0001:000011f0       ??__EcoreLog@U2@@YAXXZ     100021f0 f   moc_PToolsPlugin.obj
 0001:00001270       ??__EioLog@U2@@YAXXZ       10002270 f   moc_PToolsPlugin.obj
 0001:000012f0       ??__EperfLog@U2@@YAXXZ     100022f0 f   moc_PToolsPlugin.obj
 0001:00001370       ??__EscriptLog@U2@@YAXXZ   10002370 f   moc_PToolsPlugin.obj
 0001:000013f0       ??__EtaskLog@U2@@YAXXZ     100023f0 f   moc_PToolsPlugin.obj
 0001:00001470       ??__EuiLog@U2@@YAXXZ       10002470 f   moc_PToolsPlugin.obj
 0001:000014f0       ??__EuserActLog@U2@@YAXXZ  100024f0 f   moc_PToolsPlugin.obj
 0001:00001570       ??__E?_Generic_object@?$_Error_objects@H@std@@2V_Generic_error_category@2@A@@YAXXZ 10002570 f   moc_PToolsTests.obj
 0001:00001580       ??__E?_Iostream_object@?$_Error_objects@H@std@@2V_Iostream_error_category@2@A@@YAXXZ 10002580 f   moc_PToolsTests.obj
 0001:00001590       ??__E?_System_object@?$_Error_objects@H@std@@2V_System_error_category@2@A@@YAXXZ 10002590 f   moc_PToolsTests.obj
 0001:000015a0       ??__E?staticMetaObject@Gtest_PToolsAlignerTask@U2@@2UQMetaObject@@B@@YAXXZ 100025a0 f   moc_PToolsTests.obj
 0001:000015b0       ??__EalgoLog@U2@@YAXXZ     100025b0 f   moc_PToolsTests.obj
 0001:00001630       ??__EcmdLog@U2@@YAXXZ      10002630 f   moc_PToolsTests.obj
 0001:000016b0       ??__EcoreLog@U2@@YAXXZ     100026b0 f   moc_PToolsTests.obj
 0001:00001730       ??__EioLog@U2@@YAXXZ       10002730 f   moc_PToolsTests.obj
 0001:000017b0       ??__EperfLog@U2@@YAXXZ     100027b0 f   moc_PToolsTests.obj
 0001:00001830       ??__EscriptLog@U2@@YAXXZ   10002830 f   moc_PToolsTests.obj
 0001:000018b0       ??__EtaskLog@U2@@YAXXZ     100028b0 f   moc_PToolsTests.obj
 0001:00001930       ??__EuiLog@U2@@YAXXZ       10002930 f   moc_PToolsTests.obj
 0001:000019b0       ??__EuserActLog@U2@@YAXXZ  100029b0 f   moc_PToolsTests.obj
 0001:00001a28       ??__E_Fac_tidy_reg@std@@YAXXZ 10002a28 f   msvcprt:locale0_implib.obj
 0001:00001cfe       __catch$??0?$QList@H@@QAE@ABV0@@Z$0 10002cfe f i PToolsAligner.obj
 0001:00001dbe       __catch$??0?$QList@V?$QSharedDataPointer@VAtomData@U2@@@@@@QAE@ABV0@@Z$0 10002dbe f i PToolsAligner.obj
 0001:00002fa6       __catch$?_Copy@?$basic_string@DU?$char_traits@D@std@@V?$allocator@D@2@@std@@QAEXII@Z$0 10003fa6 f i PToolsAligner.obj
 0001:00002fe3       __catch$?_Copy@?$basic_string@DU?$char_traits@D@std@@V?$allocator@D@2@@std@@QAEXII@Z$1 10003fe3 f i PToolsAligner.obj
 0001:00003520       __catch$?align@PToolsAligner@U2@@UAE?AVStructuralAlignment@2@ABVStructuralAlignmentTaskSettings@2@AAVTaskStateInfo@2@@Z$0 10004520 f   PToolsAligner.obj
 0001:000035c7       __catch$?align@PToolsAligner@U2@@UAE?AVStructuralAlignment@2@ABVStructuralAlignmentTaskSettings@2@AAVTaskStateInfo@2@@Z$1 100045c7 f   PToolsAligner.obj
 0001:000039c0       ?createRigidBody@U2@@YAPAVRigidbody@PTools@@ABVBioStruct3DReference@1@@Z 100049c0 f   PToolsAligner.obj
 0001:00004460       ?getSubsetSize@U2@@YAHABVBioStruct3DReference@1@@Z 10005460 f   PToolsAligner.obj
 0001:00004bf4       __catch$?reallocData@?$QVector@N@@AAEXHHV?$QFlags@W4AllocationOption@QArrayData@@@@@Z$0 10005bf4 f i PToolsAligner.obj
 0001:00004c06       __catch$?reallocData@?$QVector@N@@AAEXHHV?$QFlags@W4AllocationOption@QArrayData@@@@@Z$2 10005c06 f i PToolsAligner.obj
 0001:0000514e       __catch$??0?$QList@PAVXMLTestFactory@U2@@@@QAE@ABV0@@Z$0 1000614e f i PToolsPlugin.obj
 0001:000059a5       __catch$?append@?$QList@PAVXMLTestFactory@U2@@@@QAEXABQAVXMLTestFactory@U2@@@Z$4 100069a5 f i PToolsPlugin.obj
 0001:00005c91       __catch$?detach_helper_grow@?$QList@PAVXMLTestFactory@U2@@@@AAEPAUNode@1@HH@Z$2 10006c91 f i PToolsPlugin.obj
 0001:00005c91       __catch$?detach_helper_grow@?$QList@PAVXMLTestFactory@U2@@@@AAEPAUNode@1@HH@Z$0 10006c91 f i PToolsPlugin.obj
 0001:00005eee       __catch$??0?$QList@VQString@@@@QAE@ABV0@@Z$0 10006eee f i PToolsTests.obj
 0001:00006270       ?alignmentToStr@U2@@YA?AVQString@@ABVStructuralAlignment@1@N@Z 10007270 f   PToolsTests.obj
 0001:00006485       __catch$?append@?$QList@H@@QAEXABH@Z$4 10007485 f i PToolsTests.obj
 0001:0000665c       __catch$?detach_helper@?$QList@H@@AAEXH@Z$0 1000765c f i PToolsTests.obj
 0001:00006781       __catch$?detach_helper_grow@?$QList@H@@AAEPAUNode@1@HH@Z$0 10007781 f i PToolsTests.obj
 0001:00006781       __catch$?detach_helper_grow@?$QList@H@@AAEPAUNode@1@HH@Z$2 10007781 f i PToolsTests.obj
 0001:00006d70       ?isEqual@U2@@YA_NABVStructuralAlignment@1@0N@Z 10007d70 f   PToolsTests.obj
 0001:00007042       __catch$?node_copy@?$QList@VQString@@@@AAEXPAUNode@1@00@Z$2 10008042 f i PToolsTests.obj
 0001:0000a2a2       __catch$??$?6U?$char_traits@D@std@@@std@@YAAAV?$basic_ostream@DU?$char_traits@D@std@@@0@AAV10@PBD@Z$0 1000b2a2 f i coord3d.obj
 0001:0000bbbf       __catch$??4?$vector@UCoord3D@PTools@@V?$allocator@UCoord3D@PTools@@@std@@@std@@QAEAAV01@ABV01@@Z$0 1000cbbf f i coordsarray.obj
 0001:0000da32       __catch$??$getline@DU?$char_traits@D@std@@V?$allocator@D@2@@std@@YAAAV?$basic_istream@DU?$char_traits@D@std@@@0@$$QAV10@AAV?$basic_string@DU?$char_traits@D@std@@V?$allocator@D@2@@0@D@Z$0 1000ea32 f i pdbio.obj
 0001:000110bc       __catch$??$_Uninit_copy@PAVAtomproperty@PTools@@PAV12@V?$allocator@VAtomproperty@PTools@@@std@@@std@@YAPAVAtomproperty@PTools@@PAV12@00AAU?$_Wrap_alloc@V?$allocator@VAtomproperty@PTools@@@std@@@0@U_Nonscalar_ptr_iterator_tag@0@@Z$0 100120bc f i rigidbody.obj
 0001:0001120c       __catch$??$_Uninit_move@PAVAtomproperty@PTools@@PAV12@V?$allocator@VAtomproperty@PTools@@@std@@V12@@std@@YAPAVAtomproperty@PTools@@PAV12@00AAU?$_Wrap_alloc@V?$allocator@VAtomproperty@PTools@@@std@@@0@0U_Nonscalar_ptr_iterator_tag@0@@Z$0 1001220c f i rigidbody.obj
 0001:00011bca       __catch$??4?$vector@VAtomproperty@PTools@@V?$allocator@VAtomproperty@PTools@@@std@@@std@@QAEAAV01@ABV01@@Z$0 10012bca f i rigidbody.obj
 0001:00013540       __catch$?_Reallocate@?$vector@UCoord3D@PTools@@V?$allocator@UCoord3D@PTools@@@std@@@std@@IAEXI@Z$0 10014540 f i rigidbody.obj
 0001:0001364f       __catch$?_Reallocate@?$vector@VAtomproperty@PTools@@V?$allocator@VAtomproperty@PTools@@@std@@@std@@IAEXI@Z$0 1001464f f i rigidbody.obj
 0001:00014274       __catch$??$_Uninit_fill_n@PAV?$vector@NV?$allocator@N@std@@@std@@IV12@V?$allocator@V?$vector@NV?$allocator@N@std@@@std@@@2@V12@@std@@YAXPAV?$vector@NV?$allocator@N@std@@@0@IPBV10@AAU?$_Wrap_alloc@V?$allocator@V?$vector@NV?$allocator@N@std@@@std@@@std@@@0@0U_Nonscalar_ptr_iterator_tag@0@@Z$0 10015274 f i superpose.obj
 0001:00014a10       ?MakeTensor@PTools@@YAXAAVRigidbody@1@0QAY02N@Z 10015a10 f   superpose.obj
 0001:00014d30       ?Mat33xMat33@PTools@@YAXQAY02N00@Z 10015d30 f   superpose.obj
 0001:00014e50       ?Mat33xcoord3D@PTools@@YAXQAY02NAAUCoord3D@1@1@Z 10015e50 f   superpose.obj
 0001:00015980       ?XRotMatrix@PTools@@YAXNQAY02N@Z 10016980 f   superpose.obj
 0001:000159f0       ?YRotMatrix@PTools@@YAXNQAY02N@Z 100169f0 f   superpose.obj
 0001:00015a60       ?ZRotMatrix@PTools@@YAXNQAY02N@Z 10016a60 f   superpose.obj
 0001:00015c29       __catch$?_Construct_n@?$vector@V?$vector@NV?$allocator@N@std@@@std@@V?$allocator@V?$vector@NV?$allocator@N@std@@@std@@@2@@std@@QAEXIPBV?$vector@NV?$allocator@N@std@@@2@@Z$0 10016c29 f i superpose.obj
 0001:00015fe0       ?rigidToMatrix@PTools@@YAXABVRigidbody@1@AAV?$vector@V?$vector@NV?$allocator@N@std@@@std@@V?$allocator@V?$vector@NV?$allocator@N@std@@@std@@@2@@std@@@Z 10016fe0 f   superpose.obj
 0001:0001788f       ?ArrayUnwindFilter@@YAHPAU_EXCEPTION_POINTERS@@@Z 1001888f f   MSVCRT:ehvecdtr.obj
 0001:00017906       _pre_c_init                10018906 f   MSVCRT:crtdll.obj
 0001:00017b73       ___DllMainCRTStartup       10018b73 f   MSVCRT:crtdll.obj
 0001:00017cc0       $$000000                   10018cc0     MSVCRT:sehprolg4.obj
 0001:00018340       __ehhandler$??0?$QList@H@@QAE@ABV0@@Z 10019340 f   PToolsAligner.obj
 0001:00018360       __ehhandler$??0?$QList@V?$QSharedDataPointer@VAtomData@U2@@@@@@QAE@ABV0@@Z 10019360 f   PToolsAligner.obj
 0001:00018380       __unwindfunclet$??0Atom@PTools@@QAE@VAtomproperty@1@UCoord3D@1@@Z$0 10019380 f   PToolsAligner.obj
 0001:00018388       __ehhandler$??0Atom@PTools@@QAE@VAtomproperty@1@UCoord3D@1@@Z 10019388 f   PToolsAligner.obj
 0001:000183b0       __unwindfunclet$??0Atomproperty@PTools@@QAE@ABV01@@Z$0 100193b0 f   PToolsAligner.obj
 0001:000183b8       __unwindfunclet$??0Atomproperty@PTools@@QAE@ABV01@@Z$1 100193b8 f   PToolsAligner.obj
 0001:000183c3       __unwindfunclet$??0Atomproperty@PTools@@QAE@ABV01@@Z$2 100193c3 f   PToolsAligner.obj
 0001:000183ce       __unwindfunclet$??0Atomproperty@PTools@@QAE@ABV01@@Z$3 100193ce f   PToolsAligner.obj
 0001:000183d9       __ehhandler$??0Atomproperty@PTools@@QAE@ABV01@@Z 100193d9 f   PToolsAligner.obj
 0001:00018400       __unwindfunclet$??0Atomproperty@PTools@@QAE@XZ$0 10019400 f   PToolsAligner.obj
 0001:00018408       __unwindfunclet$??0Atomproperty@PTools@@QAE@XZ$1 10019408 f   PToolsAligner.obj
 0001:00018413       __unwindfunclet$??0Atomproperty@PTools@@QAE@XZ$2 10019413 f   PToolsAligner.obj
 0001:0001841e       __unwindfunclet$??0Atomproperty@PTools@@QAE@XZ$3 1001941e f   PToolsAligner.obj
 0001:00018429       __unwindfunclet$??0Atomproperty@PTools@@QAE@XZ$4 10019429 f   PToolsAligner.obj
 0001:00018434       __ehhandler$??0Atomproperty@PTools@@QAE@XZ 10019434 f   PToolsAligner.obj
 0001:00018450       __unwindfunclet$??1Bond@U2@@QAE@XZ$0 10019450 f   PToolsAligner.obj
 0001:00018458       __ehhandler$??1Bond@U2@@QAE@XZ 10019458 f   PToolsAligner.obj
 0001:00018480       __unwindfunclet$??1Molecule3DModel@U2@@QAE@XZ$0 10019480 f   PToolsAligner.obj
 0001:00018488       __ehhandler$??1Molecule3DModel@U2@@QAE@XZ 10019488 f   PToolsAligner.obj
 0001:000184b0       __unwindfunclet$??1MoleculeData@U2@@QAE@XZ$0 100194b0 f   PToolsAligner.obj
 0001:000184bb       __unwindfunclet$??1MoleculeData@U2@@QAE@XZ$1 100194bb f   PToolsAligner.obj
 0001:000184c6       __ehhandler$??1MoleculeData@U2@@QAE@XZ 100194c6 f   PToolsAligner.obj
 0001:000184f0       __unwindfunclet$??__EalgoLog@U2@@YAXXZ$0 100194f0 f   PToolsAligner.obj
 0001:000184f9       __ehhandler$??__EalgoLog@U2@@YAXXZ 100194f9 f   PToolsAligner.obj
 0001:00018520       __unwindfunclet$??__EcmdLog@U2@@YAXXZ$0 10019520 f   PToolsAligner.obj
 0001:00018529       __ehhandler$??__EcmdLog@U2@@YAXXZ 10019529 f   PToolsAligner.obj
 0001:00018550       __unwindfunclet$??__EcoreLog@U2@@YAXXZ$0 10019550 f   PToolsAligner.obj
 0001:00018559       __ehhandler$??__EcoreLog@U2@@YAXXZ 10019559 f   PToolsAligner.obj
 0001:00018580       __unwindfunclet$??__EioLog@U2@@YAXXZ$0 10019580 f   PToolsAligner.obj
 0001:00018589       __ehhandler$??__EioLog@U2@@YAXXZ 10019589 f   PToolsAligner.obj
 0001:000185b0       __unwindfunclet$??__EperfLog@U2@@YAXXZ$0 100195b0 f   PToolsAligner.obj
 0001:000185b9       __ehhandler$??__EperfLog@U2@@YAXXZ 100195b9 f   PToolsAligner.obj
 0001:000185e0       __unwindfunclet$??__EscriptLog@U2@@YAXXZ$0 100195e0 f   PToolsAligner.obj
 0001:000185e9       __ehhandler$??__EscriptLog@U2@@YAXXZ 100195e9 f   PToolsAligner.obj
 0001:00018610       __unwindfunclet$??__EtaskLog@U2@@YAXXZ$0 10019610 f   PToolsAligner.obj
 0001:00018619       __ehhandler$??__EtaskLog@U2@@YAXXZ 10019619 f   PToolsAligner.obj
 0001:00018640       __unwindfunclet$??__EuiLog@U2@@YAXXZ$0 10019640 f   PToolsAligner.obj
 0001:00018649       __ehhandler$??__EuiLog@U2@@YAXXZ 10019649 f   PToolsAligner.obj
 0001:00018670       __unwindfunclet$??__EuserActLog@U2@@YAXXZ$0 10019670 f   PToolsAligner.obj
 0001:00018679       __ehhandler$??__EuserActLog@U2@@YAXXZ 10019679 f   PToolsAligner.obj
 0001:000186a0       __unwindfunclet$?SetType@Atomproperty@PTools@@QAEXV?$basic_string@DU?$char_traits@D@std@@V?$allocator@D@2@@std@@@Z$0 100196a0 f   PToolsAligner.obj
 0001:000186a8       __ehhandler$?SetType@Atomproperty@PTools@@QAEXV?$basic_string@DU?$char_traits@D@std@@V?$allocator@D@2@@std@@@Z 100196a8 f   PToolsAligner.obj
 0001:000186d0       __ehhandler$?_Copy@?$basic_string@DU?$char_traits@D@std@@V?$allocator@D@2@@std@@QAEXII@Z 100196d0 f   PToolsAligner.obj
 0001:000186f0       __unwindfunclet$?align@PToolsAligner@U2@@UAE?AVStructuralAlignment@2@ABVStructuralAlignmentTaskSettings@2@AAVTaskStateInfo@2@@Z$3 100196f0 f   PToolsAligner.obj
 0001:000186f9       __unwindfunclet$?align@PToolsAligner@U2@@UAE?AVStructuralAlignment@2@ABVStructuralAlignmentTaskSettings@2@AAVTaskStateInfo@2@@Z$4 100196f9 f   PToolsAligner.obj
 0001:00018702       __unwindfunclet$?align@PToolsAligner@U2@@UAE?AVStructuralAlignment@2@ABVStructuralAlignmentTaskSettings@2@AAVTaskStateInfo@2@@Z$5 10019702 f   PToolsAligner.obj
 0001:0001870b       __unwindfunclet$?align@PToolsAligner@U2@@UAE?AVStructuralAlignment@2@ABVStructuralAlignmentTaskSettings@2@AAVTaskStateInfo@2@@Z$6 1001970b f   PToolsAligner.obj
 0001:00018714       __unwindfunclet$?align@PToolsAligner@U2@@UAE?AVStructuralAlignment@2@ABVStructuralAlignmentTaskSettings@2@AAVTaskStateInfo@2@@Z$7 10019714 f   PToolsAligner.obj
 0001:0001871d       __unwindfunclet$?align@PToolsAligner@U2@@UAE?AVStructuralAlignment@2@ABVStructuralAlignmentTaskSettings@2@AAVTaskStateInfo@2@@Z$8 1001971d f   PToolsAligner.obj
 0001:00018737       __unwindfunclet$?align@PToolsAligner@U2@@UAE?AVStructuralAlignment@2@ABVStructuralAlignmentTaskSettings@2@AAVTaskStateInfo@2@@Z$9 10019737 f   PToolsAligner.obj
 0001:0001873f       __unwindfunclet$?align@PToolsAligner@U2@@UAE?AVStructuralAlignment@2@ABVStructuralAlignmentTaskSettings@2@AAVTaskStateInfo@2@@Z$10 1001973f f   PToolsAligner.obj
 0001:00018747       __unwindfunclet$?align@PToolsAligner@U2@@UAE?AVStructuralAlignment@2@ABVStructuralAlignmentTaskSettings@2@AAVTaskStateInfo@2@@Z$11 10019747 f   PToolsAligner.obj
 0001:00018750       __unwindfunclet$?align@PToolsAligner@U2@@UAE?AVStructuralAlignment@2@ABVStructuralAlignmentTaskSettings@2@AAVTaskStateInfo@2@@Z$12 10019750 f   PToolsAligner.obj
 0001:00018758       __unwindfunclet$?align@PToolsAligner@U2@@UAE?AVStructuralAlignment@2@ABVStructuralAlignmentTaskSettings@2@AAVTaskStateInfo@2@@Z$13 10019758 f   PToolsAligner.obj
 0001:00018761       __unwindfunclet$?align@PToolsAligner@U2@@UAE?AVStructuralAlignment@2@ABVStructuralAlignmentTaskSettings@2@AAVTaskStateInfo@2@@Z$14 10019761 f   PToolsAligner.obj
 0001:0001876a       __unwindfunclet$?align@PToolsAligner@U2@@UAE?AVStructuralAlignment@2@ABVStructuralAlignmentTaskSettings@2@AAVTaskStateInfo@2@@Z$15 1001976a f   PToolsAligner.obj
 0001:00018773       __unwindfunclet$?align@PToolsAligner@U2@@UAE?AVStructuralAlignment@2@ABVStructuralAlignmentTaskSettings@2@AAVTaskStateInfo@2@@Z$16 10019773 f   PToolsAligner.obj
 0001:0001877c       __ehhandler$?align@PToolsAligner@U2@@UAE?AVStructuralAlignment@2@ABVStructuralAlignmentTaskSettings@2@AAVTaskStateInfo@2@@Z 1001977c f   PToolsAligner.obj
 0001:000187a0       __unwindfunclet$?createRigidBody@U2@@YAPAVRigidbody@PTools@@ABVBioStruct3DReference@1@@Z$0 100197a0 f   PToolsAligner.obj
 0001:000187ae       __unwindfunclet$?createRigidBody@U2@@YAPAVRigidbody@PTools@@ABVBioStruct3DReference@1@@Z$1 100197ae f   PToolsAligner.obj
 0001:000187b9       __unwindfunclet$?createRigidBody@U2@@YAPAVRigidbody@PTools@@ABVBioStruct3DReference@1@@Z$2 100197b9 f   PToolsAligner.obj
 0001:000187c4       __unwindfunclet$?createRigidBody@U2@@YAPAVRigidbody@PTools@@ABVBioStruct3DReference@1@@Z$3 100197c4 f   PToolsAligner.obj
 0001:000187cf       __unwindfunclet$?createRigidBody@U2@@YAPAVRigidbody@PTools@@ABVBioStruct3DReference@1@@Z$5 100197cf f   PToolsAligner.obj
 0001:000187da       __unwindfunclet$?createRigidBody@U2@@YAPAVRigidbody@PTools@@ABVBioStruct3DReference@1@@Z$6 100197da f   PToolsAligner.obj
 0001:000187e5       __unwindfunclet$?createRigidBody@U2@@YAPAVRigidbody@PTools@@ABVBioStruct3DReference@1@@Z$12 100197e5 f   PToolsAligner.obj
 0001:000187f0       __unwindfunclet$?createRigidBody@U2@@YAPAVRigidbody@PTools@@ABVBioStruct3DReference@1@@Z$13 100197f0 f   PToolsAligner.obj
 0001:000187fb       __unwindfunclet$?createRigidBody@U2@@YAPAVRigidbody@PTools@@ABVBioStruct3DReference@1@@Z$9 100197fb f   PToolsAligner.obj
 0001:00018806       __ehhandler$?createRigidBody@U2@@YAPAVRigidbody@PTools@@ABVBioStruct3DReference@1@@Z 10019806 f   PToolsAligner.obj
 0001:00018830       __unwindfunclet$?getSubsetSize@U2@@YAHABVBioStruct3DReference@1@@Z$0 10019830 f   PToolsAligner.obj
 0001:00018838       __unwindfunclet$?getSubsetSize@U2@@YAHABVBioStruct3DReference@1@@Z$1 10019838 f   PToolsAligner.obj
 0001:00018840       __ehhandler$?getSubsetSize@U2@@YAHABVBioStruct3DReference@1@@Z 10019840 f   PToolsAligner.obj
 0001:00018860       __unwindfunclet$?node_destruct@?$QList@VBond@U2@@@@AAEXPAUNode@1@0@Z$0 10019860 f   PToolsAligner.obj
 0001:00018868       __ehhandler$?node_destruct@?$QList@VBond@U2@@@@AAEXPAUNode@1@0@Z 10019868 f   PToolsAligner.obj
 0001:00018890       __ehhandler$?reallocData@?$QVector@N@@AAEXHHV?$QFlags@W4AllocationOption@QArrayData@@@@@Z 10019890 f   PToolsAligner.obj
 0001:000188b0       __ehhandler$??0?$QList@PAVXMLTestFactory@U2@@@@QAE@ABV0@@Z 100198b0 f   PToolsPlugin.obj
 0001:000188d0       __unwindfunclet$??0Gtest_PToolsAlignerTask@U2@@QAE@PAVXMLTestFormat@1@ABVQString@@PAVGTest@1@PBVGTestEnvironment@1@ABV?$QList@PAVGTest@U2@@@@ABVQDomElement@@@Z$0 100198d0 f   PToolsPlugin.obj
 0001:000188d9       __unwindfunclet$??0Gtest_PToolsAlignerTask@U2@@QAE@PAVXMLTestFormat@1@ABVQString@@PAVGTest@1@PBVGTestEnvironment@1@ABV?$QList@PAVGTest@U2@@@@ABVQDomElement@@@Z$1 100198d9 f   PToolsPlugin.obj
 0001:000188e8       __unwindfunclet$??0Gtest_PToolsAlignerTask@U2@@QAE@PAVXMLTestFormat@1@ABVQString@@PAVGTest@1@PBVGTestEnvironment@1@ABV?$QList@PAVGTest@U2@@@@ABVQDomElement@@@Z$2 100198e8 f   PToolsPlugin.obj
 0001:000188f7       __unwindfunclet$??0Gtest_PToolsAlignerTask@U2@@QAE@PAVXMLTestFormat@1@ABVQString@@PAVGTest@1@PBVGTestEnvironment@1@ABV?$QList@PAVGTest@U2@@@@ABVQDomElement@@@Z$3 100198f7 f   PToolsPlugin.obj
 0001:00018906       __unwindfunclet$??0Gtest_PToolsAlignerTask@U2@@QAE@PAVXMLTestFormat@1@ABVQString@@PAVGTest@1@PBVGTestEnvironment@1@ABV?$QList@PAVGTest@U2@@@@ABVQDomElement@@@Z$4 10019906 f   PToolsPlugin.obj
 0001:00018915       __ehhandler$??0Gtest_PToolsAlignerTask@U2@@QAE@PAVXMLTestFormat@1@ABVQString@@PAVGTest@1@PBVGTestEnvironment@1@ABV?$QList@PAVGTest@U2@@@@ABVQDomElement@@@Z 10019915 f   PToolsPlugin.obj
 0001:00018930       __unwindfunclet$??0Gtest_PToolsAlignerTaskFactory@Gtest_PToolsAlignerTask@U2@@QAE@XZ$0 10019930 f   PToolsPlugin.obj
 0001:00018939       __unwindfunclet$??0Gtest_PToolsAlignerTaskFactory@Gtest_PToolsAlignerTask@U2@@QAE@XZ$1 10019939 f   PToolsPlugin.obj
 0001:00018942       __ehhandler$??0Gtest_PToolsAlignerTaskFactory@Gtest_PToolsAlignerTask@U2@@QAE@XZ 10019942 f   PToolsPlugin.obj
 0001:00018960       __unwindfunclet$??0PToolsPlugin@U2@@QAE@XZ$0 10019960 f   PToolsPlugin.obj
 0001:00018969       __unwindfunclet$??0PToolsPlugin@U2@@QAE@XZ$1 10019969 f   PToolsPlugin.obj
 0001:00018972       __unwindfunclet$??0PToolsPlugin@U2@@QAE@XZ$2 10019972 f   PToolsPlugin.obj
 0001:0001897b       __unwindfunclet$??0PToolsPlugin@U2@@QAE@XZ$3 1001997b f   PToolsPlugin.obj
 0001:00018984       __unwindfunclet$??0PToolsPlugin@U2@@QAE@XZ$4 10019984 f   PToolsPlugin.obj
 0001:0001898f       __unwindfunclet$??0PToolsPlugin@U2@@QAE@XZ$6 1001998f f   PToolsPlugin.obj
 0001:00018997       __ehhandler$??0PToolsPlugin@U2@@QAE@XZ 10019997 f   PToolsPlugin.obj
 0001:000189c0       __unwindfunclet$??1?$GAutoDeleteList@VXMLTestFactory@U2@@@U2@@UAE@XZ$0 100199c0 f   PToolsPlugin.obj
 0001:000189c9       __unwindfunclet$??1?$GAutoDeleteList@VXMLTestFactory@U2@@@U2@@UAE@XZ$1 100199c9 f   PToolsPlugin.obj
 0001:000189d4       __ehhandler$??1?$GAutoDeleteList@VXMLTestFactory@U2@@@U2@@UAE@XZ 100199d4 f   PToolsPlugin.obj
 0001:000189f0       __unwindfunclet$??1Gtest_PToolsAlignerTask@U2@@UAE@XZ$0 100199f0 f   PToolsPlugin.obj
 0001:000189f9       __unwindfunclet$??1Gtest_PToolsAlignerTask@U2@@UAE@XZ$1 100199f9 f   PToolsPlugin.obj
 0001:00018a08       __unwindfunclet$??1Gtest_PToolsAlignerTask@U2@@UAE@XZ$2 10019a08 f   PToolsPlugin.obj
 0001:00018a17       __unwindfunclet$??1Gtest_PToolsAlignerTask@U2@@UAE@XZ$3 10019a17 f   PToolsPlugin.obj
 0001:00018a26       __ehhandler$??1Gtest_PToolsAlignerTask@U2@@UAE@XZ 10019a26 f   PToolsPlugin.obj
 0001:00018a50       __unwindfunclet$??_GGtest_PToolsAlignerTask@U2@@UAEPAXI@Z$0 10019a50 f   PToolsPlugin.obj
 0001:00018a59       __unwindfunclet$??_GGtest_PToolsAlignerTask@U2@@UAEPAXI@Z$1 10019a59 f   PToolsPlugin.obj
 0001:00018a68       __unwindfunclet$??_GGtest_PToolsAlignerTask@U2@@UAEPAXI@Z$2 10019a68 f   PToolsPlugin.obj
 0001:00018a77       __unwindfunclet$??_GGtest_PToolsAlignerTask@U2@@UAEPAXI@Z$3 10019a77 f   PToolsPlugin.obj
 0001:00018a86       __ehhandler$??_GGtest_PToolsAlignerTask@U2@@UAEPAXI@Z 10019a86 f   PToolsPlugin.obj
 0001:00018ab0       __unwindfunclet$??__EalgoLog@U2@@YAXXZ$0 10019ab0 f   PToolsPlugin.obj
 0001:00018ab9       __ehhandler$??__EalgoLog@U2@@YAXXZ 10019ab9 f   PToolsPlugin.obj
 0001:00018ae0       __unwindfunclet$??__EcmdLog@U2@@YAXXZ$0 10019ae0 f   PToolsPlugin.obj
 0001:00018ae9       __ehhandler$??__EcmdLog@U2@@YAXXZ 10019ae9 f   PToolsPlugin.obj
 0001:00018b10       __unwindfunclet$??__EcoreLog@U2@@YAXXZ$0 10019b10 f   PToolsPlugin.obj
 0001:00018b19       __ehhandler$??__EcoreLog@U2@@YAXXZ 10019b19 f   PToolsPlugin.obj
 0001:00018b40       __unwindfunclet$??__EioLog@U2@@YAXXZ$0 10019b40 f   PToolsPlugin.obj
 0001:00018b49       __ehhandler$??__EioLog@U2@@YAXXZ 10019b49 f   PToolsPlugin.obj
 0001:00018b70       __unwindfunclet$??__EperfLog@U2@@YAXXZ$0 10019b70 f   PToolsPlugin.obj
 0001:00018b79       __ehhandler$??__EperfLog@U2@@YAXXZ 10019b79 f   PToolsPlugin.obj
 0001:00018ba0       __unwindfunclet$??__EscriptLog@U2@@YAXXZ$0 10019ba0 f   PToolsPlugin.obj
 0001:00018ba9       __ehhandler$??__EscriptLog@U2@@YAXXZ 10019ba9 f   PToolsPlugin.obj
 0001:00018bd0       __unwindfunclet$??__EtaskLog@U2@@YAXXZ$0 10019bd0 f   PToolsPlugin.obj
 0001:00018bd9       __ehhandler$??__EtaskLog@U2@@YAXXZ 10019bd9 f   PToolsPlugin.obj
 0001:00018c00       __unwindfunclet$??__EuiLog@U2@@YAXXZ$0 10019c00 f   PToolsPlugin.obj
 0001:00018c09       __ehhandler$??__EuiLog@U2@@YAXXZ 10019c09 f   PToolsPlugin.obj
 0001:00018c30       __unwindfunclet$??__EuserActLog@U2@@YAXXZ$0 10019c30 f   PToolsPlugin.obj
 0001:00018c39       __ehhandler$??__EuserActLog@U2@@YAXXZ 10019c39 f   PToolsPlugin.obj
 0001:00018c60       __ehhandler$?append@?$QList@PAVXMLTestFactory@U2@@@@QAEXABQAVXMLTestFactory@U2@@@Z 10019c60 f   PToolsPlugin.obj
 0001:00018c80       __unwindfunclet$?createFactory@Gtest_PToolsAlignerTask@U2@@SAPAVXMLTestFactory@2@XZ$0 10019c80 f   PToolsPlugin.obj
 0001:00018c8b       __unwindfunclet$?createFactory@Gtest_PToolsAlignerTask@U2@@SAPAVXMLTestFactory@2@XZ$1 10019c8b f   PToolsPlugin.obj
 0001:00018c94       __unwindfunclet$?createFactory@Gtest_PToolsAlignerTask@U2@@SAPAVXMLTestFactory@2@XZ$2 10019c94 f   PToolsPlugin.obj
 0001:00018c9d       __ehhandler$?createFactory@Gtest_PToolsAlignerTask@U2@@SAPAVXMLTestFactory@2@XZ 10019c9d f   PToolsPlugin.obj
 0001:00018cc0       __unwindfunclet$?createTest@Gtest_PToolsAlignerTaskFactory@Gtest_PToolsAlignerTask@U2@@UAEPAVGTest@3@PAVXMLTestFormat@3@ABVQString@@PAV43@PBVGTestEnvironment@3@ABV?$QList@PAVGTest@U2@@@@ABVQDomElement@@@Z$0 10019cc0 f   PToolsPlugin.obj
 0001:00018ccb       __ehhandler$?createTest@Gtest_PToolsAlignerTaskFactory@Gtest_PToolsAlignerTask@U2@@UAEPAVGTest@3@PAVXMLTestFormat@3@ABVQString@@PAV43@PBVGTestEnvironment@3@ABV?$QList@PAVGTest@U2@@@@ABVQDomElement@@@Z 10019ccb f   PToolsPlugin.obj
 0001:00018cf0       __unwindfunclet$?createTestFactories@StructualAlignerTests@U2@@SA?AV?$QList@PAVXMLTestFactory@U2@@@@XZ$0 10019cf0 f   PToolsPlugin.obj
 0001:00018d09       __ehhandler$?createTestFactories@StructualAlignerTests@U2@@SA?AV?$QList@PAVXMLTestFactory@U2@@@@XZ 10019d09 f   PToolsPlugin.obj
 0001:00018d30       __ehhandler$?detach_helper_grow@?$QList@PAVXMLTestFactory@U2@@@@AAEPAUNode@1@HH@Z 10019d30 f   PToolsPlugin.obj
 0001:00018d50       __ehhandler$??0?$QList@VQString@@@@QAE@ABV0@@Z 10019d50 f   PToolsTests.obj
 0001:00018d70       __unwindfunclet$??H@YA?BVQString@@ABV0@0@Z$0 10019d70 f   PToolsTests.obj
 0001:00018d8a       __ehhandler$??H@YA?BVQString@@ABV0@0@Z 10019d8a f   PToolsTests.obj
 0001:00018db0       __unwindfunclet$??H@YA?BVQString@@ABV0@PBD@Z$0 10019db0 f   PToolsTests.obj
 0001:00018dca       __unwindfunclet$??H@YA?BVQString@@ABV0@PBD@Z$1 10019dca f   PToolsTests.obj
 0001:00018dd3       __ehhandler$??H@YA?BVQString@@ABV0@PBD@Z 10019dd3 f   PToolsTests.obj
 0001:00018df0       __unwindfunclet$??H@YA?BVQString@@PBDABV0@@Z$0 10019df0 f   PToolsTests.obj
 0001:00018e0a       __ehhandler$??H@YA?BVQString@@PBDABV0@@Z 10019e0a f   PToolsTests.obj
 0001:00018e30       __unwindfunclet$??__EalgoLog@U2@@YAXXZ$0 10019e30 f   PToolsTests.obj
 0001:00018e39       __ehhandler$??__EalgoLog@U2@@YAXXZ 10019e39 f   PToolsTests.obj
 0001:00018e60       __unwindfunclet$??__EcmdLog@U2@@YAXXZ$0 10019e60 f   PToolsTests.obj
 0001:00018e69       __ehhandler$??__EcmdLog@U2@@YAXXZ 10019e69 f   PToolsTests.obj
 0001:00018e90       __unwindfunclet$??__EcoreLog@U2@@YAXXZ$0 10019e90 f   PToolsTests.obj
 0001:00018e99       __ehhandler$??__EcoreLog@U2@@YAXXZ 10019e99 f   PToolsTests.obj
 0001:00018ec0       __unwindfunclet$??__EioLog@U2@@YAXXZ$0 10019ec0 f   PToolsTests.obj
 0001:00018ec9       __ehhandler$??__EioLog@U2@@YAXXZ 10019ec9 f   PToolsTests.obj
 0001:00018ef0       __unwindfunclet$??__EperfLog@U2@@YAXXZ$0 10019ef0 f   PToolsTests.obj
 0001:00018ef9       __ehhandler$??__EperfLog@U2@@YAXXZ 10019ef9 f   PToolsTests.obj
 0001:00018f20       __unwindfunclet$??__EscriptLog@U2@@YAXXZ$0 10019f20 f   PToolsTests.obj
 0001:00018f29       __ehhandler$??__EscriptLog@U2@@YAXXZ 10019f29 f   PToolsTests.obj
 0001:00018f50       __unwindfunclet$??__EtaskLog@U2@@YAXXZ$0 10019f50 f   PToolsTests.obj
 0001:00018f59       __ehhandler$??__EtaskLog@U2@@YAXXZ 10019f59 f   PToolsTests.obj
 0001:00018f80       __unwindfunclet$??__EuiLog@U2@@YAXXZ$0 10019f80 f   PToolsTests.obj
 0001:00018f89       __ehhandler$??__EuiLog@U2@@YAXXZ 10019f89 f   PToolsTests.obj
 0001:00018fb0       __unwindfunclet$??__EuserActLog@U2@@YAXXZ$0 10019fb0 f   PToolsTests.obj
 0001:00018fb9       __ehhandler$??__EuserActLog@U2@@YAXXZ 10019fb9 f   PToolsTests.obj
 0001:00018fe0       __unwindfunclet$?alignmentToStr@U2@@YA?AVQString@@ABVStructuralAlignment@1@N@Z$0 10019fe0 f   PToolsTests.obj
 0001:00018fe9       __unwindfunclet$?alignmentToStr@U2@@YA?AVQString@@ABVStructuralAlignment@1@N@Z$1 10019fe9 f   PToolsTests.obj
 0001:00018ff2       __unwindfunclet$?alignmentToStr@U2@@YA?AVQString@@ABVStructuralAlignment@1@N@Z$2 10019ff2 f   PToolsTests.obj
 0001:0001900c       __unwindfunclet$?alignmentToStr@U2@@YA?AVQString@@ABVStructuralAlignment@1@N@Z$3 1001a00c f   PToolsTests.obj
 0001:00019015       __unwindfunclet$?alignmentToStr@U2@@YA?AVQString@@ABVStructuralAlignment@1@N@Z$4 1001a015 f   PToolsTests.obj
 0001:0001901e       __ehhandler$?alignmentToStr@U2@@YA?AVQString@@ABVStructuralAlignment@1@N@Z 1001a01e f   PToolsTests.obj
 0001:00019040       __ehhandler$?append@?$QList@H@@QAEXABH@Z 1001a040 f   PToolsTests.obj
 0001:00019060       __ehhandler$?detach_helper@?$QList@H@@AAEXH@Z 1001a060 f   PToolsTests.obj
 0001:00019080       __ehhandler$?detach_helper_grow@?$QList@H@@AAEPAUNode@1@HH@Z 1001a080 f   PToolsTests.obj
 0001:000190a0       __unwindfunclet$?init@Gtest_PToolsAlignerTask@U2@@QAEXPAVXMLTestFormat@2@ABVQDomElement@@@Z$0 1001a0a0 f   PToolsTests.obj
 0001:000190a9       __unwindfunclet$?init@Gtest_PToolsAlignerTask@U2@@QAEXPAVXMLTestFormat@2@ABVQDomElement@@@Z$1 1001a0a9 f   PToolsTests.obj
 0001:000190b2       __unwindfunclet$?init@Gtest_PToolsAlignerTask@U2@@QAEXPAVXMLTestFormat@2@ABVQDomElement@@@Z$2 1001a0b2 f   PToolsTests.obj
 0001:000190bb       __unwindfunclet$?init@Gtest_PToolsAlignerTask@U2@@QAEXPAVXMLTestFormat@2@ABVQDomElement@@@Z$3 1001a0bb f   PToolsTests.obj
 0001:000190c4       __unwindfunclet$?init@Gtest_PToolsAlignerTask@U2@@QAEXPAVXMLTestFormat@2@ABVQDomElement@@@Z$4 1001a0c4 f   PToolsTests.obj
 0001:000190cd       __unwindfunclet$?init@Gtest_PToolsAlignerTask@U2@@QAEXPAVXMLTestFormat@2@ABVQDomElement@@@Z$5 1001a0cd f   PToolsTests.obj
 0001:000190d6       __unwindfunclet$?init@Gtest_PToolsAlignerTask@U2@@QAEXPAVXMLTestFormat@2@ABVQDomElement@@@Z$6 1001a0d6 f   PToolsTests.obj
 0001:000190df       __unwindfunclet$?init@Gtest_PToolsAlignerTask@U2@@QAEXPAVXMLTestFormat@2@ABVQDomElement@@@Z$7 1001a0df f   PToolsTests.obj
 0001:000190e8       __unwindfunclet$?init@Gtest_PToolsAlignerTask@U2@@QAEXPAVXMLTestFormat@2@ABVQDomElement@@@Z$8 1001a0e8 f   PToolsTests.obj
 0001:000190f1       __unwindfunclet$?init@Gtest_PToolsAlignerTask@U2@@QAEXPAVXMLTestFormat@2@ABVQDomElement@@@Z$9 1001a0f1 f   PToolsTests.obj
 0001:000190fa       __unwindfunclet$?init@Gtest_PToolsAlignerTask@U2@@QAEXPAVXMLTestFormat@2@ABVQDomElement@@@Z$10 1001a0fa f   PToolsTests.obj
 0001:00019103       __unwindfunclet$?init@Gtest_PToolsAlignerTask@U2@@QAEXPAVXMLTestFormat@2@ABVQDomElement@@@Z$11 1001a103 f   PToolsTests.obj
 0001:0001910c       __unwindfunclet$?init@Gtest_PToolsAlignerTask@U2@@QAEXPAVXMLTestFormat@2@ABVQDomElement@@@Z$12 1001a10c f   PToolsTests.obj
 0001:00019115       __unwindfunclet$?init@Gtest_PToolsAlignerTask@U2@@QAEXPAVXMLTestFormat@2@ABVQDomElement@@@Z$13 1001a115 f   PToolsTests.obj
 0001:0001911e       __unwindfunclet$?init@Gtest_PToolsAlignerTask@U2@@QAEXPAVXMLTestFormat@2@ABVQDomElement@@@Z$14 1001a11e f   PToolsTests.obj
 0001:00019127       __unwindfunclet$?init@Gtest_PToolsAlignerTask@U2@@QAEXPAVXMLTestFormat@2@ABVQDomElement@@@Z$15 1001a127 f   PToolsTests.obj
 0001:0001912f       __unwindfunclet$?init@Gtest_PToolsAlignerTask@U2@@QAEXPAVXMLTestFormat@2@ABVQDomElement@@@Z$16 1001a12f f   PToolsTests.obj
 0001:00019138       __unwindfunclet$?init@Gtest_PToolsAlignerTask@U2@@QAEXPAVXMLTestFormat@2@ABVQDomElement@@@Z$17 1001a138 f   PToolsTests.obj
 0001:00019141       __unwindfunclet$?init@Gtest_PToolsAlignerTask@U2@@QAEXPAVXMLTestFormat@2@ABVQDomElement@@@Z$18 1001a141 f   PToolsTests.obj
 0001:00019149       __unwindfunclet$?init@Gtest_PToolsAlignerTask@U2@@QAEXPAVXMLTestFormat@2@ABVQDomElement@@@Z$19 1001a149 f   PToolsTests.obj
 0001:00019152       __unwindfunclet$?init@Gtest_PToolsAlignerTask@U2@@QAEXPAVXMLTestFormat@2@ABVQDomElement@@@Z$20 1001a152 f   PToolsTests.obj
 0001:0001915b       __unwindfunclet$?init@Gtest_PToolsAlignerTask@U2@@QAEXPAVXMLTestFormat@2@ABVQDomElement@@@Z$21 1001a15b f   PToolsTests.obj
 0001:00019164       __ehhandler$?init@Gtest_PToolsAlignerTask@U2@@QAEXPAVXMLTestFormat@2@ABVQDomElement@@@Z 1001a164 f   PToolsTests.obj
 0001:00019180       __unwindfunclet$?keys@?$QMap@HV?$QHash@HV?$QSharedDataPointer@VAtomData@U2@@@@@@@@QBE?AV?$QList@H@@XZ$0 1001a180 f   PToolsTests.obj
 0001:00019199       __ehhandler$?keys@?$QMap@HV?$QHash@HV?$QSharedDataPointer@VAtomData@U2@@@@@@@@QBE?AV?$QList@H@@XZ 1001a199 f   PToolsTests.obj
 0001:000191c0       __unwindfunclet$?keys@?$QMap@HV?$QSharedDataPointer@VMoleculeData@U2@@@@@@QBE?AV?$QList@H@@XZ$0 1001a1c0 f   PToolsTests.obj
 0001:000191d9       __ehhandler$?keys@?$QMap@HV?$QSharedDataPointer@VMoleculeData@U2@@@@@@QBE?AV?$QList@H@@XZ 1001a1d9 f   PToolsTests.obj
 0001:00019200       __unwindfunclet$?node_copy@?$QList@VQString@@@@AAEXPAUNode@1@00@Z$5 1001a200 f   PToolsTests.obj
 0001:00019211       __ehhandler$?node_copy@?$QList@VQString@@@@AAEXPAUNode@1@00@Z 1001a211 f   PToolsTests.obj
 0001:00019230       __unwindfunclet$?report@Gtest_PToolsAlignerTask@U2@@UAE?AW4ReportResult@Task@2@XZ$0 1001a230 f   PToolsTests.obj
 0001:00019239       __unwindfunclet$?report@Gtest_PToolsAlignerTask@U2@@UAE?AW4ReportResult@Task@2@XZ$1 1001a239 f   PToolsTests.obj
 0001:00019242       __unwindfunclet$?report@Gtest_PToolsAlignerTask@U2@@UAE?AW4ReportResult@Task@2@XZ$2 1001a242 f   PToolsTests.obj
 0001:0001924b       __unwindfunclet$?report@Gtest_PToolsAlignerTask@U2@@UAE?AW4ReportResult@Task@2@XZ$3 1001a24b f   PToolsTests.obj
 0001:00019254       __unwindfunclet$?report@Gtest_PToolsAlignerTask@U2@@UAE?AW4ReportResult@Task@2@XZ$4 1001a254 f   PToolsTests.obj
 0001:0001925d       __unwindfunclet$?report@Gtest_PToolsAlignerTask@U2@@UAE?AW4ReportResult@Task@2@XZ$5 1001a25d f   PToolsTests.obj
 0001:00019266       __ehhandler$?report@Gtest_PToolsAlignerTask@U2@@UAE?AW4ReportResult@Task@2@XZ 1001a266 f   PToolsTests.obj
 0001:00019290       __unwindfunclet$?run@Gtest_PToolsAlignerTask@U2@@UAEXXZ$4 1001a290 f   PToolsTests.obj
 0001:00019298       __unwindfunclet$?run@Gtest_PToolsAlignerTask@U2@@UAEXXZ$5 1001a298 f   PToolsTests.obj
 0001:000192a0       __unwindfunclet$?run@Gtest_PToolsAlignerTask@U2@@UAEXXZ$6 1001a2a0 f   PToolsTests.obj
 0001:000192a9       __unwindfunclet$?run@Gtest_PToolsAlignerTask@U2@@UAEXXZ$7 1001a2a9 f   PToolsTests.obj
 0001:000192b1       __unwindfunclet$?run@Gtest_PToolsAlignerTask@U2@@UAEXXZ$8 1001a2b1 f   PToolsTests.obj
 0001:000192b9       __unwindfunclet$?run@Gtest_PToolsAlignerTask@U2@@UAEXXZ$9 1001a2b9 f   PToolsTests.obj
 0001:000192c2       __unwindfunclet$?run@Gtest_PToolsAlignerTask@U2@@UAEXXZ$10 1001a2c2 f   PToolsTests.obj
 0001:000192ce       __unwindfunclet$?run@Gtest_PToolsAlignerTask@U2@@UAEXXZ$11 1001a2ce f   PToolsTests.obj
 0001:000192d6       __unwindfunclet$?run@Gtest_PToolsAlignerTask@U2@@UAEXXZ$12 1001a2d6 f   PToolsTests.obj
 0001:000192df       __unwindfunclet$?run@Gtest_PToolsAlignerTask@U2@@UAEXXZ$0 1001a2df f   PToolsTests.obj
 0001:000192e8       __unwindfunclet$?run@Gtest_PToolsAlignerTask@U2@@UAEXXZ$1 1001a2e8 f   PToolsTests.obj
 0001:000192f1       __unwindfunclet$?run@Gtest_PToolsAlignerTask@U2@@UAEXXZ$2 1001a2f1 f   PToolsTests.obj
 0001:000192fa       __unwindfunclet$?run@Gtest_PToolsAlignerTask@U2@@UAEXXZ$3 1001a2fa f   PToolsTests.obj
 0001:00019303       __ehhandler$?run@Gtest_PToolsAlignerTask@U2@@UAEXXZ 1001a303 f   PToolsTests.obj
 0001:00019330       __unwindfunclet$??0AtomSelection@PTools@@QAE@ABV01@@Z$0 1001a330 f   atomselection.obj
 0001:0001933b       __ehhandler$??0AtomSelection@PTools@@QAE@ABV01@@Z 1001a33b f   atomselection.obj
 0001:00019360       __unwindfunclet$??0AtomSelection@PTools@@QAE@ABVRigidbody@1@@Z$0 1001a360 f   atomselection.obj
 0001:0001936b       __ehhandler$??0AtomSelection@PTools@@QAE@ABVRigidbody@1@@Z 1001a36b f   atomselection.obj
 0001:00019390       __unwindfunclet$??7PTools@@YA?AVAtomSelection@0@ABV10@@Z$0 1001a390 f   atomselection.obj
 0001:000193a9       __unwindfunclet$??7PTools@@YA?AVAtomSelection@0@ABV10@@Z$1 1001a3a9 f   atomselection.obj
 0001:000193b1       __ehhandler$??7PTools@@YA?AVAtomSelection@0@ABV10@@Z 1001a3b1 f   atomselection.obj
 0001:000193d0       __unwindfunclet$??IPTools@@YA?AVAtomSelection@0@ABV10@0@Z$0 1001a3d0 f   atomselection.obj
 0001:000193d8       __unwindfunclet$??IPTools@@YA?AVAtomSelection@0@ABV10@0@Z$2 1001a3d8 f   atomselection.obj
 0001:000193e3       __unwindfunclet$??IPTools@@YA?AVAtomSelection@0@ABV10@0@Z$3 1001a3e3 f   atomselection.obj
 0001:000193ee       __ehhandler$??IPTools@@YA?AVAtomSelection@0@ABV10@0@Z 1001a3ee f   atomselection.obj
 0001:00019410       __unwindfunclet$??UPTools@@YA?AVAtomSelection@0@ABV10@0@Z$0 1001a410 f   atomselection.obj
 0001:00019418       __unwindfunclet$??UPTools@@YA?AVAtomSelection@0@ABV10@0@Z$5 1001a418 f   atomselection.obj
 0001:00019420       __unwindfunclet$??UPTools@@YA?AVAtomSelection@0@ABV10@0@Z$1 1001a420 f   atomselection.obj
 0001:00019428       __unwindfunclet$??UPTools@@YA?AVAtomSelection@0@ABV10@0@Z$6 1001a428 f   atomselection.obj
 0001:00019430       __unwindfunclet$??UPTools@@YA?AVAtomSelection@0@ABV10@0@Z$2 1001a430 f   atomselection.obj
 0001:00019438       __unwindfunclet$??UPTools@@YA?AVAtomSelection@0@ABV10@0@Z$7 1001a438 f   atomselection.obj
 0001:00019443       __unwindfunclet$??UPTools@@YA?AVAtomSelection@0@ABV10@0@Z$4 1001a443 f   atomselection.obj
 0001:0001944b       __unwindfunclet$??UPTools@@YA?AVAtomSelection@0@ABV10@0@Z$8 1001a44b f   atomselection.obj
 0001:00019456       __ehhandler$??UPTools@@YA?AVAtomSelection@0@ABV10@0@Z 1001a456 f   atomselection.obj
 0001:00019480       __unwindfunclet$?CreateRigid@AtomSelection@PTools@@QAE?AVRigidbody@2@XZ$0 1001a480 f   atomselection.obj
 0001:000194a2       __unwindfunclet$?CreateRigid@AtomSelection@PTools@@QAE?AVRigidbody@2@XZ$1 1001a4a2 f   atomselection.obj
 0001:000194ad       __ehhandler$?CreateRigid@AtomSelection@PTools@@QAE?AVRigidbody@2@XZ 1001a4ad f   atomselection.obj
 0001:000194e0       __unwindfunclet$??$?6U?$char_traits@D@std@@@std@@YAAAV?$basic_ostream@DU?$char_traits@D@std@@@0@AAV10@PBD@Z$3 1001a4e0 f   coord3d.obj
 0001:000194e8       __unwindfunclet$??$?6U?$char_traits@D@std@@@std@@YAAAV?$basic_ostream@DU?$char_traits@D@std@@@0@AAV10@PBD@Z$2 1001a4e8 f   coord3d.obj
 0001:000194f0       __ehhandler$??$?6U?$char_traits@D@std@@@std@@YAAAV?$basic_ostream@DU?$char_traits@D@std@@@0@AAV10@PBD@Z 1001a4f0 f   coord3d.obj
 0001:00019510       __unwindfunclet$??0?$basic_stringbuf@DU?$char_traits@D@std@@V?$allocator@D@2@@std@@QAE@H@Z$0 1001a510 f   coord3d.obj
 0001:00019519       __ehhandler$??0?$basic_stringbuf@DU?$char_traits@D@std@@V?$allocator@D@2@@std@@QAE@H@Z 1001a519 f   coord3d.obj
 0001:00019540       __unwindfunclet$??0?$basic_stringstream@DU?$char_traits@D@std@@V?$allocator@D@2@@std@@QAE@H@Z$0 1001a540 f   coord3d.obj
 0001:0001955d       __unwindfunclet$??0?$basic_stringstream@DU?$char_traits@D@std@@V?$allocator@D@2@@std@@QAE@H@Z$1 1001a55d f   coord3d.obj
 0001:00019569       __unwindfunclet$??0?$basic_stringstream@DU?$char_traits@D@std@@V?$allocator@D@2@@std@@QAE@H@Z$4 1001a569 f   coord3d.obj
 0001:00019572       __ehhandler$??0?$basic_stringstream@DU?$char_traits@D@std@@V?$allocator@D@2@@std@@QAE@H@Z 1001a572 f   coord3d.obj
 0001:00019590       __unwindfunclet$??0sentry@?$basic_ostream@DU?$char_traits@D@std@@@std@@QAE@AAV12@@Z$0 1001a590 f   coord3d.obj
 0001:00019598       __ehhandler$??0sentry@?$basic_ostream@DU?$char_traits@D@std@@@std@@QAE@AAV12@@Z 1001a598 f   coord3d.obj
 0001:000195c0       __unwindfunclet$?toString@Coord3D@PTools@@QAE?AV?$basic_string@DU?$char_traits@D@std@@V?$allocator@D@2@@std@@_N@Z$2 1001a5c0 f   coord3d.obj
 0001:000195da       __unwindfunclet$?toString@Coord3D@PTools@@QAE?AV?$basic_string@DU?$char_traits@D@std@@V?$allocator@D@2@@std@@_N@Z$3 1001a5da f   coord3d.obj
 0001:000195e6       __unwindfunclet$?toString@Coord3D@PTools@@QAE?AV?$basic_string@DU?$char_traits@D@std@@V?$allocator@D@2@@std@@_N@Z$6 1001a5e6 f   coord3d.obj
 0001:000195f2       __unwindfunclet$?toString@Coord3D@PTools@@QAE?AV?$basic_string@DU?$char_traits@D@std@@V?$allocator@D@2@@std@@_N@Z$0 1001a5f2 f   coord3d.obj
 0001:000195fd       __ehhandler$?toString@Coord3D@PTools@@QAE?AV?$basic_string@DU?$char_traits@D@std@@V?$allocator@D@2@@std@@_N@Z 1001a5fd f   coord3d.obj
 0001:00019620       __unwindfunclet$??0?$Array2D@N@@QAE@HH@Z$0 1001a620 f   coordsarray.obj
 0001:00019628       __ehhandler$??0?$Array2D@N@@QAE@HH@Z 1001a628 f   coordsarray.obj
 0001:00019650       __unwindfunclet$??0CoordsArray@PTools@@QAE@ABV01@@Z$0 1001a650 f   coordsarray.obj
 0001:00019658       __unwindfunclet$??0CoordsArray@PTools@@QAE@ABV01@@Z$1 1001a658 f   coordsarray.obj
 0001:00019663       __ehhandler$??0CoordsArray@PTools@@QAE@ABV01@@Z 1001a663 f   coordsarray.obj
 0001:00019680       __ehhandler$??4?$vector@UCoord3D@PTools@@V?$allocator@UCoord3D@PTools@@@std@@@std@@QAEAAV01@ABV01@@Z 1001a680 f   coordsarray.obj
 0001:000196a0       __unwindfunclet$?GetCoords@CoordsArray@PTools@@QBEXIAAUCoord3D@2@@Z$0 1001a6a0 f   coordsarray.obj
 0001:000196a8       __ehhandler$?GetCoords@CoordsArray@PTools@@QBEXIAAUCoord3D@2@@Z 1001a6a8 f   coordsarray.obj
 0001:000196d0       __unwindfunclet$?GetMatrix@CoordsArray@PTools@@QBE?AV?$Array2D@N@@XZ$1 1001a6d0 f   coordsarray.obj
 0001:000196d8       __unwindfunclet$?GetMatrix@CoordsArray@PTools@@QBE?AV?$Array2D@N@@XZ$0 1001a6d8 f   coordsarray.obj
 0001:000196f1       __ehhandler$?GetMatrix@CoordsArray@PTools@@QBE?AV?$Array2D@N@@XZ 1001a6f1 f   coordsarray.obj
 0001:00019710       __unwindfunclet$??$?HDU?$char_traits@D@std@@V?$allocator@D@1@@std@@YA?AV?$basic_string@DU?$char_traits@D@std@@V?$allocator@D@2@@0@PBDABV10@@Z$0 1001a710 f   pdbio.obj
 0001:00019729       __ehhandler$??$?HDU?$char_traits@D@std@@V?$allocator@D@1@@std@@YA?AV?$basic_string@DU?$char_traits@D@std@@V?$allocator@D@2@@0@PBDABV10@@Z 1001a729 f   pdbio.obj
 0001:00019750       __unwindfunclet$??$getline@DU?$char_traits@D@std@@V?$allocator@D@2@@std@@YAAAV?$basic_istream@DU?$char_traits@D@std@@@0@$$QAV10@AAV?$basic_string@DU?$char_traits@D@std@@V?$allocator@D@2@@0@D@Z$3 1001a750 f   pdbio.obj
 0001:00019758       __unwindfunclet$??$getline@DU?$char_traits@D@std@@V?$allocator@D@2@@std@@YAAAV?$basic_istream@DU?$char_traits@D@std@@@0@$$QAV10@AAV?$basic_string@DU?$char_traits@D@std@@V?$allocator@D@2@@0@D@Z$2 1001a758 f   pdbio.obj
 0001:00019760       __ehhandler$??$getline@DU?$char_traits@D@std@@V?$allocator@D@2@@std@@YAAAV?$basic_istream@DU?$char_traits@D@std@@@0@$$QAV10@AAV?$basic_string@DU?$char_traits@D@std@@V?$allocator@D@2@@0@D@Z 1001a760 f   pdbio.obj
 0001:00019780       __unwindfunclet$??$use_facet@V?$codecvt@DDH@std@@@std@@YAABV?$codecvt@DDH@0@ABVlocale@0@@Z$0 1001a780 f   pdbio.obj
 0001:00019789       __ehhandler$??$use_facet@V?$codecvt@DDH@std@@@std@@YAABV?$codecvt@DDH@0@ABVlocale@0@@Z 1001a789 f   pdbio.obj
 0001:000197b0       __unwindfunclet$??0?$basic_filebuf@DU?$char_traits@D@std@@@std@@QAE@PAU_iobuf@@@Z$0 1001a7b0 f   pdbio.obj
 0001:000197b9       __ehhandler$??0?$basic_filebuf@DU?$char_traits@D@std@@@std@@QAE@PAU_iobuf@@@Z 1001a7b9 f   pdbio.obj
 0001:000197e0       __unwindfunclet$??0?$basic_ifstream@DU?$char_traits@D@std@@@std@@QAE@PBDHH@Z$0 1001a7e0 f   pdbio.obj
 0001:000197fd       __unwindfunclet$??0?$basic_ifstream@DU?$char_traits@D@std@@@std@@QAE@PBDHH@Z$1 1001a7fd f   pdbio.obj
 0001:00019809       __unwindfunclet$??0?$basic_ifstream@DU?$char_traits@D@std@@@std@@QAE@PBDHH@Z$4 1001a809 f   pdbio.obj
 0001:00019812       __unwindfunclet$??0?$basic_ifstream@DU?$char_traits@D@std@@@std@@QAE@PBDHH@Z$2 1001a812 f   pdbio.obj
 0001:0001981d       __ehhandler$??0?$basic_ifstream@DU?$char_traits@D@std@@@std@@QAE@PBDHH@Z 1001a81d f   pdbio.obj
 0001:00019840       __unwindfunclet$??0?$basic_ostringstream@DU?$char_traits@D@std@@V?$allocator@D@2@@std@@QAE@H@Z$0 1001a840 f   pdbio.obj
 0001:0001985d       __unwindfunclet$??0?$basic_ostringstream@DU?$char_traits@D@std@@V?$allocator@D@2@@std@@QAE@H@Z$1 1001a85d f   pdbio.obj
 0001:00019869       __unwindfunclet$??0?$basic_ostringstream@DU?$char_traits@D@std@@V?$allocator@D@2@@std@@QAE@H@Z$4 1001a869 f   pdbio.obj
 0001:00019872       __ehhandler$??0?$basic_ostringstream@DU?$char_traits@D@std@@V?$allocator@D@2@@std@@QAE@H@Z 1001a872 f   pdbio.obj
 0001:00019890       __unwindfunclet$??0sentry@?$basic_istream@DU?$char_traits@D@std@@@std@@QAE@AAV12@_N@Z$0 1001a890 f   pdbio.obj
 0001:00019898       __ehhandler$??0sentry@?$basic_istream@DU?$char_traits@D@std@@@std@@QAE@AAV12@_N@Z 1001a898 f   pdbio.obj
 0001:000198c0       __unwindfunclet$?ReadPDB@PTools@@YAXAAV?$basic_ifstream@DU?$char_traits@D@std@@@std@@AAVRigidbody@1@@Z$0 1001a8c0 f   pdbio.obj
 0001:000198c8       __unwindfunclet$?ReadPDB@PTools@@YAXAAV?$basic_ifstream@DU?$char_traits@D@std@@@std@@AAVRigidbody@1@@Z$1 1001a8c8 f   pdbio.obj
 0001:000198d0       __unwindfunclet$?ReadPDB@PTools@@YAXAAV?$basic_ifstream@DU?$char_traits@D@std@@@std@@AAVRigidbody@1@@Z$2 1001a8d0 f   pdbio.obj
 0001:000198d8       __unwindfunclet$?ReadPDB@PTools@@YAXAAV?$basic_ifstream@DU?$char_traits@D@std@@@std@@AAVRigidbody@1@@Z$3 1001a8d8 f   pdbio.obj
 0001:000198e0       __unwindfunclet$?ReadPDB@PTools@@YAXAAV?$basic_ifstream@DU?$char_traits@D@std@@@std@@AAVRigidbody@1@@Z$7 1001a8e0 f   pdbio.obj
 0001:000198eb       __unwindfunclet$?ReadPDB@PTools@@YAXAAV?$basic_ifstream@DU?$char_traits@D@std@@@std@@AAVRigidbody@1@@Z$15 1001a8eb f   pdbio.obj
 0001:000198f6       __unwindfunclet$?ReadPDB@PTools@@YAXAAV?$basic_ifstream@DU?$char_traits@D@std@@@std@@AAVRigidbody@1@@Z$16 1001a8f6 f   pdbio.obj
 0001:00019901       __unwindfunclet$?ReadPDB@PTools@@YAXAAV?$basic_ifstream@DU?$char_traits@D@std@@@std@@AAVRigidbody@1@@Z$17 1001a901 f   pdbio.obj
 0001:0001990c       __unwindfunclet$?ReadPDB@PTools@@YAXAAV?$basic_ifstream@DU?$char_traits@D@std@@@std@@AAVRigidbody@1@@Z$13 1001a90c f   pdbio.obj
 0001:00019917       __unwindfunclet$?ReadPDB@PTools@@YAXAAV?$basic_ifstream@DU?$char_traits@D@std@@@std@@AAVRigidbody@1@@Z$18 1001a917 f   pdbio.obj
 0001:00019922       __ehhandler$?ReadPDB@PTools@@YAXAAV?$basic_ifstream@DU?$char_traits@D@std@@@std@@AAVRigidbody@1@@Z 1001a922 f   pdbio.obj
 0001:00019950       __unwindfunclet$?ReadPDB@PTools@@YAXV?$basic_string@DU?$char_traits@D@std@@V?$allocator@D@2@@std@@AAVRigidbody@1@@Z$0 1001a950 f   pdbio.obj
 0001:00019958       __unwindfunclet$?ReadPDB@PTools@@YAXV?$basic_string@DU?$char_traits@D@std@@V?$allocator@D@2@@std@@AAVRigidbody@1@@Z$1 1001a958 f   pdbio.obj
 0001:00019960       __unwindfunclet$?ReadPDB@PTools@@YAXV?$basic_string@DU?$char_traits@D@std@@V?$allocator@D@2@@std@@AAVRigidbody@1@@Z$2 1001a960 f   pdbio.obj
 0001:0001996b       __unwindfunclet$?ReadPDB@PTools@@YAXV?$basic_string@DU?$char_traits@D@std@@V?$allocator@D@2@@std@@AAVRigidbody@1@@Z$3 1001a96b f   pdbio.obj
 0001:00019976       __unwindfunclet$?ReadPDB@PTools@@YAXV?$basic_string@DU?$char_traits@D@std@@V?$allocator@D@2@@std@@AAVRigidbody@1@@Z$4 1001a976 f   pdbio.obj
 0001:0001997e       __unwindfunclet$?ReadPDB@PTools@@YAXV?$basic_string@DU?$char_traits@D@std@@V?$allocator@D@2@@std@@AAVRigidbody@1@@Z$5 1001a97e f   pdbio.obj
 0001:00019986       __ehhandler$?ReadPDB@PTools@@YAXV?$basic_string@DU?$char_traits@D@std@@V?$allocator@D@2@@std@@AAVRigidbody@1@@Z 1001a986 f   pdbio.obj
 0001:000199b0       __unwindfunclet$?SetChainId@Atomproperty@PTools@@QAEXV?$basic_string@DU?$char_traits@D@std@@V?$allocator@D@2@@std@@@Z$0 1001a9b0 f   pdbio.obj
 0001:000199b8       __ehhandler$?SetChainId@Atomproperty@PTools@@QAEXV?$basic_string@DU?$char_traits@D@std@@V?$allocator@D@2@@std@@@Z 1001a9b8 f   pdbio.obj
 0001:000199e0       __unwindfunclet$?SetExtra@Atomproperty@PTools@@QAEXV?$basic_string@DU?$char_traits@D@std@@V?$allocator@D@2@@std@@@Z$0 1001a9e0 f   pdbio.obj
 0001:000199e8       __ehhandler$?SetExtra@Atomproperty@PTools@@QAEXV?$basic_string@DU?$char_traits@D@std@@V?$allocator@D@2@@std@@@Z 1001a9e8 f   pdbio.obj
 0001:00019a10       __unwindfunclet$?SetResidType@Atomproperty@PTools@@QAEXV?$basic_string@DU?$char_traits@D@std@@V?$allocator@D@2@@std@@@Z$0 1001aa10 f   pdbio.obj
 0001:00019a18       __ehhandler$?SetResidType@Atomproperty@PTools@@QAEXV?$basic_string@DU?$char_traits@D@std@@V?$allocator@D@2@@std@@@Z 1001aa18 f   pdbio.obj
 0001:00019a40       __unwindfunclet$?WritePDB@PTools@@YAXABVRigidbody@1@V?$basic_string@DU?$char_traits@D@std@@V?$allocator@D@2@@std@@@Z$0 1001aa40 f   pdbio.obj
 0001:00019a48       __unwindfunclet$?WritePDB@PTools@@YAXABVRigidbody@1@V?$basic_string@DU?$char_traits@D@std@@V?$allocator@D@2@@std@@@Z$1 1001aa48 f   pdbio.obj
 0001:00019a53       __ehhandler$?WritePDB@PTools@@YAXABVRigidbody@1@V?$basic_string@DU?$char_traits@D@std@@V?$allocator@D@2@@std@@@Z 1001aa53 f   pdbio.obj
 0001:00019a80       __unwindfunclet$?_Endwrite@?$basic_filebuf@DU?$char_traits@D@std@@@std@@IAE_NXZ$0 1001aa80 f   pdbio.obj
 0001:00019a88       __ehhandler$?_Endwrite@?$basic_filebuf@DU?$char_traits@D@std@@@std@@IAE_NXZ 1001aa88 f   pdbio.obj
 0001:00019ab0       __unwindfunclet$?isAtom@PTools@@YA_NABV?$basic_string@DU?$char_traits@D@std@@V?$allocator@D@2@@std@@@Z$0 1001aab0 f   pdbio.obj
 0001:00019ab8       __unwindfunclet$?isAtom@PTools@@YA_NABV?$basic_string@DU?$char_traits@D@std@@V?$allocator@D@2@@std@@@Z$1 1001aab8 f   pdbio.obj
 0001:00019ac0       __ehhandler$?isAtom@PTools@@YA_NABV?$basic_string@DU?$char_traits@D@std@@V?$allocator@D@2@@std@@@Z 1001aac0 f   pdbio.obj
 0001:00019af0       __unwindfunclet$?isHeteroAtom@PTools@@YA_NABV?$basic_string@DU?$char_traits@D@std@@V?$allocator@D@2@@std@@@Z$0 1001aaf0 f   pdbio.obj
 0001:00019af8       __ehhandler$?isHeteroAtom@PTools@@YA_NABV?$basic_string@DU?$char_traits@D@std@@V?$allocator@D@2@@std@@@Z 1001aaf8 f   pdbio.obj
 0001:00019b20       __unwindfunclet$?open@?$basic_filebuf@DU?$char_traits@D@std@@@std@@QAEPAV12@PBDHH@Z$0 1001ab20 f   pdbio.obj
 0001:00019b28       __ehhandler$?open@?$basic_filebuf@DU?$char_traits@D@std@@@std@@QAEPAV12@PBDHH@Z 1001ab28 f   pdbio.obj
 0001:00019b50       __unwindfunclet$?overflow@?$basic_filebuf@DU?$char_traits@D@std@@@std@@MAEHH@Z$0 1001ab50 f   pdbio.obj
 0001:00019b58       __ehhandler$?overflow@?$basic_filebuf@DU?$char_traits@D@std@@@std@@MAEHH@Z 1001ab58 f   pdbio.obj
 0001:00019b80       __unwindfunclet$?readatomtype@PTools@@YA?AV?$basic_string@DU?$char_traits@D@std@@V?$allocator@D@2@@std@@ABV23@@Z$0 1001ab80 f   pdbio.obj
 0001:00019b88       __ehhandler$?readatomtype@PTools@@YA?AV?$basic_string@DU?$char_traits@D@std@@V?$allocator@D@2@@std@@ABV23@@Z 1001ab88 f   pdbio.obj
 0001:00019bb0       __unwindfunclet$?readresidtype@PTools@@YA?AV?$basic_string@DU?$char_traits@D@std@@V?$allocator@D@2@@std@@ABV23@@Z$0 1001abb0 f   pdbio.obj
 0001:00019bb8       __ehhandler$?readresidtype@PTools@@YA?AV?$basic_string@DU?$char_traits@D@std@@V?$allocator@D@2@@std@@ABV23@@Z 1001abb8 f   pdbio.obj
 0001:00019be0       __unwindfunclet$?strip@PTools@@YA?AV?$basic_string@DU?$char_traits@D@std@@V?$allocator@D@2@@std@@ABV23@PBD@Z$0 1001abe0 f   pdbio.obj
 0001:00019bf9       __ehhandler$?strip@PTools@@YA?AV?$basic_string@DU?$char_traits@D@std@@V?$allocator@D@2@@std@@ABV23@PBD@Z 1001abf9 f   pdbio.obj
 0001:00019c20       __unwindfunclet$?uflow@?$basic_filebuf@DU?$char_traits@D@std@@@std@@MAEHXZ$0 1001ac20 f   pdbio.obj
 0001:00019c28       __ehhandler$?uflow@?$basic_filebuf@DU?$char_traits@D@std@@@std@@MAEHXZ 1001ac28 f   pdbio.obj
 0001:00019c50       __unwindfunclet$??$_Uninit_copy@PAVAtomproperty@PTools@@PAV12@V?$allocator@VAtomproperty@PTools@@@std@@@std@@YAPAVAtomproperty@PTools@@PAV12@00AAU?$_Wrap_alloc@V?$allocator@VAtomproperty@PTools@@@std@@@0@U_Nonscalar_ptr_iterator_tag@0@@Z$2 1001ac50 f   rigidbody.obj
 0001:00019c61       __ehhandler$??$_Uninit_copy@PAVAtomproperty@PTools@@PAV12@V?$allocator@VAtomproperty@PTools@@@std@@@std@@YAPAVAtomproperty@PTools@@PAV12@00AAU?$_Wrap_alloc@V?$allocator@VAtomproperty@PTools@@@std@@@0@U_Nonscalar_ptr_iterator_tag@0@@Z 1001ac61 f   rigidbody.obj
 0001:00019c80       __unwindfunclet$??$_Uninit_move@PAVAtomproperty@PTools@@PAV12@V?$allocator@VAtomproperty@PTools@@@std@@V12@@std@@YAPAVAtomproperty@PTools@@PAV12@00AAU?$_Wrap_alloc@V?$allocator@VAtomproperty@PTools@@@std@@@0@0U_Nonscalar_ptr_iterator_tag@0@@Z$2 1001ac80 f   rigidbody.obj
 0001:00019c91       __ehhandler$??$_Uninit_move@PAVAtomproperty@PTools@@PAV12@V?$allocator@VAtomproperty@PTools@@@std@@V12@@std@@YAPAVAtomproperty@PTools@@PAV12@00AAU?$_Wrap_alloc@V?$allocator@VAtomproperty@PTools@@@std@@@0@0U_Nonscalar_ptr_iterator_tag@0@@Z 1001ac91 f   rigidbody.obj
 0001:00019cb0       __unwindfunclet$??$construct@VAtomproperty@PTools@@AAV12@@?$_Wrap_alloc@V?$allocator@VAtomproperty@PTools@@@std@@@std@@QAEXPAVAtomproperty@PTools@@AAV23@@Z$0 1001acb0 f   rigidbody.obj
 0001:00019cc1       __ehhandler$??$construct@VAtomproperty@PTools@@AAV12@@?$_Wrap_alloc@V?$allocator@VAtomproperty@PTools@@@std@@@std@@QAEXPAVAtomproperty@PTools@@AAV23@@Z 1001acc1 f   rigidbody.obj
 0001:00019ce0       __unwindfunclet$??$construct@VAtomproperty@PTools@@AAV12@@?$allocator@VAtomproperty@PTools@@@std@@QAEXPAVAtomproperty@PTools@@AAV23@@Z$0 1001ace0 f   rigidbody.obj
 0001:00019cf1       __ehhandler$??$construct@VAtomproperty@PTools@@AAV12@@?$allocator@VAtomproperty@PTools@@@std@@QAEXPAVAtomproperty@PTools@@AAV23@@Z 1001acf1 f   rigidbody.obj
 0001:00019d10       __unwindfunclet$??$construct@VAtomproperty@PTools@@AAV12@@?$allocator_traits@V?$allocator@VAtomproperty@PTools@@@std@@@std@@SAXAAV?$allocator@VAtomproperty@PTools@@@1@PAVAtomproperty@PTools@@AAV34@@Z$0 1001ad10 f   rigidbody.obj
 0001:00019d21       __ehhandler$??$construct@VAtomproperty@PTools@@AAV12@@?$allocator_traits@V?$allocator@VAtomproperty@PTools@@@std@@@std@@SAXAAV?$allocator@VAtomproperty@PTools@@@1@PAVAtomproperty@PTools@@AAV34@@Z 1001ad21 f   rigidbody.obj
 0001:00019d40       __unwindfunclet$??$construct@VAtomproperty@PTools@@ABV12@@?$_Wrap_alloc@V?$allocator@VAtomproperty@PTools@@@std@@@std@@QAEXPAVAtomproperty@PTools@@ABV23@@Z$0 1001ad40 f   rigidbody.obj
 0001:00019d51       __ehhandler$??$construct@VAtomproperty@PTools@@ABV12@@?$_Wrap_alloc@V?$allocator@VAtomproperty@PTools@@@std@@@std@@QAEXPAVAtomproperty@PTools@@ABV23@@Z 1001ad51 f   rigidbody.obj
 0001:00019d70       __unwindfunclet$??$construct@VAtomproperty@PTools@@ABV12@@?$allocator_traits@V?$allocator@VAtomproperty@PTools@@@std@@@std@@SAXAAV?$allocator@VAtomproperty@PTools@@@1@PAVAtomproperty@PTools@@ABV34@@Z$0 1001ad70 f   rigidbody.obj
 0001:00019d81       __ehhandler$??$construct@VAtomproperty@PTools@@ABV12@@?$allocator_traits@V?$allocator@VAtomproperty@PTools@@@std@@@std@@SAXAAV?$allocator@VAtomproperty@PTools@@@1@PAVAtomproperty@PTools@@ABV34@@Z 1001ad81 f   rigidbody.obj
 0001:00019da0       __unwindfunclet$??$construct@VAtomproperty@PTools@@V12@@?$_Wrap_alloc@V?$allocator@VAtomproperty@PTools@@@std@@@std@@QAEXPAVAtomproperty@PTools@@$$QAV23@@Z$0 1001ada0 f   rigidbody.obj
 0001:00019db1       __ehhandler$??$construct@VAtomproperty@PTools@@V12@@?$_Wrap_alloc@V?$allocator@VAtomproperty@PTools@@@std@@@std@@QAEXPAVAtomproperty@PTools@@$$QAV23@@Z 1001adb1 f   rigidbody.obj
 0001:00019dd0       __unwindfunclet$??$construct@VAtomproperty@PTools@@V12@@?$allocator@VAtomproperty@PTools@@@std@@QAEXPAVAtomproperty@PTools@@$$QAV23@@Z$0 1001add0 f   rigidbody.obj
 0001:00019de1       __ehhandler$??$construct@VAtomproperty@PTools@@V12@@?$allocator@VAtomproperty@PTools@@@std@@QAEXPAVAtomproperty@PTools@@$$QAV23@@Z 1001ade1 f   rigidbody.obj
 0001:00019e00       __unwindfunclet$??$construct@VAtomproperty@PTools@@V12@@?$allocator_traits@V?$allocator@VAtomproperty@PTools@@@std@@@std@@SAXAAV?$allocator@VAtomproperty@PTools@@@1@PAVAtomproperty@PTools@@$$QAV34@@Z$0 1001ae00 f   rigidbody.obj
 0001:00019e11       __ehhandler$??$construct@VAtomproperty@PTools@@V12@@?$allocator_traits@V?$allocator@VAtomproperty@PTools@@@std@@@std@@SAXAAV?$allocator@VAtomproperty@PTools@@@1@PAVAtomproperty@PTools@@$$QAV34@@Z 1001ae11 f   rigidbody.obj
 0001:00019e30       __unwindfunclet$??0Rigidbody@PTools@@QAE@ABV01@@Z$0 1001ae30 f   rigidbody.obj
 0001:00019e3b       __unwindfunclet$??0Rigidbody@PTools@@QAE@ABV01@@Z$1 1001ae3b f   rigidbody.obj
 0001:00019e49       __unwindfunclet$??0Rigidbody@PTools@@QAE@ABV01@@Z$2 1001ae49 f   rigidbody.obj
 0001:00019e57       __unwindfunclet$??0Rigidbody@PTools@@QAE@ABV01@@Z$3 1001ae57 f   rigidbody.obj
 0001:00019e65       __ehhandler$??0Rigidbody@PTools@@QAE@ABV01@@Z 1001ae65 f   rigidbody.obj
 0001:00019e80       __unwindfunclet$??0Rigidbody@PTools@@QAE@V?$basic_string@DU?$char_traits@D@std@@V?$allocator@D@2@@std@@@Z$0 1001ae80 f   rigidbody.obj
 0001:00019e88       __unwindfunclet$??0Rigidbody@PTools@@QAE@V?$basic_string@DU?$char_traits@D@std@@V?$allocator@D@2@@std@@@Z$1 1001ae88 f   rigidbody.obj
 0001:00019e93       __unwindfunclet$??0Rigidbody@PTools@@QAE@V?$basic_string@DU?$char_traits@D@std@@V?$allocator@D@2@@std@@@Z$2 1001ae93 f   rigidbody.obj
 0001:00019ea1       __unwindfunclet$??0Rigidbody@PTools@@QAE@V?$basic_string@DU?$char_traits@D@std@@V?$allocator@D@2@@std@@@Z$3 1001aea1 f   rigidbody.obj
 0001:00019eaf       __unwindfunclet$??0Rigidbody@PTools@@QAE@V?$basic_string@DU?$char_traits@D@std@@V?$allocator@D@2@@std@@@Z$4 1001aeaf f   rigidbody.obj
 0001:00019ebd       __ehhandler$??0Rigidbody@PTools@@QAE@V?$basic_string@DU?$char_traits@D@std@@V?$allocator@D@2@@std@@@Z 1001aebd f   rigidbody.obj
 0001:00019ee0       __unwindfunclet$??0Rigidbody@PTools@@QAE@XZ$0 1001aee0 f   rigidbody.obj
 0001:00019eeb       __unwindfunclet$??0Rigidbody@PTools@@QAE@XZ$1 1001aeeb f   rigidbody.obj
 0001:00019ef9       __unwindfunclet$??0Rigidbody@PTools@@QAE@XZ$2 1001aef9 f   rigidbody.obj
 0001:00019f07       __unwindfunclet$??0Rigidbody@PTools@@QAE@XZ$3 1001af07 f   rigidbody.obj
 0001:00019f15       __ehhandler$??0Rigidbody@PTools@@QAE@XZ 1001af15 f   rigidbody.obj
 0001:00019f30       __ehhandler$??4?$vector@VAtomproperty@PTools@@V?$allocator@VAtomproperty@PTools@@@std@@@std@@QAEAAV01@ABV01@@Z 1001af30 f   rigidbody.obj
 0001:00019f50       __unwindfunclet$??HRigidbody@PTools@@QAE?AV01@ABV01@@Z$0 1001af50 f   rigidbody.obj
 0001:00019f69       __ehhandler$??HRigidbody@PTools@@QAE?AV01@ABV01@@Z 1001af69 f   rigidbody.obj
 0001:00019f90       __unwindfunclet$?AddAtom@Rigidbody@PTools@@QAEXABVAtom@2@@Z$0 1001af90 f   rigidbody.obj
 0001:00019f9b       __ehhandler$?AddAtom@Rigidbody@PTools@@QAEXABVAtom@2@@Z 1001af9b f   rigidbody.obj
 0001:00019fd0       __unwindfunclet$?Backbone@Rigidbody@PTools@@QAE?AVAtomSelection@2@XZ$0 1001afd0 f   rigidbody.obj
 0001:00019ff2       __unwindfunclet$?Backbone@Rigidbody@PTools@@QAE?AVAtomSelection@2@XZ$1 1001aff2 f   rigidbody.obj
 0001:00019ffd       __unwindfunclet$?Backbone@Rigidbody@PTools@@QAE?AVAtomSelection@2@XZ$2 1001affd f   rigidbody.obj
 0001:0001a005       __ehhandler$?Backbone@Rigidbody@PTools@@QAE?AVAtomSelection@2@XZ 1001b005 f   rigidbody.obj
 0001:0001a030       __unwindfunclet$?CopyAtom@Rigidbody@PTools@@UBE?AVAtom@2@I@Z$2 1001b030 f   rigidbody.obj
 0001:0001a03b       __ehhandler$?CopyAtom@Rigidbody@PTools@@UBE?AVAtom@2@I@Z 1001b03b f   rigidbody.obj
 0001:0001a060       __unwindfunclet$?SelectAllAtoms@Rigidbody@PTools@@QBE?AVAtomSelection@2@XZ$0 1001b060 f   rigidbody.obj
 0001:0001a079       __ehhandler$?SelectAllAtoms@Rigidbody@PTools@@QBE?AVAtomSelection@2@XZ 1001b079 f   rigidbody.obj
 0001:0001a0a0       __unwindfunclet$?SelectAtomType@Rigidbody@PTools@@QAE?AVAtomSelection@2@V?$basic_string@DU?$char_traits@D@std@@V?$allocator@D@2@@std@@@Z$0 1001b0a0 f   rigidbody.obj
 0001:0001a0a8       __unwindfunclet$?SelectAtomType@Rigidbody@PTools@@QAE?AVAtomSelection@2@V?$basic_string@DU?$char_traits@D@std@@V?$allocator@D@2@@std@@@Z$1 1001b0a8 f   rigidbody.obj
 0001:0001a0c1       __unwindfunclet$?SelectAtomType@Rigidbody@PTools@@QAE?AVAtomSelection@2@V?$basic_string@DU?$char_traits@D@std@@V?$allocator@D@2@@std@@@Z$2 1001b0c1 f   rigidbody.obj
 0001:0001a0c9       __ehhandler$?SelectAtomType@Rigidbody@PTools@@QAE?AVAtomSelection@2@V?$basic_string@DU?$char_traits@D@std@@V?$allocator@D@2@@std@@@Z 1001b0c9 f   rigidbody.obj
 0001:0001a0f0       __unwindfunclet$?SelectChainId@Rigidbody@PTools@@QAE?AVAtomSelection@2@V?$basic_string@DU?$char_traits@D@std@@V?$allocator@D@2@@std@@@Z$0 1001b0f0 f   rigidbody.obj
 0001:0001a0f8       __unwindfunclet$?SelectChainId@Rigidbody@PTools@@QAE?AVAtomSelection@2@V?$basic_string@DU?$char_traits@D@std@@V?$allocator@D@2@@std@@@Z$1 1001b0f8 f   rigidbody.obj
 0001:0001a111       __unwindfunclet$?SelectChainId@Rigidbody@PTools@@QAE?AVAtomSelection@2@V?$basic_string@DU?$char_traits@D@std@@V?$allocator@D@2@@std@@@Z$2 1001b111 f   rigidbody.obj
 0001:0001a119       __ehhandler$?SelectChainId@Rigidbody@PTools@@QAE?AVAtomSelection@2@V?$basic_string@DU?$char_traits@D@std@@V?$allocator@D@2@@std@@@Z 1001b119 f   rigidbody.obj
 0001:0001a140       __unwindfunclet$?SelectResRange@Rigidbody@PTools@@QAE?AVAtomSelection@2@II@Z$0 1001b140 f   rigidbody.obj
 0001:0001a159       __ehhandler$?SelectResRange@Rigidbody@PTools@@QAE?AVAtomSelection@2@II@Z 1001b159 f   rigidbody.obj
 0001:0001a180       __unwindfunclet$?SelectResidType@Rigidbody@PTools@@QAE?AVAtomSelection@2@V?$basic_string@DU?$char_traits@D@std@@V?$allocator@D@2@@std@@@Z$0 1001b180 f   rigidbody.obj
 0001:0001a188       __unwindfunclet$?SelectResidType@Rigidbody@PTools@@QAE?AVAtomSelection@2@V?$basic_string@DU?$char_traits@D@std@@V?$allocator@D@2@@std@@@Z$1 1001b188 f   rigidbody.obj
 0001:0001a1a1       __unwindfunclet$?SelectResidType@Rigidbody@PTools@@QAE?AVAtomSelection@2@V?$basic_string@DU?$char_traits@D@std@@V?$allocator@D@2@@std@@@Z$2 1001b1a1 f   rigidbody.obj
 0001:0001a1a9       __ehhandler$?SelectResidType@Rigidbody@PTools@@QAE?AVAtomSelection@2@V?$basic_string@DU?$char_traits@D@std@@V?$allocator@D@2@@std@@@Z 1001b1a9 f   rigidbody.obj
 0001:0001a1d0       __unwindfunclet$?SetAtom@Rigidbody@PTools@@QAEXIABVAtom@2@@Z$0 1001b1d0 f   rigidbody.obj
 0001:0001a1d8       __unwindfunclet$?SetAtom@Rigidbody@PTools@@QAEXIABVAtom@2@@Z$1 1001b1d8 f   rigidbody.obj
 0001:0001a1e3       __ehhandler$?SetAtom@Rigidbody@PTools@@QAEXIABVAtom@2@@Z 1001b1e3 f   rigidbody.obj
 0001:0001a210       __ehhandler$?_Reallocate@?$vector@UCoord3D@PTools@@V?$allocator@UCoord3D@PTools@@@std@@@std@@IAEXI@Z 1001b210 f   rigidbody.obj
 0001:0001a230       __ehhandler$?_Reallocate@?$vector@VAtomproperty@PTools@@V?$allocator@VAtomproperty@PTools@@@std@@@std@@IAEXI@Z 1001b230 f   rigidbody.obj
 0001:0001a250       __unwindfunclet$?construct@?$allocator@VAtomproperty@PTools@@@std@@QAEXPAVAtomproperty@PTools@@ABV34@@Z$0 1001b250 f   rigidbody.obj
 0001:0001a261       __ehhandler$?construct@?$allocator@VAtomproperty@PTools@@@std@@QAEXPAVAtomproperty@PTools@@ABV34@@Z 1001b261 f   rigidbody.obj
 0001:0001a280       __unwindfunclet$?isBackbone@PTools@@YA_NABV?$basic_string@DU?$char_traits@D@std@@V?$allocator@D@2@@std@@@Z$0 1001b280 f   rigidbody.obj
 0001:0001a288       __unwindfunclet$?isBackbone@PTools@@YA_NABV?$basic_string@DU?$char_traits@D@std@@V?$allocator@D@2@@std@@@Z$1 1001b288 f   rigidbody.obj
 0001:0001a290       __unwindfunclet$?isBackbone@PTools@@YA_NABV?$basic_string@DU?$char_traits@D@std@@V?$allocator@D@2@@std@@@Z$2 1001b290 f   rigidbody.obj
 0001:0001a298       __unwindfunclet$?isBackbone@PTools@@YA_NABV?$basic_string@DU?$char_traits@D@std@@V?$allocator@D@2@@std@@@Z$4 1001b298 f   rigidbody.obj
 0001:0001a2ab       __ehhandler$?isBackbone@PTools@@YA_NABV?$basic_string@DU?$char_traits@D@std@@V?$allocator@D@2@@std@@@Z 1001b2ab f   rigidbody.obj
 0001:0001a2d0       __unwindfunclet$?push_back@?$vector@VAtomproperty@PTools@@V?$allocator@VAtomproperty@PTools@@@std@@@std@@QAEXABVAtomproperty@PTools@@@Z$0 1001b2d0 f   rigidbody.obj
 0001:0001a2e1       __unwindfunclet$?push_back@?$vector@VAtomproperty@PTools@@V?$allocator@VAtomproperty@PTools@@@std@@@std@@QAEXABVAtomproperty@PTools@@@Z$1 1001b2e1 f   rigidbody.obj
 0001:0001a2f2       __ehhandler$?push_back@?$vector@VAtomproperty@PTools@@V?$allocator@VAtomproperty@PTools@@@std@@@std@@QAEXABVAtomproperty@PTools@@@Z 1001b2f2 f   rigidbody.obj
 0001:0001a310       __unwindfunclet$?Rmsd@PTools@@YANABVAtomSelection@1@0@Z$0 1001b310 f   rmsd.obj
 0001:0001a31b       __unwindfunclet$?Rmsd@PTools@@YANABVAtomSelection@1@0@Z$1 1001b31b f   rmsd.obj
 0001:0001a326       __ehhandler$?Rmsd@PTools@@YANABVAtomSelection@1@0@Z 1001b326 f   rmsd.obj
 0001:0001a360       __unwindfunclet$??$_Uninit_fill_n@PAV?$vector@NV?$allocator@N@std@@@std@@IV12@V?$allocator@V?$vector@NV?$allocator@N@std@@@std@@@2@V12@@std@@YAXPAV?$vector@NV?$allocator@N@std@@@0@IPBV10@AAU?$_Wrap_alloc@V?$allocator@V?$vector@NV?$allocator@N@std@@@std@@@std@@@0@0U_Nonscalar_ptr_iterator_tag@0@@Z$2 1001b360 f   superpose.obj
 0001:0001a371       __ehhandler$??$_Uninit_fill_n@PAV?$vector@NV?$allocator@N@std@@@std@@IV12@V?$allocator@V?$vector@NV?$allocator@N@std@@@std@@@2@V12@@std@@YAXPAV?$vector@NV?$allocator@N@std@@@0@IPBV10@AAU?$_Wrap_alloc@V?$allocator@V?$vector@NV?$allocator@N@std@@@std@@@std@@@0@0U_Nonscalar_ptr_iterator_tag@0@@Z 1001b371 f   superpose.obj
 0001:0001a390       __unwindfunclet$??$construct@V?$vector@NV?$allocator@N@std@@@std@@ABV12@@?$_Wrap_alloc@V?$allocator@V?$vector@NV?$allocator@N@std@@@std@@@std@@@std@@QAEXPAV?$vector@NV?$allocator@N@std@@@1@ABV21@@Z$0 1001b390 f   superpose.obj
 0001:0001a3a1       __ehhandler$??$construct@V?$vector@NV?$allocator@N@std@@@std@@ABV12@@?$_Wrap_alloc@V?$allocator@V?$vector@NV?$allocator@N@std@@@std@@@std@@@std@@QAEXPAV?$vector@NV?$allocator@N@std@@@1@ABV21@@Z 1001b3a1 f   superpose.obj
 0001:0001a3c0       __unwindfunclet$??$construct@V?$vector@NV?$allocator@N@std@@@std@@ABV12@@?$allocator_traits@V?$allocator@V?$vector@NV?$allocator@N@std@@@std@@@std@@@std@@SAXAAV?$allocator@V?$vector@NV?$allocator@N@std@@@std@@@1@PAV?$vector@NV?$allocator@N@std@@@1@ABV31@@Z$0 1001b3c0 f   superpose.obj
 0001:0001a3d1       __ehhandler$??$construct@V?$vector@NV?$allocator@N@std@@@std@@ABV12@@?$allocator_traits@V?$allocator@V?$vector@NV?$allocator@N@std@@@std@@@std@@@std@@SAXAAV?$allocator@V?$vector@NV?$allocator@N@std@@@std@@@1@PAV?$vector@NV?$allocator@N@std@@@1@ABV31@@Z 1001b3d1 f   superpose.obj
 0001:0001a3f0       __unwindfunclet$?MakeTensor@PTools@@YAXAAVRigidbody@1@0QAY02N@Z$0 1001b3f0 f   superpose.obj
 0001:0001a3f8       __unwindfunclet$?MakeTensor@PTools@@YAXAAVRigidbody@1@0QAY02N@Z$1 1001b3f8 f   superpose.obj
 0001:0001a400       __unwindfunclet$?MakeTensor@PTools@@YAXAAVRigidbody@1@0QAY02N@Z$2 1001b400 f   superpose.obj
 0001:0001a408       __unwindfunclet$?MakeTensor@PTools@@YAXAAVRigidbody@1@0QAY02N@Z$3 1001b408 f   superpose.obj
 0001:0001a410       __unwindfunclet$?MakeTensor@PTools@@YAXAAVRigidbody@1@0QAY02N@Z$4 1001b410 f   superpose.obj
 0001:0001a418       __unwindfunclet$?MakeTensor@PTools@@YAXAAVRigidbody@1@0QAY02N@Z$5 1001b418 f   superpose.obj
 0001:0001a420       __ehhandler$?MakeTensor@PTools@@YAXAAVRigidbody@1@0QAY02N@Z 1001b420 f   superpose.obj
 0001:0001a450       __ehhandler$?_Construct_n@?$vector@V?$vector@NV?$allocator@N@std@@@std@@V?$allocator@V?$vector@NV?$allocator@N@std@@@std@@@2@@std@@QAEXIPBV?$vector@NV?$allocator@N@std@@@2@@Z 1001b450 f   superpose.obj
 0001:0001a470       __unwindfunclet$?construct@?$allocator@V?$vector@NV?$allocator@N@std@@@std@@@std@@QAEXPAV?$vector@NV?$allocator@N@std@@@2@ABV32@@Z$0 1001b470 f   superpose.obj
 0001:0001a481       __ehhandler$?construct@?$allocator@V?$vector@NV?$allocator@N@std@@@std@@@std@@QAEXPAV?$vector@NV?$allocator@N@std@@@2@ABV32@@Z 1001b481 f   superpose.obj
 0001:0001a4a0       __unwindfunclet$?superpose@PTools@@YA?AUSuperpose_t@@ABVRigidbody@1@0H@Z$0 1001b4a0 f   superpose.obj
 0001:0001a4ab       __unwindfunclet$?superpose@PTools@@YA?AUSuperpose_t@@ABVRigidbody@1@0H@Z$1 1001b4ab f   superpose.obj
 0001:0001a4b6       __unwindfunclet$?superpose@PTools@@YA?AUSuperpose_t@@ABVRigidbody@1@0H@Z$7 1001b4b6 f   superpose.obj
 0001:0001a4c1       __unwindfunclet$?superpose@PTools@@YA?AUSuperpose_t@@ABVRigidbody@1@0H@Z$2 1001b4c1 f   superpose.obj
 0001:0001a4cc       __unwindfunclet$?superpose@PTools@@YA?AUSuperpose_t@@ABVRigidbody@1@0H@Z$3 1001b4cc f   superpose.obj
 0001:0001a4ee       __unwindfunclet$?superpose@PTools@@YA?AUSuperpose_t@@ABVRigidbody@1@0H@Z$4 1001b4ee f   superpose.obj
 0001:0001a4f9       __unwindfunclet$?superpose@PTools@@YA?AUSuperpose_t@@ABVRigidbody@1@0H@Z$5 1001b4f9 f   superpose.obj
 0001:0001a504       __unwindfunclet$?superpose@PTools@@YA?AUSuperpose_t@@ABVRigidbody@1@0H@Z$6 1001b504 f   superpose.obj
 0001:0001a50f       __ehhandler$?superpose@PTools@@YA?AUSuperpose_t@@ABVRigidbody@1@0H@Z 1001b50f f   superpose.obj
 0001:0001a540       __unwindfunclet$??__EalgoLog@U2@@YAXXZ$0 1001b540 f   moc_PToolsPlugin.obj
 0001:0001a549       __ehhandler$??__EalgoLog@U2@@YAXXZ 1001b549 f   moc_PToolsPlugin.obj
 0001:0001a570       __unwindfunclet$??__EcmdLog@U2@@YAXXZ$0 1001b570 f   moc_PToolsPlugin.obj
 0001:0001a579       __ehhandler$??__EcmdLog@U2@@YAXXZ 1001b579 f   moc_PToolsPlugin.obj
 0001:0001a5a0       __unwindfunclet$??__EcoreLog@U2@@YAXXZ$0 1001b5a0 f   moc_PToolsPlugin.obj
 0001:0001a5a9       __ehhandler$??__EcoreLog@U2@@YAXXZ 1001b5a9 f   moc_PToolsPlugin.obj
 0001:0001a5d0       __unwindfunclet$??__EioLog@U2@@YAXXZ$0 1001b5d0 f   moc_PToolsPlugin.obj
 0001:0001a5d9       __ehhandler$??__EioLog@U2@@YAXXZ 1001b5d9 f   moc_PToolsPlugin.obj
 0001:0001a600       __unwindfunclet$??__EperfLog@U2@@YAXXZ$0 1001b600 f   moc_PToolsPlugin.obj
 0001:0001a609       __ehhandler$??__EperfLog@U2@@YAXXZ 1001b609 f   moc_PToolsPlugin.obj
 0001:0001a630       __unwindfunclet$??__EscriptLog@U2@@YAXXZ$0 1001b630 f   moc_PToolsPlugin.obj
 0001:0001a639       __ehhandler$??__EscriptLog@U2@@YAXXZ 1001b639 f   moc_PToolsPlugin.obj
 0001:0001a660       __unwindfunclet$??__EtaskLog@U2@@YAXXZ$0 1001b660 f   moc_PToolsPlugin.obj
 0001:0001a669       __ehhandler$??__EtaskLog@U2@@YAXXZ 1001b669 f   moc_PToolsPlugin.obj
 0001:0001a690       __unwindfunclet$??__EuiLog@U2@@YAXXZ$0 1001b690 f   moc_PToolsPlugin.obj
 0001:0001a699       __ehhandler$??__EuiLog@U2@@YAXXZ 1001b699 f   moc_PToolsPlugin.obj
 0001:0001a6c0       __unwindfunclet$??__EuserActLog@U2@@YAXXZ$0 1001b6c0 f   moc_PToolsPlugin.obj
 0001:0001a6c9       __ehhandler$??__EuserActLog@U2@@YAXXZ 1001b6c9 f   moc_PToolsPlugin.obj
 0001:0001a6f0       __unwindfunclet$??__EalgoLog@U2@@YAXXZ$0 1001b6f0 f   moc_PToolsTests.obj
 0001:0001a6f9       __ehhandler$??__EalgoLog@U2@@YAXXZ 1001b6f9 f   moc_PToolsTests.obj
 0001:0001a720       __unwindfunclet$??__EcmdLog@U2@@YAXXZ$0 1001b720 f   moc_PToolsTests.obj
 0001:0001a729       __ehhandler$??__EcmdLog@U2@@YAXXZ 1001b729 f   moc_PToolsTests.obj
 0001:0001a750       __unwindfunclet$??__EcoreLog@U2@@YAXXZ$0 1001b750 f   moc_PToolsTests.obj
 0001:0001a759       __ehhandler$??__EcoreLog@U2@@YAXXZ 1001b759 f   moc_PToolsTests.obj
 0001:0001a780       __unwindfunclet$??__EioLog@U2@@YAXXZ$0 1001b780 f   moc_PToolsTests.obj
 0001:0001a789       __ehhandler$??__EioLog@U2@@YAXXZ 1001b789 f   moc_PToolsTests.obj
 0001:0001a7b0       __unwindfunclet$??__EperfLog@U2@@YAXXZ$0 1001b7b0 f   moc_PToolsTests.obj
 0001:0001a7b9       __ehhandler$??__EperfLog@U2@@YAXXZ 1001b7b9 f   moc_PToolsTests.obj
 0001:0001a7e0       __unwindfunclet$??__EscriptLog@U2@@YAXXZ$0 1001b7e0 f   moc_PToolsTests.obj
 0001:0001a7e9       __ehhandler$??__EscriptLog@U2@@YAXXZ 1001b7e9 f   moc_PToolsTests.obj
 0001:0001a810       __unwindfunclet$??__EtaskLog@U2@@YAXXZ$0 1001b810 f   moc_PToolsTests.obj
 0001:0001a819       __ehhandler$??__EtaskLog@U2@@YAXXZ 1001b819 f   moc_PToolsTests.obj
 0001:0001a840       __unwindfunclet$??__EuiLog@U2@@YAXXZ$0 1001b840 f   moc_PToolsTests.obj
 0001:0001a849       __ehhandler$??__EuiLog@U2@@YAXXZ 1001b849 f   moc_PToolsTests.obj
 0001:0001a870       __unwindfunclet$??__EuserActLog@U2@@YAXXZ$0 1001b870 f   moc_PToolsTests.obj
 0001:0001a879       __ehhandler$??__EuserActLog@U2@@YAXXZ 1001b879 f   moc_PToolsTests.obj
 0001:0001a8a0       ??__F?_Generic_object@?$_Error_objects@H@std@@2V_Generic_error_category@2@A@@YAXXZ 1001b8a0 f   PToolsAligner.obj
 0001:0001a8b0       ??__F?_Iostream_object@?$_Error_objects@H@std@@2V_Iostream_error_category@2@A@@YAXXZ 1001b8b0 f   PToolsAligner.obj
 0001:0001a8c0       ??__F?_System_object@?$_Error_objects@H@std@@2V_System_error_category@2@A@@YAXXZ 1001b8c0 f   PToolsAligner.obj
 0001:0001a8d0       ??__FalgoLog@U2@@YAXXZ     1001b8d0 f   PToolsAligner.obj
 0001:0001a8e0       ??__FcmdLog@U2@@YAXXZ      1001b8e0 f   PToolsAligner.obj
 0001:0001a8f0       ??__FcoreLog@U2@@YAXXZ     1001b8f0 f   PToolsAligner.obj
 0001:0001a900       ??__FioLog@U2@@YAXXZ       1001b900 f   PToolsAligner.obj
 0001:0001a910       ??__FperfLog@U2@@YAXXZ     1001b910 f   PToolsAligner.obj
 0001:0001a920       ??__FscriptLog@U2@@YAXXZ   1001b920 f   PToolsAligner.obj
 0001:0001a930       ??__FtaskLog@U2@@YAXXZ     1001b930 f   PToolsAligner.obj
 0001:0001a940       ??__FuiLog@U2@@YAXXZ       1001b940 f   PToolsAligner.obj
 0001:0001a950       ??__FuserActLog@U2@@YAXXZ  1001b950 f   PToolsAligner.obj
 0001:0001a960       ??__F?_Generic_object@?$_Error_objects@H@std@@2V_Generic_error_category@2@A@@YAXXZ 1001b960 f   PToolsPlugin.obj
 0001:0001a970       ??__F?_Iostream_object@?$_Error_objects@H@std@@2V_Iostream_error_category@2@A@@YAXXZ 1001b970 f   PToolsPlugin.obj
 0001:0001a980       ??__F?_System_object@?$_Error_objects@H@std@@2V_System_error_category@2@A@@YAXXZ 1001b980 f   PToolsPlugin.obj
 0001:0001a990       ??__FPTOOLS_ID@U2@@YAXXZ   1001b990 f   PToolsPlugin.obj
 0001:0001a9a0       ??__FalgoLog@U2@@YAXXZ     1001b9a0 f   PToolsPlugin.obj
 0001:0001a9b0       ??__FcmdLog@U2@@YAXXZ      1001b9b0 f   PToolsPlugin.obj
 0001:0001a9c0       ??__FcoreLog@U2@@YAXXZ     1001b9c0 f   PToolsPlugin.obj
 0001:0001a9d0       ??__FioLog@U2@@YAXXZ       1001b9d0 f   PToolsPlugin.obj
 0001:0001a9e0       ??__FperfLog@U2@@YAXXZ     1001b9e0 f   PToolsPlugin.obj
 0001:0001a9f0       ??__FscriptLog@U2@@YAXXZ   1001b9f0 f   PToolsPlugin.obj
 0001:0001aa00       ??__FtaskLog@U2@@YAXXZ     1001ba00 f   PToolsPlugin.obj
 0001:0001aa10       ??__FuiLog@U2@@YAXXZ       1001ba10 f   PToolsPlugin.obj
 0001:0001aa20       ??__FuserActLog@U2@@YAXXZ  1001ba20 f   PToolsPlugin.obj
 0001:0001aa30       ??__F?ACCURACY_ATTR@Gtest_PToolsAlignerTask@U2@@2VQString@@B@@YAXXZ 1001ba30 f   PToolsTests.obj
 0001:0001aa40       ??__F?MOBO_ATTR@Gtest_PToolsAlignerTask@U2@@2VQString@@B@@YAXXZ 1001ba40 f   PToolsTests.obj
 0001:0001aa50       ??__F?REFO_ATTR@Gtest_PToolsAlignerTask@U2@@2VQString@@B@@YAXXZ 1001ba50 f   PToolsTests.obj
 0001:0001aa60       ??__F?RMSD_ATTR@Gtest_PToolsAlignerTask@U2@@2VQString@@B@@YAXXZ 1001ba60 f   PToolsTests.obj
 0001:0001aa70       ??__F?TRANSFORM_ATTR@Gtest_PToolsAlignerTask@U2@@2VQString@@B@@YAXXZ 1001ba70 f   PToolsTests.obj
 0001:0001aa80       ??__F?_Generic_object@?$_Error_objects@H@std@@2V_Generic_error_category@2@A@@YAXXZ 1001ba80 f   PToolsTests.obj
 0001:0001aa90       ??__F?_Iostream_object@?$_Error_objects@H@std@@2V_Iostream_error_category@2@A@@YAXXZ 1001ba90 f   PToolsTests.obj
 0001:0001aaa0       ??__F?_System_object@?$_Error_objects@H@std@@2V_System_error_category@2@A@@YAXXZ 1001baa0 f   PToolsTests.obj
 0001:0001aab0       ??__FalgoLog@U2@@YAXXZ     1001bab0 f   PToolsTests.obj
 0001:0001aac0       ??__FcmdLog@U2@@YAXXZ      1001bac0 f   PToolsTests.obj
 0001:0001aad0       ??__FcoreLog@U2@@YAXXZ     1001bad0 f   PToolsTests.obj
 0001:0001aae0       ??__FioLog@U2@@YAXXZ       1001bae0 f   PToolsTests.obj
 0001:0001aaf0       ??__FperfLog@U2@@YAXXZ     1001baf0 f   PToolsTests.obj
 0001:0001ab00       ??__FscriptLog@U2@@YAXXZ   1001bb00 f   PToolsTests.obj
 0001:0001ab10       ??__FtaskLog@U2@@YAXXZ     1001bb10 f   PToolsTests.obj
 0001:0001ab20       ??__FuiLog@U2@@YAXXZ       1001bb20 f   PToolsTests.obj
 0001:0001ab30       ??__FuserActLog@U2@@YAXXZ  1001bb30 f   PToolsTests.obj
 0001:0001ab40       ??__F?_Generic_object@?$_Error_objects@H@std@@2V_Generic_error_category@2@A@@YAXXZ 1001bb40 f   atom.obj
 0001:0001ab50       ??__F?_Iostream_object@?$_Error_objects@H@std@@2V_Iostream_error_category@2@A@@YAXXZ 1001bb50 f   atom.obj
 0001:0001ab60       ??__F?_System_object@?$_Error_objects@H@std@@2V_System_error_category@2@A@@YAXXZ 1001bb60 f   atom.obj
 0001:0001ab70       ??__F?_Generic_object@?$_Error_objects@H@std@@2V_Generic_error_category@2@A@@YAXXZ 1001bb70 f   atomselection.obj
 0001:0001ab80       ??__F?_Iostream_object@?$_Error_objects@H@std@@2V_Iostream_error_category@2@A@@YAXXZ 1001bb80 f   atomselection.obj
 0001:0001ab90       ??__F?_System_object@?$_Error_objects@H@std@@2V_System_error_category@2@A@@YAXXZ 1001bb90 f   atomselection.obj
 0001:0001aba0       ??__F?_Generic_object@?$_Error_objects@H@std@@2V_Generic_error_category@2@A@@YAXXZ 1001bba0 f   basetypes.obj
 0001:0001abb0       ??__F?_Iostream_object@?$_Error_objects@H@std@@2V_Iostream_error_category@2@A@@YAXXZ 1001bbb0 f   basetypes.obj
 0001:0001abc0       ??__F?_System_object@?$_Error_objects@H@std@@2V_System_error_category@2@A@@YAXXZ 1001bbc0 f   basetypes.obj
 0001:0001abd0       ??__F?_Generic_object@?$_Error_objects@H@std@@2V_Generic_error_category@2@A@@YAXXZ 1001bbd0 f   coord3d.obj
 0001:0001abe0       ??__F?_Iostream_object@?$_Error_objects@H@std@@2V_Iostream_error_category@2@A@@YAXXZ 1001bbe0 f   coord3d.obj
 0001:0001abf0       ??__F?_System_object@?$_Error_objects@H@std@@2V_System_error_category@2@A@@YAXXZ 1001bbf0 f   coord3d.obj
 0001:0001ac00       ??__F?_Generic_object@?$_Error_objects@H@std@@2V_Generic_error_category@2@A@@YAXXZ 1001bc00 f   coordsarray.obj
 0001:0001ac10       ??__F?_Iostream_object@?$_Error_objects@H@std@@2V_Iostream_error_category@2@A@@YAXXZ 1001bc10 f   coordsarray.obj
 0001:0001ac20       ??__F?_System_object@?$_Error_objects@H@std@@2V_System_error_category@2@A@@YAXXZ 1001bc20 f   coordsarray.obj
 0001:0001ac30       ??__F?_Generic_object@?$_Error_objects@H@std@@2V_Generic_error_category@2@A@@YAXXZ 1001bc30 f   geometry.obj
 0001:0001ac40       ??__F?_Iostream_object@?$_Error_objects@H@std@@2V_Iostream_error_category@2@A@@YAXXZ 1001bc40 f   geometry.obj
 0001:0001ac50       ??__F?_System_object@?$_Error_objects@H@std@@2V_System_error_category@2@A@@YAXXZ 1001bc50 f   geometry.obj
 0001:0001ac60       ??__F?_Generic_object@?$_Error_objects@H@std@@2V_Generic_error_category@2@A@@YAXXZ 1001bc60 f   pdbio.obj
 0001:0001ac70       ??__F?_Iostream_object@?$_Error_objects@H@std@@2V_Iostream_error_category@2@A@@YAXXZ 1001bc70 f   pdbio.obj
 0001:0001ac80       ??__F?_System_object@?$_Error_objects@H@std@@2V_System_error_category@2@A@@YAXXZ 1001bc80 f   pdbio.obj
 0001:0001ac90       ??__F?_Generic_object@?$_Error_objects@H@std@@2V_Generic_error_category@2@A@@YAXXZ 1001bc90 f   rigidbody.obj
 0001:0001aca0       ??__F?_Iostream_object@?$_Error_objects@H@std@@2V_Iostream_error_category@2@A@@YAXXZ 1001bca0 f   rigidbody.obj
 0001:0001acb0       ??__F?_System_object@?$_Error_objects@H@std@@2V_System_error_category@2@A@@YAXXZ 1001bcb0 f   rigidbody.obj
 0001:0001acc0       ??__F?_Generic_object@?$_Error_objects@H@std@@2V_Generic_error_category@2@A@@YAXXZ 1001bcc0 f   rmsd.obj
 0001:0001acd0       ??__F?_Iostream_object@?$_Error_objects@H@std@@2V_Iostream_error_category@2@A@@YAXXZ 1001bcd0 f   rmsd.obj
 0001:0001ace0       ??__F?_System_object@?$_Error_objects@H@std@@2V_System_error_category@2@A@@YAXXZ 1001bce0 f   rmsd.obj
 0001:0001acf0       ??__F?_Generic_object@?$_Error_objects@H@std@@2V_Generic_error_category@2@A@@YAXXZ 1001bcf0 f   superpose.obj
 0001:0001ad00       ??__F?_Iostream_object@?$_Error_objects@H@std@@2V_Iostream_error_category@2@A@@YAXXZ 1001bd00 f   superpose.obj
 0001:0001ad10       ??__F?_System_object@?$_Error_objects@H@std@@2V_System_error_category@2@A@@YAXXZ 1001bd10 f   superpose.obj
 0001:0001ad20       ??__F?_Generic_object@?$_Error_objects@H@std@@2V_Generic_error_category@2@A@@YAXXZ 1001bd20 f   moc_PToolsPlugin.obj
 0001:0001ad30       ??__F?_Iostream_object@?$_Error_objects@H@std@@2V_Iostream_error_category@2@A@@YAXXZ 1001bd30 f   moc_PToolsPlugin.obj
 0001:0001ad40       ??__F?_System_object@?$_Error_objects@H@std@@2V_System_error_category@2@A@@YAXXZ 1001bd40 f   moc_PToolsPlugin.obj
 0001:0001ad50       ??__FalgoLog@U2@@YAXXZ     1001bd50 f   moc_PToolsPlugin.obj
 0001:0001ad60       ??__FcmdLog@U2@@YAXXZ      1001bd60 f   moc_PToolsPlugin.obj
 0001:0001ad70       ??__FcoreLog@U2@@YAXXZ     1001bd70 f   moc_PToolsPlugin.obj
 0001:0001ad80       ??__FioLog@U2@@YAXXZ       1001bd80 f   moc_PToolsPlugin.obj
 0001:0001ad90       ??__FperfLog@U2@@YAXXZ     1001bd90 f   moc_PToolsPlugin.obj
 0001:0001ada0       ??__FscriptLog@U2@@YAXXZ   1001bda0 f   moc_PToolsPlugin.obj
 0001:0001adb0       ??__FtaskLog@U2@@YAXXZ     1001bdb0 f   moc_PToolsPlugin.obj
 0001:0001adc0       ??__FuiLog@U2@@YAXXZ       1001bdc0 f   moc_PToolsPlugin.obj
 0001:0001add0       ??__FuserActLog@U2@@YAXXZ  1001bdd0 f   moc_PToolsPlugin.obj
 0001:0001ade0       ??__F?_Generic_object@?$_Error_objects@H@std@@2V_Generic_error_category@2@A@@YAXXZ 1001bde0 f   moc_PToolsTests.obj
 0001:0001adf0       ??__F?_Iostream_object@?$_Error_objects@H@std@@2V_Iostream_error_category@2@A@@YAXXZ 1001bdf0 f   moc_PToolsTests.obj
 0001:0001ae00       ??__F?_System_object@?$_Error_objects@H@std@@2V_System_error_category@2@A@@YAXXZ 1001be00 f   moc_PToolsTests.obj
 0001:0001ae10       ??__FalgoLog@U2@@YAXXZ     1001be10 f   moc_PToolsTests.obj
 0001:0001ae20       ??__FcmdLog@U2@@YAXXZ      1001be20 f   moc_PToolsTests.obj
 0001:0001ae30       ??__FcoreLog@U2@@YAXXZ     1001be30 f   moc_PToolsTests.obj
 0001:0001ae40       ??__FioLog@U2@@YAXXZ       1001be40 f   moc_PToolsTests.obj
 0001:0001ae50       ??__FperfLog@U2@@YAXXZ     1001be50 f   moc_PToolsTests.obj
 0001:0001ae60       ??__FscriptLog@U2@@YAXXZ   1001be60 f   moc_PToolsTests.obj
 0001:0001ae70       ??__FtaskLog@U2@@YAXXZ     1001be70 f   moc_PToolsTests.obj
 0001:0001ae80       ??__FuiLog@U2@@YAXXZ       1001be80 f   moc_PToolsTests.obj
 0001:0001ae90       ??__FuserActLog@U2@@YAXXZ  1001be90 f   moc_PToolsTests.obj
 0001:0001ae9b       ??__F_Fac_tidy_reg@std@@YAXXZ 1001be9b f   msvcprt:locale0_implib.obj
 0002:000003c8       __Fac_tidy_reg$initializer$ 1001c3c8     msvcprt:locale0_implib.obj
 0002:000003cc       _algoLog$initializer$      1001c3cc     PToolsAligner.obj
 0002:000003d0       _cmdLog$initializer$       1001c3d0     PToolsAligner.obj
 0002:000003d4       _coreLog$initializer$      1001c3d4     PToolsAligner.obj
 0002:000003d8       _ioLog$initializer$        1001c3d8     PToolsAligner.obj
 0002:000003dc       _perfLog$initializer$      1001c3dc     PToolsAligner.obj
 0002:000003e0       _scriptLog$initializer$    1001c3e0     PToolsAligner.obj
 0002:000003e4       _taskLog$initializer$      1001c3e4     PToolsAligner.obj
 0002:000003e8       _uiLog$initializer$        1001c3e8     PToolsAligner.obj
 0002:000003ec       _userActLog$initializer$   1001c3ec     PToolsAligner.obj
 0002:000003f0       ?_Generic_object$initializer$@?$_Error_objects@H@std@@2P6AXXZA 1001c3f0     PToolsAligner.obj
 0002:000003f4       ?_Iostream_object$initializer$@?$_Error_objects@H@std@@2P6AXXZA 1001c3f4     PToolsAligner.obj
 0002:000003f8       ?_System_object$initializer$@?$_Error_objects@H@std@@2P6AXXZA 1001c3f8     PToolsAligner.obj
 0002:000003fc       _algoLog$initializer$      1001c3fc     PToolsPlugin.obj
 0002:00000400       _cmdLog$initializer$       1001c400     PToolsPlugin.obj
 0002:00000404       _coreLog$initializer$      1001c404     PToolsPlugin.obj
 0002:00000408       _ioLog$initializer$        1001c408     PToolsPlugin.obj
 0002:0000040c       _perfLog$initializer$      1001c40c     PToolsPlugin.obj
 0002:00000410       _scriptLog$initializer$    1001c410     PToolsPlugin.obj
 0002:00000414       _taskLog$initializer$      1001c414     PToolsPlugin.obj
 0002:00000418       _uiLog$initializer$        1001c418     PToolsPlugin.obj
 0002:0000041c       _userActLog$initializer$   1001c41c     PToolsPlugin.obj
 0002:00000420       _PTOOLS_ID$initializer$    1001c420     PToolsPlugin.obj
 0002:00000424       _algoLog$initializer$      1001c424     PToolsTests.obj
 0002:00000428       _cmdLog$initializer$       1001c428     PToolsTests.obj
 0002:0000042c       _coreLog$initializer$      1001c42c     PToolsTests.obj
 0002:00000430       _ioLog$initializer$        1001c430     PToolsTests.obj
 0002:00000434       _perfLog$initializer$      1001c434     PToolsTests.obj
 0002:00000438       _scriptLog$initializer$    1001c438     PToolsTests.obj
 0002:0000043c       _taskLog$initializer$      1001c43c     PToolsTests.obj
 0002:00000440       _uiLog$initializer$        1001c440     PToolsTests.obj
 0002:00000444       _userActLog$initializer$   1001c444     PToolsTests.obj
 0002:00000448       ?REFO_ATTR$initializer$@Gtest_PToolsAlignerTask@U2@@2P6AXXZA 1001c448     PToolsTests.obj
 0002:0000044c       ?MOBO_ATTR$initializer$@Gtest_PToolsAlignerTask@U2@@2P6AXXZA 1001c44c     PToolsTests.obj
 0002:00000450       ?RMSD_ATTR$initializer$@Gtest_PToolsAlignerTask@U2@@2P6AXXZA 1001c450     PToolsTests.obj
 0002:00000454       ?ACCURACY_ATTR$initializer$@Gtest_PToolsAlignerTask@U2@@2P6AXXZA 1001c454     PToolsTests.obj
 0002:00000458       ?TRANSFORM_ATTR$initializer$@Gtest_PToolsAlignerTask@U2@@2P6AXXZA 1001c458     PToolsTests.obj
 0002:0000045c       _algoLog$initializer$      1001c45c     moc_PToolsPlugin.obj
 0002:00000460       _cmdLog$initializer$       1001c460     moc_PToolsPlugin.obj
 0002:00000464       _coreLog$initializer$      1001c464     moc_PToolsPlugin.obj
 0002:00000468       _ioLog$initializer$        1001c468     moc_PToolsPlugin.obj
 0002:0000046c       _perfLog$initializer$      1001c46c     moc_PToolsPlugin.obj
 0002:00000470       _scriptLog$initializer$    1001c470     moc_PToolsPlugin.obj
 0002:00000474       _taskLog$initializer$      1001c474     moc_PToolsPlugin.obj
 0002:00000478       _uiLog$initializer$        1001c478     moc_PToolsPlugin.obj
 0002:0000047c       _userActLog$initializer$   1001c47c     moc_PToolsPlugin.obj
 0002:00000480       ?staticMetaObject$initializer$@PToolsPlugin@U2@@2P6AXXZA 1001c480     moc_PToolsPlugin.obj
 0002:00000484       _algoLog$initializer$      1001c484     moc_PToolsTests.obj
 0002:00000488       _cmdLog$initializer$       1001c488     moc_PToolsTests.obj
 0002:0000048c       _coreLog$initializer$      1001c48c     moc_PToolsTests.obj
 0002:00000490       _ioLog$initializer$        1001c490     moc_PToolsTests.obj
 0002:00000494       _perfLog$initializer$      1001c494     moc_PToolsTests.obj
 0002:00000498       _scriptLog$initializer$    1001c498     moc_PToolsTests.obj
 0002:0000049c       _taskLog$initializer$      1001c49c     moc_PToolsTests.obj
 0002:000004a0       _uiLog$initializer$        1001c4a0     moc_PToolsTests.obj
 0002:000004a4       _userActLog$initializer$   1001c4a4     moc_PToolsTests.obj
 0002:000004a8       ?staticMetaObject$initializer$@Gtest_PToolsAlignerTask@U2@@2P6AXXZA 1001c4a8     moc_PToolsTests.obj
 0002:000004b4       _pcinit                    1001c4b4     MSVCRT:crtdll.obj
 0002:000004b8       _pinit                     1001c4b8     MSVCRT:atonexit.obj
 0002:00000d38       _qt_meta_stringdata_U2__PToolsPlugin 1001cd38     moc_PToolsPlugin.obj
 0002:00000d5c       _qt_meta_data_U2__PToolsPlugin 1001cd5c     moc_PToolsPlugin.obj
 0002:00000d98       _qt_meta_stringdata_U2__Gtest_PToolsAlignerTask 1001cd98     moc_PToolsTests.obj
 0002:00000dc4       _qt_meta_data_U2__Gtest_PToolsAlignerTask 1001cdc4     moc_PToolsTests.obj
 0002:00000e10       _GS_ExceptionPointers      1001ce10     MSVCRT:gs_report.obj
 0002:00001c88       __catchsym$?_Copy@?$basic_string@DU?$char_traits@D@std@@V?$allocator@D@2@@std@@QAEXII@Z$5 1001dc88     PToolsAligner.obj
 0002:00001c98       __catchsym$?_Copy@?$basic_string@DU?$char_traits@D@std@@V?$allocator@D@2@@std@@QAEXII@Z$4 1001dc98     PToolsAligner.obj
 0002:00001ca8       __unwindtable$?_Copy@?$basic_string@DU?$char_traits@D@std@@V?$allocator@D@2@@std@@QAEXII@Z 1001dca8     PToolsAligner.obj
 0002:00001cc8       __ehfuncinfo$?_Copy@?$basic_string@DU?$char_traits@D@std@@V?$allocator@D@2@@std@@QAEXII@Z 1001dcc8     PToolsAligner.obj
 0002:00001cec       __tryblocktable$?_Copy@?$basic_string@DU?$char_traits@D@std@@V?$allocator@D@2@@std@@QAEXII@Z 1001dcec     PToolsAligner.obj
 0002:00001d14       __unwindtable$??__EalgoLog@U2@@YAXXZ 1001dd14     PToolsAligner.obj
 0002:00001d1c       __ehfuncinfo$??__EalgoLog@U2@@YAXXZ 1001dd1c     PToolsAligner.obj
 0002:00001d40       __unwindtable$??__EcmdLog@U2@@YAXXZ 1001dd40     PToolsAligner.obj
 0002:00001d48       __ehfuncinfo$??__EcmdLog@U2@@YAXXZ 1001dd48     PToolsAligner.obj
 0002:00001d6c       __unwindtable$??__EcoreLog@U2@@YAXXZ 1001dd6c     PToolsAligner.obj
 0002:00001d74       __ehfuncinfo$??__EcoreLog@U2@@YAXXZ 1001dd74     PToolsAligner.obj
 0002:00001d98       __unwindtable$??__EioLog@U2@@YAXXZ 1001dd98     PToolsAligner.obj
 0002:00001da0       __ehfuncinfo$??__EioLog@U2@@YAXXZ 1001dda0     PToolsAligner.obj
 0002:00001dc4       __unwindtable$??__EperfLog@U2@@YAXXZ 1001ddc4     PToolsAligner.obj
 0002:00001dcc       __ehfuncinfo$??__EperfLog@U2@@YAXXZ 1001ddcc     PToolsAligner.obj
 0002:00001df0       __unwindtable$??__EscriptLog@U2@@YAXXZ 1001ddf0     PToolsAligner.obj
 0002:00001df8       __ehfuncinfo$??__EscriptLog@U2@@YAXXZ 1001ddf8     PToolsAligner.obj
 0002:00001e1c       __unwindtable$??__EtaskLog@U2@@YAXXZ 1001de1c     PToolsAligner.obj
 0002:00001e24       __ehfuncinfo$??__EtaskLog@U2@@YAXXZ 1001de24     PToolsAligner.obj
 0002:00001e48       __unwindtable$??__EuiLog@U2@@YAXXZ 1001de48     PToolsAligner.obj
 0002:00001e50       __ehfuncinfo$??__EuiLog@U2@@YAXXZ 1001de50     PToolsAligner.obj
 0002:00001e74       __unwindtable$??__EuserActLog@U2@@YAXXZ 1001de74     PToolsAligner.obj
 0002:00001e7c       __ehfuncinfo$??__EuserActLog@U2@@YAXXZ 1001de7c     PToolsAligner.obj
 0002:00001ea0       __unwindtable$??1Bond@U2@@QAE@XZ 1001dea0     PToolsAligner.obj
 0002:00001ea8       __ehfuncinfo$??1Bond@U2@@QAE@XZ 1001dea8     PToolsAligner.obj
 0002:00001ecc       __catchsym$??0?$QList@V?$QSharedDataPointer@VAtomData@U2@@@@@@QAE@ABV0@@Z$2 1001decc     PToolsAligner.obj
 0002:00001edc       __unwindtable$??0?$QList@V?$QSharedDataPointer@VAtomData@U2@@@@@@QAE@ABV0@@Z 1001dedc     PToolsAligner.obj
 0002:00001eec       __tryblocktable$??0?$QList@V?$QSharedDataPointer@VAtomData@U2@@@@@@QAE@ABV0@@Z 1001deec     PToolsAligner.obj
 0002:00001f00       __ehfuncinfo$??0?$QList@V?$QSharedDataPointer@VAtomData@U2@@@@@@QAE@ABV0@@Z 1001df00     PToolsAligner.obj
 0002:00001f24       __unwindtable$?node_destruct@?$QList@VBond@U2@@@@AAEXPAUNode@1@0@Z 1001df24     PToolsAligner.obj
 0002:00001f34       __ehfuncinfo$?node_destruct@?$QList@VBond@U2@@@@AAEXPAUNode@1@0@Z 1001df34     PToolsAligner.obj
 0002:00001f58       __unwindtable$??1Molecule3DModel@U2@@QAE@XZ 1001df58     PToolsAligner.obj
 0002:00001f60       __ehfuncinfo$??1Molecule3DModel@U2@@QAE@XZ 1001df60     PToolsAligner.obj
 0002:00001f84       __unwindtable$??1MoleculeData@U2@@QAE@XZ 1001df84     PToolsAligner.obj
 0002:00001f94       __ehfuncinfo$??1MoleculeData@U2@@QAE@XZ 1001df94     PToolsAligner.obj
 0002:00001fb8       __catchsym$??0?$QList@H@@QAE@ABV0@@Z$2 1001dfb8     PToolsAligner.obj
 0002:00001fc8       __unwindtable$??0?$QList@H@@QAE@ABV0@@Z 1001dfc8     PToolsAligner.obj
 0002:00001fd8       __tryblocktable$??0?$QList@H@@QAE@ABV0@@Z 1001dfd8     PToolsAligner.obj
 0002:00001fec       __ehfuncinfo$??0?$QList@H@@QAE@ABV0@@Z 1001dfec     PToolsAligner.obj
 0002:00002010       __tryblocktable$?align@PToolsAligner@U2@@UAE?AVStructuralAlignment@2@ABVStructuralAlignmentTaskSettings@2@AAVTaskStateInfo@2@@Z 1001e010     PToolsAligner.obj
 0002:00002024       __catchsym$?align@PToolsAligner@U2@@UAE?AVStructuralAlignment@2@ABVStructuralAlignmentTaskSettings@2@AAVTaskStateInfo@2@@Z$19 1001e024     PToolsAligner.obj
 0002:00002044       __ehfuncinfo$?align@PToolsAligner@U2@@UAE?AVStructuralAlignment@2@ABVStructuralAlignmentTaskSettings@2@AAVTaskStateInfo@2@@Z 1001e044     PToolsAligner.obj
 0002:00002068       __unwindtable$?align@PToolsAligner@U2@@UAE?AVStructuralAlignment@2@ABVStructuralAlignmentTaskSettings@2@AAVTaskStateInfo@2@@Z 1001e068     PToolsAligner.obj
 0002:000020e8       __catchsym$?reallocData@?$QVector@N@@AAEXHHV?$QFlags@W4AllocationOption@QArrayData@@@@@Z$5 1001e0e8     PToolsAligner.obj
 0002:000020f8       __catchsym$?reallocData@?$QVector@N@@AAEXHHV?$QFlags@W4AllocationOption@QArrayData@@@@@Z$4 1001e0f8     PToolsAligner.obj
 0002:00002108       __unwindtable$?reallocData@?$QVector@N@@AAEXHHV?$QFlags@W4AllocationOption@QArrayData@@@@@Z 1001e108     PToolsAligner.obj
 0002:00002128       __ehfuncinfo$?reallocData@?$QVector@N@@AAEXHHV?$QFlags@W4AllocationOption@QArrayData@@@@@Z 1001e128     PToolsAligner.obj
 0002:0000214c       __tryblocktable$?reallocData@?$QVector@N@@AAEXHHV?$QFlags@W4AllocationOption@QArrayData@@@@@Z 1001e14c     PToolsAligner.obj
 0002:00002174       __ehfuncinfo$??0Atomproperty@PTools@@QAE@XZ 1001e174     PToolsAligner.obj
 0002:00002198       __unwindtable$??0Atomproperty@PTools@@QAE@XZ 1001e198     PToolsAligner.obj
 0002:000021c0       __unwindtable$?SetType@Atomproperty@PTools@@QAEXV?$basic_string@DU?$char_traits@D@std@@V?$allocator@D@2@@std@@@Z 1001e1c0     PToolsAligner.obj
 0002:000021c8       __ehfuncinfo$?SetType@Atomproperty@PTools@@QAEXV?$basic_string@DU?$char_traits@D@std@@V?$allocator@D@2@@std@@@Z 1001e1c8     PToolsAligner.obj
 0002:000021ec       __unwindtable$??0Atomproperty@PTools@@QAE@ABV01@@Z 1001e1ec     PToolsAligner.obj
 0002:0000220c       __ehfuncinfo$??0Atomproperty@PTools@@QAE@ABV01@@Z 1001e20c     PToolsAligner.obj
 0002:00002230       __unwindtable$??0Atom@PTools@@QAE@VAtomproperty@1@UCoord3D@1@@Z 1001e230     PToolsAligner.obj
 0002:00002238       __ehfuncinfo$??0Atom@PTools@@QAE@VAtomproperty@1@UCoord3D@1@@Z 1001e238     PToolsAligner.obj
 0002:0000225c       __ehfuncinfo$?createRigidBody@U2@@YAPAVRigidbody@PTools@@ABVBioStruct3DReference@1@@Z 1001e25c     PToolsAligner.obj
 0002:00002280       __unwindtable$?createRigidBody@U2@@YAPAVRigidbody@PTools@@ABVBioStruct3DReference@1@@Z 1001e280     PToolsAligner.obj
 0002:000022c8       __unwindtable$?getSubsetSize@U2@@YAHABVBioStruct3DReference@1@@Z 1001e2c8     PToolsAligner.obj
 0002:000022d8       __ehfuncinfo$?getSubsetSize@U2@@YAHABVBioStruct3DReference@1@@Z 1001e2d8     PToolsAligner.obj
 0002:000022fc       __unwindtable$??__EalgoLog@U2@@YAXXZ 1001e2fc     PToolsPlugin.obj
 0002:00002304       __ehfuncinfo$??__EalgoLog@U2@@YAXXZ 1001e304     PToolsPlugin.obj
 0002:00002328       __unwindtable$??__EcmdLog@U2@@YAXXZ 1001e328     PToolsPlugin.obj
 0002:00002330       __ehfuncinfo$??__EcmdLog@U2@@YAXXZ 1001e330     PToolsPlugin.obj
 0002:00002354       __unwindtable$??__EcoreLog@U2@@YAXXZ 1001e354     PToolsPlugin.obj
 0002:0000235c       __ehfuncinfo$??__EcoreLog@U2@@YAXXZ 1001e35c     PToolsPlugin.obj
 0002:00002380       __unwindtable$??__EioLog@U2@@YAXXZ 1001e380     PToolsPlugin.obj
 0002:00002388       __ehfuncinfo$??__EioLog@U2@@YAXXZ 1001e388     PToolsPlugin.obj
 0002:000023ac       __unwindtable$??__EperfLog@U2@@YAXXZ 1001e3ac     PToolsPlugin.obj
 0002:000023b4       __ehfuncinfo$??__EperfLog@U2@@YAXXZ 1001e3b4     PToolsPlugin.obj
 0002:000023d8       __unwindtable$??__EscriptLog@U2@@YAXXZ 1001e3d8     PToolsPlugin.obj
 0002:000023e0       __ehfuncinfo$??__EscriptLog@U2@@YAXXZ 1001e3e0     PToolsPlugin.obj
 0002:00002404       __unwindtable$??__EtaskLog@U2@@YAXXZ 1001e404     PToolsPlugin.obj
 0002:0000240c       __ehfuncinfo$??__EtaskLog@U2@@YAXXZ 1001e40c     PToolsPlugin.obj
 0002:00002430       __unwindtable$??__EuiLog@U2@@YAXXZ 1001e430     PToolsPlugin.obj
 0002:00002438       __ehfuncinfo$??__EuiLog@U2@@YAXXZ 1001e438     PToolsPlugin.obj
 0002:0000245c       __unwindtable$??__EuserActLog@U2@@YAXXZ 1001e45c     PToolsPlugin.obj
 0002:00002464       __ehfuncinfo$??__EuserActLog@U2@@YAXXZ 1001e464     PToolsPlugin.obj
 0002:00002488       __ehfuncinfo$??0PToolsPlugin@U2@@QAE@XZ 1001e488     PToolsPlugin.obj
 0002:000024ac       __unwindtable$??0PToolsPlugin@U2@@QAE@XZ 1001e4ac     PToolsPlugin.obj
 0002:000024ec       __unwindtable$?createTestFactories@StructualAlignerTests@U2@@SA?AV?$QList@PAVXMLTestFactory@U2@@@@XZ 1001e4ec     PToolsPlugin.obj
 0002:000024f4       __ehfuncinfo$?createTestFactories@StructualAlignerTests@U2@@SA?AV?$QList@PAVXMLTestFactory@U2@@@@XZ 1001e4f4     PToolsPlugin.obj
 0002:00002518       __ehfuncinfo$??0Gtest_PToolsAlignerTask@U2@@QAE@PAVXMLTestFormat@1@ABVQString@@PAVGTest@1@PBVGTestEnvironment@1@ABV?$QList@PAVGTest@U2@@@@ABVQDomElement@@@Z 1001e518     PToolsPlugin.obj
 0002:0000253c       __unwindtable$??0Gtest_PToolsAlignerTask@U2@@QAE@PAVXMLTestFormat@1@ABVQString@@PAVGTest@1@PBVGTestEnvironment@1@ABV?$QList@PAVGTest@U2@@@@ABVQDomElement@@@Z 1001e53c     PToolsPlugin.obj
 0002:00002564       __unwindtable$??0Gtest_PToolsAlignerTaskFactory@Gtest_PToolsAlignerTask@U2@@QAE@XZ 1001e564     PToolsPlugin.obj
 0002:0000257c       __ehfuncinfo$??0Gtest_PToolsAlignerTaskFactory@Gtest_PToolsAlignerTask@U2@@QAE@XZ 1001e57c     PToolsPlugin.obj
 0002:000025a0       __unwindtable$?createTest@Gtest_PToolsAlignerTaskFactory@Gtest_PToolsAlignerTask@U2@@UAEPAVGTest@3@PAVXMLTestFormat@3@ABVQString@@PAV43@PBVGTestEnvironment@3@ABV?$QList@PAVGTest@U2@@@@ABVQDomElement@@@Z 1001e5a0     PToolsPlugin.obj
 0002:000025a8       __ehfuncinfo$?createTest@Gtest_PToolsAlignerTaskFactory@Gtest_PToolsAlignerTask@U2@@UAEPAVGTest@3@PAVXMLTestFormat@3@ABVQString@@PAV43@PBVGTestEnvironment@3@ABV?$QList@PAVGTest@U2@@@@ABVQDomElement@@@Z 1001e5a8     PToolsPlugin.obj
 0002:000025cc       __unwindtable$?createFactory@Gtest_PToolsAlignerTask@U2@@SAPAVXMLTestFactory@2@XZ 1001e5cc     PToolsPlugin.obj
 0002:000025ec       __ehfuncinfo$?createFactory@Gtest_PToolsAlignerTask@U2@@SAPAVXMLTestFactory@2@XZ 1001e5ec     PToolsPlugin.obj
 0002:00002610       __unwindtable$??1Gtest_PToolsAlignerTask@U2@@UAE@XZ 1001e610     PToolsPlugin.obj
 0002:00002630       __ehfuncinfo$??1Gtest_PToolsAlignerTask@U2@@UAE@XZ 1001e630     PToolsPlugin.obj
 0002:00002654       __unwindtable$??_GGtest_PToolsAlignerTask@U2@@UAEPAXI@Z 1001e654     PToolsPlugin.obj
 0002:00002674       __ehfuncinfo$??_GGtest_PToolsAlignerTask@U2@@UAEPAXI@Z 1001e674     PToolsPlugin.obj
 0002:00002698       __unwindtable$??1?$GAutoDeleteList@VXMLTestFactory@U2@@@U2@@UAE@XZ 1001e698     PToolsPlugin.obj
 0002:000026a8       __ehfuncinfo$??1?$GAutoDeleteList@VXMLTestFactory@U2@@@U2@@UAE@XZ 1001e6a8     PToolsPlugin.obj
 0002:000026cc       __catchsym$??0?$QList@PAVXMLTestFactory@U2@@@@QAE@ABV0@@Z$2 1001e6cc     PToolsPlugin.obj
 0002:000026dc       __unwindtable$??0?$QList@PAVXMLTestFactory@U2@@@@QAE@ABV0@@Z 1001e6dc     PToolsPlugin.obj
 0002:000026ec       __tryblocktable$??0?$QList@PAVXMLTestFactory@U2@@@@QAE@ABV0@@Z 1001e6ec     PToolsPlugin.obj
 0002:00002700       __ehfuncinfo$??0?$QList@PAVXMLTestFactory@U2@@@@QAE@ABV0@@Z 1001e700     PToolsPlugin.obj
 0002:00002724       __catchsym$?append@?$QList@PAVXMLTestFactory@U2@@@@QAEXABQAVXMLTestFactory@U2@@@Z$6 1001e724     PToolsPlugin.obj
 0002:00002734       __tryblocktable$?append@?$QList@PAVXMLTestFactory@U2@@@@QAEXABQAVXMLTestFactory@U2@@@Z 1001e734     PToolsPlugin.obj
 0002:00002748       __ehfuncinfo$?append@?$QList@PAVXMLTestFactory@U2@@@@QAEXABQAVXMLTestFactory@U2@@@Z 1001e748     PToolsPlugin.obj
 0002:0000276c       __unwindtable$?append@?$QList@PAVXMLTestFactory@U2@@@@QAEXABQAVXMLTestFactory@U2@@@Z 1001e76c     PToolsPlugin.obj
 0002:0000279c       __catchsym$?detach_helper_grow@?$QList@PAVXMLTestFactory@U2@@@@AAEPAUNode@1@HH@Z$5 1001e79c     PToolsPlugin.obj
 0002:000027ac       __catchsym$?detach_helper_grow@?$QList@PAVXMLTestFactory@U2@@@@AAEPAUNode@1@HH@Z$4 1001e7ac     PToolsPlugin.obj
 0002:000027bc       __unwindtable$?detach_helper_grow@?$QList@PAVXMLTestFactory@U2@@@@AAEPAUNode@1@HH@Z 1001e7bc     PToolsPlugin.obj
 0002:000027dc       __ehfuncinfo$?detach_helper_grow@?$QList@PAVXMLTestFactory@U2@@@@AAEPAUNode@1@HH@Z 1001e7dc     PToolsPlugin.obj
 0002:00002800       __tryblocktable$?detach_helper_grow@?$QList@PAVXMLTestFactory@U2@@@@AAEPAUNode@1@HH@Z 1001e800     PToolsPlugin.obj
 0002:00002828       __unwindtable$??H@YA?BVQString@@ABV0@0@Z 1001e828     PToolsTests.obj
 0002:00002830       __ehfuncinfo$??H@YA?BVQString@@ABV0@0@Z 1001e830     PToolsTests.obj
 0002:00002854       __unwindtable$??H@YA?BVQString@@ABV0@PBD@Z 1001e854     PToolsTests.obj
 0002:00002864       __ehfuncinfo$??H@YA?BVQString@@ABV0@PBD@Z 1001e864     PToolsTests.obj
 0002:00002888       __unwindtable$??H@YA?BVQString@@PBDABV0@@Z 1001e888     PToolsTests.obj
 0002:00002890       __ehfuncinfo$??H@YA?BVQString@@PBDABV0@@Z 1001e890     PToolsTests.obj
 0002:000028b4       __catchsym$??0?$QList@VQString@@@@QAE@ABV0@@Z$2 1001e8b4     PToolsTests.obj
 0002:000028c4       __unwindtable$??0?$QList@VQString@@@@QAE@ABV0@@Z 1001e8c4     PToolsTests.obj
 0002:000028d4       __tryblocktable$??0?$QList@VQString@@@@QAE@ABV0@@Z 1001e8d4     PToolsTests.obj
 0002:000028e8       __ehfuncinfo$??0?$QList@VQString@@@@QAE@ABV0@@Z 1001e8e8     PToolsTests.obj
 0002:0000290c       __catchsym$?node_copy@?$QList@VQString@@@@AAEXPAUNode@1@00@Z$6 1001e90c     PToolsTests.obj
 0002:0000291c       __tryblocktable$?node_copy@?$QList@VQString@@@@AAEXPAUNode@1@00@Z 1001e91c     PToolsTests.obj
 0002:00002930       __ehfuncinfo$?node_copy@?$QList@VQString@@@@AAEXPAUNode@1@00@Z 1001e930     PToolsTests.obj
 0002:00002954       __unwindtable$?node_copy@?$QList@VQString@@@@AAEXPAUNode@1@00@Z 1001e954     PToolsTests.obj
 0002:00002984       __unwindtable$?keys@?$QMap@HV?$QSharedDataPointer@VMoleculeData@U2@@@@@@QBE?AV?$QList@H@@XZ 1001e984     PToolsTests.obj
 0002:0000298c       __ehfuncinfo$?keys@?$QMap@HV?$QSharedDataPointer@VMoleculeData@U2@@@@@@QBE?AV?$QList@H@@XZ 1001e98c     PToolsTests.obj
 0002:000029b0       __unwindtable$?keys@?$QMap@HV?$QHash@HV?$QSharedDataPointer@VAtomData@U2@@@@@@@@QBE?AV?$QList@H@@XZ 1001e9b0     PToolsTests.obj
 0002:000029b8       __ehfuncinfo$?keys@?$QMap@HV?$QHash@HV?$QSharedDataPointer@VAtomData@U2@@@@@@@@QBE?AV?$QList@H@@XZ 1001e9b8     PToolsTests.obj
 0002:000029dc       __unwindtable$??__EalgoLog@U2@@YAXXZ 1001e9dc     PToolsTests.obj
 0002:000029e4       __ehfuncinfo$??__EalgoLog@U2@@YAXXZ 1001e9e4     PToolsTests.obj
 0002:00002a08       __unwindtable$??__EcmdLog@U2@@YAXXZ 1001ea08     PToolsTests.obj
 0002:00002a10       __ehfuncinfo$??__EcmdLog@U2@@YAXXZ 1001ea10     PToolsTests.obj
 0002:00002a34       __unwindtable$??__EcoreLog@U2@@YAXXZ 1001ea34     PToolsTests.obj
 0002:00002a3c       __ehfuncinfo$??__EcoreLog@U2@@YAXXZ 1001ea3c     PToolsTests.obj
 0002:00002a60       __unwindtable$??__EioLog@U2@@YAXXZ 1001ea60     PToolsTests.obj
 0002:00002a68       __ehfuncinfo$??__EioLog@U2@@YAXXZ 1001ea68     PToolsTests.obj
 0002:00002a8c       __unwindtable$??__EperfLog@U2@@YAXXZ 1001ea8c     PToolsTests.obj
 0002:00002a94       __ehfuncinfo$??__EperfLog@U2@@YAXXZ 1001ea94     PToolsTests.obj
 0002:00002ab8       __unwindtable$??__EscriptLog@U2@@YAXXZ 1001eab8     PToolsTests.obj
 0002:00002ac0       __ehfuncinfo$??__EscriptLog@U2@@YAXXZ 1001eac0     PToolsTests.obj
 0002:00002ae4       __unwindtable$??__EtaskLog@U2@@YAXXZ 1001eae4     PToolsTests.obj
 0002:00002aec       __ehfuncinfo$??__EtaskLog@U2@@YAXXZ 1001eaec     PToolsTests.obj
 0002:00002b10       __unwindtable$??__EuiLog@U2@@YAXXZ 1001eb10     PToolsTests.obj
 0002:00002b18       __ehfuncinfo$??__EuiLog@U2@@YAXXZ 1001eb18     PToolsTests.obj
 0002:00002b3c       __unwindtable$??__EuserActLog@U2@@YAXXZ 1001eb3c     PToolsTests.obj
 0002:00002b44       __ehfuncinfo$??__EuserActLog@U2@@YAXXZ 1001eb44     PToolsTests.obj
 0002:00002b68       __catchsym$?append@?$QList@H@@QAEXABH@Z$6 1001eb68     PToolsTests.obj
 0002:00002b78       __tryblocktable$?append@?$QList@H@@QAEXABH@Z 1001eb78     PToolsTests.obj
 0002:00002b8c       __ehfuncinfo$?append@?$QList@H@@QAEXABH@Z 1001eb8c     PToolsTests.obj
 0002:00002bb0       __unwindtable$?append@?$QList@H@@QAEXABH@Z 1001ebb0     PToolsTests.obj
 0002:00002be0       __catchsym$?detach_helper_grow@?$QList@H@@AAEPAUNode@1@HH@Z$5 1001ebe0     PToolsTests.obj
 0002:00002bf0       __catchsym$?detach_helper_grow@?$QList@H@@AAEPAUNode@1@HH@Z$4 1001ebf0     PToolsTests.obj
 0002:00002c00       __unwindtable$?detach_helper_grow@?$QList@H@@AAEPAUNode@1@HH@Z 1001ec00     PToolsTests.obj
 0002:00002c20       __ehfuncinfo$?detach_helper_grow@?$QList@H@@AAEPAUNode@1@HH@Z 1001ec20     PToolsTests.obj
 0002:00002c44       __tryblocktable$?detach_helper_grow@?$QList@H@@AAEPAUNode@1@HH@Z 1001ec44     PToolsTests.obj
 0002:00002c6c       __catchsym$?detach_helper@?$QList@H@@AAEXH@Z$2 1001ec6c     PToolsTests.obj
 0002:00002c7c       __unwindtable$?detach_helper@?$QList@H@@AAEXH@Z 1001ec7c     PToolsTests.obj
 0002:00002c8c       __tryblocktable$?detach_helper@?$QList@H@@AAEXH@Z 1001ec8c     PToolsTests.obj
 0002:00002ca0       __ehfuncinfo$?detach_helper@?$QList@H@@AAEXH@Z 1001eca0     PToolsTests.obj
 0002:00002cc4       __ehfuncinfo$?init@Gtest_PToolsAlignerTask@U2@@QAEXPAVXMLTestFormat@2@ABVQDomElement@@@Z 1001ecc4     PToolsTests.obj
 0002:00002ce8       __unwindtable$?init@Gtest_PToolsAlignerTask@U2@@QAEXPAVXMLTestFormat@2@ABVQDomElement@@@Z 1001ece8     PToolsTests.obj
 0002:00002db8       __ehfuncinfo$?run@Gtest_PToolsAlignerTask@U2@@UAEXXZ 1001edb8     PToolsTests.obj
 0002:00002ddc       __unwindtable$?run@Gtest_PToolsAlignerTask@U2@@UAEXXZ 1001eddc     PToolsTests.obj
 0002:00002e74       __ehfuncinfo$?report@Gtest_PToolsAlignerTask@U2@@UAE?AW4ReportResult@Task@2@XZ 1001ee74     PToolsTests.obj
 0002:00002e98       __unwindtable$?report@Gtest_PToolsAlignerTask@U2@@UAE?AW4ReportResult@Task@2@XZ 1001ee98     PToolsTests.obj
 0002:00002ed0       __ehfuncinfo$?alignmentToStr@U2@@YA?AVQString@@ABVStructuralAlignment@1@N@Z 1001eed0     PToolsTests.obj
 0002:00002ef4       __unwindtable$?alignmentToStr@U2@@YA?AVQString@@ABVStructuralAlignment@1@N@Z 1001eef4     PToolsTests.obj
 0002:00002f1c       __unwindtable$??0AtomSelection@PTools@@QAE@ABV01@@Z 1001ef1c     atomselection.obj
 0002:00002f24       __ehfuncinfo$??0AtomSelection@PTools@@QAE@ABV01@@Z 1001ef24     atomselection.obj
 0002:00002f48       __unwindtable$??0AtomSelection@PTools@@QAE@ABVRigidbody@1@@Z 1001ef48     atomselection.obj
 0002:00002f50       __ehfuncinfo$??0AtomSelection@PTools@@QAE@ABVRigidbody@1@@Z 1001ef50     atomselection.obj
 0002:00002f74       __unwindtable$?CreateRigid@AtomSelection@PTools@@QAE?AVRigidbody@2@XZ 1001ef74     atomselection.obj
 0002:00002f84       __ehfuncinfo$?CreateRigid@AtomSelection@PTools@@QAE?AVRigidbody@2@XZ 1001ef84     atomselection.obj
 0002:00002fa8       __unwindtable$??IPTools@@YA?AVAtomSelection@0@ABV10@0@Z 1001efa8     atomselection.obj
 0002:00002fc0       __ehfuncinfo$??IPTools@@YA?AVAtomSelection@0@ABV10@0@Z 1001efc0     atomselection.obj
 0002:00002fe4       __ehfuncinfo$??UPTools@@YA?AVAtomSelection@0@ABV10@0@Z 1001efe4     atomselection.obj
 0002:00003008       __unwindtable$??UPTools@@YA?AVAtomSelection@0@ABV10@0@Z 1001f008     atomselection.obj
 0002:00003048       __unwindtable$??7PTools@@YA?AVAtomSelection@0@ABV10@@Z 1001f048     atomselection.obj
 0002:00003058       __ehfuncinfo$??7PTools@@YA?AVAtomSelection@0@ABV10@@Z 1001f058     atomselection.obj
 0002:0000307c       __unwindtable$?toString@Coord3D@PTools@@QAE?AV?$basic_string@DU?$char_traits@D@std@@V?$allocator@D@2@@std@@_N@Z 1001f07c     coord3d.obj
 0002:0000309c       __ehfuncinfo$?toString@Coord3D@PTools@@QAE?AV?$basic_string@DU?$char_traits@D@std@@V?$allocator@D@2@@std@@_N@Z 1001f09c     coord3d.obj
 0002:000030c0       __unwindtable$??0?$basic_stringstream@DU?$char_traits@D@std@@V?$allocator@D@2@@std@@QAE@H@Z 1001f0c0     coord3d.obj
 0002:000030d8       __ehfuncinfo$??0?$basic_stringstream@DU?$char_traits@D@std@@V?$allocator@D@2@@std@@QAE@H@Z 1001f0d8     coord3d.obj
 0002:000030fc       __unwindtable$??0?$basic_stringbuf@DU?$char_traits@D@std@@V?$allocator@D@2@@std@@QAE@H@Z 1001f0fc     coord3d.obj
 0002:00003104       __ehfuncinfo$??0?$basic_stringbuf@DU?$char_traits@D@std@@V?$allocator@D@2@@std@@QAE@H@Z 1001f104     coord3d.obj
 0002:00003128       __catchsym$??$?6U?$char_traits@D@std@@@std@@YAAAV?$basic_ostream@DU?$char_traits@D@std@@@0@AAV10@PBD@Z$4 1001f128     coord3d.obj
 0002:00003138       __tryblocktable$??$?6U?$char_traits@D@std@@@std@@YAAAV?$basic_ostream@DU?$char_traits@D@std@@@0@AAV10@PBD@Z 1001f138     coord3d.obj
 0002:0000314c       __unwindtable$??$?6U?$char_traits@D@std@@@std@@YAAAV?$basic_ostream@DU?$char_traits@D@std@@@0@AAV10@PBD@Z 1001f14c     coord3d.obj
 0002:0000316c       __ehfuncinfo$??$?6U?$char_traits@D@std@@@std@@YAAAV?$basic_ostream@DU?$char_traits@D@std@@@0@AAV10@PBD@Z 1001f16c     coord3d.obj
 0002:00003190       __unwindtable$??0sentry@?$basic_ostream@DU?$char_traits@D@std@@@std@@QAE@AAV12@@Z 1001f190     coord3d.obj
 0002:00003198       __ehfuncinfo$??0sentry@?$basic_ostream@DU?$char_traits@D@std@@@std@@QAE@AAV12@@Z 1001f198     coord3d.obj
 0002:000031bc       __unwindtable$??0?$Array2D@N@@QAE@HH@Z 1001f1bc     coordsarray.obj
 0002:000031c4       __ehfuncinfo$??0?$Array2D@N@@QAE@HH@Z 1001f1c4     coordsarray.obj
 0002:000031e8       __catchsym$??4?$vector@UCoord3D@PTools@@V?$allocator@UCoord3D@PTools@@@std@@@std@@QAEAAV01@ABV01@@Z$2 1001f1e8     coordsarray.obj
 0002:000031f8       __unwindtable$??4?$vector@UCoord3D@PTools@@V?$allocator@UCoord3D@PTools@@@std@@@std@@QAEAAV01@ABV01@@Z 1001f1f8     coordsarray.obj
 0002:00003208       __tryblocktable$??4?$vector@UCoord3D@PTools@@V?$allocator@UCoord3D@PTools@@@std@@@std@@QAEAAV01@ABV01@@Z 1001f208     coordsarray.obj
 0002:0000321c       __ehfuncinfo$??4?$vector@UCoord3D@PTools@@V?$allocator@UCoord3D@PTools@@@std@@@std@@QAEAAV01@ABV01@@Z 1001f21c     coordsarray.obj
 0002:00003240       __unwindtable$??0CoordsArray@PTools@@QAE@ABV01@@Z 1001f240     coordsarray.obj
 0002:00003250       __ehfuncinfo$??0CoordsArray@PTools@@QAE@ABV01@@Z 1001f250     coordsarray.obj
 0002:00003274       __unwindtable$?GetCoords@CoordsArray@PTools@@QBEXIAAUCoord3D@2@@Z 1001f274     coordsarray.obj
 0002:0000327c       __ehfuncinfo$?GetCoords@CoordsArray@PTools@@QBEXIAAUCoord3D@2@@Z 1001f27c     coordsarray.obj
 0002:000032a0       __unwindtable$?GetMatrix@CoordsArray@PTools@@QBE?AV?$Array2D@N@@XZ 1001f2a0     coordsarray.obj
 0002:000032b0       __ehfuncinfo$?GetMatrix@CoordsArray@PTools@@QBE?AV?$Array2D@N@@XZ 1001f2b0     coordsarray.obj
 0002:00003348       __unwindtable$??0sentry@?$basic_istream@DU?$char_traits@D@std@@@std@@QAE@AAV12@_N@Z 1001f348     pdbio.obj
 0002:00003350       __ehfuncinfo$??0sentry@?$basic_istream@DU?$char_traits@D@std@@@std@@QAE@AAV12@_N@Z 1001f350     pdbio.obj
 0002:00003374       __unwindtable$?SetResidType@Atomproperty@PTools@@QAEXV?$basic_string@DU?$char_traits@D@std@@V?$allocator@D@2@@std@@@Z 1001f374     pdbio.obj
 0002:0000337c       __ehfuncinfo$?SetResidType@Atomproperty@PTools@@QAEXV?$basic_string@DU?$char_traits@D@std@@V?$allocator@D@2@@std@@@Z 1001f37c     pdbio.obj
 0002:000033a0       __unwindtable$?SetChainId@Atomproperty@PTools@@QAEXV?$basic_string@DU?$char_traits@D@std@@V?$allocator@D@2@@std@@@Z 1001f3a0     pdbio.obj
 0002:000033a8       __ehfuncinfo$?SetChainId@Atomproperty@PTools@@QAEXV?$basic_string@DU?$char_traits@D@std@@V?$allocator@D@2@@std@@@Z 1001f3a8     pdbio.obj
 0002:000033cc       __unwindtable$?SetExtra@Atomproperty@PTools@@QAEXV?$basic_string@DU?$char_traits@D@std@@V?$allocator@D@2@@std@@@Z 1001f3cc     pdbio.obj
 0002:000033d4       __ehfuncinfo$?SetExtra@Atomproperty@PTools@@QAEXV?$basic_string@DU?$char_traits@D@std@@V?$allocator@D@2@@std@@@Z 1001f3d4     pdbio.obj
 0002:000033f8       __ehfuncinfo$?ReadPDB@PTools@@YAXAAV?$basic_ifstream@DU?$char_traits@D@std@@@std@@AAVRigidbody@1@@Z 1001f3f8     pdbio.obj
 0002:0000341c       __unwindtable$?ReadPDB@PTools@@YAXAAV?$basic_ifstream@DU?$char_traits@D@std@@@std@@AAVRigidbody@1@@Z 1001f41c     pdbio.obj
 0002:0000346c       __ehfuncinfo$?ReadPDB@PTools@@YAXV?$basic_string@DU?$char_traits@D@std@@V?$allocator@D@2@@std@@AAVRigidbody@1@@Z 1001f46c     pdbio.obj
 0002:00003490       __unwindtable$?ReadPDB@PTools@@YAXV?$basic_string@DU?$char_traits@D@std@@V?$allocator@D@2@@std@@AAVRigidbody@1@@Z 1001f490     pdbio.obj
 0002:000034c0       __unwindtable$?WritePDB@PTools@@YAXABVRigidbody@1@V?$basic_string@DU?$char_traits@D@std@@V?$allocator@D@2@@std@@@Z 1001f4c0     pdbio.obj
 0002:000034d0       __ehfuncinfo$?WritePDB@PTools@@YAXABVRigidbody@1@V?$basic_string@DU?$char_traits@D@std@@V?$allocator@D@2@@std@@@Z 1001f4d0     pdbio.obj
 0002:000034f4       __unwindtable$?strip@PTools@@YA?AV?$basic_string@DU?$char_traits@D@std@@V?$allocator@D@2@@std@@ABV23@PBD@Z 1001f4f4     pdbio.obj
 0002:000034fc       __ehfuncinfo$?strip@PTools@@YA?AV?$basic_string@DU?$char_traits@D@std@@V?$allocator@D@2@@std@@ABV23@PBD@Z 1001f4fc     pdbio.obj
 0002:00003520       __unwindtable$?isAtom@PTools@@YA_NABV?$basic_string@DU?$char_traits@D@std@@V?$allocator@D@2@@std@@@Z 1001f520     pdbio.obj
 0002:00003530       __ehfuncinfo$?isAtom@PTools@@YA_NABV?$basic_string@DU?$char_traits@D@std@@V?$allocator@D@2@@std@@@Z 1001f530     pdbio.obj
 0002:00003554       __unwindtable$?isHeteroAtom@PTools@@YA_NABV?$basic_string@DU?$char_traits@D@std@@V?$allocator@D@2@@std@@@Z 1001f554     pdbio.obj
 0002:0000355c       __ehfuncinfo$?isHeteroAtom@PTools@@YA_NABV?$basic_string@DU?$char_traits@D@std@@V?$allocator@D@2@@std@@@Z 1001f55c     pdbio.obj
 0002:00003580       __unwindtable$?readatomtype@PTools@@YA?AV?$basic_string@DU?$char_traits@D@std@@V?$allocator@D@2@@std@@ABV23@@Z 1001f580     pdbio.obj
 0002:00003588       __ehfuncinfo$?readatomtype@PTools@@YA?AV?$basic_string@DU?$char_traits@D@std@@V?$allocator@D@2@@std@@ABV23@@Z 1001f588     pdbio.obj
 0002:000035ac       __unwindtable$?readresidtype@PTools@@YA?AV?$basic_string@DU?$char_traits@D@std@@V?$allocator@D@2@@std@@ABV23@@Z 1001f5ac     pdbio.obj
 0002:000035b4       __ehfuncinfo$?readresidtype@PTools@@YA?AV?$basic_string@DU?$char_traits@D@std@@V?$allocator@D@2@@std@@ABV23@@Z 1001f5b4     pdbio.obj
 0002:000035d8       __unwindtable$??0?$basic_ifstream@DU?$char_traits@D@std@@@std@@QAE@PBDHH@Z 1001f5d8     pdbio.obj
 0002:000035f8       __ehfuncinfo$??0?$basic_ifstream@DU?$char_traits@D@std@@@std@@QAE@PBDHH@Z 1001f5f8     pdbio.obj
 0002:0000361c       __unwindtable$??0?$basic_filebuf@DU?$char_traits@D@std@@@std@@QAE@PAU_iobuf@@@Z 1001f61c     pdbio.obj
 0002:00003624       __ehfuncinfo$??0?$basic_filebuf@DU?$char_traits@D@std@@@std@@QAE@PAU_iobuf@@@Z 1001f624     pdbio.obj
 0002:00003648       __unwindtable$?open@?$basic_filebuf@DU?$char_traits@D@std@@@std@@QAEPAV12@PBDHH@Z 1001f648     pdbio.obj
 0002:00003650       __ehfuncinfo$?open@?$basic_filebuf@DU?$char_traits@D@std@@@std@@QAEPAV12@PBDHH@Z 1001f650     pdbio.obj
 0002:00003674       __unwindtable$?overflow@?$basic_filebuf@DU?$char_traits@D@std@@@std@@MAEHH@Z 1001f674     pdbio.obj
 0002:0000367c       __ehfuncinfo$?overflow@?$basic_filebuf@DU?$char_traits@D@std@@@std@@MAEHH@Z 1001f67c     pdbio.obj
 0002:000036a0       __unwindtable$?uflow@?$basic_filebuf@DU?$char_traits@D@std@@@std@@MAEHXZ 1001f6a0     pdbio.obj
 0002:000036a8       __ehfuncinfo$?uflow@?$basic_filebuf@DU?$char_traits@D@std@@@std@@MAEHXZ 1001f6a8     pdbio.obj
 0002:000036cc       __unwindtable$?_Endwrite@?$basic_filebuf@DU?$char_traits@D@std@@@std@@IAE_NXZ 1001f6cc     pdbio.obj
 0002:000036d4       __ehfuncinfo$?_Endwrite@?$basic_filebuf@DU?$char_traits@D@std@@@std@@IAE_NXZ 1001f6d4     pdbio.obj
 0002:000036f8       __unwindtable$??0?$basic_ostringstream@DU?$char_traits@D@std@@V?$allocator@D@2@@std@@QAE@H@Z 1001f6f8     pdbio.obj
 0002:00003710       __ehfuncinfo$??0?$basic_ostringstream@DU?$char_traits@D@std@@V?$allocator@D@2@@std@@QAE@H@Z 1001f710     pdbio.obj
 0002:00003734       __unwindtable$??$?HDU?$char_traits@D@std@@V?$allocator@D@1@@std@@YA?AV?$basic_string@DU?$char_traits@D@std@@V?$allocator@D@2@@0@PBDABV10@@Z 1001f734     pdbio.obj
 0002:0000373c       __ehfuncinfo$??$?HDU?$char_traits@D@std@@V?$allocator@D@1@@std@@YA?AV?$basic_string@DU?$char_traits@D@std@@V?$allocator@D@2@@0@PBDABV10@@Z 1001f73c     pdbio.obj
 0002:00003760       __unwindtable$??$use_facet@V?$codecvt@DDH@std@@@std@@YAABV?$codecvt@DDH@0@ABVlocale@0@@Z 1001f760     pdbio.obj
 0002:00003768       __ehfuncinfo$??$use_facet@V?$codecvt@DDH@std@@@std@@YAABV?$codecvt@DDH@0@ABVlocale@0@@Z 1001f768     pdbio.obj
 0002:0000378c       __catchsym$??$getline@DU?$char_traits@D@std@@V?$allocator@D@2@@std@@YAAAV?$basic_istream@DU?$char_traits@D@std@@@0@$$QAV10@AAV?$basic_string@DU?$char_traits@D@std@@V?$allocator@D@2@@0@D@Z$4 1001f78c     pdbio.obj
 0002:0000379c       __tryblocktable$??$getline@DU?$char_traits@D@std@@V?$allocator@D@2@@std@@YAAAV?$basic_istream@DU?$char_traits@D@std@@@0@$$QAV10@AAV?$basic_string@DU?$char_traits@D@std@@V?$allocator@D@2@@0@D@Z 1001f79c     pdbio.obj
 0002:000037b0       __unwindtable$??$getline@DU?$char_traits@D@std@@V?$allocator@D@2@@std@@YAAAV?$basic_istream@DU?$char_traits@D@std@@@0@$$QAV10@AAV?$basic_string@DU?$char_traits@D@std@@V?$allocator@D@2@@0@D@Z 1001f7b0     pdbio.obj
 0002:000037d0       __ehfuncinfo$??$getline@DU?$char_traits@D@std@@V?$allocator@D@2@@std@@YAAAV?$basic_istream@DU?$char_traits@D@std@@@0@$$QAV10@AAV?$basic_string@DU?$char_traits@D@std@@V?$allocator@D@2@@0@D@Z 1001f7d0     pdbio.obj
 0002:00003868       __catchsym$?_Reallocate@?$vector@UCoord3D@PTools@@V?$allocator@UCoord3D@PTools@@@std@@@std@@IAEXI@Z$2 1001f868     rigidbody.obj
 0002:00003878       __unwindtable$?_Reallocate@?$vector@UCoord3D@PTools@@V?$allocator@UCoord3D@PTools@@@std@@@std@@IAEXI@Z 1001f878     rigidbody.obj
 0002:00003888       __tryblocktable$?_Reallocate@?$vector@UCoord3D@PTools@@V?$allocator@UCoord3D@PTools@@@std@@@std@@IAEXI@Z 1001f888     rigidbody.obj
 0002:0000389c       __ehfuncinfo$?_Reallocate@?$vector@UCoord3D@PTools@@V?$allocator@UCoord3D@PTools@@@std@@@std@@IAEXI@Z 1001f89c     rigidbody.obj
 0002:000038c0       __unwindtable$?construct@?$allocator@VAtomproperty@PTools@@@std@@QAEXPAVAtomproperty@PTools@@ABV34@@Z 1001f8c0     rigidbody.obj
 0002:000038c8       __ehfuncinfo$?construct@?$allocator@VAtomproperty@PTools@@@std@@QAEXPAVAtomproperty@PTools@@ABV34@@Z 1001f8c8     rigidbody.obj
 0002:000038ec       __catchsym$??4?$vector@VAtomproperty@PTools@@V?$allocator@VAtomproperty@PTools@@@std@@@std@@QAEAAV01@ABV01@@Z$2 1001f8ec     rigidbody.obj
 0002:000038fc       __unwindtable$??4?$vector@VAtomproperty@PTools@@V?$allocator@VAtomproperty@PTools@@@std@@@std@@QAEAAV01@ABV01@@Z 1001f8fc     rigidbody.obj
 0002:0000390c       __tryblocktable$??4?$vector@VAtomproperty@PTools@@V?$allocator@VAtomproperty@PTools@@@std@@@std@@QAEAAV01@ABV01@@Z 1001f90c     rigidbody.obj
 0002:00003920       __ehfuncinfo$??4?$vector@VAtomproperty@PTools@@V?$allocator@VAtomproperty@PTools@@@std@@@std@@QAEAAV01@ABV01@@Z 1001f920     rigidbody.obj
 0002:00003944       __unwindtable$?push_back@?$vector@VAtomproperty@PTools@@V?$allocator@VAtomproperty@PTools@@@std@@@std@@QAEXABVAtomproperty@PTools@@@Z 1001f944     rigidbody.obj
 0002:00003954       __ehfuncinfo$?push_back@?$vector@VAtomproperty@PTools@@V?$allocator@VAtomproperty@PTools@@@std@@@std@@QAEXABVAtomproperty@PTools@@@Z 1001f954     rigidbody.obj
 0002:00003978       __catchsym$?_Reallocate@?$vector@VAtomproperty@PTools@@V?$allocator@VAtomproperty@PTools@@@std@@@std@@IAEXI@Z$2 1001f978     rigidbody.obj
 0002:00003988       __unwindtable$?_Reallocate@?$vector@VAtomproperty@PTools@@V?$allocator@VAtomproperty@PTools@@@std@@@std@@IAEXI@Z 1001f988     rigidbody.obj
 0002:00003998       __tryblocktable$?_Reallocate@?$vector@VAtomproperty@PTools@@V?$allocator@VAtomproperty@PTools@@@std@@@std@@IAEXI@Z 1001f998     rigidbody.obj
 0002:000039ac       __ehfuncinfo$?_Reallocate@?$vector@VAtomproperty@PTools@@V?$allocator@VAtomproperty@PTools@@@std@@@std@@IAEXI@Z 1001f9ac     rigidbody.obj
 0002:000039d0       __unwindtable$??0Rigidbody@PTools@@QAE@XZ 1001f9d0     rigidbody.obj
 0002:000039f0       __ehfuncinfo$??0Rigidbody@PTools@@QAE@XZ 1001f9f0     rigidbody.obj
 0002:00003a14       __ehfuncinfo$??0Rigidbody@PTools@@QAE@V?$basic_string@DU?$char_traits@D@std@@V?$allocator@D@2@@std@@@Z 1001fa14     rigidbody.obj
 0002:00003a38       __unwindtable$??0Rigidbody@PTools@@QAE@V?$basic_string@DU?$char_traits@D@std@@V?$allocator@D@2@@std@@@Z 1001fa38     rigidbody.obj
 0002:00003a60       __unwindtable$??0Rigidbody@PTools@@QAE@ABV01@@Z 1001fa60     rigidbody.obj
 0002:00003a80       __ehfuncinfo$??0Rigidbody@PTools@@QAE@ABV01@@Z 1001fa80     rigidbody.obj
 0002:00003aa4       __unwindtable$?CopyAtom@Rigidbody@PTools@@UBE?AVAtom@2@I@Z 1001faa4     rigidbody.obj
 0002:00003aac       __ehfuncinfo$?CopyAtom@Rigidbody@PTools@@UBE?AVAtom@2@I@Z 1001faac     rigidbody.obj
 0002:00003ad0       __unwindtable$?SetAtom@Rigidbody@PTools@@QAEXIABVAtom@2@@Z 1001fad0     rigidbody.obj
 0002:00003ae0       __ehfuncinfo$?SetAtom@Rigidbody@PTools@@QAEXIABVAtom@2@@Z 1001fae0     rigidbody.obj
 0002:00003b04       __unwindtable$?AddAtom@Rigidbody@PTools@@QAEXABVAtom@2@@Z 1001fb04     rigidbody.obj
 0002:00003b0c       __ehfuncinfo$?AddAtom@Rigidbody@PTools@@QAEXABVAtom@2@@Z 1001fb0c     rigidbody.obj
 0002:00003b30       __unwindtable$?SelectAllAtoms@Rigidbody@PTools@@QBE?AVAtomSelection@2@XZ 1001fb30     rigidbody.obj
 0002:00003b38       __ehfuncinfo$?SelectAllAtoms@Rigidbody@PTools@@QBE?AVAtomSelection@2@XZ 1001fb38     rigidbody.obj
 0002:00003b5c       __unwindtable$?SelectAtomType@Rigidbody@PTools@@QAE?AVAtomSelection@2@V?$basic_string@DU?$char_traits@D@std@@V?$allocator@D@2@@std@@@Z 1001fb5c     rigidbody.obj
 0002:00003b74       __ehfuncinfo$?SelectAtomType@Rigidbody@PTools@@QAE?AVAtomSelection@2@V?$basic_string@DU?$char_traits@D@std@@V?$allocator@D@2@@std@@@Z 1001fb74     rigidbody.obj
 0002:00003b98       __unwindtable$?SelectResidType@Rigidbody@PTools@@QAE?AVAtomSelection@2@V?$basic_string@DU?$char_traits@D@std@@V?$allocator@D@2@@std@@@Z 1001fb98     rigidbody.obj
 0002:00003bb0       __ehfuncinfo$?SelectResidType@Rigidbody@PTools@@QAE?AVAtomSelection@2@V?$basic_string@DU?$char_traits@D@std@@V?$allocator@D@2@@std@@@Z 1001fbb0     rigidbody.obj
 0002:00003bd4       __unwindtable$?SelectChainId@Rigidbody@PTools@@QAE?AVAtomSelection@2@V?$basic_string@DU?$char_traits@D@std@@V?$allocator@D@2@@std@@@Z 1001fbd4     rigidbody.obj
 0002:00003bec       __ehfuncinfo$?SelectChainId@Rigidbody@PTools@@QAE?AVAtomSelection@2@V?$basic_string@DU?$char_traits@D@std@@V?$allocator@D@2@@std@@@Z 1001fbec     rigidbody.obj
 0002:00003c10       __unwindtable$?SelectResRange@Rigidbody@PTools@@QAE?AVAtomSelection@2@II@Z 1001fc10     rigidbody.obj
 0002:00003c18       __ehfuncinfo$?SelectResRange@Rigidbody@PTools@@QAE?AVAtomSelection@2@II@Z 1001fc18     rigidbody.obj
 0002:00003c3c       __unwindtable$?Backbone@Rigidbody@PTools@@QAE?AVAtomSelection@2@XZ 1001fc3c     rigidbody.obj
 0002:00003c54       __ehfuncinfo$?Backbone@Rigidbody@PTools@@QAE?AVAtomSelection@2@XZ 1001fc54     rigidbody.obj
 0002:00003c78       __unwindtable$??HRigidbody@PTools@@QAE?AV01@ABV01@@Z 1001fc78     rigidbody.obj
 0002:00003c80       __ehfuncinfo$??HRigidbody@PTools@@QAE?AV01@ABV01@@Z 1001fc80     rigidbody.obj
 0002:00003ca4       __unwindtable$?isBackbone@PTools@@YA_NABV?$basic_string@DU?$char_traits@D@std@@V?$allocator@D@2@@std@@@Z 1001fca4     rigidbody.obj
 0002:00003cc4       __ehfuncinfo$?isBackbone@PTools@@YA_NABV?$basic_string@DU?$char_traits@D@std@@V?$allocator@D@2@@std@@@Z 1001fcc4     rigidbody.obj
 0002:00003ce8       __unwindtable$??$construct@VAtomproperty@PTools@@AAV12@@?$_Wrap_alloc@V?$allocator@VAtomproperty@PTools@@@std@@@std@@QAEXPAVAtomproperty@PTools@@AAV23@@Z 1001fce8     rigidbody.obj
 0002:00003cf0       __ehfuncinfo$??$construct@VAtomproperty@PTools@@AAV12@@?$_Wrap_alloc@V?$allocator@VAtomproperty@PTools@@@std@@@std@@QAEXPAVAtomproperty@PTools@@AAV23@@Z 1001fcf0     rigidbody.obj
 0002:00003d14       __unwindtable$??$construct@VAtomproperty@PTools@@ABV12@@?$_Wrap_alloc@V?$allocator@VAtomproperty@PTools@@@std@@@std@@QAEXPAVAtomproperty@PTools@@ABV23@@Z 1001fd14     rigidbody.obj
 0002:00003d1c       __ehfuncinfo$??$construct@VAtomproperty@PTools@@ABV12@@?$_Wrap_alloc@V?$allocator@VAtomproperty@PTools@@@std@@@std@@QAEXPAVAtomproperty@PTools@@ABV23@@Z 1001fd1c     rigidbody.obj
 0002:00003d40       __unwindtable$??$construct@VAtomproperty@PTools@@AAV12@@?$allocator_traits@V?$allocator@VAtomproperty@PTools@@@std@@@std@@SAXAAV?$allocator@VAtomproperty@PTools@@@1@PAVAtomproperty@PTools@@AAV34@@Z 1001fd40     rigidbody.obj
 0002:00003d48       __ehfuncinfo$??$construct@VAtomproperty@PTools@@AAV12@@?$allocator_traits@V?$allocator@VAtomproperty@PTools@@@std@@@std@@SAXAAV?$allocator@VAtomproperty@PTools@@@1@PAVAtomproperty@PTools@@AAV34@@Z 1001fd48     rigidbody.obj
 0002:00003d6c       __unwindtable$??$construct@VAtomproperty@PTools@@ABV12@@?$allocator_traits@V?$allocator@VAtomproperty@PTools@@@std@@@std@@SAXAAV?$allocator@VAtomproperty@PTools@@@1@PAVAtomproperty@PTools@@ABV34@@Z 1001fd6c     rigidbody.obj
 0002:00003d74       __ehfuncinfo$??$construct@VAtomproperty@PTools@@ABV12@@?$allocator_traits@V?$allocator@VAtomproperty@PTools@@@std@@@std@@SAXAAV?$allocator@VAtomproperty@PTools@@@1@PAVAtomproperty@PTools@@ABV34@@Z 1001fd74     rigidbody.obj
 0002:00003d98       __unwindtable$??$construct@VAtomproperty@PTools@@AAV12@@?$allocator@VAtomproperty@PTools@@@std@@QAEXPAVAtomproperty@PTools@@AAV23@@Z 1001fd98     rigidbody.obj
 0002:00003da0       __ehfuncinfo$??$construct@VAtomproperty@PTools@@AAV12@@?$allocator@VAtomproperty@PTools@@@std@@QAEXPAVAtomproperty@PTools@@AAV23@@Z 1001fda0     rigidbody.obj
 0002:00003dc4       __catchsym$??$_Uninit_copy@PAVAtomproperty@PTools@@PAV12@V?$allocator@VAtomproperty@PTools@@@std@@@std@@YAPAVAtomproperty@PTools@@PAV12@00AAU?$_Wrap_alloc@V?$allocator@VAtomproperty@PTools@@@std@@@0@U_Nonscalar_ptr_iterator_tag@0@@Z$3 1001fdc4     rigidbody.obj
 0002:00003dd4       __tryblocktable$??$_Uninit_copy@PAVAtomproperty@PTools@@PAV12@V?$allocator@VAtomproperty@PTools@@@std@@@std@@YAPAVAtomproperty@PTools@@PAV12@00AAU?$_Wrap_alloc@V?$allocator@VAtomproperty@PTools@@@std@@@0@U_Nonscalar_ptr_iterator_tag@0@@Z 1001fdd4     rigidbody.obj
 0002:00003de8       __unwindtable$??$_Uninit_copy@PAVAtomproperty@PTools@@PAV12@V?$allocator@VAtomproperty@PTools@@@std@@@std@@YAPAVAtomproperty@PTools@@PAV12@00AAU?$_Wrap_alloc@V?$allocator@VAtomproperty@PTools@@@std@@@0@U_Nonscalar_ptr_iterator_tag@0@@Z 1001fde8     rigidbody.obj
 0002:00003e00       __ehfuncinfo$??$_Uninit_copy@PAVAtomproperty@PTools@@PAV12@V?$allocator@VAtomproperty@PTools@@@std@@@std@@YAPAVAtomproperty@PTools@@PAV12@00AAU?$_Wrap_alloc@V?$allocator@VAtomproperty@PTools@@@std@@@0@U_Nonscalar_ptr_iterator_tag@0@@Z 1001fe00     rigidbody.obj
 0002:00003e24       __catchsym$??$_Uninit_move@PAVAtomproperty@PTools@@PAV12@V?$allocator@VAtomproperty@PTools@@@std@@V12@@std@@YAPAVAtomproperty@PTools@@PAV12@00AAU?$_Wrap_alloc@V?$allocator@VAtomproperty@PTools@@@std@@@0@0U_Nonscalar_ptr_iterator_tag@0@@Z$3 1001fe24     rigidbody.obj
 0002:00003e34       __tryblocktable$??$_Uninit_move@PAVAtomproperty@PTools@@PAV12@V?$allocator@VAtomproperty@PTools@@@std@@V12@@std@@YAPAVAtomproperty@PTools@@PAV12@00AAU?$_Wrap_alloc@V?$allocator@VAtomproperty@PTools@@@std@@@0@0U_Nonscalar_ptr_iterator_tag@0@@Z 1001fe34     rigidbody.obj
 0002:00003e48       __unwindtable$??$_Uninit_move@PAVAtomproperty@PTools@@PAV12@V?$allocator@VAtomproperty@PTools@@@std@@V12@@std@@YAPAVAtomproperty@PTools@@PAV12@00AAU?$_Wrap_alloc@V?$allocator@VAtomproperty@PTools@@@std@@@0@0U_Nonscalar_ptr_iterator_tag@0@@Z 1001fe48     rigidbody.obj
 0002:00003e60       __ehfuncinfo$??$_Uninit_move@PAVAtomproperty@PTools@@PAV12@V?$allocator@VAtomproperty@PTools@@@std@@V12@@std@@YAPAVAtomproperty@PTools@@PAV12@00AAU?$_Wrap_alloc@V?$allocator@VAtomproperty@PTools@@@std@@@0@0U_Nonscalar_ptr_iterator_tag@0@@Z 1001fe60     rigidbody.obj
 0002:00003e84       __unwindtable$??$construct@VAtomproperty@PTools@@V12@@?$_Wrap_alloc@V?$allocator@VAtomproperty@PTools@@@std@@@std@@QAEXPAVAtomproperty@PTools@@$$QAV23@@Z 1001fe84     rigidbody.obj
 0002:00003e8c       __ehfuncinfo$??$construct@VAtomproperty@PTools@@V12@@?$_Wrap_alloc@V?$allocator@VAtomproperty@PTools@@@std@@@std@@QAEXPAVAtomproperty@PTools@@$$QAV23@@Z 1001fe8c     rigidbody.obj
 0002:00003eb0       __unwindtable$??$construct@VAtomproperty@PTools@@V12@@?$allocator_traits@V?$allocator@VAtomproperty@PTools@@@std@@@std@@SAXAAV?$allocator@VAtomproperty@PTools@@@1@PAVAtomproperty@PTools@@$$QAV34@@Z 1001feb0     rigidbody.obj
 0002:00003eb8       __ehfuncinfo$??$construct@VAtomproperty@PTools@@V12@@?$allocator_traits@V?$allocator@VAtomproperty@PTools@@@std@@@std@@SAXAAV?$allocator@VAtomproperty@PTools@@@1@PAVAtomproperty@PTools@@$$QAV34@@Z 1001feb8     rigidbody.obj
 0002:00003edc       __unwindtable$??$construct@VAtomproperty@PTools@@V12@@?$allocator@VAtomproperty@PTools@@@std@@QAEXPAVAtomproperty@PTools@@$$QAV23@@Z 1001fedc     rigidbody.obj
 0002:00003ee4       __ehfuncinfo$??$construct@VAtomproperty@PTools@@V12@@?$allocator@VAtomproperty@PTools@@@std@@QAEXPAVAtomproperty@PTools@@$$QAV23@@Z 1001fee4     rigidbody.obj
 0002:00003f08       __unwindtable$?Rmsd@PTools@@YANABVAtomSelection@1@0@Z 1001ff08     rmsd.obj
 0002:00003f18       __ehfuncinfo$?Rmsd@PTools@@YANABVAtomSelection@1@0@Z 1001ff18     rmsd.obj
 0002:00003f3c       __ehfuncinfo$?superpose@PTools@@YA?AUSuperpose_t@@ABVRigidbody@1@0H@Z 1001ff3c     superpose.obj
 0002:00003f60       __unwindtable$?superpose@PTools@@YA?AUSuperpose_t@@ABVRigidbody@1@0H@Z 1001ff60     superpose.obj
 0002:00003fa0       __unwindtable$?construct@?$allocator@V?$vector@NV?$allocator@N@std@@@std@@@std@@QAEXPAV?$vector@NV?$allocator@N@std@@@2@ABV32@@Z 1001ffa0     superpose.obj
 0002:00003fa8       __ehfuncinfo$?construct@?$allocator@V?$vector@NV?$allocator@N@std@@@std@@@std@@QAEXPAV?$vector@NV?$allocator@N@std@@@2@ABV32@@Z 1001ffa8     superpose.obj
 0002:00003fcc       __catchsym$?_Construct_n@?$vector@V?$vector@NV?$allocator@N@std@@@std@@V?$allocator@V?$vector@NV?$allocator@N@std@@@std@@@2@@std@@QAEXIPBV?$vector@NV?$allocator@N@std@@@2@@Z$2 1001ffcc     superpose.obj
 0002:00003fdc       __unwindtable$?_Construct_n@?$vector@V?$vector@NV?$allocator@N@std@@@std@@V?$allocator@V?$vector@NV?$allocator@N@std@@@std@@@2@@std@@QAEXIPBV?$vector@NV?$allocator@N@std@@@2@@Z 1001ffdc     superpose.obj
 0002:00003fec       __tryblocktable$?_Construct_n@?$vector@V?$vector@NV?$allocator@N@std@@@std@@V?$allocator@V?$vector@NV?$allocator@N@std@@@std@@@2@@std@@QAEXIPBV?$vector@NV?$allocator@N@std@@@2@@Z 1001ffec     superpose.obj
 0002:00004000       __ehfuncinfo$?_Construct_n@?$vector@V?$vector@NV?$allocator@N@std@@@std@@V?$allocator@V?$vector@NV?$allocator@N@std@@@std@@@2@@std@@QAEXIPBV?$vector@NV?$allocator@N@std@@@2@@Z 10020000     superpose.obj
 0002:00004024       __ehfuncinfo$?MakeTensor@PTools@@YAXAAVRigidbody@1@0QAY02N@Z 10020024     superpose.obj
 0002:00004048       __unwindtable$?MakeTensor@PTools@@YAXAAVRigidbody@1@0QAY02N@Z 10020048     superpose.obj
 0002:00004088       __catchsym$??$_Uninit_fill_n@PAV?$vector@NV?$allocator@N@std@@@std@@IV12@V?$allocator@V?$vector@NV?$allocator@N@std@@@std@@@2@V12@@std@@YAXPAV?$vector@NV?$allocator@N@std@@@0@IPBV10@AAU?$_Wrap_alloc@V?$allocator@V?$vector@NV?$allocator@N@std@@@std@@@std@@@0@0U_Nonscalar_ptr_iterator_tag@0@@Z$3 10020088     superpose.obj
 0002:00004098       __tryblocktable$??$_Uninit_fill_n@PAV?$vector@NV?$allocator@N@std@@@std@@IV12@V?$allocator@V?$vector@NV?$allocator@N@std@@@std@@@2@V12@@std@@YAXPAV?$vector@NV?$allocator@N@std@@@0@IPBV10@AAU?$_Wrap_alloc@V?$allocator@V?$vector@NV?$allocator@N@std@@@std@@@std@@@0@0U_Nonscalar_ptr_iterator_tag@0@@Z 10020098     superpose.obj
 0002:000040ac       __unwindtable$??$_Uninit_fill_n@PAV?$vector@NV?$allocator@N@std@@@std@@IV12@V?$allocator@V?$vector@NV?$allocator@N@std@@@std@@@2@V12@@std@@YAXPAV?$vector@NV?$allocator@N@std@@@0@IPBV10@AAU?$_Wrap_alloc@V?$allocator@V?$vector@NV?$allocator@N@std@@@std@@@std@@@0@0U_Nonscalar_ptr_iterator_tag@0@@Z 100200ac     superpose.obj
 0002:000040c4       __ehfuncinfo$??$_Uninit_fill_n@PAV?$vector@NV?$allocator@N@std@@@std@@IV12@V?$allocator@V?$vector@NV?$allocator@N@std@@@std@@@2@V12@@std@@YAXPAV?$vector@NV?$allocator@N@std@@@0@IPBV10@AAU?$_Wrap_alloc@V?$allocator@V?$vector@NV?$allocator@N@std@@@std@@@std@@@0@0U_Nonscalar_ptr_iterator_tag@0@@Z 100200c4     superpose.obj
 0002:000040e8       __unwindtable$??$construct@V?$vector@NV?$allocator@N@std@@@std@@ABV12@@?$_Wrap_alloc@V?$allocator@V?$vector@NV?$allocator@N@std@@@std@@@std@@@std@@QAEXPAV?$vector@NV?$allocator@N@std@@@1@ABV21@@Z 100200e8     superpose.obj
 0002:000040f0       __ehfuncinfo$??$construct@V?$vector@NV?$allocator@N@std@@@std@@ABV12@@?$_Wrap_alloc@V?$allocator@V?$vector@NV?$allocator@N@std@@@std@@@std@@@std@@QAEXPAV?$vector@NV?$allocator@N@std@@@1@ABV21@@Z 100200f0     superpose.obj
 0002:00004114       __unwindtable$??$construct@V?$vector@NV?$allocator@N@std@@@std@@ABV12@@?$allocator_traits@V?$allocator@V?$vector@NV?$allocator@N@std@@@std@@@std@@@std@@SAXAAV?$allocator@V?$vector@NV?$allocator@N@std@@@std@@@1@PAV?$vector@NV?$allocator@N@std@@@1@ABV31@@Z 10020114     superpose.obj
 0002:0000411c       __ehfuncinfo$??$construct@V?$vector@NV?$allocator@N@std@@@std@@ABV12@@?$allocator_traits@V?$allocator@V?$vector@NV?$allocator@N@std@@@std@@@std@@@std@@SAXAAV?$allocator@V?$vector@NV?$allocator@N@std@@@std@@@1@PAV?$vector@NV?$allocator@N@std@@@1@ABV31@@Z 1002011c     superpose.obj
 0002:00004178       __unwindtable$??__EalgoLog@U2@@YAXXZ 10020178     moc_PToolsPlugin.obj
 0002:00004180       __ehfuncinfo$??__EalgoLog@U2@@YAXXZ 10020180     moc_PToolsPlugin.obj
 0002:000041a4       __unwindtable$??__EcmdLog@U2@@YAXXZ 100201a4     moc_PToolsPlugin.obj
 0002:000041ac       __ehfuncinfo$??__EcmdLog@U2@@YAXXZ 100201ac     moc_PToolsPlugin.obj
 0002:000041d0       __unwindtable$??__EcoreLog@U2@@YAXXZ 100201d0     moc_PToolsPlugin.obj
 0002:000041d8       __ehfuncinfo$??__EcoreLog@U2@@YAXXZ 100201d8     moc_PToolsPlugin.obj
 0002:000041fc       __unwindtable$??__EioLog@U2@@YAXXZ 100201fc     moc_PToolsPlugin.obj
 0002:00004204       __ehfuncinfo$??__EioLog@U2@@YAXXZ 10020204     moc_PToolsPlugin.obj
 0002:00004228       __unwindtable$??__EperfLog@U2@@YAXXZ 10020228     moc_PToolsPlugin.obj
 0002:00004230       __ehfuncinfo$??__EperfLog@U2@@YAXXZ 10020230     moc_PToolsPlugin.obj
 0002:00004254       __unwindtable$??__EscriptLog@U2@@YAXXZ 10020254     moc_PToolsPlugin.obj
 0002:0000425c       __ehfuncinfo$??__EscriptLog@U2@@YAXXZ 1002025c     moc_PToolsPlugin.obj
 0002:00004280       __unwindtable$??__EtaskLog@U2@@YAXXZ 10020280     moc_PToolsPlugin.obj
 0002:00004288       __ehfuncinfo$??__EtaskLog@U2@@YAXXZ 10020288     moc_PToolsPlugin.obj
 0002:000042ac       __unwindtable$??__EuiLog@U2@@YAXXZ 100202ac     moc_PToolsPlugin.obj
 0002:000042b4       __ehfuncinfo$??__EuiLog@U2@@YAXXZ 100202b4     moc_PToolsPlugin.obj
 0002:000042d8       __unwindtable$??__EuserActLog@U2@@YAXXZ 100202d8     moc_PToolsPlugin.obj
 0002:000042e0       __ehfuncinfo$??__EuserActLog@U2@@YAXXZ 100202e0     moc_PToolsPlugin.obj
 0002:00004304       __unwindtable$??__EalgoLog@U2@@YAXXZ 10020304     moc_PToolsTests.obj
 0002:0000430c       __ehfuncinfo$??__EalgoLog@U2@@YAXXZ 1002030c     moc_PToolsTests.obj
 0002:00004330       __unwindtable$??__EcmdLog@U2@@YAXXZ 10020330     moc_PToolsTests.obj
 0002:00004338       __ehfuncinfo$??__EcmdLog@U2@@YAXXZ 10020338     moc_PToolsTests.obj
 0002:0000435c       __unwindtable$??__EcoreLog@U2@@YAXXZ 1002035c     moc_PToolsTests.obj
 0002:00004364       __ehfuncinfo$??__EcoreLog@U2@@YAXXZ 10020364     moc_PToolsTests.obj
 0002:00004388       __unwindtable$??__EioLog@U2@@YAXXZ 10020388     moc_PToolsTests.obj
 0002:00004390       __ehfuncinfo$??__EioLog@U2@@YAXXZ 10020390     moc_PToolsTests.obj
 0002:000043b4       __unwindtable$??__EperfLog@U2@@YAXXZ 100203b4     moc_PToolsTests.obj
 0002:000043bc       __ehfuncinfo$??__EperfLog@U2@@YAXXZ 100203bc     moc_PToolsTests.obj
 0002:000043e0       __unwindtable$??__EscriptLog@U2@@YAXXZ 100203e0     moc_PToolsTests.obj
 0002:000043e8       __ehfuncinfo$??__EscriptLog@U2@@YAXXZ 100203e8     moc_PToolsTests.obj
 0002:0000440c       __unwindtable$??__EtaskLog@U2@@YAXXZ 1002040c     moc_PToolsTests.obj
 0002:00004414       __ehfuncinfo$??__EtaskLog@U2@@YAXXZ 10020414     moc_PToolsTests.obj
 0002:00004438       __unwindtable$??__EuiLog@U2@@YAXXZ 10020438     moc_PToolsTests.obj
 0002:00004440       __ehfuncinfo$??__EuiLog@U2@@YAXXZ 10020440     moc_PToolsTests.obj
 0002:00004464       __unwindtable$??__EuserActLog@U2@@YAXXZ 10020464     moc_PToolsTests.obj
 0002:0000446c       __ehfuncinfo$??__EuserActLog@U2@@YAXXZ 1002046c     moc_PToolsTests.obj
 0002:00004490       __sehtable$__onexit        10020490     MSVCRT:atonexit.obj
 0002:000044b0       __sehtable$??_M@YGXPAXIHP6EX0@Z@Z 100204b0     MSVCRT:ehvecdtr.obj
 0002:000044d0       __sehtable$?__ArrayUnwind@@YGXPAXIHP6EX0@Z@Z 100204d0     MSVCRT:ehvecdtr.obj
 0002:000044f0       __sehtable$___DllMainCRTStartup 100204f0     MSVCRT:crtdll.obj
 0002:00004518       __sehtable$__IsNonwritableInCurrentImage 10020518     MSVCRT:pesect.obj
 0002:00004540       .edata                     10020540     ptools.exp
 0002:00004568       rgpv                       10020568     ptools.exp
 0002:0000456c       rgszName                   1002056c     ptools.exp
 0002:00004570       rgwOrd                     10020570     ptools.exp
 0002:00004572       szName                     10020572     ptools.exp
 0002:0000457d       $N00001                    1002057d     ptools.exp
 0002:000050ec       .idata$6                   100210ec     U2Core:U2Core.dll
 0002:00005342       .idata$6                   10021342     U2Algorithm:U2Algorithm.dll
 0002:000055aa       .idata$6                   100215aa     U2Test:U2Test.dll
 0002:000055e8       .idata$6                   100215e8     Qt5Xml:Qt5Xml.dll
 0002:00005d74       .idata$6                   10021d74     Qt5Core:Qt5Core.dll
 0002:00006976       .idata$6                   10022976     msvcprt:MSVCP120.dll
 0002:00006c2c       .idata$6                   10022c2c     MSVCRT:MSVCR120.dll
 0002:00006e40       .idata$6                   10022e40     kernel32:KERNEL32.dll
 0003:00000710       __Tuple_alloc              10023710     PToolsAligner.obj
 0003:00000711       _ignore                    10023711     PToolsAligner.obj
 0003:00000712       _allocator_arg             10023712     PToolsAligner.obj
 0003:00000713       _piecewise_construct       10023713     PToolsAligner.obj
 0003:00000714       _taskLog                   10023714     PToolsAligner.obj
 0003:0000071c       _algoLog                   1002371c     PToolsAligner.obj
 0003:00000724       _userActLog                10023724     PToolsAligner.obj
 0003:0000072c       _ioLog                     1002372c     PToolsAligner.obj
 0003:00000734       _coreLog                   10023734     PToolsAligner.obj
 0003:0000073c       _uiLog                     1002373c     PToolsAligner.obj
 0003:00000744       _scriptLog                 10023744     PToolsAligner.obj
 0003:0000074c       _perfLog                   1002374c     PToolsAligner.obj
 0003:00000754       _cmdLog                    10023754     PToolsAligner.obj
 0003:00000764       __Tuple_alloc              10023764     PToolsPlugin.obj
 0003:00000765       _ignore                    10023765     PToolsPlugin.obj
 0003:00000766       _allocator_arg             10023766     PToolsPlugin.obj
 0003:00000767       _piecewise_construct       10023767     PToolsPlugin.obj
 0003:00000768       _taskLog                   10023768     PToolsPlugin.obj
 0003:00000770       _algoLog                   10023770     PToolsPlugin.obj
 0003:00000778       _PTOOLS_ID                 10023778     PToolsPlugin.obj
 0003:0000077c       _userActLog                1002377c     PToolsPlugin.obj
 0003:00000784       _ioLog                     10023784     PToolsPlugin.obj
 0003:0000078c       _coreLog                   1002378c     PToolsPlugin.obj
 0003:00000794       _uiLog                     10023794     PToolsPlugin.obj
 0003:0000079c       _scriptLog                 1002379c     PToolsPlugin.obj
 0003:000007a4       _perfLog                   100237a4     PToolsPlugin.obj
 0003:000007ac       _cmdLog                    100237ac     PToolsPlugin.obj
 0003:000007b4       __Tuple_alloc              100237b4     PToolsTests.obj
 0003:000007b5       _ignore                    100237b5     PToolsTests.obj
 0003:000007b6       _allocator_arg             100237b6     PToolsTests.obj
 0003:000007b7       _piecewise_construct       100237b7     PToolsTests.obj
 0003:000007b8       _taskLog                   100237b8     PToolsTests.obj
 0003:000007c0       _algoLog                   100237c0     PToolsTests.obj
 0003:000007c8       _userActLog                100237c8     PToolsTests.obj
 0003:000007d0       _ioLog                     100237d0     PToolsTests.obj
 0003:000007d8       _coreLog                   100237d8     PToolsTests.obj
 0003:000007e0       _uiLog                     100237e0     PToolsTests.obj
 0003:000007f0       _scriptLog                 100237f0     PToolsTests.obj
 0003:000007f8       _perfLog                   100237f8     PToolsTests.obj
 0003:00000800       _cmdLog                    10023800     PToolsTests.obj
 0003:00000814       _allocator_arg             10023814     atom.obj
 0003:00000815       _piecewise_construct       10023815     atom.obj
 0003:00000816       _allocator_arg             10023816     atomselection.obj
 0003:00000817       _piecewise_construct       10023817     atomselection.obj
 0003:00000818       _allocator_arg             10023818     basetypes.obj
 0003:00000819       _piecewise_construct       10023819     basetypes.obj
 0003:0000081a       _allocator_arg             1002381a     coord3d.obj
 0003:0000081b       _piecewise_construct       1002381b     coord3d.obj
 0003:0000081c       _allocator_arg             1002381c     coordsarray.obj
 0003:0000081d       _piecewise_construct       1002381d     coordsarray.obj
 0003:0000081e       _allocator_arg             1002381e     geometry.obj
 0003:0000081f       _piecewise_construct       1002381f     geometry.obj
 0003:00000820       _allocator_arg             10023820     pdbio.obj
 0003:00000821       _piecewise_construct       10023821     pdbio.obj
 0003:0000082c       _allocator_arg             1002382c     rigidbody.obj
 0003:0000082d       _piecewise_construct       1002382d     rigidbody.obj
 0003:0000082e       _allocator_arg             1002382e     rmsd.obj
 0003:0000082f       _piecewise_construct       1002382f     rmsd.obj
 0003:00000830       _allocator_arg             10023830     superpose.obj
 0003:00000831       _piecewise_construct       10023831     superpose.obj
 0003:00000834       __Tuple_alloc              10023834     moc_PToolsPlugin.obj
 0003:00000835       _ignore                    10023835     moc_PToolsPlugin.obj
 0003:00000836       _allocator_arg             10023836     moc_PToolsPlugin.obj
 0003:00000837       _piecewise_construct       10023837     moc_PToolsPlugin.obj
 0003:00000838       _taskLog                   10023838     moc_PToolsPlugin.obj
 0003:00000840       _algoLog                   10023840     moc_PToolsPlugin.obj
 0003:00000848       _userActLog                10023848     moc_PToolsPlugin.obj
 0003:00000850       _ioLog                     10023850     moc_PToolsPlugin.obj
 0003:00000858       _coreLog                   10023858     moc_PToolsPlugin.obj
 0003:00000860       _uiLog                     10023860     moc_PToolsPlugin.obj
 0003:00000868       _scriptLog                 10023868     moc_PToolsPlugin.obj
 0003:00000870       _perfLog                   10023870     moc_PToolsPlugin.obj
 0003:00000878       _cmdLog                    10023878     moc_PToolsPlugin.obj
 0003:00000880       __Tuple_alloc              10023880     moc_PToolsTests.obj
 0003:00000881       _ignore                    10023881     moc_PToolsTests.obj
 0003:00000882       _allocator_arg             10023882     moc_PToolsTests.obj
 0003:00000883       _piecewise_construct       10023883     moc_PToolsTests.obj
 0003:00000884       _taskLog                   10023884     moc_PToolsTests.obj
 0003:0000088c       _algoLog                   1002388c     moc_PToolsTests.obj
 0003:00000894       _userActLog                10023894     moc_PToolsTests.obj
 0003:0000089c       _ioLog                     1002389c     moc_PToolsTests.obj
 0003:000008a4       _coreLog                   100238a4     moc_PToolsTests.obj
 0003:000008ac       _uiLog                     100238ac     moc_PToolsTests.obj
 0003:000008b4       _scriptLog                 100238b4     moc_PToolsTests.obj
 0003:000008bc       _perfLog                   100238bc     moc_PToolsTests.obj
 0003:000008c4       _cmdLog                    100238c4     moc_PToolsTests.obj
 0003:000008cc       __Fac_head                 100238cc     msvcprt:locale0_implib.obj
 0003:000008d0       __Fac_tidy_reg             100238d0     msvcprt:locale0_implib.obj
 0003:000008d4       ___proc_attached           100238d4     MSVCRT:crtdll.obj
 0003:000008d8       _GS_ExceptionRecord        100238d8     MSVCRT:gs_report.obj
 0003:00000928       _GS_ContextRecord          10023928     MSVCRT:gs_report.obj
 0003:00000bf4       _DebuggerWasPresent        10023bf4     MSVCRT:gs_report.obj
 0004:00000060       $R000000                   10024060     * linker generated manifest res *

 Exports

  ordinal    name

        1    _ugene_plugin_init
               exported name: ugene_plugin_init
